 dna_flexibility

 Timestamp is 5c7621ff (Wed Feb 27 12:37:03 2019)

 Preferred load address is 10000000

 Start         Length     Name                   Class
 0001:00000000 00003e54H .text$di                CODE
 0001:00003e60 0000acbeH .text$mn                CODE
 0001:0000eb20 000024b4H .text$x                 CODE
 0001:00010fe0 00000e6aH .text$yd                CODE
 0002:00000000 000008b8H .idata$5                DATA
 0002:000008b8 00000004H .CRT$XCA                DATA
 0002:000008bc 00000320H .CRT$XCU                DATA
 0002:00000bdc 00000004H .CRT$XCZ                DATA
 0002:00000be0 00000004H .CRT$XIA                DATA
 0002:00000be4 00000004H .CRT$XIAA               DATA
 0002:00000be8 00000004H .CRT$XIC                DATA
 0002:00000bec 00000004H .CRT$XIZ                DATA
 0002:00000bf0 000024a0H .rdata                  DATA
 0002:00003090 00000078H .rdata$debug            DATA
 0002:00003108 000010b4H .rdata$r                DATA
 0002:000041c0 00000280H .rdata$sxdata           DATA
 0002:00004440 00000004H .rtc$IAA                DATA
 0002:00004444 00000004H .rtc$IZZ                DATA
 0002:00004448 00000004H .rtc$TAA                DATA
 0002:0000444c 00000004H .rtc$TZZ                DATA
 0002:00004450 0000286cH .xdata$x                DATA
 0002:00006cc0 00000058H .edata                  DATA
 0002:00006d18 000000b4H .idata$2                DATA
 0002:00006dcc 00000014H .idata$3                DATA
 0002:00006de0 000008b8H .idata$4                DATA
 0002:00007698 00006368H .idata$6                DATA
 0003:00000000 00000324H .data                   DATA
 0003:00000324 000006e8H .data$r                 DATA
 0003:00000a10 000006f4H .bss                    DATA
 0004:00000000 00000058H .rsrc$01                DATA
 0004:00000060 00000180H .rsrc$02                DATA

  Address         Publics by Value              Rva+Base       Lib:Object

 0000:00000000       __except_list              00000000     <absolute>
 0000:00000000       ___guard_fids_table        00000000     <absolute>
 0000:00000000       ___guard_flags             00000000     <absolute>
 0000:00000000       ___guard_fids_count        00000000     <absolute>
 0000:000000a0       ___safe_se_handler_count   000000a0     <absolute>
 0000:00009876       __ldused                   00009876     <absolute>
 0000:00009876       __fltused                  00009876     <absolute>
 0000:00000000       ___ImageBase               10000000     <linker-defined>
 0001:00003e60       ??$_Allocate@D@std@@YAPADIPAD@Z 10004e60 f i DNAFlexDialog.obj
 0001:00003e90       ??$addressof@D@std@@YAPADAAD@Z 10004e90 f i DNAFlexDialog.obj
 0001:00003ea0       ??$atomic@H@?$QAtomicOpsBySize@$03@@CAPAJPAH@Z 10004ea0 f i DNAFlexDialog.obj
 0001:00003eb0       ??$construct@PADAAPAD@?$_Wrap_alloc@V?$allocator@D@std@@@std@@QAEXPAPADAAPAD@Z 10004eb0 f i DNAFlexDialog.obj
 0001:00003ed0       ??$construct@PADAAPAD@?$allocator@D@std@@QAEXPAPADAAPAD@Z 10004ed0 f i DNAFlexDialog.obj
 0001:00003ef0       ??$construct@PADAAPAD@?$allocator_traits@V?$allocator@D@std@@@std@@SAXAAV?$allocator@D@1@PAPADAAPAD@Z 10004ef0 f i DNAFlexDialog.obj
 0001:00003f10       ??$deref@H@?$QAtomicOpsBySize@$03@@SA_NAAH@Z 10004f10 f i DNAFlexDialog.obj
 0001:00003f30       ??$destroy@PAD@?$_Wrap_alloc@V?$allocator@D@std@@@std@@QAEXPAPAD@Z 10004f30 f i DNAFlexDialog.obj
 0001:00003f40       ??$destroy@PAD@?$allocator@D@std@@QAEXPAPAD@Z 10004f40 f i DNAFlexDialog.obj
 0001:00003f50       ??$destroy@PAD@?$allocator_traits@V?$allocator@D@std@@@std@@SAXAAV?$allocator@D@1@PAPAD@Z 10004f50 f i DNAFlexDialog.obj
 0001:00003f60       ??$forward@AAPAD@std@@YAAAPADAAPAD@Z 10004f60 f i DNAFlexDialog.obj
 0001:00003f70       ??$load@H@?$QGenericAtomicOps@U?$QAtomicOpsBySize@$03@@@@SAHABH@Z 10004f70 f i DNAFlexDialog.obj
 0001:00003f80       ??$ref@H@?$QAtomicOpsBySize@$03@@SA_NAAH@Z 10004f80 f i DNAFlexDialog.obj
 0001:00003fa0       ??0?$AbstractId@H@U2@@IAE@ABH@Z 10004fa0 f i DNAFlexDialog.obj
 0001:00003fc0       ??0?$QFlags@W4AlignmentFlag@Qt@@@@QAE@PQPrivate@0@H@Z 10004fc0 f i DNAFlexDialog.obj
 0001:00003fd0       ??0?$QFlags@W4StandardButton@QDialogButtonBox@@@@QAE@VQFlag@@@Z 10004fd0 f i DNAFlexDialog.obj
 0001:00003fe0       ??0?$QFlags@W4StandardButton@QDialogButtonBox@@@@QAE@W4StandardButton@QDialogButtonBox@@@Z 10004fe0 f i DNAFlexDialog.obj
 0001:00003ff0       ??0?$QFlags@W4StandardButton@QMessageBox@@@@QAE@W4StandardButton@QMessageBox@@@Z 10004ff0 f i DNAFlexDialog.obj
 0001:00004000       ??0?$QFlags@W4WindowType@Qt@@@@QAE@PQPrivate@0@H@Z 10005000 f i DNAFlexDialog.obj
 0001:00004010       ??0?$_String_alloc@$0A@U?$_String_base_types@DV?$allocator@D@std@@@std@@@std@@QAE@ABV?$allocator@D@1@@Z 10005010 f i DNAFlexDialog.obj
 0001:00004030       ??0?$_String_val@U?$_Simple_types@D@std@@@std@@QAE@XZ 10005030 f i DNAFlexDialog.obj
 0001:00004050       ??0?$_Wrap_alloc@V?$allocator@D@std@@@std@@QAE@XZ 10005050 f i DNAFlexDialog.obj
 0001:00004060       ??0?$allocator@D@std@@QAE@XZ 10005060 f i DNAFlexDialog.obj
 0001:00004070       ??0?$basic_string@DU?$char_traits@D@std@@V?$allocator@D@2@@std@@QAE@PBD@Z 10005070 f i DNAFlexDialog.obj
 0001:000040d0       ??0AbstractInt32Id@U2@@IAE@H@Z 100050d0 f i DNAFlexDialog.obj
 0001:000040f0       ??0DNAFlexDialog@U2@@QAE@PAVADVSequenceObjectContext@1@@Z 100050f0 f   DNAFlexDialog.obj
 0001:000044c0       ??0QFlag@@QAE@H@Z          100054c0 f i DNAFlexDialog.obj
 0001:000044d0       ??0ServiceType@U2@@QAE@H@Z 100054d0 f i DNAFlexDialog.obj
 0001:000044f0       ??0_Generic_error_category@std@@QAE@XZ 100054f0 f i DNAFlexDialog.obj
 0001:00004500       ??0_Ignore@std@@QAE@XZ     10005500 f i DNAFlexDialog.obj
 0001:00004510       ??0_Iostream_error_category@std@@QAE@XZ 10005510 f i DNAFlexDialog.obj
 0001:00004520       ??0_System_error_category@std@@QAE@XZ 10005520 f i DNAFlexDialog.obj
 0001:00004530       ??0error_category@std@@QAE@XZ 10005530 f i DNAFlexDialog.obj
 0001:00004540       ??0error_condition@std@@QAE@HABVerror_category@1@@Z 10005540 f i DNAFlexDialog.obj
 0001:00004560       ??1?$AbstractId@H@U2@@MAE@XZ 10005560 f i DNAFlexDialog.obj
 0001:00004570       ??1?$basic_string@DU?$char_traits@D@std@@V?$allocator@D@2@@std@@QAE@XZ 10005570 f i DNAFlexDialog.obj
 0001:000045a0       ??1AbstractInt32Id@U2@@UAE@XZ 100055a0 f i DNAFlexDialog.obj
 0001:000045b0       ??1DNAFlexDialog@U2@@UAE@XZ 100055b0 f i DNAFlexDialog.obj
 0001:000045c0       ??1ServiceType@U2@@UAE@XZ  100055c0 f i DNAFlexDialog.obj
 0001:000045d0       ??1_Generic_error_category@std@@UAE@XZ 100055d0 f i DNAFlexDialog.obj
 0001:000045e0       ??1_Iostream_error_category@std@@UAE@XZ 100055e0 f i DNAFlexDialog.obj
 0001:000045f0       ??1_System_error_category@std@@UAE@XZ 100055f0 f i DNAFlexDialog.obj
 0001:00004600       ??1error_category@std@@UAE@XZ 10005600 f i DNAFlexDialog.obj
 0001:00004610       ??2@YAPAXIPAX@Z            10005610 f i DNAFlexDialog.obj
 0001:00004620       ??3@YAXPAX0@Z              10005620 f i DNAFlexDialog.obj
 0001:00004630       ??8error_category@std@@QBE_NABV01@@Z 10005630 f i DNAFlexDialog.obj
 0001:00004640       ??8error_condition@std@@QBE_NABV01@@Z 10005640 f i DNAFlexDialog.obj
 0001:00004660       ??BQFlag@@QBEHXZ           10005660 f i DNAFlexDialog.obj
 0001:00004670       ??C?$QSharedDataPointer@VAnnotationData@U2@@@@QAEPAVAnnotationData@U2@@XZ 10005670 f i DNAFlexDialog.obj
 0001:00004690       ??C?$QSharedDataPointer@VAnnotationData@U2@@@@QBEPBVAnnotationData@U2@@XZ 10005690 f i DNAFlexDialog.obj
 0001:00004900       ??U?$QFlags@W4StandardButton@QDialogButtonBox@@@@QBE?AV0@W4StandardButton@QDialogButtonBox@@@Z 10005900 f i DNAFlexDialog.obj
 0001:00004920       ??U@YA?AV?$QFlags@W4StandardButton@QDialogButtonBox@@@@W4StandardButton@QDialogButtonBox@@0@Z 10005920 f i DNAFlexDialog.obj
 0001:00004930       ??_EDNAFlexDialog@U2@@W7AEPAXI@Z 10005930 f i DNAFlexDialog.obj
 0001:00004938       ??_EQDialogButtonBox@@W7AEPAXI@Z 10005938 f i DNAFlexDialog.obj
 0001:00004940       ??_EQDoubleSpinBox@@W7AEPAXI@Z 10005940 f i DNAFlexDialog.obj
 0001:00004948       ??_EQGridLayout@@W7AEPAXI@Z 10005948 f i DNAFlexDialog.obj
 0001:00004950       ??_EQGroupBox@@W7AEPAXI@Z  10005950 f i DNAFlexDialog.obj
 0001:00004958       ??_EQHBoxLayout@@W7AEPAXI@Z 10005958 f i DNAFlexDialog.obj
 0001:00004960       ??_EQLabel@@W7AEPAXI@Z     10005960 f i DNAFlexDialog.obj
 0001:00004968       ??_EQPushButton@@W7AEPAXI@Z 10005968 f i DNAFlexDialog.obj
 0001:00004970       ??_EQSpinBox@@W7AEPAXI@Z   10005970 f i DNAFlexDialog.obj
 0001:00004978       ??_EQTabWidget@@W7AEPAXI@Z 10005978 f i DNAFlexDialog.obj
 0001:00004980       ??_EQVBoxLayout@@W7AEPAXI@Z 10005980 f i DNAFlexDialog.obj
 0001:00004988       ??_EQWidget@@W7AEPAXI@Z    10005988 f i DNAFlexDialog.obj
 0001:00004990       ??_G?$AbstractId@H@U2@@MAEPAXI@Z 10005990 f i DNAFlexDialog.obj
 0001:00004990       ??_E?$AbstractId@H@U2@@MAEPAXI@Z 10005990 f i DNAFlexDialog.obj
 0001:000049c0       ??_GAbstractInt32Id@U2@@UAEPAXI@Z 100059c0 f i DNAFlexDialog.obj
 0001:000049c0       ??_EAbstractInt32Id@U2@@UAEPAXI@Z 100059c0 f i DNAFlexDialog.obj
 0001:000049f0       ??_GAnnotationData@U2@@QAEPAXI@Z 100059f0 f i DNAFlexDialog.obj
 0001:00004a20       ??_GCreateAnnotationWidgetController@U2@@UAEPAXI@Z 10005a20 f i DNAFlexDialog.obj
 0001:00004a20       ??_ECreateAnnotationWidgetController@U2@@UAEPAXI@Z 10005a20 f i DNAFlexDialog.obj
 0001:00004a50       ??_GDNAFlexDialog@U2@@UAEPAXI@Z 10005a50 f i DNAFlexDialog.obj
 0001:00004a50       ??_EDNAFlexDialog@U2@@UAEPAXI@Z 10005a50 f i DNAFlexDialog.obj
 0001:00004a80       ??_EHelpButton@U2@@UAEPAXI@Z 10005a80 f i DNAFlexDialog.obj
 0001:00004a80       ??_GHelpButton@U2@@UAEPAXI@Z 10005a80 f i DNAFlexDialog.obj
 0001:00004ab0       ??_EQDialogButtonBox@@UAEPAXI@Z 10005ab0 f i DNAFlexDialog.obj
 0001:00004ab0       ??_GQDialogButtonBox@@UAEPAXI@Z 10005ab0 f i DNAFlexDialog.obj
 0001:00004ae0       ??_EQDoubleSpinBox@@UAEPAXI@Z 10005ae0 f i DNAFlexDialog.obj
 0001:00004ae0       ??_GQDoubleSpinBox@@UAEPAXI@Z 10005ae0 f i DNAFlexDialog.obj
 0001:00004b10       ??_EQGridLayout@@UAEPAXI@Z 10005b10 f i DNAFlexDialog.obj
 0001:00004b10       ??_GQGridLayout@@UAEPAXI@Z 10005b10 f i DNAFlexDialog.obj
 0001:00004b40       ??_GQGroupBox@@UAEPAXI@Z   10005b40 f i DNAFlexDialog.obj
 0001:00004b40       ??_EQGroupBox@@UAEPAXI@Z   10005b40 f i DNAFlexDialog.obj
 0001:00004b70       ??_EQHBoxLayout@@UAEPAXI@Z 10005b70 f i DNAFlexDialog.obj
 0001:00004b70       ??_GQHBoxLayout@@UAEPAXI@Z 10005b70 f i DNAFlexDialog.obj
 0001:00004ba0       ??_GQLabel@@UAEPAXI@Z      10005ba0 f i DNAFlexDialog.obj
 0001:00004ba0       ??_EQLabel@@UAEPAXI@Z      10005ba0 f i DNAFlexDialog.obj
 0001:00004bd0       ??_GQPushButton@@UAEPAXI@Z 10005bd0 f i DNAFlexDialog.obj
 0001:00004bd0       ??_EQPushButton@@UAEPAXI@Z 10005bd0 f i DNAFlexDialog.obj
 0001:00004c00       ??_EQSpacerItem@@UAEPAXI@Z 10005c00 f i DNAFlexDialog.obj
 0001:00004c00       ??_GQSpacerItem@@UAEPAXI@Z 10005c00 f i DNAFlexDialog.obj
 0001:00004c30       ??_GQSpinBox@@UAEPAXI@Z    10005c30 f i DNAFlexDialog.obj
 0001:00004c30       ??_EQSpinBox@@UAEPAXI@Z    10005c30 f i DNAFlexDialog.obj
 0001:00004c60       ??_EQTabWidget@@UAEPAXI@Z  10005c60 f i DNAFlexDialog.obj
 0001:00004c60       ??_GQTabWidget@@UAEPAXI@Z  10005c60 f i DNAFlexDialog.obj
 0001:00004c90       ??_EQVBoxLayout@@UAEPAXI@Z 10005c90 f i DNAFlexDialog.obj
 0001:00004c90       ??_GQVBoxLayout@@UAEPAXI@Z 10005c90 f i DNAFlexDialog.obj
 0001:00004cc0       ??_GQWidget@@UAEPAXI@Z     10005cc0 f i DNAFlexDialog.obj
 0001:00004cc0       ??_EQWidget@@UAEPAXI@Z     10005cc0 f i DNAFlexDialog.obj
 0001:00004cf0       ??_GServiceType@U2@@UAEPAXI@Z 10005cf0 f i DNAFlexDialog.obj
 0001:00004cf0       ??_EServiceType@U2@@UAEPAXI@Z 10005cf0 f i DNAFlexDialog.obj
 0001:00004d20       ??_E_Generic_error_category@std@@UAEPAXI@Z 10005d20 f i DNAFlexDialog.obj
 0001:00004d20       ??_G_Generic_error_category@std@@UAEPAXI@Z 10005d20 f i DNAFlexDialog.obj
 0001:00004d50       ??_G_Iostream_error_category@std@@UAEPAXI@Z 10005d50 f i DNAFlexDialog.obj
 0001:00004d50       ??_E_Iostream_error_category@std@@UAEPAXI@Z 10005d50 f i DNAFlexDialog.obj
 0001:00004d80       ??_G_System_error_category@std@@UAEPAXI@Z 10005d80 f i DNAFlexDialog.obj
 0001:00004d80       ??_E_System_error_category@std@@UAEPAXI@Z 10005d80 f i DNAFlexDialog.obj
 0001:00004db0       ??_Gerror_category@std@@UAEPAXI@Z 10005db0 f i DNAFlexDialog.obj
 0001:00004db0       ??_Eerror_category@std@@UAEPAXI@Z 10005db0 f i DNAFlexDialog.obj
 0001:00004de0       ?_Copy@?$basic_string@DU?$char_traits@D@std@@V?$allocator@D@2@@std@@QAEXII@Z 10005de0 f i DNAFlexDialog.obj
 0001:00004f30       ?_Eos@?$basic_string@DU?$char_traits@D@std@@V?$allocator@D@2@@std@@QAEXI@Z 10005f30 f i DNAFlexDialog.obj
 0001:00004f60       ?_Getal@?$_String_alloc@$0A@U?$_String_base_types@DV?$allocator@D@std@@@std@@@std@@QBE?AU?$_Wrap_alloc@V?$allocator@D@std@@@2@XZ 10005f60 f i DNAFlexDialog.obj
 0001:00004f70       ?_Grow@?$basic_string@DU?$char_traits@D@std@@V?$allocator@D@2@@std@@QAE_NI_N@Z 10005f70 f i DNAFlexDialog.obj
 0001:00005020       ?_Inside@?$basic_string@DU?$char_traits@D@std@@V?$allocator@D@2@@std@@QAE_NPBD@Z 10006020 f i DNAFlexDialog.obj
 0001:00005060       ?_Myptr@?$_String_val@U?$_Simple_types@D@std@@@std@@QAEPADXZ 10006060 f i DNAFlexDialog.obj
 0001:00005070       ?_Myptr@?$_String_val@U?$_Simple_types@D@std@@@std@@QBEPBDXZ 10006070 f i DNAFlexDialog.obj
 0001:00005080       ?_Tidy@?$basic_string@DU?$char_traits@D@std@@V?$allocator@D@2@@std@@QAEX_NI@Z 10006080 f i DNAFlexDialog.obj
 0001:000050d0       ?_Xlen@?$basic_string@DU?$char_traits@D@std@@V?$allocator@D@2@@std@@QBEXXZ 100060d0 f i DNAFlexDialog.obj
 0001:000050e0       ?_Xran@?$basic_string@DU?$char_traits@D@std@@V?$allocator@D@2@@std@@QBEXXZ 100060e0 f i DNAFlexDialog.obj
 0001:000050f0       ?accept@DNAFlexDialog@U2@@UAEXXZ 100060f0 f   DNAFlexDialog.obj
 0001:000053b0       ?allocate@?$_Wrap_alloc@V?$allocator@D@std@@@std@@QAEPADI@Z 100063b0 f i DNAFlexDialog.obj
 0001:000053e0       ?allocate@?$allocator@D@std@@QAEPADI@Z 100063e0 f i DNAFlexDialog.obj
 0001:00005410       ?assign@?$basic_string@DU?$char_traits@D@std@@V?$allocator@D@2@@std@@QAEAAV12@ABV12@II@Z 10006410 f i DNAFlexDialog.obj
 0001:00005530       ?assign@?$basic_string@DU?$char_traits@D@std@@V?$allocator@D@2@@std@@QAEAAV12@PBD@Z 10006530 f i DNAFlexDialog.obj
 0001:00005570       ?assign@?$basic_string@DU?$char_traits@D@std@@V?$allocator@D@2@@std@@QAEAAV12@PBDI@Z 10006570 f i DNAFlexDialog.obj
 0001:00005670       ?assign@?$char_traits@D@std@@SAXAADABD@Z 10006670 f i DNAFlexDialog.obj
 0001:00005680       ?category@error_code@std@@QBEABVerror_category@2@XZ 10006680 f i DNAFlexDialog.obj
 0001:00005690       ?category@error_condition@std@@QBEABVerror_category@2@XZ 10006690 f i DNAFlexDialog.obj
 0001:000056a0       ?clone@?$QSharedDataPointer@VAnnotationData@U2@@@@IAEPAVAnnotationData@U2@@XZ 100066a0 f i DNAFlexDialog.obj
 0001:00005710       ?copy@?$char_traits@D@std@@SAPADPADPBDI@Z 10006710 f i DNAFlexDialog.obj
 0001:00005730       ?data_ptr@?$QStaticStringData@$08@@QBEPAU?$QTypedArrayData@G@@XZ 10006730 f i DNAFlexDialog.obj
 0001:00005740       ?data_ptr@?$QStaticStringData@$09@@QBEPAU?$QTypedArrayData@G@@XZ 10006740 f i DNAFlexDialog.obj
 0001:00005750       ?data_ptr@?$QStaticStringData@$0BA@@@QBEPAU?$QTypedArrayData@G@@XZ 10006750 f i DNAFlexDialog.obj
 0001:00005760       ?data_ptr@?$QStaticStringData@$0BB@@@QBEPAU?$QTypedArrayData@G@@XZ 10006760 f i DNAFlexDialog.obj
 0001:00005770       ?data_ptr@?$QStaticStringData@$0BF@@@QBEPAU?$QTypedArrayData@G@@XZ 10006770 f i DNAFlexDialog.obj
 0001:00005780       ?data_ptr@?$QStaticStringData@$0BG@@@QBEPAU?$QTypedArrayData@G@@XZ 10006780 f i DNAFlexDialog.obj
 0001:00005790       ?data_ptr@?$QStaticStringData@$0L@@@QBEPAU?$QTypedArrayData@G@@XZ 10006790 f i DNAFlexDialog.obj
 0001:000057a0       ?data_ptr@?$QStaticStringData@$0M@@@QBEPAU?$QTypedArrayData@G@@XZ 100067a0 f i DNAFlexDialog.obj
 0001:000057b0       ?data_ptr@?$QStaticStringData@$0N@@@QBEPAU?$QTypedArrayData@G@@XZ 100067b0 f i DNAFlexDialog.obj
 0001:000057c0       ?data_ptr@?$QStaticStringData@$0O@@@QBEPAU?$QTypedArrayData@G@@XZ 100067c0 f i DNAFlexDialog.obj
 0001:000057d0       ?deallocate@?$_Wrap_alloc@V?$allocator@D@std@@@std@@QAEXPADI@Z 100067d0 f i DNAFlexDialog.obj
 0001:000057f0       ?deallocate@?$allocator@D@std@@QAEXPADI@Z 100067f0 f i DNAFlexDialog.obj
 0001:00005810       ?default_error_condition@_System_error_category@std@@UBE?AVerror_condition@2@H@Z 10006810 f i DNAFlexDialog.obj
 0001:00005850       ?default_error_condition@error_category@std@@UBE?AVerror_condition@2@H@Z 10006850 f i DNAFlexDialog.obj
 0001:00005870       ?deref@?$QBasicAtomicInteger@H@@QAE_NXZ 10006870 f i DNAFlexDialog.obj
 0001:00005880       ?detach@?$QSharedDataPointer@VAnnotationData@U2@@@@QAEXXZ 10006880 f i DNAFlexDialog.obj
 0001:00005890       ?detach_helper@?$QSharedDataPointer@VAnnotationData@U2@@@@AAEXXZ 10006890 f i DNAFlexDialog.obj
 0001:00005930       ?equivalent@error_category@std@@UBE_NABVerror_code@2@H@Z 10006930 f i DNAFlexDialog.obj
 0001:00005950       ?equivalent@error_category@std@@UBE_NHABVerror_condition@2@@Z 10006950 f i DNAFlexDialog.obj
 0001:00005990       ?erase@?$basic_string@DU?$char_traits@D@std@@V?$allocator@D@2@@std@@QAEAAV12@I@Z 10006990 f i DNAFlexDialog.obj
 0001:000059d0       ?erase@?$basic_string@DU?$char_traits@D@std@@V?$allocator@D@2@@std@@QAEAAV12@II@Z 100069d0 f i DNAFlexDialog.obj
 0001:00005a70       ?generic_category@std@@YAABVerror_category@1@XZ 10006a70 f i DNAFlexDialog.obj
 0001:00005a80       ?isValid@AbstractInt32Id@U2@@UBE_NXZ 10006a80 f i DNAFlexDialog.obj
 0001:00005a90       ?length@?$char_traits@D@std@@SAIPBD@Z 10006a90 f i DNAFlexDialog.obj
 0001:00005ab0       ?load@?$QBasicAtomicInteger@H@@QBEHXZ 10006ab0 f i DNAFlexDialog.obj
 0001:00005ac0       ?max_size@?$_Wrap_alloc@V?$allocator@D@std@@@std@@QBEIXZ 10006ac0 f i DNAFlexDialog.obj
 0001:00005ad0       ?max_size@?$allocator@D@std@@QBEIXZ 10006ad0 f i DNAFlexDialog.obj
 0001:00005ae0       ?max_size@?$allocator_traits@V?$allocator@D@std@@@std@@SAIABV?$allocator@D@2@@Z 10006ae0 f i DNAFlexDialog.obj
 0001:00005af0       ?max_size@?$basic_string@DU?$char_traits@D@std@@V?$allocator@D@2@@std@@QBEIXZ 10006af0 f i DNAFlexDialog.obj
 0001:00005b00       ?message@_Generic_error_category@std@@UBE?AV?$basic_string@DU?$char_traits@D@std@@V?$allocator@D@2@@2@H@Z 10006b00 f i DNAFlexDialog.obj
 0001:00005b80       ?message@_Iostream_error_category@std@@UBE?AV?$basic_string@DU?$char_traits@D@std@@V?$allocator@D@2@@2@H@Z 10006b80 f i DNAFlexDialog.obj
 0001:00005bd0       ?message@_System_error_category@std@@UBE?AV?$basic_string@DU?$char_traits@D@std@@V?$allocator@D@2@@2@H@Z 10006bd0 f i DNAFlexDialog.obj
 0001:00005c50       ?move@?$char_traits@D@std@@SAPADPADPBDI@Z 10006c50 f i DNAFlexDialog.obj
 0001:00005c70       ?name@_Generic_error_category@std@@UBEPBDXZ 10006c70 f i DNAFlexDialog.obj
 0001:00005c80       ?name@_Iostream_error_category@std@@UBEPBDXZ 10006c80 f i DNAFlexDialog.obj
 0001:00005c90       ?name@_System_error_category@std@@UBEPBDXZ 10006c90 f i DNAFlexDialog.obj
 0001:00005ca0       ?qt_noop@@YAXXZ            10006ca0 f i DNAFlexDialog.obj
 0001:00005cb0       ?ref@?$QBasicAtomicInteger@H@@QAE_NXZ 10006cb0 f i DNAFlexDialog.obj
 0001:00005cd0       ?retranslateUi@Ui_DNAFlexDialog@@QAEXPAVQDialog@@@Z 10006cd0 f i DNAFlexDialog.obj
 0001:00005f90       ?setupUi@Ui_DNAFlexDialog@@QAEXPAVQDialog@@@Z 10006f90 f i DNAFlexDialog.obj
 0001:00006b60       ?size@?$basic_string@DU?$char_traits@D@std@@V?$allocator@D@2@@std@@QBEIXZ 10007b60 f i DNAFlexDialog.obj
 0001:00006b70       ?sl_defaultSettings@DNAFlexDialog@U2@@AAEXXZ 10007b70 f   DNAFlexDialog.obj
 0001:00006bb0       ?sl_rememberSettings@DNAFlexDialog@U2@@AAEXXZ 10007bb0 f   DNAFlexDialog.obj
 0001:00006bc0       ?sl_spinThresholdChanged@DNAFlexDialog@U2@@AAEXN@Z 10007bc0 f   DNAFlexDialog.obj
 0001:00006be0       ?sl_spinWindowSizeChanged@DNAFlexDialog@U2@@AAEXH@Z 10007be0 f   DNAFlexDialog.obj
 0001:00006bf0       ?sl_spinWindowStepChanged@DNAFlexDialog@U2@@AAEXH@Z 10007bf0 f   DNAFlexDialog.obj
 0001:00006c00       ?sl_updateSizes@DNAFlexDialog@U2@@AAEXH@Z 10007c00 f   DNAFlexDialog.obj
 0001:00006cc0       ?system_category@std@@YAABVerror_category@1@XZ 10007cc0 f i DNAFlexDialog.obj
 0001:00006cd0       ?tr@DNAFlexDialog@U2@@SA?AVQString@@PBD0H@Z 10007cd0 f i DNAFlexDialog.obj
 0001:00006d00       ?updateHighFlexValues@DNAFlexDialog@U2@@AAEXXZ 10007d00 f   DNAFlexDialog.obj
 0001:00006d40       ?value@error_code@std@@QBEHXZ 10007d40 f i DNAFlexDialog.obj
 0001:00006d50       ?value@error_condition@std@@QBEHXZ 10007d50 f i DNAFlexDialog.obj
 0001:00006d60       _hypot                     10007d60 f i DNAFlexDialog.obj
 0001:00006d90       ??$internalConstruct@UNormalDeleter@QtSharedPointer@@@?$QSharedPointer@VGSequenceGraphData@U2@@@@AAEXPAVGSequenceGraphData@U2@@UNormalDeleter@QtSharedPointer@@@Z 10007d90 f i DNAFlexGraph.obj
 0001:00006df0       ??$qMin@_J@@YAAB_JAB_J0@Z  10007df0 f i DNAFlexGraph.obj
 0001:00006e20       ??$store@HH@?$QGenericAtomicOps@U?$QAtomicOpsBySize@$03@@@@SAXAAHH@Z 10007e20 f i DNAFlexGraph.obj
 0001:00006e30       ??0?$CustomDeleter@VGSequenceGraphData@U2@@UNormalDeleter@QtSharedPointer@@@QtSharedPointer@@QAE@PAVGSequenceGraphData@U2@@UNormalDeleter@1@@Z 10007e30 f i DNAFlexGraph.obj
 0001:00006e40       ??0?$QList@V?$QSharedPointer@VGSequenceGraphData@U2@@@@@@QAE@$$QAV0@@Z 10007e40 f i DNAFlexGraph.obj
 0001:00006e60       ??0?$QList@V?$QSharedPointer@VGSequenceGraphData@U2@@@@@@QAE@XZ 10007e60 f i DNAFlexGraph.obj
 0001:00006e70       ??0?$QMap@VQString@@VQColor@@@@QAE@XZ 10007e70 f i DNAFlexGraph.obj
 0001:00006e80       ??0?$QSharedPointer@VGSequenceGraphData@U2@@@@QAE@ABV0@@Z 10007e80 f i DNAFlexGraph.obj
 0001:00006ec0       ??0?$QSharedPointer@VGSequenceGraphData@U2@@@@QAE@PAVGSequenceGraphData@U2@@@Z 10007ec0 f i DNAFlexGraph.obj
 0001:00006f30       ??0DNAFlexGraphFactory@U2@@QAE@PAVQObject@@@Z 10007f30 f   DNAFlexGraph.obj
 0001:00006fb0       ??0ExternalRefCountData@QtSharedPointer@@QAE@P6AXPAU01@@Z@Z 10007fb0 f i DNAFlexGraph.obj
 0001:00006fd0       ??1?$QList@V?$QSharedPointer@VGSequenceGraphData@U2@@@@@@QAE@XZ 10007fd0 f i DNAFlexGraph.obj
 0001:00007020       ??1?$QMap@VQString@@VQColor@@@@QAE@XZ 10008020 f i DNAFlexGraph.obj
 0001:00007090       ??1?$QSharedPointer@VGSequenceGraphData@U2@@@@QAE@XZ 10008090 f i DNAFlexGraph.obj
 0001:000070d0       ??1DNAFlexGraphFactory@U2@@UAE@XZ 100080d0 f i DNAFlexGraph.obj
 0001:000070e0       ??1ExternalRefCountData@QtSharedPointer@@QAE@XZ 100080e0 f i DNAFlexGraph.obj
 0001:000070f0       ??3ExternalRefCountData@QtSharedPointer@@SAXPAX0@Z 100080f0 f i DNAFlexGraph.obj
 0001:00007100       ??3ExternalRefCountData@QtSharedPointer@@SAXPAX@Z 10008100 f i DNAFlexGraph.obj
 0001:00007110       ??C?$QSharedPointer@VGSequenceGraphData@U2@@@@QBEPAVGSequenceGraphData@U2@@XZ 10008110 f i DNAFlexGraph.obj
 0001:00007120       ??_G?$QSharedPointer@VGSequenceGraphData@U2@@@@QAEPAXI@Z 10008120 f i DNAFlexGraph.obj
 0001:00007170       ??_EDNAFlexGraphFactory@U2@@UAEPAXI@Z 10008170 f i DNAFlexGraph.obj
 0001:00007170       ??_GDNAFlexGraphFactory@U2@@UAEPAXI@Z 10008170 f i DNAFlexGraph.obj
 0001:000071a0       ??_GExternalRefCountData@QtSharedPointer@@QAEPAXI@Z 100081a0 f i DNAFlexGraph.obj
 0001:000071c0       ??_EGSequenceGraphData@U2@@UAEPAXI@Z 100081c0 f i DNAFlexGraph.obj
 0001:000071c0       ??_GGSequenceGraphData@U2@@UAEPAXI@Z 100081c0 f i DNAFlexGraph.obj
 0001:000071f0       ??_GGSequenceGraphDrawer@U2@@UAEPAXI@Z 100081f0 f i DNAFlexGraph.obj
 0001:000071f0       ??_EGSequenceGraphDrawer@U2@@UAEPAXI@Z 100081f0 f i DNAFlexGraph.obj
 0001:00007220       ??_GQString@@QAEPAXI@Z     10008220 f i DNAFlexGraph.obj
 0001:00007250       ?append@?$QList@V?$QSharedPointer@VGSequenceGraphData@U2@@@@@@QAEXABV?$QSharedPointer@VGSequenceGraphData@U2@@@@@Z 10008250 f i DNAFlexGraph.obj
 0001:00007350       ?create@?$ExternalRefCountWithCustomDeleter@VGSequenceGraphData@U2@@UNormalDeleter@QtSharedPointer@@@QtSharedPointer@@SAPAU12@PAVGSequenceGraphData@U2@@UNormalDeleter@2@P6AXPAUExternalRefCountData@2@@Z@Z 10008350 f i DNAFlexGraph.obj
 0001:00007390       ?createGraphs@DNAFlexGraphFactory@U2@@UAE?AV?$QList@V?$QSharedPointer@VGSequenceGraphData@U2@@@@@@PAVGSequenceGraphView@2@@Z 10008390 f   DNAFlexGraph.obj
 0001:000074a0       ?data@?$QSharedPointer@VGSequenceGraphData@U2@@@@QBEPAVGSequenceGraphData@U2@@XZ 100084a0 f i DNAFlexGraph.obj
 0001:000074b0       ?dealloc@?$QList@V?$QSharedPointer@VGSequenceGraphData@U2@@@@@@AAEXPAUData@QListData@@@Z 100084b0 f i DNAFlexGraph.obj
 0001:000074e0       ?deleter@?$ExternalRefCountWithCustomDeleter@VGSequenceGraphData@U2@@UNormalDeleter@QtSharedPointer@@@QtSharedPointer@@SAXPAUExternalRefCountData@2@@Z 100084e0 f i DNAFlexGraph.obj
 0001:00007500       ?deref@?$QSharedPointer@VGSequenceGraphData@U2@@@@AAEXXZ 10008500 f i DNAFlexGraph.obj
 0001:00007540       ?deref@?$QSharedPointer@VGSequenceGraphData@U2@@@@CAXPAUExternalRefCountData@QtSharedPointer@@@Z 10008540 f i DNAFlexGraph.obj
 0001:00007580       ?deref@RefCount@QtPrivate@@QAE_NXZ 10008580 f i DNAFlexGraph.obj
 0001:000075a0       ?destroy@?$QMapData@VQString@@VQColor@@@@QAEXXZ 100085a0 f i DNAFlexGraph.obj
 0001:000075f0       ?destroy@ExternalRefCountData@QtSharedPointer@@QAEXXZ 100085f0 f i DNAFlexGraph.obj
 0001:00007600       ?destroySubTree@?$QMapNode@VQString@@VQColor@@@@QAEXXZ 10008600 f i DNAFlexGraph.obj
 0001:00007630       ?detach_helper_grow@?$QList@V?$QSharedPointer@VGSequenceGraphData@U2@@@@@@AAEPAUNode@1@HH@Z 10008630 f i DNAFlexGraph.obj
 0001:000077a0       ?enableSharedFromThis@?$QSharedPointer@VGSequenceGraphData@U2@@@@AAAXZZ 100087a0 f i DNAFlexGraph.obj
 0001:000077b0       ?execute@?$CustomDeleter@VGSequenceGraphData@U2@@UNormalDeleter@QtSharedPointer@@@QtSharedPointer@@QAEXXZ 100087b0 f i DNAFlexGraph.obj
 0001:000077c0       ?getDrawer@DNAFlexGraphFactory@U2@@UAEPAVGSequenceGraphDrawer@2@PAVGSequenceGraphView@2@@Z 100087c0 f   DNAFlexGraph.obj
 0001:000078a0       ?isEnabled@DNAFlexGraphFactory@U2@@UBE_NPBVU2SequenceObject@2@@Z 100088a0 f   DNAFlexGraph.obj
 0001:00007920       ?isShared@RefCount@QtPrivate@@QBE_NXZ 10008920 f i DNAFlexGraph.obj
 0001:00007940       ?leftNode@?$QMapNode@VQString@@VQColor@@@@QBEPAU1@XZ 10008940 f i DNAFlexGraph.obj
 0001:00007980       ?node_construct@?$QList@V?$QSharedPointer@VGSequenceGraphData@U2@@@@@@AAEXPAUNode@1@ABV?$QSharedPointer@VGSequenceGraphData@U2@@@@@Z 10008980 f i DNAFlexGraph.obj
 0001:000079e0       ?node_copy@?$QList@V?$QSharedPointer@VGSequenceGraphData@U2@@@@@@AAEXPAUNode@1@00@Z 100089e0 f i DNAFlexGraph.obj
 0001:00007ab0       ?node_destruct@?$QList@V?$QSharedPointer@VGSequenceGraphData@U2@@@@@@AAEXPAUNode@1@0@Z 10008ab0 f i DNAFlexGraph.obj
 0001:00007b10       ?node_destruct@?$QList@V?$QSharedPointer@VGSequenceGraphData@U2@@@@@@AAEXPAUNode@1@@Z 10008b10 f i DNAFlexGraph.obj
 0001:00007b60       ?ref@?$QSharedPointer@VGSequenceGraphData@U2@@@@ABEXXZ 10008b60 f i DNAFlexGraph.obj
 0001:00007b80       ?rightNode@?$QMapNode@VQString@@VQColor@@@@QBEPAU1@XZ 10008b80 f i DNAFlexGraph.obj
 0001:00007b90       ?root@?$QMapData@VQString@@VQColor@@@@QBEPAU?$QMapNode@VQString@@VQColor@@@@XZ 10008b90 f i DNAFlexGraph.obj
 0001:00007ba0       ?setQObjectShared@ExternalRefCountData@QtSharedPointer@@QAAXZZ 10008ba0 f i DNAFlexGraph.obj
 0001:00007bb0       ?store@?$QBasicAtomicInteger@H@@QAEXH@Z 10008bb0 f i DNAFlexGraph.obj
 0001:00007bc0       ?tr@DNAFlexGraphFactory@U2@@SA?AVQString@@PBD0H@Z 10008bc0 f i DNAFlexGraph.obj
 0001:00007bf0       ??0?$QFlags@W4AllocationOption@QArrayData@@@@QAE@W4AllocationOption@QArrayData@@@Z 10008bf0 f i DNAFlexGraphAlgorithm.obj
 0001:00007c00       ??0DNAFlexGraphAlgorithm@U2@@QAE@XZ 10008c00 f   DNAFlexGraphAlgorithm.obj
 0001:00007c20       ??1DNAFlexGraphAlgorithm@U2@@UAE@XZ 10008c20 f   DNAFlexGraphAlgorithm.obj
 0001:00007c30       ??_EDNAFlexGraphAlgorithm@U2@@UAEPAXI@Z 10008c30 f i DNAFlexGraphAlgorithm.obj
 0001:00007c30       ??_GDNAFlexGraphAlgorithm@U2@@UAEPAXI@Z 10008c30 f i DNAFlexGraphAlgorithm.obj
 0001:00007c60       ?allocate@?$QTypedArrayData@M@@SAPAU1@IV?$QFlags@W4AllocationOption@QArrayData@@@@@Z 10008c60 f i DNAFlexGraphAlgorithm.obj
 0001:00007c80       ?append@?$QVector@M@@QAEXABM@Z 10008c80 f i DNAFlexGraphAlgorithm.obj
 0001:00007d00       ?begin@?$QTypedArrayData@M@@QAEPAMPAM@Z 10008d00 f i DNAFlexGraphAlgorithm.obj
 0001:00007d10       ?calculate@DNAFlexGraphAlgorithm@U2@@UAEXAAV?$QVector@M@@PAVU2SequenceObject@2@ABVU2Region@2@PBVGSequenceGraphWindowData@2@AAVU2OpStatus@2@@Z 10008d10 f   DNAFlexGraphAlgorithm.obj
 0001:00007fa0       ?data@?$QTypedArrayData@M@@QAEPAMXZ 10008fa0 f i DNAFlexGraphAlgorithm.obj
 0001:00007fb0       ?deallocate@?$QTypedArrayData@M@@SAXPAUQArrayData@@@Z 10008fb0 f i DNAFlexGraphAlgorithm.obj
 0001:00007fd0       ?defaultConstruct@?$QVector@M@@AAEXPAM0@Z 10008fd0 f i DNAFlexGraphAlgorithm.obj
 0001:00007ff0       ?destruct@?$QVector@M@@AAEXPAM0@Z 10008ff0 f i DNAFlexGraphAlgorithm.obj
 0001:00008000       ?end@?$QTypedArrayData@M@@QAEPAMPAM@Z 10009000 f i DNAFlexGraphAlgorithm.obj
 0001:00008020       ?freeData@?$QVector@M@@AAEXPAU?$QTypedArrayData@M@@@Z 10009020 f i DNAFlexGraphAlgorithm.obj
 0001:00008050       ?isDetached@?$QVector@M@@QBE_NXZ 10009050 f i DNAFlexGraphAlgorithm.obj
 0001:00008080       ?reallocData@?$QVector@M@@AAEXHHV?$QFlags@W4AllocationOption@QArrayData@@@@@Z 10009080 f i DNAFlexGraphAlgorithm.obj
 0001:000082c0       ?reserve@?$QVector@M@@QAEXH@Z 100092c0 f i DNAFlexGraphAlgorithm.obj
 0001:00008310       ?sharedNull@?$QTypedArrayData@M@@SAPAU1@XZ 10009310 f i DNAFlexGraphAlgorithm.obj
 0001:00008320       ?tr@DNAFlexPlugin@U2@@SA?AVQString@@PBD0H@Z 10009320 f i DNAFlexGraphAlgorithm.obj
 0001:00008350       ??$?0VDNAFlexDialog@U2@@@?$QWeakPointer@VQObject@@@@AAE@PAVDNAFlexDialog@U2@@_N@Z 10009350 f i DNAFlexPlugin.obj
 0001:00008390       ??$qobject_cast@PAVADVSingleSequenceWidget@U2@@@@YAPAVADVSingleSequenceWidget@U2@@PAVQObject@@@Z 10009390 f i DNAFlexPlugin.obj
 0001:000083b0       ??$qobject_cast@PAVAnnotatedDNAView@U2@@@@YAPAVAnnotatedDNAView@U2@@PAVQObject@@@Z 100093b0 f i DNAFlexPlugin.obj
 0001:000083d0       ??$qobject_cast@PAVGObjectViewAction@U2@@@@YAPAVGObjectViewAction@U2@@PAVQObject@@@Z 100093d0 f i DNAFlexPlugin.obj
 0001:000083f0       ??0?$QFlags@W4ADVGlobalActionFlag@U2@@@@QAE@W4ADVGlobalActionFlag@U2@@@Z 100093f0 f i DNAFlexPlugin.obj
 0001:00008400       ??0?$QForeachContainer@$$CBV?$QList@PAVADVSequenceWidget@U2@@@@@@QAE@ABV?$QList@PAVADVSequenceWidget@U2@@@@@Z 10009400 f i DNAFlexPlugin.obj
 0001:00008440       ??0?$QList@PAVADVSequenceWidget@U2@@@@QAE@ABV0@@Z 10009440 f i DNAFlexPlugin.obj
 0001:00008500       ??0?$QObjectScopedPointer@VDNAFlexDialog@U2@@@U2@@QAE@PAVDNAFlexDialog@1@@Z 10009500 f i DNAFlexPlugin.obj
 0001:00008540       ??0?$QPointer@VDNAFlexDialog@U2@@@@QAE@PAVDNAFlexDialog@U2@@@Z 10009540 f i DNAFlexPlugin.obj
 0001:00008580       ??0DNAFlexPlugin@U2@@QAE@XZ 10009580 f   DNAFlexPlugin.obj
 0001:00008670       ??0DNAFlexViewContext@U2@@QAE@PAVQObject@@@Z 10009670 f   DNAFlexPlugin.obj
 0001:00008730       ??0GObjectViewFactoryId@U2@@QAE@PBD@Z 10009730 f i DNAFlexPlugin.obj
 0001:00008770       ??0QLatin1Char@@QAE@D@Z    10009770 f i DNAFlexPlugin.obj
 0001:00008780       ??0const_iterator@?$QList@PAVADVSequenceWidget@U2@@@@QAE@PAUNode@1@@Z 10009780 f i DNAFlexPlugin.obj
 0001:00008790       ??1?$QForeachContainer@$$CBV?$QList@PAVADVSequenceWidget@U2@@@@@@QAE@XZ 10009790 f i DNAFlexPlugin.obj
 0001:000087c0       ??1?$QList@PAVADVSequenceWidget@U2@@@@QAE@XZ 100097c0 f i DNAFlexPlugin.obj
 0001:000087f0       ??1?$QObjectScopedPointer@VDNAFlexDialog@U2@@@U2@@QAE@XZ 100097f0 f i DNAFlexPlugin.obj
 0001:00008870       ??1?$QPointer@VDNAFlexDialog@U2@@@@QAE@XZ 10009870 f i DNAFlexPlugin.obj
 0001:00008890       ??1?$QWeakPointer@VQObject@@@@QAE@XZ 10009890 f i DNAFlexPlugin.obj
 0001:000088b0       ??1DNAFlexPlugin@U2@@UAE@XZ 100098b0 f i DNAFlexPlugin.obj
 0001:000088c0       ??1DNAFlexViewContext@U2@@UAE@XZ 100098c0 f i DNAFlexPlugin.obj
 0001:000088d0       ??1GObjectViewFactoryId@U2@@QAE@XZ 100098d0 f i DNAFlexPlugin.obj
 0001:000088e0       ??9@YA_NABVQString@@0@Z    100098e0 f i DNAFlexPlugin.obj
 0001:00008900       ??9const_iterator@?$QList@PAVADVSequenceWidget@U2@@@@QBE_NABV01@@Z 10009900 f i DNAFlexPlugin.obj
 0001:00008920       ??C?$QObjectScopedPointer@VDNAFlexDialog@U2@@@U2@@QBEPAVDNAFlexDialog@1@XZ 10009920 f i DNAFlexPlugin.obj
 0001:00008940       ??C?$QPointer@VDNAFlexDialog@U2@@@@QBEPAVDNAFlexDialog@U2@@XZ 10009940 f i DNAFlexPlugin.obj
 0001:00008960       ??Dconst_iterator@?$QList@PAVADVSequenceWidget@U2@@@@QBEABQAVADVSequenceWidget@U2@@XZ 10009960 f i DNAFlexPlugin.obj
 0001:00008970       ??Econst_iterator@?$QList@PAVADVSequenceWidget@U2@@@@QAEAAV01@XZ 10009970 f i DNAFlexPlugin.obj
 0001:00008976       ??_EDNAFlexViewContext@U2@@W7AEPAXI@Z 10009976 f i DNAFlexPlugin.obj
 0001:00008980       ??_EADVGlobalAction@U2@@UAEPAXI@Z 10009980 f i DNAFlexPlugin.obj
 0001:00008980       ??_GADVGlobalAction@U2@@UAEPAXI@Z 10009980 f i DNAFlexPlugin.obj
 0001:000089b0       ??_EDNAFlexPlugin@U2@@UAEPAXI@Z 100099b0 f i DNAFlexPlugin.obj
 0001:000089b0       ??_GDNAFlexPlugin@U2@@UAEPAXI@Z 100099b0 f i DNAFlexPlugin.obj
 0001:000089e0       ??_GDNAFlexViewContext@U2@@UAEPAXI@Z 100099e0 f i DNAFlexPlugin.obj
 0001:000089e0       ??_EDNAFlexViewContext@U2@@UAEPAXI@Z 100099e0 f i DNAFlexPlugin.obj
 0001:00008a10       ??_EGraphAction@U2@@UAEPAXI@Z 10009a10 f i DNAFlexPlugin.obj
 0001:00008a10       ??_GGraphAction@U2@@UAEPAXI@Z 10009a10 f i DNAFlexPlugin.obj
 0001:00008a40       ?begin@?$QList@PAVADVSequenceWidget@U2@@@@QBE?AVconst_iterator@1@XZ 10009a40 f i DNAFlexPlugin.obj
 0001:00008a60       ?data@?$QPointer@VDNAFlexDialog@U2@@@@QBEPAVDNAFlexDialog@U2@@XZ 10009a60 f i DNAFlexPlugin.obj
 0001:00008a80       ?data@?$QWeakPointer@VQObject@@@@QBEPAVQObject@@XZ 10009a80 f i DNAFlexPlugin.obj
 0001:00008aa0       ?dealloc@?$QList@PAVADVSequenceWidget@U2@@@@AAEXPAUData@QListData@@@Z 10009aa0 f i DNAFlexPlugin.obj
 0001:00008ac0       ?end@?$QList@PAVADVSequenceWidget@U2@@@@QBE?AVconst_iterator@1@XZ 10009ac0 f i DNAFlexPlugin.obj
 0001:00008ae0       ?initViewContext@DNAFlexViewContext@U2@@EAEXPAVGObjectView@2@@Z 10009ae0 f   DNAFlexPlugin.obj
 0001:00008d30       ?isNull@?$QObjectScopedPointer@VDNAFlexDialog@U2@@@U2@@QBE_NXZ 10009d30 f i DNAFlexPlugin.obj
 0001:00008d50       ?isNull@?$QPointer@VDNAFlexDialog@U2@@@@QBE_NXZ 10009d50 f i DNAFlexPlugin.obj
 0001:00008d70       ?isNull@?$QWeakPointer@VQObject@@@@QBE_NXZ 10009d70 f i DNAFlexPlugin.obj
 0001:00008d90       ?node_copy@?$QList@PAVADVSequenceWidget@U2@@@@AAEXPAUNode@1@00@Z 10009d90 f i DNAFlexPlugin.obj
 0001:00008dc0       ?node_destruct@?$QList@PAVADVSequenceWidget@U2@@@@AAEXPAUNode@1@0@Z 10009dc0 f i DNAFlexPlugin.obj
 0001:00008dd0       ?ref@RefCount@QtPrivate@@QAE_NXZ 10009dd0 f i DNAFlexPlugin.obj
 0001:00008df0       ?sl_sequenceWidgetAdded@DNAFlexViewContext@U2@@AAEXPAVADVSequenceWidget@2@@Z 10009df0 f   DNAFlexPlugin.obj
 0001:00008f20       ?sl_showDNAFlexDialog@DNAFlexViewContext@U2@@AAEXXZ 10009f20 f   DNAFlexPlugin.obj
 0001:000092d0       ?t@Node@?$QList@PAVADVSequenceWidget@U2@@@@QAEAAPAVADVSequenceWidget@U2@@XZ 1000a2d0 f i DNAFlexPlugin.obj
 0001:000092e0       ?tr@DNAFlexViewContext@U2@@SA?AVQString@@PBD0H@Z 1000a2e0 f i DNAFlexPlugin.obj
 0001:00009310       _ugene_plugin_init         1000a310 f   DNAFlexPlugin.obj
 0001:00009330       ??$?0VAnnotationTableObject@U2@@@?$QWeakPointer@VQObject@@@@AAE@PAVAnnotationTableObject@U2@@_N@Z 1000a330 f i DNAFlexTask.obj
 0001:00009370       ??$qobject_cast@PAVFindHighFlexRegions@U2@@@@YAPAVFindHighFlexRegions@U2@@PAVQObject@@@Z 1000a370 f i DNAFlexTask.obj
 0001:00009390       ??0?$QFlags@W4TaskFlag@U2@@@@QAE@VQFlag@@@Z 1000a390 f i DNAFlexTask.obj
 0001:000093a0       ??0?$QFlags@W4TaskFlag@U2@@@@QAE@W4TaskFlag@U2@@@Z 1000a3a0 f i DNAFlexTask.obj
 0001:000093b0       ??0?$QForeachContainer@$$CBV?$QList@VHighFlexResult@U2@@@@@@QAE@ABV?$QList@VHighFlexResult@U2@@@@@Z 1000a3b0 f i DNAFlexTask.obj
 0001:000093f0       ??0?$QList@PAVTask@U2@@@@QAE@$$QAV0@@Z 1000a3f0 f i DNAFlexTask.obj
 0001:00009410       ??0?$QList@PAVTask@U2@@@@QAE@XZ 1000a410 f i DNAFlexTask.obj
 0001:00009420       ??0?$QList@V?$QSharedDataPointer@VAnnotationData@U2@@@@@@QAE@$$QAV0@@Z 1000a420 f i DNAFlexTask.obj
 0001:00009440       ??0?$QList@V?$QSharedDataPointer@VAnnotationData@U2@@@@@@QAE@XZ 1000a440 f i DNAFlexTask.obj
 0001:00009450       ??0?$QList@VHighFlexResult@U2@@@@QAE@ABV0@@Z 1000a450 f i DNAFlexTask.obj
 0001:00009510       ??0?$QPointer@VAnnotationTableObject@U2@@@@QAE@PAVAnnotationTableObject@U2@@@Z 1000a510 f i DNAFlexTask.obj
 0001:00009550       ??0?$QSharedDataPointer@VAnnotationData@U2@@@@QAE@ABV0@@Z 1000a550 f i DNAFlexTask.obj
 0001:00009570       ??0?$QSharedDataPointer@VAnnotationData@U2@@@@QAE@PAVAnnotationData@U2@@@Z 1000a570 f i DNAFlexTask.obj
 0001:00009590       ??0DNAFlexTask@U2@@QAE@ABVHighFlexSettings@1@PAVAnnotationTableObject@1@ABVQString@@22ABVDNASequence@1@@Z 1000a590 f   DNAFlexTask.obj
 0001:000096d0       ??0const_iterator@?$QList@VHighFlexResult@U2@@@@QAE@PAUNode@1@@Z 1000a6d0 f i DNAFlexTask.obj
 0001:000096e0       ??1?$QForeachContainer@$$CBV?$QList@VHighFlexResult@U2@@@@@@QAE@XZ 1000a6e0 f i DNAFlexTask.obj
 0001:000096f0       ??1?$QList@PAVTask@U2@@@@QAE@XZ 1000a6f0 f i DNAFlexTask.obj
 0001:00009720       ??1?$QList@V?$QSharedDataPointer@VAnnotationData@U2@@@@@@QAE@XZ 1000a720 f i DNAFlexTask.obj
 0001:00009770       ??1?$QList@VHighFlexResult@U2@@@@QAE@XZ 1000a770 f i DNAFlexTask.obj
 0001:000097d0       ??1?$QPointer@VAnnotationTableObject@U2@@@@QAE@XZ 1000a7d0 f i DNAFlexTask.obj
 0001:000097f0       ??1?$QSharedDataPointer@VAnnotationData@U2@@@@QAE@XZ 1000a7f0 f i DNAFlexTask.obj
 0001:00009820       ??1DNAFlexTask@U2@@UAE@XZ  1000a820 f i DNAFlexTask.obj
 0001:000098e0       ??6?$QVector@VU2Region@U2@@@@QAEAAV0@ABVU2Region@U2@@@Z 1000a8e0 f i DNAFlexTask.obj
 0001:00009900       ??9const_iterator@?$QList@VHighFlexResult@U2@@@@QBE_NABV01@@Z 1000a900 f i DNAFlexTask.obj
 0001:00009920       ??B?$QPointer@VAnnotationTableObject@U2@@@@QBEPAVAnnotationTableObject@U2@@XZ 1000a920 f i DNAFlexTask.obj
 0001:00009940       ??Dconst_iterator@?$QList@VHighFlexResult@U2@@@@QBEABVHighFlexResult@U2@@XZ 1000a940 f i DNAFlexTask.obj
 0001:00009950       ??Econst_iterator@?$QList@VHighFlexResult@U2@@@@QAEAAV01@XZ 1000a950 f i DNAFlexTask.obj
 0001:00009960       ??U?$QFlags@W4TaskFlag@U2@@@@QBE?AV0@W4TaskFlag@U2@@@Z 1000a960 f i DNAFlexTask.obj
 0001:00009980       ??_G?$QSharedDataPointer@VAnnotationData@U2@@@@QAEPAXI@Z 1000a980 f i DNAFlexTask.obj
 0001:000099d0       ??_ECreateAnnotationsTask@U2@@UAEPAXI@Z 1000a9d0 f i DNAFlexTask.obj
 0001:000099d0       ??_GCreateAnnotationsTask@U2@@UAEPAXI@Z 1000a9d0 f i DNAFlexTask.obj
 0001:00009a00       ??_EDNAFlexTask@U2@@UAEPAXI@Z 1000aa00 f i DNAFlexTask.obj
 0001:00009a00       ??_GDNAFlexTask@U2@@UAEPAXI@Z 1000aa00 f i DNAFlexTask.obj
 0001:00009a30       ??_GU2Qualifier@U2@@QAEPAXI@Z 1000aa30 f i DNAFlexTask.obj
 0001:00009a60       ?allocate@?$QTypedArrayData@VU2Qualifier@U2@@@@SAPAU1@IV?$QFlags@W4AllocationOption@QArrayData@@@@@Z 1000aa60 f i DNAFlexTask.obj
 0001:00009a80       ?allocate@?$QTypedArrayData@VU2Region@U2@@@@SAPAU1@IV?$QFlags@W4AllocationOption@QArrayData@@@@@Z 1000aa80 f i DNAFlexTask.obj
 0001:00009aa0       ?append@?$QList@PAVTask@U2@@@@QAEXABQAVTask@U2@@@Z 1000aaa0 f i DNAFlexTask.obj
 0001:00009b30       ?append@?$QList@V?$QSharedDataPointer@VAnnotationData@U2@@@@@@QAEXABV?$QSharedDataPointer@VAnnotationData@U2@@@@@Z 1000ab30 f i DNAFlexTask.obj
 0001:00009c00       ?append@?$QVector@VU2Qualifier@U2@@@@QAEXABVU2Qualifier@U2@@@Z 1000ac00 f i DNAFlexTask.obj
 0001:00009cd0       ?append@?$QVector@VU2Region@U2@@@@QAEXABVU2Region@U2@@@Z 1000acd0 f i DNAFlexTask.obj
 0001:00009d50       ?begin@?$QList@VHighFlexResult@U2@@@@QBE?AVconst_iterator@1@XZ 1000ad50 f i DNAFlexTask.obj
 0001:00009d70       ?begin@?$QTypedArrayData@VU2Qualifier@U2@@@@QAEPAVU2Qualifier@U2@@PAV23@@Z 1000ad70 f i DNAFlexTask.obj
 0001:00009d80       ?begin@?$QTypedArrayData@VU2Region@U2@@@@QAEPAVU2Region@U2@@PAV23@@Z 1000ad80 f i DNAFlexTask.obj
 0001:00009d90       ?data@?$QPointer@VAnnotationTableObject@U2@@@@QBEPAVAnnotationTableObject@U2@@XZ 1000ad90 f i DNAFlexTask.obj
 0001:00009db0       ?data@?$QTypedArrayData@VU2Qualifier@U2@@@@QAEPAVU2Qualifier@U2@@XZ 1000adb0 f i DNAFlexTask.obj
 0001:00009dc0       ?data@?$QTypedArrayData@VU2Region@U2@@@@QAEPAVU2Region@U2@@XZ 1000adc0 f i DNAFlexTask.obj
 0001:00009dd0       ?dealloc@?$QList@PAVTask@U2@@@@AAEXPAUData@QListData@@@Z 1000add0 f i DNAFlexTask.obj
 0001:00009df0       ?dealloc@?$QList@V?$QSharedDataPointer@VAnnotationData@U2@@@@@@AAEXPAUData@QListData@@@Z 1000adf0 f i DNAFlexTask.obj
 0001:00009e20       ?dealloc@?$QList@VHighFlexResult@U2@@@@AAEXPAUData@QListData@@@Z 1000ae20 f i DNAFlexTask.obj
 0001:00009e70       ?deallocate@?$QTypedArrayData@VU2Qualifier@U2@@@@SAXPAUQArrayData@@@Z 1000ae70 f i DNAFlexTask.obj
 0001:00009e90       ?deallocate@?$QTypedArrayData@VU2Region@U2@@@@SAXPAUQArrayData@@@Z 1000ae90 f i DNAFlexTask.obj
 0001:00009eb0       ?defaultConstruct@?$QVector@VU2Qualifier@U2@@@@AAEXPAVU2Qualifier@U2@@0@Z 1000aeb0 f i DNAFlexTask.obj
 0001:00009f20       ?defaultConstruct@?$QVector@VU2Region@U2@@@@AAEXPAVU2Region@U2@@0@Z 1000af20 f i DNAFlexTask.obj
 0001:00009f40       ?destruct@?$QVector@VU2Qualifier@U2@@@@AAEXPAVU2Qualifier@U2@@0@Z 1000af40 f i DNAFlexTask.obj
 0001:00009f70       ?destruct@?$QVector@VU2Region@U2@@@@AAEXPAVU2Region@U2@@0@Z 1000af70 f i DNAFlexTask.obj
 0001:00009f80       ?detach_helper_grow@?$QList@PAVTask@U2@@@@AAEPAUNode@1@HH@Z 1000af80 f i DNAFlexTask.obj
 0001:0000a090       ?detach_helper_grow@?$QList@V?$QSharedDataPointer@VAnnotationData@U2@@@@@@AAEPAUNode@1@HH@Z 1000b090 f i DNAFlexTask.obj
 0001:0000a200       ?end@?$QList@VHighFlexResult@U2@@@@QBE?AVconst_iterator@1@XZ 1000b200 f i DNAFlexTask.obj
 0001:0000a220       ?end@?$QTypedArrayData@VU2Qualifier@U2@@@@QAEPAVU2Qualifier@U2@@PAV23@@Z 1000b220 f i DNAFlexTask.obj
 0001:0000a240       ?end@?$QTypedArrayData@VU2Region@U2@@@@QAEPAVU2Region@U2@@PAV23@@Z 1000b240 f i DNAFlexTask.obj
 0001:0000a260       ?freeData@?$QVector@VU2Qualifier@U2@@@@AAEXPAU?$QTypedArrayData@VU2Qualifier@U2@@@@@Z 1000b260 f i DNAFlexTask.obj
 0001:0000a2b0       ?freeData@?$QVector@VU2Region@U2@@@@AAEXPAU?$QTypedArrayData@VU2Region@U2@@@@@Z 1000b2b0 f i DNAFlexTask.obj
 0001:0000a2e0       ?getAnnotationsFromResults@DNAFlexTask@U2@@QAE?AV?$QList@V?$QSharedDataPointer@VAnnotationData@U2@@@@@@ABV?$QList@VHighFlexResult@U2@@@@@Z 1000b2e0 f   DNAFlexTask.obj
 0001:0000a8a0       ?isDetached@?$QVector@VU2Qualifier@U2@@@@QBE_NXZ 1000b8a0 f i DNAFlexTask.obj
 0001:0000a8d0       ?isDetached@?$QVector@VU2Region@U2@@@@QBE_NXZ 1000b8d0 f i DNAFlexTask.obj
 0001:0000a900       ?isEmpty@?$QList@V?$QSharedDataPointer@VAnnotationData@U2@@@@@@QBE_NXZ 1000b900 f i DNAFlexTask.obj
 0001:0000a910       ?isNull@?$QPointer@VAnnotationTableObject@U2@@@@QBE_NXZ 1000b910 f i DNAFlexTask.obj
 0001:0000a930       ?node_construct@?$QList@PAVTask@U2@@@@AAEXPAUNode@1@ABQAVTask@U2@@@Z 1000b930 f i DNAFlexTask.obj
 0001:0000a950       ?node_construct@?$QList@V?$QSharedDataPointer@VAnnotationData@U2@@@@@@AAEXPAUNode@1@ABV?$QSharedDataPointer@VAnnotationData@U2@@@@@Z 1000b950 f i DNAFlexTask.obj
 0001:0000a980       ?node_copy@?$QList@PAVTask@U2@@@@AAEXPAUNode@1@00@Z 1000b980 f i DNAFlexTask.obj
 0001:0000a9b0       ?node_copy@?$QList@V?$QSharedDataPointer@VAnnotationData@U2@@@@@@AAEXPAUNode@1@00@Z 1000b9b0 f i DNAFlexTask.obj
 0001:0000a9f0       ?node_copy@?$QList@VHighFlexResult@U2@@@@AAEXPAUNode@1@00@Z 1000b9f0 f i DNAFlexTask.obj
 0001:0000aab0       ?node_destruct@?$QList@PAVTask@U2@@@@AAEXPAUNode@1@0@Z 1000bab0 f i DNAFlexTask.obj
 0001:0000aac0       ?node_destruct@?$QList@PAVTask@U2@@@@AAEXPAUNode@1@@Z 1000bac0 f i DNAFlexTask.obj
 0001:0000aad0       ?node_destruct@?$QList@V?$QSharedDataPointer@VAnnotationData@U2@@@@@@AAEXPAUNode@1@0@Z 1000bad0 f i DNAFlexTask.obj
 0001:0000ab20       ?node_destruct@?$QList@V?$QSharedDataPointer@VAnnotationData@U2@@@@@@AAEXPAUNode@1@@Z 1000bb20 f i DNAFlexTask.obj
 0001:0000ab60       ?node_destruct@?$QList@VHighFlexResult@U2@@@@AAEXPAUNode@1@0@Z 1000bb60 f i DNAFlexTask.obj
 0001:0000ab90       ?onSubTaskFinished@DNAFlexTask@U2@@UAE?AV?$QList@PAVTask@U2@@@@PAVTask@2@@Z 1000bb90 f   DNAFlexTask.obj
 0001:0000aee0       ?reallocData@?$QVector@VU2Qualifier@U2@@@@AAEXHHV?$QFlags@W4AllocationOption@QArrayData@@@@@Z 1000bee0 f i DNAFlexTask.obj
 0001:0000b110       ?reallocData@?$QVector@VU2Region@U2@@@@AAEXHHV?$QFlags@W4AllocationOption@QArrayData@@@@@Z 1000c110 f i DNAFlexTask.obj
 0001:0000b350       ?sharedNull@?$QTypedArrayData@VU2Qualifier@U2@@@@SAPAU1@XZ 1000c350 f i DNAFlexTask.obj
 0001:0000b360       ?sharedNull@?$QTypedArrayData@VU2Region@U2@@@@SAPAU1@XZ 1000c360 f i DNAFlexTask.obj
 0001:0000b370       ?t@Node@?$QList@VHighFlexResult@U2@@@@QAEAAVHighFlexResult@U2@@XZ 1000c370 f i DNAFlexTask.obj
 0001:0000b380       ?tr@DNAFlexTask@U2@@SA?AVQString@@PBD0H@Z 1000c380 f i DNAFlexTask.obj
 0001:0000b3b0       ??0?$QList@VHighFlexResult@U2@@@@QAE@XZ 1000c3b0 f i FindHighFlexRegions.obj
 0001:0000b3c0       ??0FindHighFlexRegions@U2@@QAE@ABVDNASequence@1@ABVHighFlexSettings@1@@Z 1000c3c0 f   FindHighFlexRegions.obj
 0001:0000b480       ??0FindHighFlexRegionsListener@U2@@QAE@XZ 1000c480 f i FindHighFlexRegions.obj
 0001:0000b490       ??1FindHighFlexRegions@U2@@UAE@XZ 1000c490 f i FindHighFlexRegions.obj
 0001:0000b510       ??1FindHighFlexRegionsListener@U2@@UAE@XZ 1000c510 f i FindHighFlexRegions.obj
 0001:0000b517       ??_EFindHighFlexRegions@U2@@WJA@AEPAXI@Z 1000c517 f i FindHighFlexRegions.obj
 0001:0000b530       ??_EFindHighFlexRegions@U2@@UAEPAXI@Z 1000c530 f i FindHighFlexRegions.obj
 0001:0000b530       ??_GFindHighFlexRegions@U2@@UAEPAXI@Z 1000c530 f i FindHighFlexRegions.obj
 0001:0000b5c0       ??_GFindHighFlexRegionsListener@U2@@UAEPAXI@Z 1000c5c0 f i FindHighFlexRegions.obj
 0001:0000b5c0       ??_EFindHighFlexRegionsListener@U2@@UAEPAXI@Z 1000c5c0 f i FindHighFlexRegions.obj
 0001:0000b5f0       ?append@?$QList@VHighFlexResult@U2@@@@QAEXABVHighFlexResult@U2@@@Z 1000c5f0 f i FindHighFlexRegions.obj
 0001:0000b6b0       ?detach_helper_grow@?$QList@VHighFlexResult@U2@@@@AAEPAUNode@1@HH@Z 1000c6b0 f i FindHighFlexRegions.obj
 0001:0000b830       ?getResults@FindHighFlexRegions@U2@@QBE?AV?$QList@VHighFlexResult@U2@@@@XZ 1000c830 f   FindHighFlexRegions.obj
 0001:0000b860       ?node_construct@?$QList@VHighFlexResult@U2@@@@AAEXPAUNode@1@ABVHighFlexResult@U2@@@Z 1000c860 f i FindHighFlexRegions.obj
 0001:0000b8b0       ?node_destruct@?$QList@VHighFlexResult@U2@@@@AAEXPAUNode@1@@Z 1000c8b0 f i FindHighFlexRegions.obj
 0001:0000b8d0       ?onResult@FindHighFlexRegions@U2@@UAEXABVHighFlexResult@2@@Z 1000c8d0 f   FindHighFlexRegions.obj
 0001:0000b8e0       ?run@FindHighFlexRegions@U2@@UAEXXZ 1000c8e0 f   FindHighFlexRegions.obj
 0001:0000b930       ?tr@FindHighFlexRegions@U2@@SA?AVQString@@PBD0H@Z 1000c930 f i FindHighFlexRegions.obj
 0001:0000b960       ??0HighFlexResult@U2@@QAE@ABVU2Region@1@NHN@Z 1000c960 f i FindHighFlexRegionsAlgorithm.obj
 0001:0000b990       ?addToResults@FindHighFlexRegionsAlgorithm@U2@@CAXPAVFindHighFlexRegionsListener@2@ABVHighFlexResult@2@@Z 1000c990 f   FindHighFlexRegionsAlgorithm.obj
 0001:0000bb00       ?find@FindHighFlexRegionsAlgorithm@U2@@SAXPAVFindHighFlexRegionsListener@2@ABVHighFlexSettings@2@VQByteArray@@HAAH3@Z 1000cb00 f   FindHighFlexRegionsAlgorithm.obj
 0001:0000bf00       ?flexibilityAngle@FindHighFlexRegionsAlgorithm@U2@@SANDD@Z 1000cf00 f   FindHighFlexRegionsAlgorithm.obj
 0001:0000c1d0       ??0HighFlexSettings@U2@@QAE@XZ 1000d1d0 f   HighFlexSettings.obj
 0001:0000c220       ??H@YA?BVQString@@ABV0@0@Z 1000d220 f i HighFlexSettings.obj
 0001:0000c290       ??H@YA?BVQString@@ABV0@PBD@Z 1000d290 f i HighFlexSettings.obj
 0001:0000c330       ?rememberSettings@HighFlexSettings@U2@@QAEXXZ 1000d330 f   HighFlexSettings.obj
 0001:0000c500       ?restoreDefaults@HighFlexSettings@U2@@QAEXXZ 1000d500 f   HighFlexSettings.obj
 0001:0000c670       ?restoreRememberedSettings@HighFlexSettings@U2@@AAE_NXZ 1000d670 f   HighFlexSettings.obj
 0001:0000c950       ??C?$QScopedPointer@VQObjectData@@U?$QScopedPointerDeleter@VQObjectData@@@@@@QBEPAVQObjectData@@XZ 1000d950 f i moc_DNAFlexDialog.obj
 0001:0000c960       ?metaObject@DNAFlexDialog@U2@@UBEPBUQMetaObject@@XZ 1000d960 f   moc_DNAFlexDialog.obj
 0001:0000c980       ?qt_metacall@DNAFlexDialog@U2@@UAEHW4Call@QMetaObject@@HPAPAX@Z 1000d980 f   moc_DNAFlexDialog.obj
 0001:0000c9f0       ?qt_metacast@DNAFlexDialog@U2@@UAEPAXPBD@Z 1000d9f0 f   moc_DNAFlexDialog.obj
 0001:0000ca90       ?qt_static_metacall@DNAFlexDialog@U2@@CAXPAVQObject@@W4Call@QMetaObject@@HPAPAX@Z 1000da90 f   moc_DNAFlexDialog.obj
 0001:0000cb30       ?metaObject@DNAFlexGraphFactory@U2@@UBEPBUQMetaObject@@XZ 1000db30 f   moc_DNAFlexGraph.obj
 0001:0000cb50       ?qt_metacall@DNAFlexGraphFactory@U2@@UAEHW4Call@QMetaObject@@HPAPAX@Z 1000db50 f   moc_DNAFlexGraph.obj
 0001:0000cb60       ?qt_metacast@DNAFlexGraphFactory@U2@@UAEPAXPBD@Z 1000db60 f   moc_DNAFlexGraph.obj
 0001:0000cbc0       ?qt_static_metacall@DNAFlexGraphFactory@U2@@CAXPAVQObject@@W4Call@QMetaObject@@HPAPAX@Z 1000dbc0 f   moc_DNAFlexGraph.obj
 0001:0000cbd0       ??$acquireMemoryFence@H@?$QGenericAtomicOps@U?$QAtomicOpsBySize@$03@@@@SAXABH@Z 1000dbd0 f i moc_DNAFlexPlugin.obj
 0001:0000cbe0       ??$loadAcquire@H@?$QGenericAtomicOps@U?$QAtomicOpsBySize@$03@@@@SAHABH@Z 1000dbe0 f i moc_DNAFlexPlugin.obj
 0001:0000cbf0       ??$orderedMemoryFence@H@?$QGenericAtomicOps@U?$QAtomicOpsBySize@$03@@@@SAXABH@Z 1000dbf0 f i moc_DNAFlexPlugin.obj
 0001:0000cc00       ??$qMetaTypeId@PAVADVSequenceWidget@U2@@@@YAHXZ 1000dc00 f i moc_DNAFlexPlugin.obj
 0001:0000cc10       ??$qRegisterMetaType@PAVADVSequenceWidget@U2@@@@YAHXZ 1000dc10 f i moc_DNAFlexPlugin.obj
 0001:0000cc20       ??$qRegisterNormalizedMetaType@PAVADVSequenceWidget@U2@@@@YAHABVQByteArray@@PAPAVADVSequenceWidget@U2@@W4DefinedType@?$MetaTypeDefinedHelper@PAVADVSequenceWidget@U2@@$00@QtPrivate@@@Z 1000dc20 f i moc_DNAFlexPlugin.obj
 0001:0000cc80       ??$releaseMemoryFence@H@?$QGenericAtomicOps@U?$QAtomicOpsBySize@$03@@@@SAXABH@Z 1000dc80 f i moc_DNAFlexPlugin.obj
 0001:0000cc90       ??$storeRelease@HH@?$QGenericAtomicOps@U?$QAtomicOpsBySize@$03@@@@SAXAAHH@Z 1000dc90 f i moc_DNAFlexPlugin.obj
 0001:0000cca0       ??0?$QFlags@W4TypeFlag@QMetaType@@@@QAE@VQFlag@@@Z 1000dca0 f i moc_DNAFlexPlugin.obj
 0001:0000ccb0       ??_5?$QFlags@W4TypeFlag@QMetaType@@@@QAEAAV0@W4TypeFlag@QMetaType@@@Z 1000dcb0 f i moc_DNAFlexPlugin.obj
 0001:0000ccc0       ?Construct@?$QMetaTypeFunctionHelper@PAVADVSequenceWidget@U2@@$00@QtMetaTypePrivate@@SAPAXPAXPBX@Z 1000dcc0 f i moc_DNAFlexPlugin.obj
 0001:0000ccf0       ?Create@?$QMetaTypeFunctionHelper@PAVADVSequenceWidget@U2@@$00@QtMetaTypePrivate@@SAPAXPBX@Z 1000dcf0 f i moc_DNAFlexPlugin.obj
 0001:0000cd30       ?Delete@?$QMetaTypeFunctionHelper@PAVADVSequenceWidget@U2@@$00@QtMetaTypePrivate@@SAXPAX@Z 1000dd30 f i moc_DNAFlexPlugin.obj
 0001:0000cd40       ?Destruct@?$QMetaTypeFunctionHelper@PAVADVSequenceWidget@U2@@$00@QtMetaTypePrivate@@SAXPAX@Z 1000dd40 f i moc_DNAFlexPlugin.obj
 0001:0000cd50       ?loadAcquire@?$QBasicAtomicInteger@H@@QBEHXZ 1000dd50 f i moc_DNAFlexPlugin.obj
 0001:0000cd60       ?metaObject@DNAFlexPlugin@U2@@UBEPBUQMetaObject@@XZ 1000dd60 f   moc_DNAFlexPlugin.obj
 0001:0000cd80       ?metaObject@DNAFlexViewContext@U2@@UBEPBUQMetaObject@@XZ 1000dd80 f   moc_DNAFlexPlugin.obj
 0001:0000cda0       ?qt_metacall@DNAFlexPlugin@U2@@UAEHW4Call@QMetaObject@@HPAPAX@Z 1000dda0 f   moc_DNAFlexPlugin.obj
 0001:0000cdb0       ?qt_metacall@DNAFlexViewContext@U2@@UAEHW4Call@QMetaObject@@HPAPAX@Z 1000ddb0 f   moc_DNAFlexPlugin.obj
 0001:0000ce10       ?qt_metacast@DNAFlexPlugin@U2@@UAEPAXPBD@Z 1000de10 f   moc_DNAFlexPlugin.obj
 0001:0000ce70       ?qt_metacast@DNAFlexViewContext@U2@@UAEPAXPBD@Z 1000de70 f   moc_DNAFlexPlugin.obj
 0001:0000ced0       ?qt_metatype_id@?$QMetaTypeId2@PAVADVSequenceWidget@U2@@@@SAHXZ 1000ded0 f i moc_DNAFlexPlugin.obj
 0001:0000cee0       ?qt_metatype_id@?$QMetaTypeIdHelper@PAVADVSequenceWidget@U2@@$00@QtPrivate@@SAHXZ 1000dee0 f i moc_DNAFlexPlugin.obj
 0001:0000cef0       ?qt_metatype_id@?$QMetaTypeIdQObject@PAVADVSequenceWidget@U2@@$00@@SAHXZ 1000def0 f i moc_DNAFlexPlugin.obj
 0001:0000cfd0       ?qt_static_metacall@DNAFlexPlugin@U2@@CAXPAVQObject@@W4Call@QMetaObject@@HPAPAX@Z 1000dfd0 f   moc_DNAFlexPlugin.obj
 0001:0000cfe0       ?qt_static_metacall@DNAFlexViewContext@U2@@CAXPAVQObject@@W4Call@QMetaObject@@HPAPAX@Z 1000dfe0 f   moc_DNAFlexPlugin.obj
 0001:0000d050       ?registerConverter@?$AssociativeContainerConverterHelper@PAVADVSequenceWidget@U2@@$0A@@QtPrivate@@SA_NH@Z 1000e050 f i moc_DNAFlexPlugin.obj
 0001:0000d060       ?registerConverter@?$IsPair@PAVADVSequenceWidget@U2@@@QtPrivate@@SA_NH@Z 1000e060 f i moc_DNAFlexPlugin.obj
 0001:0000d070       ?registerConverter@?$MetaTypeSmartPointerHelper@PAVADVSequenceWidget@U2@@X@QtPrivate@@SA_NH@Z 1000e070 f i moc_DNAFlexPlugin.obj
 0001:0000d080       ?registerConverter@?$SequentialContainerConverterHelper@PAVADVSequenceWidget@U2@@$0A@@QtPrivate@@SA_NH@Z 1000e080 f i moc_DNAFlexPlugin.obj
 0001:0000d090       ?storeRelease@?$QBasicAtomicInteger@H@@QAEXH@Z 1000e090 f i moc_DNAFlexPlugin.obj
 0001:0000d0a0       ?value@?$MetaObjectForType@PAVADVSequenceWidget@U2@@$00@QtPrivate@@SAPBUQMetaObject@@XZ 1000e0a0 f i moc_DNAFlexPlugin.obj
 0001:0000d0b0       ?metaObject@DNAFlexTask@U2@@UBEPBUQMetaObject@@XZ 1000e0b0 f   moc_DNAFlexTask.obj
 0001:0000d0d0       ?qt_metacall@DNAFlexTask@U2@@UAEHW4Call@QMetaObject@@HPAPAX@Z 1000e0d0 f   moc_DNAFlexTask.obj
 0001:0000d0e0       ?qt_metacast@DNAFlexTask@U2@@UAEPAXPBD@Z 1000e0e0 f   moc_DNAFlexTask.obj
 0001:0000d140       ?qt_static_metacall@DNAFlexTask@U2@@CAXPAVQObject@@W4Call@QMetaObject@@HPAPAX@Z 1000e140 f   moc_DNAFlexTask.obj
 0001:0000d150       ?metaObject@FindHighFlexRegions@U2@@UBEPBUQMetaObject@@XZ 1000e150 f   moc_FindHighFlexRegions.obj
 0001:0000d170       ?qt_metacall@FindHighFlexRegions@U2@@UAEHW4Call@QMetaObject@@HPAPAX@Z 1000e170 f   moc_FindHighFlexRegions.obj
 0001:0000d180       ?qt_metacast@FindHighFlexRegions@U2@@UAEPAXPBD@Z 1000e180 f   moc_FindHighFlexRegions.obj
 0001:0000d220       ?qt_static_metacall@FindHighFlexRegions@U2@@CAXPAVQObject@@W4Call@QMetaObject@@HPAPAX@Z 1000e220 f   moc_FindHighFlexRegions.obj
 0001:0000d230       ??0initializer@?A0xf1761197@@QAE@XZ 1000e230 f i qrc_dna_flexibility.obj
 0001:0000d250       ??1initializer@?A0xf1761197@@QAE@XZ 1000e250 f i qrc_dna_flexibility.obj
 0001:0000d270       ?qCleanupResources_dna_flexibility@@YAHXZ 1000e270 f   qrc_dna_flexibility.obj
 0001:0000d290       ?qInitResources_dna_flexibility@@YAHXZ 1000e290 f   qrc_dna_flexibility.obj
 0001:0000d2b0       ??0Logger@U2@@QAE@ABVQString@@@Z 1000e2b0 f   U2Core:U2Core.dll
 0001:0000d2b6       ??1Logger@U2@@UAE@XZ       1000e2b6 f   U2Core:U2Core.dll
 0001:0000d2bc       ?isCoR@U2OpStatus@U2@@UBE_NXZ 1000e2bc f   U2Core:U2Core.dll
 0001:0000d2c2       ??0GObjectReference@U2@@QAE@PBVGObject@1@_N@Z 1000e2c2 f   U2Core:U2Core.dll
 0001:0000d2c8       ??1GObjectReference@U2@@QAE@XZ 1000e2c8 f   U2Core:U2Core.dll
 0001:0000d2ce       ??4GObjectReference@U2@@QAEAAV01@ABV01@@Z 1000e2ce f   U2Core:U2Core.dll
 0001:0000d2d4       ??0DNASequence@U2@@QAE@ABVQByteArray@@PBVDNAAlphabet@1@@Z 1000e2d4 f   U2Core:U2Core.dll
 0001:0000d2da       ??1DNASequence@U2@@QAE@XZ  1000e2da f   U2Core:U2Core.dll
 0001:0000d2e0       ??1AnnotationData@U2@@QAE@XZ 1000e2e0 f   U2Core:U2Core.dll
 0001:0000d2e6       ??0AnnotationData@U2@@QAE@ABV01@@Z 1000e2e6 f   U2Core:U2Core.dll
 0001:0000d2ec       ?getTaskScheduler@AppContext@U2@@SAPAVTaskScheduler@2@XZ 1000e2ec f   U2Core:U2Core.dll
 0001:0000d2f2       ?getSequenceLength@U2SequenceObject@U2@@QBE_JXZ 1000e2f2 f   U2Core:U2Core.dll
 0001:0000d2f8       ?getWholeSequenceData@U2SequenceObject@U2@@QBE?AVQByteArray@@AAVU2OpStatus@2@@Z 1000e2f8 f   U2Core:U2Core.dll
 0001:0000d2fe       ??0U2OpStatusImpl@U2@@QAE@XZ 1000e2fe f   U2Core:U2Core.dll
 0001:0000d304       ?getError@U2OpStatusImpl@U2@@UBE?AVQString@@XZ 1000e304 f   U2Core:U2Core.dll
 0001:0000d30a       ??1U2OpStatusImpl@U2@@UAE@XZ 1000e30a f   U2Core:U2Core.dll
 0001:0000d310       ?errorTitle@L10N@U2@@SA?AVQString@@XZ 1000e310 f   U2Core:U2Core.dll
 0001:0000d316       ?getAlphabet@U2SequenceObject@U2@@QBEPBVDNAAlphabet@2@XZ 1000e316 f   U2Core:U2Core.dll
 0001:0000d31c       ?NUCL_DNA_DEFAULT@BaseDNAAlphabetIds@U2@@SA?BVQString@@XZ 1000e31c f   U2Core:U2Core.dll
 0001:0000d322       ?getMainWindow@AppContext@U2@@SAPAVMainWindow@2@XZ 1000e322 f   U2Core:U2Core.dll
 0001:0000d328       ?error@Logger@U2@@QAEXABVQString@@@Z 1000e328 f   U2Core:U2Core.dll
 0001:0000d32e       ??0Plugin@U2@@QAE@ABVQString@@0_NW4PluginState@1@@Z 1000e32e f   U2Core:U2Core.dll
 0001:0000d334       ??1Plugin@U2@@UAE@XZ       1000e334 f   U2Core:U2Core.dll
 0001:0000d33a       ??CU2Location@U2@@QAEPAVU2LocationData@1@XZ 1000e33a f   U2Core:U2Core.dll
 0001:0000d340       ??0U2Qualifier@U2@@QAE@XZ  1000e340 f   U2Core:U2Core.dll
 0001:0000d346       ??0U2Qualifier@U2@@QAE@ABVQString@@0@Z 1000e346 f   U2Core:U2Core.dll
 0001:0000d34c       ??1U2Qualifier@U2@@QAE@XZ  1000e34c f   U2Core:U2Core.dll
 0001:0000d352       ??0U2Qualifier@U2@@QAE@ABV01@@Z 1000e352 f   U2Core:U2Core.dll
 0001:0000d358       ??0AnnotationData@U2@@QAE@XZ 1000e358 f   U2Core:U2Core.dll
 0001:0000d35e       ??0Task@U2@@QAE@ABVQString@@V?$QFlags@W4TaskFlag@U2@@@@@Z 1000e35e f   U2Core:U2Core.dll
 0001:0000d364       ?addSubTask@Task@U2@@QAEXPAV12@@Z 1000e364 f   U2Core:U2Core.dll
 0001:0000d36a       ?hasError@Task@U2@@QBE_NXZ 1000e36a f   U2Core:U2Core.dll
 0001:0000d370       ?getError@Task@U2@@QBE?AVQString@@XZ 1000e370 f   U2Core:U2Core.dll
 0001:0000d376       ??1Task@U2@@UAE@XZ         1000e376 f   U2Core:U2Core.dll
 0001:0000d37c       ??0CreateAnnotationsTask@U2@@QAE@PAVAnnotationTableObject@1@ABV?$QList@V?$QSharedDataPointer@VAnnotationData@U2@@@@@@ABVQString@@@Z 1000e37c f   U2Core:U2Core.dll
 0001:0000d382       ??1CreateAnnotationsTask@U2@@UAE@XZ 1000e382 f   U2Core:U2Core.dll
 0001:0000d388       ??0DNASequence@U2@@QAE@ABV01@@Z 1000e388 f   U2Core:U2Core.dll
 0001:0000d38e       ?addDescriptionQualifier@U1AnnotationUtils@U2@@SAXAAV?$QSharedDataPointer@VAnnotationData@U2@@@@ABVQString@@@Z 1000e38e f   U2Core:U2Core.dll
 0001:0000d394       ?cleanup@Task@U2@@UAEXXZ   1000e394 f   U2Core:U2Core.dll
 0001:0000d39a       ?generateReport@Task@U2@@UBE?AVQString@@XZ 1000e39a f   U2Core:U2Core.dll
 0001:0000d3a0       ?getNumParallelSubtasks@Task@U2@@UBEHXZ 1000e3a0 f   U2Core:U2Core.dll
 0001:0000d3a6       ?getParentTask@Task@U2@@UBEPAV12@XZ 1000e3a6 f   U2Core:U2Core.dll
 0001:0000d3ac       ?getSubtaskWithErrors@Task@U2@@UBEPAV12@XZ 1000e3ac f   U2Core:U2Core.dll
 0001:0000d3b2       ?getTaskId@Task@U2@@UBE_JXZ 1000e3b2 f   U2Core:U2Core.dll
 0001:0000d3b8       ?getTopLevelParentTask@Task@U2@@UAEPAV12@XZ 1000e3b8 f   U2Core:U2Core.dll
 0001:0000d3be       ?getWarnings@Task@U2@@UBE?AVQStringList@@XZ 1000e3be f   U2Core:U2Core.dll
 0001:0000d3c4       ?hasSubtasksWithErrors@Task@U2@@UBE_NXZ 1000e3c4 f   U2Core:U2Core.dll
 0001:0000d3ca       ?hasWarning@Task@U2@@UBE_NXZ 1000e3ca f   U2Core:U2Core.dll
 0001:0000d3d0       ?isNotificationReport@Task@U2@@UBE_NXZ 1000e3d0 f   U2Core:U2Core.dll
 0001:0000d3d6       ?isReportingEnabled@Task@U2@@UBE_NXZ 1000e3d6 f   U2Core:U2Core.dll
 0001:0000d3dc       ?isReportingSupported@Task@U2@@UBE_NXZ 1000e3dc f   U2Core:U2Core.dll
 0001:0000d3e2       ?isTopLevelTask@Task@U2@@UBE_NXZ 1000e3e2 f   U2Core:U2Core.dll
 0001:0000d3e8       ?metaObject@CreateAnnotationsTask@U2@@UBEPBUQMetaObject@@XZ 1000e3e8 f   U2Core:U2Core.dll
 0001:0000d3ee       ?onSubTaskFinished@Task@U2@@MAE?AV?$QList@PAVTask@U2@@@@PAV12@@Z 1000e3ee f   U2Core:U2Core.dll
 0001:0000d3f4       ?prepare@Task@U2@@UAEXXZ   1000e3f4 f   U2Core:U2Core.dll
 0001:0000d3fa       ?propagateSubtaskError@Task@U2@@UAE_NXZ 1000e3fa f   U2Core:U2Core.dll
 0001:0000d400       ?qt_metacall@CreateAnnotationsTask@U2@@UAEHW4Call@QMetaObject@@HPAPAX@Z 1000e400 f   U2Core:U2Core.dll
 0001:0000d406       ?qt_metacast@CreateAnnotationsTask@U2@@UAEPAXPBD@Z 1000e406 f   U2Core:U2Core.dll
 0001:0000d40c       ?report@CreateAnnotationsTask@U2@@UAE?AW4ReportResult@Task@2@XZ 1000e40c f   U2Core:U2Core.dll
 0001:0000d412       ?report@Task@U2@@UAE?AW4ReportResult@12@XZ 1000e412 f   U2Core:U2Core.dll
 0001:0000d418       ?run@CreateAnnotationsTask@U2@@UAEXXZ 1000e418 f   U2Core:U2Core.dll
 0001:0000d41e       ?run@Task@U2@@UAEXXZ       1000e41e f   U2Core:U2Core.dll
 0001:0000d424       ?setCollectChildrensWarningsFlag@Task@U2@@UAEX_N@Z 1000e424 f   U2Core:U2Core.dll
 0001:0000d42a       ?setNoAutoDelete@Task@U2@@UAEX_N@Z 1000e42a f   U2Core:U2Core.dll
 0001:0000d430       ?setNotificationReport@Task@U2@@UAEX_N@Z 1000e430 f   U2Core:U2Core.dll
 0001:0000d436       ?setReportingEnabled@Task@U2@@UAEX_N@Z 1000e436 f   U2Core:U2Core.dll
 0001:0000d43c       ?setReportingSupported@Task@U2@@UAEX_N@Z 1000e43c f   U2Core:U2Core.dll
 0001:0000d442       ?getSettings@AppContext@U2@@SAPAVSettings@2@XZ 1000e442 f   U2Core:U2Core.dll
 0001:0000d448       ?qt_metacast@Plugin@U2@@UAEPAXPBD@Z 1000e448 f   U2Core:U2Core.dll
 0001:0000d44e       ?qt_metacall@Plugin@U2@@UAEHW4Call@QMetaObject@@HPAPAX@Z 1000e44e f   U2Core:U2Core.dll
 0001:0000d454       ?qt_metacast@Task@U2@@UAEPAXPBD@Z 1000e454 f   U2Core:U2Core.dll
 0001:0000d45a       ?qt_metacall@Task@U2@@UAEHW4Call@QMetaObject@@HPAPAX@Z 1000e45a f   U2Core:U2Core.dll
 0001:0000d460       ??0CreateAnnotationModel@U2@@QAE@XZ 1000e460 f   U2Gui:U2Gui.dll
 0001:0000d466       ?getAnnotationObject@CreateAnnotationModel@U2@@QBEPAVAnnotationTableObject@2@XZ 1000e466 f   U2Gui:U2Gui.dll
 0001:0000d46c       ??1CreateAnnotationModel@U2@@QAE@XZ 1000e46c f   U2Gui:U2Gui.dll
 0001:0000d472       ??0CreateAnnotationWidgetController@U2@@QAE@ABVCreateAnnotationModel@1@PAVQObject@@W4AnnotationWidgetMode@01@@Z 1000e472 f   U2Gui:U2Gui.dll
 0001:0000d478       ?validate@CreateAnnotationWidgetController@U2@@QAE?AVQString@@XZ 1000e478 f   U2Gui:U2Gui.dll
 0001:0000d47e       ?prepareAnnotationObject@CreateAnnotationWidgetController@U2@@QAE_NXZ 1000e47e f   U2Gui:U2Gui.dll
 0001:0000d484       ?getWidget@CreateAnnotationWidgetController@U2@@QBEPAVQWidget@@XZ 1000e484 f   U2Gui:U2Gui.dll
 0001:0000d48a       ??1CreateAnnotationWidgetController@U2@@UAE@XZ 1000e48a f   U2Gui:U2Gui.dll
 0001:0000d490       ??0HelpButton@U2@@QAE@PAVQObject@@PAVQDialogButtonBox@@ABVQString@@@Z 1000e490 f   U2Gui:U2Gui.dll
 0001:0000d496       ??1HelpButton@U2@@UAE@XZ   1000e496 f   U2Gui:U2Gui.dll
 0001:0000d49c       ?getWidget@GObjectView@U2@@QAEPAVQWidget@@XZ 1000e49c f   U2Gui:U2Gui.dll
 0001:0000d4a2       ?metaObject@CreateAnnotationWidgetController@U2@@UBEPBUQMetaObject@@XZ 1000e4a2 f   U2Gui:U2Gui.dll
 0001:0000d4a8       ?metaObject@HelpButton@U2@@UBEPBUQMetaObject@@XZ 1000e4a8 f   U2Gui:U2Gui.dll
 0001:0000d4ae       ?qt_metacall@CreateAnnotationWidgetController@U2@@UAEHW4Call@QMetaObject@@HPAPAX@Z 1000e4ae f   U2Gui:U2Gui.dll
 0001:0000d4b4       ?qt_metacall@HelpButton@U2@@UAEHW4Call@QMetaObject@@HPAPAX@Z 1000e4b4 f   U2Gui:U2Gui.dll
 0001:0000d4ba       ?qt_metacast@CreateAnnotationWidgetController@U2@@UAEPAXPBD@Z 1000e4ba f   U2Gui:U2Gui.dll
 0001:0000d4c0       ?qt_metacast@HelpButton@U2@@UAEPAXPBD@Z 1000e4c0 f   U2Gui:U2Gui.dll
 0001:0000d4c6       ?sl_buttonClicked@HelpButton@U2@@MAEXXZ 1000e4c6 f   U2Gui:U2Gui.dll
 0001:0000d4cc       ?getObjectView@GObjectViewAction@U2@@QBEPAVGObjectView@2@XZ 1000e4cc f   U2Gui:U2Gui.dll
 0001:0000d4d2       ??0GObjectViewWindowContext@U2@@QAE@PAVQObject@@ABVGObjectViewFactoryId@1@@Z 1000e4d2 f   U2Gui:U2Gui.dll
 0001:0000d4d8       ??1GObjectViewWindowContext@U2@@UAE@XZ 1000e4d8 f   U2Gui:U2Gui.dll
 0001:0000d4de       ?buildMenu@GObjectViewWindowContext@U2@@MAEXPAVGObjectView@2@PAVQMenu@@@Z 1000e4de f   U2Gui:U2Gui.dll
 0001:0000d4e4       ?canHandle@GObjectViewObjectHandler@U2@@UAE_NPAVGObjectView@2@PAVGObject@2@@Z 1000e4e4 f   U2Gui:U2Gui.dll
 0001:0000d4ea       ?disconnectView@GObjectViewWindowContext@U2@@MAEXPAVGObjectView@2@@Z 1000e4ea f   U2Gui:U2Gui.dll
 0001:0000d4f0       ?init@GObjectViewWindowContext@U2@@UAEXXZ 1000e4f0 f   U2Gui:U2Gui.dll
 0001:0000d4f6       ?onObjectAdded@GObjectViewObjectHandler@U2@@UAEXPAVGObjectView@2@PAVGObject@2@@Z 1000e4f6 f   U2Gui:U2Gui.dll
 0001:0000d4fc       ?onObjectRemoved@GObjectViewWindowContext@U2@@UAEXPAVGObjectView@2@PAVGObject@2@@Z 1000e4fc f   U2Gui:U2Gui.dll
 0001:0000d502       ?sl_buildContextMenu@GObjectViewWindowContext@U2@@MAEXPAVGObjectView@2@PAVQMenu@@@Z 1000e502 f   U2Gui:U2Gui.dll
 0001:0000d508       ?sl_buildStaticMenu@GObjectViewWindowContext@U2@@MAEXPAVGObjectView@2@PAVQMenu@@@Z 1000e508 f   U2Gui:U2Gui.dll
 0001:0000d50e       ?sl_windowAdded@GObjectViewWindowContext@U2@@MAEXPAVMWMDIWindow@2@@Z 1000e50e f   U2Gui:U2Gui.dll
 0001:0000d514       ?sl_windowClosing@GObjectViewWindowContext@U2@@MAEXPAVMWMDIWindow@2@@Z 1000e514 f   U2Gui:U2Gui.dll
 0001:0000d51a       ?qt_metacast@GObjectViewWindowContext@U2@@UAEPAXPBD@Z 1000e51a f   U2Gui:U2Gui.dll
 0001:0000d520       ?qt_metacall@GObjectViewWindowContext@U2@@UAEHW4Call@QMetaObject@@HPAPAX@Z 1000e520 f   U2Gui:U2Gui.dll
 0001:0000d526       ?tryAddObject@AnnotatedDNAView@U2@@QAE?AVQString@@PAVGObject@2@@Z 1000e526 f   U2View:U2View.dll
 0001:0000d52c       ??1GSequenceGraphWindowData@U2@@UAE@XZ 1000e52c f   U2View:U2View.dll
 0001:0000d532       ??0GSequenceGraphDrawer@U2@@QAE@PAVGSequenceGraphView@1@ABVGSequenceGraphWindowData@1@V?$QMap@VQString@@VQColor@@@@@Z 1000e532 f   U2View:U2View.dll
 0001:0000d538       ??1GSequenceGraphDrawer@U2@@UAE@XZ 1000e538 f   U2View:U2View.dll
 0001:0000d53e       ??0GSequenceGraphData@U2@@QAE@ABVQString@@@Z 1000e53e f   U2View:U2View.dll
 0001:0000d544       ??1GSequenceGraphData@U2@@UAE@XZ 1000e544 f   U2View:U2View.dll
 0001:0000d54a       ??0GSequenceGraphFactory@U2@@QAE@ABVQString@@PAVQObject@@@Z 1000e54a f   U2View:U2View.dll
 0001:0000d550       ??1GSequenceGraphFactory@U2@@UAE@XZ 1000e550 f   U2View:U2View.dll
 0001:0000d556       ?draw@GSequenceGraphDrawer@U2@@UAEXAAVQPainter@@ABV?$QList@V?$QSharedPointer@VGSequenceGraphData@U2@@@@@@ABVQRect@@@Z 1000e556 f   U2View:U2View.dll
 0001:0000d55c       ?metaObject@GSequenceGraphDrawer@U2@@UBEPBUQMetaObject@@XZ 1000e55c f   U2View:U2View.dll
 0001:0000d562       ?qt_metacall@GSequenceGraphDrawer@U2@@UAEHW4Call@QMetaObject@@HPAPAX@Z 1000e562 f   U2View:U2View.dll
 0001:0000d568       ?qt_metacast@GSequenceGraphDrawer@U2@@UAEPAXPBD@Z 1000e568 f   U2View:U2View.dll
 0001:0000d56e       ?showSettingsDialog@GSequenceGraphDrawer@U2@@UAEXXZ 1000e56e f   U2View:U2View.dll
 0001:0000d574       ??1GSequenceGraphAlgorithm@U2@@UAE@XZ 1000e574 f   U2View:U2View.dll
 0001:0000d57a       ??0GSequenceGraphAlgorithm@U2@@IAE@XZ 1000e57a f   U2View:U2View.dll
 0001:0000d580       ?getSequenceData@GSequenceGraphAlgorithm@U2@@IAEABVQByteArray@@PAVU2SequenceObject@2@AAVU2OpStatus@2@@Z 1000e580 f   U2View:U2View.dll
 0001:0000d586       ?getNumSteps@GSequenceGraphUtils@U2@@SAHABVU2Region@2@HH@Z 1000e586 f   U2View:U2View.dll
 0001:0000d58c       ?getAlphabet@SequenceObjectContext@U2@@QBEPBVDNAAlphabet@2@XZ 1000e58c f   U2View:U2View.dll
 0001:0000d592       ??0ADVGlobalAction@U2@@QAE@PAVAnnotatedDNAView@1@ABVQIcon@@ABVQString@@HV?$QFlags@W4ADVGlobalActionFlag@U2@@@@@Z 1000e592 f   U2View:U2View.dll
 0001:0000d598       ?addAlphabetFilter@ADVGlobalAction@U2@@QAEXW4DNAAlphabetType@@@Z 1000e598 f   U2View:U2View.dll
 0001:0000d59e       ??1ADVGlobalAction@U2@@UAE@XZ 1000e59e f   U2View:U2View.dll
 0001:0000d5a4       ?getSequenceWidgets@AnnotatedDNAView@U2@@QBE?BV?$QList@PAVADVSequenceWidget@U2@@@@XZ 1000e5a4 f   U2View:U2View.dll
 0001:0000d5aa       ?getSequenceInFocus@AnnotatedDNAView@U2@@QBEPAVADVSequenceObjectContext@2@XZ 1000e5aa f   U2View:U2View.dll
 0001:0000d5b0       ?getSequenceContext@ADVSingleSequenceWidget@U2@@QBEPAVADVSequenceObjectContext@2@XZ 1000e5b0 f   U2View:U2View.dll
 0001:0000d5b6       ?getSequenceObject@ADVSingleSequenceWidget@U2@@QBEPAVU2SequenceObject@2@XZ 1000e5b6 f   U2View:U2View.dll
 0001:0000d5bc       ??0GraphAction@U2@@QAE@PAVGSequenceGraphFactory@1@@Z 1000e5bc f   U2View:U2View.dll
 0001:0000d5c2       ??1GraphAction@U2@@UAE@XZ  1000e5c2 f   U2View:U2View.dll
 0001:0000d5c8       ?addGraphAction@GraphMenuAction@U2@@SAXPAVADVSequenceObjectContext@2@PAVGraphAction@2@@Z 1000e5c8 f   U2View:U2View.dll
 0001:0000d5ce       ?metaObject@ADVGlobalAction@U2@@UBEPBUQMetaObject@@XZ 1000e5ce f   U2View:U2View.dll
 0001:0000d5d4       ?metaObject@GraphAction@U2@@UBEPBUQMetaObject@@XZ 1000e5d4 f   U2View:U2View.dll
 0001:0000d5da       ?qt_metacall@ADVGlobalAction@U2@@UAEHW4Call@QMetaObject@@HPAPAX@Z 1000e5da f   U2View:U2View.dll
 0001:0000d5e0       ?qt_metacall@GraphAction@U2@@UAEHW4Call@QMetaObject@@HPAPAX@Z 1000e5e0 f   U2View:U2View.dll
 0001:0000d5e6       ?qt_metacast@ADVGlobalAction@U2@@UAEPAXPBD@Z 1000e5e6 f   U2View:U2View.dll
 0001:0000d5ec       ?qt_metacast@GraphAction@U2@@UAEPAXPBD@Z 1000e5ec f   U2View:U2View.dll
 0001:0000d5f2       ??0QSizePolicy@@QAE@W4Policy@0@0W4ControlType@0@@Z 1000e5f2 f   Qt5Widgets:Qt5Widgets.dll
 0001:0000d5f8       ?setHorizontalStretch@QSizePolicy@@QAEXH@Z 1000e5f8 f   Qt5Widgets:Qt5Widgets.dll
 0001:0000d5fe       ?setVerticalStretch@QSizePolicy@@QAEXH@Z 1000e5fe f   Qt5Widgets:Qt5Widgets.dll
 0001:0000d604       ??0QWidget@@QAE@PAV0@V?$QFlags@W4WindowType@Qt@@@@@Z 1000e604 f   Qt5Widgets:Qt5Widgets.dll
 0001:0000d60a       ??1QWidget@@UAE@XZ         1000e60a f   Qt5Widgets:Qt5Widgets.dll
 0001:0000d610       ?setMinimumSize@QWidget@@QAEXHH@Z 1000e610 f   Qt5Widgets:Qt5Widgets.dll
 0001:0000d616       ?setWindowTitle@QWidget@@QAEXABVQString@@@Z 1000e616 f   Qt5Widgets:Qt5Widgets.dll
 0001:0000d61c       ?setWindowIcon@QWidget@@QAEXABVQIcon@@@Z 1000e61c f   Qt5Widgets:Qt5Widgets.dll
 0001:0000d622       ?setStatusTip@QWidget@@QAEXABVQString@@@Z 1000e622 f   Qt5Widgets:Qt5Widgets.dll
 0001:0000d628       ?setWhatsThis@QWidget@@QAEXABVQString@@@Z 1000e628 f   Qt5Widgets:Qt5Widgets.dll
 0001:0000d62e       ?resize@QWidget@@QAEXABVQSize@@@Z 1000e62e f   Qt5Widgets:Qt5Widgets.dll
 0001:0000d634       ?adjustSize@QWidget@@QAEXXZ 1000e634 f   Qt5Widgets:Qt5Widgets.dll
 0001:0000d63a       ?sizePolicy@QWidget@@QBE?AVQSizePolicy@@XZ 1000e63a f   Qt5Widgets:Qt5Widgets.dll
 0001:0000d640       ?setSizePolicy@QWidget@@QAEXVQSizePolicy@@@Z 1000e640 f   Qt5Widgets:Qt5Widgets.dll
 0001:0000d646       ?layout@QWidget@@QBEPAVQLayout@@XZ 1000e646 f   Qt5Widgets:Qt5Widgets.dll
 0001:0000d64c       ??0QDialog@@QAE@PAVQWidget@@V?$QFlags@W4WindowType@Qt@@@@@Z 1000e64c f   Qt5Widgets:Qt5Widgets.dll
 0001:0000d652       ??1QDialog@@UAE@XZ         1000e652 f   Qt5Widgets:Qt5Widgets.dll
 0001:0000d658       ?accept@QDialog@@UAEXXZ    1000e658 f   Qt5Widgets:Qt5Widgets.dll
 0001:0000d65e       ??0QDialogButtonBox@@QAE@PAVQWidget@@@Z 1000e65e f   Qt5Widgets:Qt5Widgets.dll
 0001:0000d664       ??1QDialogButtonBox@@UAE@XZ 1000e664 f   Qt5Widgets:Qt5Widgets.dll
 0001:0000d66a       ?setStandardButtons@QDialogButtonBox@@QAEXV?$QFlags@W4StandardButton@QDialogButtonBox@@@@@Z 1000e66a f   Qt5Widgets:Qt5Widgets.dll
 0001:0000d670       ?button@QDialogButtonBox@@QBEPAVQPushButton@@W4StandardButton@1@@Z 1000e670 f   Qt5Widgets:Qt5Widgets.dll
 0001:0000d676       ??0QSpinBox@@QAE@PAVQWidget@@@Z 1000e676 f   Qt5Widgets:Qt5Widgets.dll
 0001:0000d67c       ??1QSpinBox@@UAE@XZ        1000e67c f   Qt5Widgets:Qt5Widgets.dll
 0001:0000d682       ?setMinimum@QSpinBox@@QAEXH@Z 1000e682 f   Qt5Widgets:Qt5Widgets.dll
 0001:0000d688       ?setMaximum@QSpinBox@@QAEXH@Z 1000e688 f   Qt5Widgets:Qt5Widgets.dll
 0001:0000d68e       ?setValue@QSpinBox@@QAEXH@Z 1000e68e f   Qt5Widgets:Qt5Widgets.dll
 0001:0000d694       ??0QDoubleSpinBox@@QAE@PAVQWidget@@@Z 1000e694 f   Qt5Widgets:Qt5Widgets.dll
 0001:0000d69a       ??1QDoubleSpinBox@@UAE@XZ  1000e69a f   Qt5Widgets:Qt5Widgets.dll
 0001:0000d6a0       ?setSingleStep@QDoubleSpinBox@@QAEXN@Z 1000e6a0 f   Qt5Widgets:Qt5Widgets.dll
 0001:0000d6a6       ?setMaximum@QDoubleSpinBox@@QAEXN@Z 1000e6a6 f   Qt5Widgets:Qt5Widgets.dll
 0001:0000d6ac       ?setDecimals@QDoubleSpinBox@@QAEXH@Z 1000e6ac f   Qt5Widgets:Qt5Widgets.dll
 0001:0000d6b2       ?setValue@QDoubleSpinBox@@QAEXN@Z 1000e6b2 f   Qt5Widgets:Qt5Widgets.dll
 0001:0000d6b8       ??0QSpacerItem@@QAE@HHW4Policy@QSizePolicy@@0@Z 1000e6b8 f   Qt5Widgets:Qt5Widgets.dll
 0001:0000d6be       ??1QSpacerItem@@UAE@XZ     1000e6be f   Qt5Widgets:Qt5Widgets.dll
 0001:0000d6c4       ?addWidget@QLayout@@QAEXPAVQWidget@@@Z 1000e6c4 f   Qt5Widgets:Qt5Widgets.dll
 0001:0000d6ca       ?addWidget@QBoxLayout@@QAEXPAVQWidget@@HV?$QFlags@W4AlignmentFlag@Qt@@@@@Z 1000e6ca f   Qt5Widgets:Qt5Widgets.dll
 0001:0000d6d0       ?addLayout@QBoxLayout@@QAEXPAVQLayout@@H@Z 1000e6d0 f   Qt5Widgets:Qt5Widgets.dll
 0001:0000d6d6       ??0QHBoxLayout@@QAE@PAVQWidget@@@Z 1000e6d6 f   Qt5Widgets:Qt5Widgets.dll
 0001:0000d6dc       ??1QHBoxLayout@@UAE@XZ     1000e6dc f   Qt5Widgets:Qt5Widgets.dll
 0001:0000d6e2       ??0QVBoxLayout@@QAE@PAVQWidget@@@Z 1000e6e2 f   Qt5Widgets:Qt5Widgets.dll
 0001:0000d6e8       ??1QVBoxLayout@@UAE@XZ     1000e6e8 f   Qt5Widgets:Qt5Widgets.dll
 0001:0000d6ee       ??0QGridLayout@@QAE@XZ     1000e6ee f   Qt5Widgets:Qt5Widgets.dll
 0001:0000d6f4       ??1QGridLayout@@UAE@XZ     1000e6f4 f   Qt5Widgets:Qt5Widgets.dll
 0001:0000d6fa       ?addWidget@QGridLayout@@QAEXPAVQWidget@@HHHHV?$QFlags@W4AlignmentFlag@Qt@@@@@Z 1000e6fa f   Qt5Widgets:Qt5Widgets.dll
 0001:0000d700       ??0QGroupBox@@QAE@PAVQWidget@@@Z 1000e700 f   Qt5Widgets:Qt5Widgets.dll
 0001:0000d706       ??1QGroupBox@@UAE@XZ       1000e706 f   Qt5Widgets:Qt5Widgets.dll
 0001:0000d70c       ?setTitle@QGroupBox@@QAEXABVQString@@@Z 1000e70c f   Qt5Widgets:Qt5Widgets.dll
 0001:0000d712       ??0QTabWidget@@QAE@PAVQWidget@@@Z 1000e712 f   Qt5Widgets:Qt5Widgets.dll
 0001:0000d718       ??1QTabWidget@@UAE@XZ      1000e718 f   Qt5Widgets:Qt5Widgets.dll
 0001:0000d71e       ?addTab@QTabWidget@@QAEHPAVQWidget@@ABVQString@@@Z 1000e71e f   Qt5Widgets:Qt5Widgets.dll
 0001:0000d724       ?setTabText@QTabWidget@@QAEXHABVQString@@@Z 1000e724 f   Qt5Widgets:Qt5Widgets.dll
 0001:0000d72a       ?currentWidget@QTabWidget@@QBEPAVQWidget@@XZ 1000e72a f   Qt5Widgets:Qt5Widgets.dll
 0001:0000d730       ?widget@QTabWidget@@QBEPAVQWidget@@H@Z 1000e730 f   Qt5Widgets:Qt5Widgets.dll
 0001:0000d736       ?indexOf@QTabWidget@@QBEHPAVQWidget@@@Z 1000e736 f   Qt5Widgets:Qt5Widgets.dll
 0001:0000d73c       ?count@QTabWidget@@QBEHXZ  1000e73c f   Qt5Widgets:Qt5Widgets.dll
 0001:0000d742       ?setTabShape@QTabWidget@@QAEXW4TabShape@1@@Z 1000e742 f   Qt5Widgets:Qt5Widgets.dll
 0001:0000d748       ?setCurrentIndex@QTabWidget@@QAEXH@Z 1000e748 f   Qt5Widgets:Qt5Widgets.dll
 0001:0000d74e       ??0QLabel@@QAE@PAVQWidget@@V?$QFlags@W4WindowType@Qt@@@@@Z 1000e74e f   Qt5Widgets:Qt5Widgets.dll
 0001:0000d754       ??1QLabel@@UAE@XZ          1000e754 f   Qt5Widgets:Qt5Widgets.dll
 0001:0000d75a       ?setIndent@QLabel@@QAEXH@Z 1000e75a f   Qt5Widgets:Qt5Widgets.dll
 0001:0000d760       ?setText@QLabel@@QAEXABVQString@@@Z 1000e760 f   Qt5Widgets:Qt5Widgets.dll
 0001:0000d766       ?setText@QAbstractButton@@QAEXABVQString@@@Z 1000e766 f   Qt5Widgets:Qt5Widgets.dll
 0001:0000d76c       ??0QPushButton@@QAE@PAVQWidget@@@Z 1000e76c f   Qt5Widgets:Qt5Widgets.dll
 0001:0000d772       ??1QPushButton@@UAE@XZ     1000e772 f   Qt5Widgets:Qt5Widgets.dll
 0001:0000d778       ?warning@QMessageBox@@SA?AW4StandardButton@1@PAVQWidget@@ABVQString@@1V?$QFlags@W4StandardButton@QMessageBox@@@@W421@@Z 1000e778 f   Qt5Widgets:Qt5Widgets.dll
 0001:0000d77e       ?critical@QMessageBox@@SA?AW4StandardButton@1@PAVQWidget@@ABVQString@@1V?$QFlags@W4StandardButton@QMessageBox@@@@W421@@Z 1000e77e f   Qt5Widgets:Qt5Widgets.dll
 0001:0000d784       ?actionEvent@QWidget@@MAEXPAVQActionEvent@@@Z 1000e784 f   Qt5Widgets:Qt5Widgets.dll
 0001:0000d78a       ?addItem@QBoxLayout@@UAEXPAVQLayoutItem@@@Z 1000e78a f   Qt5Widgets:Qt5Widgets.dll
 0001:0000d790       ?addItem@QGridLayout@@MAEXPAVQLayoutItem@@@Z 1000e790 f   Qt5Widgets:Qt5Widgets.dll
 0001:0000d796       ?changeEvent@QAbstractButton@@MAEXPAVQEvent@@@Z 1000e796 f   Qt5Widgets:Qt5Widgets.dll
 0001:0000d79c       ?changeEvent@QAbstractSpinBox@@MAEXPAVQEvent@@@Z 1000e79c f   Qt5Widgets:Qt5Widgets.dll
 0001:0000d7a2       ?changeEvent@QDialogButtonBox@@MAEXPAVQEvent@@@Z 1000e7a2 f   Qt5Widgets:Qt5Widgets.dll
 0001:0000d7a8       ?changeEvent@QGroupBox@@MAEXPAVQEvent@@@Z 1000e7a8 f   Qt5Widgets:Qt5Widgets.dll
 0001:0000d7ae       ?changeEvent@QLabel@@MAEXPAVQEvent@@@Z 1000e7ae f   Qt5Widgets:Qt5Widgets.dll
 0001:0000d7b4       ?changeEvent@QTabWidget@@MAEXPAVQEvent@@@Z 1000e7b4 f   Qt5Widgets:Qt5Widgets.dll
 0001:0000d7ba       ?changeEvent@QWidget@@MAEXPAVQEvent@@@Z 1000e7ba f   Qt5Widgets:Qt5Widgets.dll
 0001:0000d7c0       ?checkStateSet@QAbstractButton@@MAEXXZ 1000e7c0 f   Qt5Widgets:Qt5Widgets.dll
 0001:0000d7c6       ?childEvent@QGroupBox@@MAEXPAVQChildEvent@@@Z 1000e7c6 f   Qt5Widgets:Qt5Widgets.dll
 0001:0000d7cc       ?childEvent@QLayout@@MAEXPAVQChildEvent@@@Z 1000e7cc f   Qt5Widgets:Qt5Widgets.dll
 0001:0000d7d2       ?clear@QAbstractSpinBox@@UAEXXZ 1000e7d2 f   Qt5Widgets:Qt5Widgets.dll
 0001:0000d7d8       ?closeEvent@QAbstractSpinBox@@MAEXPAVQCloseEvent@@@Z 1000e7d8 f   Qt5Widgets:Qt5Widgets.dll
 0001:0000d7de       ?closeEvent@QDialog@@MAEXPAVQCloseEvent@@@Z 1000e7de f   Qt5Widgets:Qt5Widgets.dll
 0001:0000d7e4       ?closeEvent@QWidget@@MAEXPAVQCloseEvent@@@Z 1000e7e4 f   Qt5Widgets:Qt5Widgets.dll
 0001:0000d7ea       ?contextMenuEvent@QAbstractSpinBox@@MAEXPAVQContextMenuEvent@@@Z 1000e7ea f   Qt5Widgets:Qt5Widgets.dll
 0001:0000d7f0       ?contextMenuEvent@QDialog@@MAEXPAVQContextMenuEvent@@@Z 1000e7f0 f   Qt5Widgets:Qt5Widgets.dll
 0001:0000d7f6       ?contextMenuEvent@QLabel@@MAEXPAVQContextMenuEvent@@@Z 1000e7f6 f   Qt5Widgets:Qt5Widgets.dll
 0001:0000d7fc       ?contextMenuEvent@QWidget@@MAEXPAVQContextMenuEvent@@@Z 1000e7fc f   Qt5Widgets:Qt5Widgets.dll
 0001:0000d802       ?controlTypes@QLayout@@UBE?AV?$QFlags@W4ControlType@QSizePolicy@@@@XZ 1000e802 f   Qt5Widgets:Qt5Widgets.dll
 0001:0000d808       ?controlTypes@QLayoutItem@@UBE?AV?$QFlags@W4ControlType@QSizePolicy@@@@XZ 1000e808 f   Qt5Widgets:Qt5Widgets.dll
 0001:0000d80e       ?count@QBoxLayout@@UBEHXZ  1000e80e f   Qt5Widgets:Qt5Widgets.dll
 0001:0000d814       ?count@QGridLayout@@UBEHXZ 1000e814 f   Qt5Widgets:Qt5Widgets.dll
 0001:0000d81a       ?devType@QWidget@@UBEHXZ   1000e81a f   Qt5Widgets:Qt5Widgets.dll
 0001:0000d820       ?done@QDialog@@UAEXH@Z     1000e820 f   Qt5Widgets:Qt5Widgets.dll
 0001:0000d826       ?dragEnterEvent@QWidget@@MAEXPAVQDragEnterEvent@@@Z 1000e826 f   Qt5Widgets:Qt5Widgets.dll
 0001:0000d82c       ?dragLeaveEvent@QWidget@@MAEXPAVQDragLeaveEvent@@@Z 1000e82c f   Qt5Widgets:Qt5Widgets.dll
 0001:0000d832       ?dragMoveEvent@QWidget@@MAEXPAVQDragMoveEvent@@@Z 1000e832 f   Qt5Widgets:Qt5Widgets.dll
 0001:0000d838       ?dropEvent@QWidget@@MAEXPAVQDropEvent@@@Z 1000e838 f   Qt5Widgets:Qt5Widgets.dll
 0001:0000d83e       ?enterEvent@QWidget@@MAEXPAVQEvent@@@Z 1000e83e f   Qt5Widgets:Qt5Widgets.dll
 0001:0000d844       ?event@QAbstractSpinBox@@UAE_NPAVQEvent@@@Z 1000e844 f   Qt5Widgets:Qt5Widgets.dll
 0001:0000d84a       ?event@QDialogButtonBox@@MAE_NPAVQEvent@@@Z 1000e84a f   Qt5Widgets:Qt5Widgets.dll
 0001:0000d850       ?event@QGroupBox@@MAE_NPAVQEvent@@@Z 1000e850 f   Qt5Widgets:Qt5Widgets.dll
 0001:0000d856       ?event@QLabel@@MAE_NPAVQEvent@@@Z 1000e856 f   Qt5Widgets:Qt5Widgets.dll
 0001:0000d85c       ?event@QPushButton@@MAE_NPAVQEvent@@@Z 1000e85c f   Qt5Widgets:Qt5Widgets.dll
 0001:0000d862       ?event@QSpinBox@@MAE_NPAVQEvent@@@Z 1000e862 f   Qt5Widgets:Qt5Widgets.dll
 0001:0000d868       ?event@QTabWidget@@MAE_NPAVQEvent@@@Z 1000e868 f   Qt5Widgets:Qt5Widgets.dll
 0001:0000d86e       ?event@QWidget@@MAE_NPAVQEvent@@@Z 1000e86e f   Qt5Widgets:Qt5Widgets.dll
 0001:0000d874       ?eventFilter@QDialog@@MAE_NPAVQObject@@PAVQEvent@@@Z 1000e874 f   Qt5Widgets:Qt5Widgets.dll
 0001:0000d87a       ?exec@QDialog@@UAEHXZ      1000e87a f   Qt5Widgets:Qt5Widgets.dll
 0001:0000d880       ?expandingDirections@QBoxLayout@@UBE?AV?$QFlags@W4Orientation@Qt@@@@XZ 1000e880 f   Qt5Widgets:Qt5Widgets.dll
 0001:0000d886       ?expandingDirections@QGridLayout@@UBE?AV?$QFlags@W4Orientation@Qt@@@@XZ 1000e886 f   Qt5Widgets:Qt5Widgets.dll
 0001:0000d88c       ?expandingDirections@QSpacerItem@@UBE?AV?$QFlags@W4Orientation@Qt@@@@XZ 1000e88c f   Qt5Widgets:Qt5Widgets.dll
 0001:0000d892       ?fixup@QDoubleSpinBox@@UBEXAAVQString@@@Z 1000e892 f   Qt5Widgets:Qt5Widgets.dll
 0001:0000d898       ?fixup@QSpinBox@@MBEXAAVQString@@@Z 1000e898 f   Qt5Widgets:Qt5Widgets.dll
 0001:0000d89e       ?focusInEvent@QAbstractSpinBox@@MAEXPAVQFocusEvent@@@Z 1000e89e f   Qt5Widgets:Qt5Widgets.dll
 0001:0000d8a4       ?focusInEvent@QGroupBox@@MAEXPAVQFocusEvent@@@Z 1000e8a4 f   Qt5Widgets:Qt5Widgets.dll
 0001:0000d8aa       ?focusInEvent@QLabel@@MAEXPAVQFocusEvent@@@Z 1000e8aa f   Qt5Widgets:Qt5Widgets.dll
 0001:0000d8b0       ?focusInEvent@QPushButton@@MAEXPAVQFocusEvent@@@Z 1000e8b0 f   Qt5Widgets:Qt5Widgets.dll
 0001:0000d8b6       ?focusInEvent@QWidget@@MAEXPAVQFocusEvent@@@Z 1000e8b6 f   Qt5Widgets:Qt5Widgets.dll
 0001:0000d8bc       ?focusNextPrevChild@QLabel@@MAE_N_N@Z 1000e8bc f   Qt5Widgets:Qt5Widgets.dll
 0001:0000d8c2       ?focusNextPrevChild@QWidget@@MAE_N_N@Z 1000e8c2 f   Qt5Widgets:Qt5Widgets.dll
 0001:0000d8c8       ?focusOutEvent@QAbstractSpinBox@@MAEXPAVQFocusEvent@@@Z 1000e8c8 f   Qt5Widgets:Qt5Widgets.dll
 0001:0000d8ce       ?focusOutEvent@QLabel@@MAEXPAVQFocusEvent@@@Z 1000e8ce f   Qt5Widgets:Qt5Widgets.dll
 0001:0000d8d4       ?focusOutEvent@QPushButton@@MAEXPAVQFocusEvent@@@Z 1000e8d4 f   Qt5Widgets:Qt5Widgets.dll
 0001:0000d8da       ?focusOutEvent@QWidget@@MAEXPAVQFocusEvent@@@Z 1000e8da f   Qt5Widgets:Qt5Widgets.dll
 0001:0000d8e0       ?geometry@QLayout@@UBE?AVQRect@@XZ 1000e8e0 f   Qt5Widgets:Qt5Widgets.dll
 0001:0000d8e6       ?geometry@QSpacerItem@@UBE?AVQRect@@XZ 1000e8e6 f   Qt5Widgets:Qt5Widgets.dll
 0001:0000d8ec       ?hasHeightForWidth@QBoxLayout@@UBE_NXZ 1000e8ec f   Qt5Widgets:Qt5Widgets.dll
 0001:0000d8f2       ?hasHeightForWidth@QGridLayout@@UBE_NXZ 1000e8f2 f   Qt5Widgets:Qt5Widgets.dll
 0001:0000d8f8       ?hasHeightForWidth@QLayoutItem@@UBE_NXZ 1000e8f8 f   Qt5Widgets:Qt5Widgets.dll
 0001:0000d8fe       ?hasHeightForWidth@QTabWidget@@UBE_NXZ 1000e8fe f   Qt5Widgets:Qt5Widgets.dll
 0001:0000d904       ?hasHeightForWidth@QWidget@@UBE_NXZ 1000e904 f   Qt5Widgets:Qt5Widgets.dll
 0001:0000d90a       ?heightForWidth@QBoxLayout@@UBEHH@Z 1000e90a f   Qt5Widgets:Qt5Widgets.dll
 0001:0000d910       ?heightForWidth@QGridLayout@@UBEHH@Z 1000e910 f   Qt5Widgets:Qt5Widgets.dll
 0001:0000d916       ?heightForWidth@QLabel@@UBEHH@Z 1000e916 f   Qt5Widgets:Qt5Widgets.dll
 0001:0000d91c       ?heightForWidth@QLayoutItem@@UBEHH@Z 1000e91c f   Qt5Widgets:Qt5Widgets.dll
 0001:0000d922       ?heightForWidth@QTabWidget@@UBEHH@Z 1000e922 f   Qt5Widgets:Qt5Widgets.dll
 0001:0000d928       ?heightForWidth@QWidget@@UBEHH@Z 1000e928 f   Qt5Widgets:Qt5Widgets.dll
 0001:0000d92e       ?hideEvent@QAbstractSpinBox@@MAEXPAVQHideEvent@@@Z 1000e92e f   Qt5Widgets:Qt5Widgets.dll
 0001:0000d934       ?hideEvent@QWidget@@MAEXPAVQHideEvent@@@Z 1000e934 f   Qt5Widgets:Qt5Widgets.dll
 0001:0000d93a       ?hitButton@QAbstractButton@@MBE_NABVQPoint@@@Z 1000e93a f   Qt5Widgets:Qt5Widgets.dll
 0001:0000d940       ?indexOf@QLayout@@UBEHPAVQWidget@@@Z 1000e940 f   Qt5Widgets:Qt5Widgets.dll
 0001:0000d946       ?initPainter@QWidget@@MBEXPAVQPainter@@@Z 1000e946 f   Qt5Widgets:Qt5Widgets.dll
 0001:0000d94c       ?inputMethodEvent@QWidget@@MAEXPAVQInputMethodEvent@@@Z 1000e94c f   Qt5Widgets:Qt5Widgets.dll
 0001:0000d952       ?inputMethodQuery@QAbstractSpinBox@@UBE?AVQVariant@@W4InputMethodQuery@Qt@@@Z 1000e952 f   Qt5Widgets:Qt5Widgets.dll
 0001:0000d958       ?inputMethodQuery@QWidget@@UBE?AVQVariant@@W4InputMethodQuery@Qt@@@Z 1000e958 f   Qt5Widgets:Qt5Widgets.dll
 0001:0000d95e       ?invalidate@QBoxLayout@@UAEXXZ 1000e95e f   Qt5Widgets:Qt5Widgets.dll
 0001:0000d964       ?invalidate@QGridLayout@@UAEXXZ 1000e964 f   Qt5Widgets:Qt5Widgets.dll
 0001:0000d96a       ?invalidate@QLayoutItem@@UAEXXZ 1000e96a f   Qt5Widgets:Qt5Widgets.dll
 0001:0000d970       ?isEmpty@QLayout@@UBE_NXZ  1000e970 f   Qt5Widgets:Qt5Widgets.dll
 0001:0000d976       ?isEmpty@QSpacerItem@@UBE_NXZ 1000e976 f   Qt5Widgets:Qt5Widgets.dll
 0001:0000d97c       ?itemAt@QBoxLayout@@UBEPAVQLayoutItem@@H@Z 1000e97c f   Qt5Widgets:Qt5Widgets.dll
 0001:0000d982       ?itemAt@QGridLayout@@UBEPAVQLayoutItem@@H@Z 1000e982 f   Qt5Widgets:Qt5Widgets.dll
 0001:0000d988       ?keyPressEvent@QAbstractSpinBox@@MAEXPAVQKeyEvent@@@Z 1000e988 f   Qt5Widgets:Qt5Widgets.dll
 0001:0000d98e       ?keyPressEvent@QDialog@@MAEXPAVQKeyEvent@@@Z 1000e98e f   Qt5Widgets:Qt5Widgets.dll
 0001:0000d994       ?keyPressEvent@QLabel@@MAEXPAVQKeyEvent@@@Z 1000e994 f   Qt5Widgets:Qt5Widgets.dll
 0001:0000d99a       ?keyPressEvent@QPushButton@@MAEXPAVQKeyEvent@@@Z 1000e99a f   Qt5Widgets:Qt5Widgets.dll
 0001:0000d9a0       ?keyPressEvent@QTabWidget@@MAEXPAVQKeyEvent@@@Z 1000e9a0 f   Qt5Widgets:Qt5Widgets.dll
 0001:0000d9a6       ?keyPressEvent@QWidget@@MAEXPAVQKeyEvent@@@Z 1000e9a6 f   Qt5Widgets:Qt5Widgets.dll
 0001:0000d9ac       ?keyReleaseEvent@QAbstractButton@@MAEXPAVQKeyEvent@@@Z 1000e9ac f   Qt5Widgets:Qt5Widgets.dll
 0001:0000d9b2       ?keyReleaseEvent@QAbstractSpinBox@@MAEXPAVQKeyEvent@@@Z 1000e9b2 f   Qt5Widgets:Qt5Widgets.dll
 0001:0000d9b8       ?keyReleaseEvent@QWidget@@MAEXPAVQKeyEvent@@@Z 1000e9b8 f   Qt5Widgets:Qt5Widgets.dll
 0001:0000d9be       ?layout@QLayout@@UAEPAV1@XZ 1000e9be f   Qt5Widgets:Qt5Widgets.dll
 0001:0000d9c4       ?layout@QLayoutItem@@UAEPAVQLayout@@XZ 1000e9c4 f   Qt5Widgets:Qt5Widgets.dll
 0001:0000d9ca       ?leaveEvent@QWidget@@MAEXPAVQEvent@@@Z 1000e9ca f   Qt5Widgets:Qt5Widgets.dll
 0001:0000d9d0       ?maximumSize@QBoxLayout@@UBE?AVQSize@@XZ 1000e9d0 f   Qt5Widgets:Qt5Widgets.dll
 0001:0000d9d6       ?maximumSize@QGridLayout@@UBE?AVQSize@@XZ 1000e9d6 f   Qt5Widgets:Qt5Widgets.dll
 0001:0000d9dc       ?maximumSize@QSpacerItem@@UBE?AVQSize@@XZ 1000e9dc f   Qt5Widgets:Qt5Widgets.dll
 0001:0000d9e2       ?metaObject@QDialogButtonBox@@UBEPBUQMetaObject@@XZ 1000e9e2 f   Qt5Widgets:Qt5Widgets.dll
 0001:0000d9e8       ?metaObject@QDoubleSpinBox@@UBEPBUQMetaObject@@XZ 1000e9e8 f   Qt5Widgets:Qt5Widgets.dll
 0001:0000d9ee       ?metaObject@QGridLayout@@UBEPBUQMetaObject@@XZ 1000e9ee f   Qt5Widgets:Qt5Widgets.dll
 0001:0000d9f4       ?metaObject@QGroupBox@@UBEPBUQMetaObject@@XZ 1000e9f4 f   Qt5Widgets:Qt5Widgets.dll
 0001:0000d9fa       ?metaObject@QHBoxLayout@@UBEPBUQMetaObject@@XZ 1000e9fa f   Qt5Widgets:Qt5Widgets.dll
 0001:0000da00       ?metaObject@QLabel@@UBEPBUQMetaObject@@XZ 1000ea00 f   Qt5Widgets:Qt5Widgets.dll
 0001:0000da06       ?metaObject@QPushButton@@UBEPBUQMetaObject@@XZ 1000ea06 f   Qt5Widgets:Qt5Widgets.dll
 0001:0000da0c       ?metaObject@QSpinBox@@UBEPBUQMetaObject@@XZ 1000ea0c f   Qt5Widgets:Qt5Widgets.dll
 0001:0000da12       ?metaObject@QTabWidget@@UBEPBUQMetaObject@@XZ 1000ea12 f   Qt5Widgets:Qt5Widgets.dll
 0001:0000da18       ?metaObject@QVBoxLayout@@UBEPBUQMetaObject@@XZ 1000ea18 f   Qt5Widgets:Qt5Widgets.dll
 0001:0000da1e       ?metaObject@QWidget@@UBEPBUQMetaObject@@XZ 1000ea1e f   Qt5Widgets:Qt5Widgets.dll
 0001:0000da24       ?metric@QWidget@@MBEHW4PaintDeviceMetric@QPaintDevice@@@Z 1000ea24 f   Qt5Widgets:Qt5Widgets.dll
 0001:0000da2a       ?minimumHeightForWidth@QBoxLayout@@UBEHH@Z 1000ea2a f   Qt5Widgets:Qt5Widgets.dll
 0001:0000da30       ?minimumHeightForWidth@QGridLayout@@UBEHH@Z 1000ea30 f   Qt5Widgets:Qt5Widgets.dll
 0001:0000da36       ?minimumHeightForWidth@QLayoutItem@@UBEHH@Z 1000ea36 f   Qt5Widgets:Qt5Widgets.dll
 0001:0000da3c       ?minimumSize@QBoxLayout@@UBE?AVQSize@@XZ 1000ea3c f   Qt5Widgets:Qt5Widgets.dll
 0001:0000da42       ?minimumSize@QGridLayout@@UBE?AVQSize@@XZ 1000ea42 f   Qt5Widgets:Qt5Widgets.dll
 0001:0000da48       ?minimumSize@QSpacerItem@@UBE?AVQSize@@XZ 1000ea48 f   Qt5Widgets:Qt5Widgets.dll
 0001:0000da4e       ?minimumSizeHint@QAbstractSpinBox@@UBE?AVQSize@@XZ 1000ea4e f   Qt5Widgets:Qt5Widgets.dll
 0001:0000da54       ?minimumSizeHint@QDialog@@UBE?AVQSize@@XZ 1000ea54 f   Qt5Widgets:Qt5Widgets.dll
 0001:0000da5a       ?minimumSizeHint@QGroupBox@@UBE?AVQSize@@XZ 1000ea5a f   Qt5Widgets:Qt5Widgets.dll
 0001:0000da60       ?minimumSizeHint@QLabel@@UBE?AVQSize@@XZ 1000ea60 f   Qt5Widgets:Qt5Widgets.dll
 0001:0000da66       ?minimumSizeHint@QPushButton@@UBE?AVQSize@@XZ 1000ea66 f   Qt5Widgets:Qt5Widgets.dll
 0001:0000da6c       ?minimumSizeHint@QTabWidget@@UBE?AVQSize@@XZ 1000ea6c f   Qt5Widgets:Qt5Widgets.dll
 0001:0000da72       ?minimumSizeHint@QWidget@@UBE?AVQSize@@XZ 1000ea72 f   Qt5Widgets:Qt5Widgets.dll
 0001:0000da78       ?mouseDoubleClickEvent@QWidget@@MAEXPAVQMouseEvent@@@Z 1000ea78 f   Qt5Widgets:Qt5Widgets.dll
 0001:0000da7e       ?mouseMoveEvent@QAbstractButton@@MAEXPAVQMouseEvent@@@Z 1000ea7e f   Qt5Widgets:Qt5Widgets.dll
 0001:0000da84       ?mouseMoveEvent@QAbstractSpinBox@@MAEXPAVQMouseEvent@@@Z 1000ea84 f   Qt5Widgets:Qt5Widgets.dll
 0001:0000da8a       ?mouseMoveEvent@QGroupBox@@MAEXPAVQMouseEvent@@@Z 1000ea8a f   Qt5Widgets:Qt5Widgets.dll
 0001:0000da90       ?mouseMoveEvent@QLabel@@MAEXPAVQMouseEvent@@@Z 1000ea90 f   Qt5Widgets:Qt5Widgets.dll
 0001:0000da96       ?mouseMoveEvent@QWidget@@MAEXPAVQMouseEvent@@@Z 1000ea96 f   Qt5Widgets:Qt5Widgets.dll
 0001:0000da9c       ?mousePressEvent@QAbstractButton@@MAEXPAVQMouseEvent@@@Z 1000ea9c f   Qt5Widgets:Qt5Widgets.dll
 0001:0000daa2       ?mousePressEvent@QAbstractSpinBox@@MAEXPAVQMouseEvent@@@Z 1000eaa2 f   Qt5Widgets:Qt5Widgets.dll
 0001:0000daa8       ?mousePressEvent@QGroupBox@@MAEXPAVQMouseEvent@@@Z 1000eaa8 f   Qt5Widgets:Qt5Widgets.dll
 0001:0000daae       ?mousePressEvent@QLabel@@MAEXPAVQMouseEvent@@@Z 1000eaae f   Qt5Widgets:Qt5Widgets.dll
 0001:0000dab4       ?mousePressEvent@QWidget@@MAEXPAVQMouseEvent@@@Z 1000eab4 f   Qt5Widgets:Qt5Widgets.dll
 0001:0000daba       ?mouseReleaseEvent@QAbstractButton@@MAEXPAVQMouseEvent@@@Z 1000eaba f   Qt5Widgets:Qt5Widgets.dll
 0001:0000dac0       ?mouseReleaseEvent@QAbstractSpinBox@@MAEXPAVQMouseEvent@@@Z 1000eac0 f   Qt5Widgets:Qt5Widgets.dll
 0001:0000dac6       ?mouseReleaseEvent@QGroupBox@@MAEXPAVQMouseEvent@@@Z 1000eac6 f   Qt5Widgets:Qt5Widgets.dll
 0001:0000dacc       ?mouseReleaseEvent@QLabel@@MAEXPAVQMouseEvent@@@Z 1000eacc f   Qt5Widgets:Qt5Widgets.dll
 0001:0000dad2       ?mouseReleaseEvent@QWidget@@MAEXPAVQMouseEvent@@@Z 1000ead2 f   Qt5Widgets:Qt5Widgets.dll
 0001:0000dad8       ?moveEvent@QWidget@@MAEXPAVQMoveEvent@@@Z 1000ead8 f   Qt5Widgets:Qt5Widgets.dll
 0001:0000dade       ?nativeEvent@QWidget@@MAE_NABVQByteArray@@PAXPAJ@Z 1000eade f   Qt5Widgets:Qt5Widgets.dll
 0001:0000dae4       ?nextCheckState@QAbstractButton@@MAEXXZ 1000eae4 f   Qt5Widgets:Qt5Widgets.dll
 0001:0000daea       ?open@QDialog@@UAEXXZ      1000eaea f   Qt5Widgets:Qt5Widgets.dll
 0001:0000daf0       ?paintEngine@QWidget@@UBEPAVQPaintEngine@@XZ 1000eaf0 f   Qt5Widgets:Qt5Widgets.dll
 0001:0000daf6       ?paintEvent@QAbstractSpinBox@@MAEXPAVQPaintEvent@@@Z 1000eaf6 f   Qt5Widgets:Qt5Widgets.dll
 0001:0000dafc       ?paintEvent@QGroupBox@@MAEXPAVQPaintEvent@@@Z 1000eafc f   Qt5Widgets:Qt5Widgets.dll
 0001:0000db02       ?paintEvent@QLabel@@MAEXPAVQPaintEvent@@@Z 1000eb02 f   Qt5Widgets:Qt5Widgets.dll
 0001:0000db08       ?paintEvent@QPushButton@@MAEXPAVQPaintEvent@@@Z 1000eb08 f   Qt5Widgets:Qt5Widgets.dll
 0001:0000db0e       ?paintEvent@QTabWidget@@MAEXPAVQPaintEvent@@@Z 1000eb0e f   Qt5Widgets:Qt5Widgets.dll
 0001:0000db14       ?paintEvent@QWidget@@MAEXPAVQPaintEvent@@@Z 1000eb14 f   Qt5Widgets:Qt5Widgets.dll
 0001:0000db1a       ?qt_metacall@QDialogButtonBox@@UAEHW4Call@QMetaObject@@HPAPAX@Z 1000eb1a f   Qt5Widgets:Qt5Widgets.dll
 0001:0000db20       ?qt_metacall@QDoubleSpinBox@@UAEHW4Call@QMetaObject@@HPAPAX@Z 1000eb20 f   Qt5Widgets:Qt5Widgets.dll
 0001:0000db26       ?qt_metacall@QGridLayout@@UAEHW4Call@QMetaObject@@HPAPAX@Z 1000eb26 f   Qt5Widgets:Qt5Widgets.dll
 0001:0000db2c       ?qt_metacall@QGroupBox@@UAEHW4Call@QMetaObject@@HPAPAX@Z 1000eb2c f   Qt5Widgets:Qt5Widgets.dll
 0001:0000db32       ?qt_metacall@QHBoxLayout@@UAEHW4Call@QMetaObject@@HPAPAX@Z 1000eb32 f   Qt5Widgets:Qt5Widgets.dll
 0001:0000db38       ?qt_metacall@QLabel@@UAEHW4Call@QMetaObject@@HPAPAX@Z 1000eb38 f   Qt5Widgets:Qt5Widgets.dll
 0001:0000db3e       ?qt_metacall@QPushButton@@UAEHW4Call@QMetaObject@@HPAPAX@Z 1000eb3e f   Qt5Widgets:Qt5Widgets.dll
 0001:0000db44       ?qt_metacall@QSpinBox@@UAEHW4Call@QMetaObject@@HPAPAX@Z 1000eb44 f   Qt5Widgets:Qt5Widgets.dll
 0001:0000db4a       ?qt_metacall@QTabWidget@@UAEHW4Call@QMetaObject@@HPAPAX@Z 1000eb4a f   Qt5Widgets:Qt5Widgets.dll
 0001:0000db50       ?qt_metacall@QVBoxLayout@@UAEHW4Call@QMetaObject@@HPAPAX@Z 1000eb50 f   Qt5Widgets:Qt5Widgets.dll
 0001:0000db56       ?qt_metacall@QWidget@@UAEHW4Call@QMetaObject@@HPAPAX@Z 1000eb56 f   Qt5Widgets:Qt5Widgets.dll
 0001:0000db5c       ?qt_metacast@QDialogButtonBox@@UAEPAXPBD@Z 1000eb5c f   Qt5Widgets:Qt5Widgets.dll
 0001:0000db62       ?qt_metacast@QDoubleSpinBox@@UAEPAXPBD@Z 1000eb62 f   Qt5Widgets:Qt5Widgets.dll
 0001:0000db68       ?qt_metacast@QGridLayout@@UAEPAXPBD@Z 1000eb68 f   Qt5Widgets:Qt5Widgets.dll
 0001:0000db6e       ?qt_metacast@QGroupBox@@UAEPAXPBD@Z 1000eb6e f   Qt5Widgets:Qt5Widgets.dll
 0001:0000db74       ?qt_metacast@QHBoxLayout@@UAEPAXPBD@Z 1000eb74 f   Qt5Widgets:Qt5Widgets.dll
 0001:0000db7a       ?qt_metacast@QLabel@@UAEPAXPBD@Z 1000eb7a f   Qt5Widgets:Qt5Widgets.dll
 0001:0000db80       ?qt_metacast@QPushButton@@UAEPAXPBD@Z 1000eb80 f   Qt5Widgets:Qt5Widgets.dll
 0001:0000db86       ?qt_metacast@QSpinBox@@UAEPAXPBD@Z 1000eb86 f   Qt5Widgets:Qt5Widgets.dll
 0001:0000db8c       ?qt_metacast@QTabWidget@@UAEPAXPBD@Z 1000eb8c f   Qt5Widgets:Qt5Widgets.dll
 0001:0000db92       ?qt_metacast@QVBoxLayout@@UAEPAXPBD@Z 1000eb92 f   Qt5Widgets:Qt5Widgets.dll
 0001:0000db98       ?qt_metacast@QWidget@@UAEPAXPBD@Z 1000eb98 f   Qt5Widgets:Qt5Widgets.dll
 0001:0000db9e       ?redirected@QWidget@@MBEPAVQPaintDevice@@PAVQPoint@@@Z 1000eb9e f   Qt5Widgets:Qt5Widgets.dll
 0001:0000dba4       ?reject@QDialog@@UAEXXZ    1000eba4 f   Qt5Widgets:Qt5Widgets.dll
 0001:0000dbaa       ?resizeEvent@QAbstractSpinBox@@MAEXPAVQResizeEvent@@@Z 1000ebaa f   Qt5Widgets:Qt5Widgets.dll
 0001:0000dbb0       ?resizeEvent@QDialog@@MAEXPAVQResizeEvent@@@Z 1000ebb0 f   Qt5Widgets:Qt5Widgets.dll
 0001:0000dbb6       ?resizeEvent@QGroupBox@@MAEXPAVQResizeEvent@@@Z 1000ebb6 f   Qt5Widgets:Qt5Widgets.dll
 0001:0000dbbc       ?resizeEvent@QTabWidget@@MAEXPAVQResizeEvent@@@Z 1000ebbc f   Qt5Widgets:Qt5Widgets.dll
 0001:0000dbc2       ?resizeEvent@QWidget@@MAEXPAVQResizeEvent@@@Z 1000ebc2 f   Qt5Widgets:Qt5Widgets.dll
 0001:0000dbc8       ?setGeometry@QBoxLayout@@UAEXABVQRect@@@Z 1000ebc8 f   Qt5Widgets:Qt5Widgets.dll
 0001:0000dbce       ?setGeometry@QGridLayout@@UAEXABVQRect@@@Z 1000ebce f   Qt5Widgets:Qt5Widgets.dll
 0001:0000dbd4       ?setGeometry@QSpacerItem@@UAEXABVQRect@@@Z 1000ebd4 f   Qt5Widgets:Qt5Widgets.dll
 0001:0000dbda       ?setVisible@QDialog@@UAEX_N@Z 1000ebda f   Qt5Widgets:Qt5Widgets.dll
 0001:0000dbe0       ?setVisible@QWidget@@UAEX_N@Z 1000ebe0 f   Qt5Widgets:Qt5Widgets.dll
 0001:0000dbe6       ?sharedPainter@QWidget@@MBEPAVQPainter@@XZ 1000ebe6 f   Qt5Widgets:Qt5Widgets.dll
 0001:0000dbec       ?showEvent@QAbstractSpinBox@@MAEXPAVQShowEvent@@@Z 1000ebec f   Qt5Widgets:Qt5Widgets.dll
 0001:0000dbf2       ?showEvent@QDialog@@MAEXPAVQShowEvent@@@Z 1000ebf2 f   Qt5Widgets:Qt5Widgets.dll
 0001:0000dbf8       ?showEvent@QTabWidget@@MAEXPAVQShowEvent@@@Z 1000ebf8 f   Qt5Widgets:Qt5Widgets.dll
 0001:0000dbfe       ?showEvent@QWidget@@MAEXPAVQShowEvent@@@Z 1000ebfe f   Qt5Widgets:Qt5Widgets.dll
 0001:0000dc04       ?sizeHint@QAbstractSpinBox@@UBE?AVQSize@@XZ 1000ec04 f   Qt5Widgets:Qt5Widgets.dll
 0001:0000dc0a       ?sizeHint@QBoxLayout@@UBE?AVQSize@@XZ 1000ec0a f   Qt5Widgets:Qt5Widgets.dll
 0001:0000dc10       ?sizeHint@QDialog@@UBE?AVQSize@@XZ 1000ec10 f   Qt5Widgets:Qt5Widgets.dll
 0001:0000dc16       ?sizeHint@QGridLayout@@UBE?AVQSize@@XZ 1000ec16 f   Qt5Widgets:Qt5Widgets.dll
 0001:0000dc1c       ?sizeHint@QLabel@@UBE?AVQSize@@XZ 1000ec1c f   Qt5Widgets:Qt5Widgets.dll
 0001:0000dc22       ?sizeHint@QPushButton@@UBE?AVQSize@@XZ 1000ec22 f   Qt5Widgets:Qt5Widgets.dll
 0001:0000dc28       ?sizeHint@QSpacerItem@@UBE?AVQSize@@XZ 1000ec28 f   Qt5Widgets:Qt5Widgets.dll
 0001:0000dc2e       ?sizeHint@QTabWidget@@UBE?AVQSize@@XZ 1000ec2e f   Qt5Widgets:Qt5Widgets.dll
 0001:0000dc34       ?sizeHint@QWidget@@UBE?AVQSize@@XZ 1000ec34 f   Qt5Widgets:Qt5Widgets.dll
 0001:0000dc3a       ?spacerItem@QLayoutItem@@UAEPAVQSpacerItem@@XZ 1000ec3a f   Qt5Widgets:Qt5Widgets.dll
 0001:0000dc40       ?spacerItem@QSpacerItem@@UAEPAV1@XZ 1000ec40 f   Qt5Widgets:Qt5Widgets.dll
 0001:0000dc46       ?stepBy@QAbstractSpinBox@@UAEXH@Z 1000ec46 f   Qt5Widgets:Qt5Widgets.dll
 0001:0000dc4c       ?stepEnabled@QAbstractSpinBox@@MBE?AV?$QFlags@W4StepEnabledFlag@QAbstractSpinBox@@@@XZ 1000ec4c f   Qt5Widgets:Qt5Widgets.dll
 0001:0000dc52       ?tabInserted@QTabWidget@@MAEXH@Z 1000ec52 f   Qt5Widgets:Qt5Widgets.dll
 0001:0000dc58       ?tabRemoved@QTabWidget@@MAEXH@Z 1000ec58 f   Qt5Widgets:Qt5Widgets.dll
 0001:0000dc5e       ?tabletEvent@QWidget@@MAEXPAVQTabletEvent@@@Z 1000ec5e f   Qt5Widgets:Qt5Widgets.dll
 0001:0000dc64       ?takeAt@QBoxLayout@@UAEPAVQLayoutItem@@H@Z 1000ec64 f   Qt5Widgets:Qt5Widgets.dll
 0001:0000dc6a       ?takeAt@QGridLayout@@UAEPAVQLayoutItem@@H@Z 1000ec6a f   Qt5Widgets:Qt5Widgets.dll
 0001:0000dc70       ?textFromValue@QDoubleSpinBox@@UBE?AVQString@@N@Z 1000ec70 f   Qt5Widgets:Qt5Widgets.dll
 0001:0000dc76       ?textFromValue@QSpinBox@@MBE?AVQString@@H@Z 1000ec76 f   Qt5Widgets:Qt5Widgets.dll
 0001:0000dc7c       ?timerEvent@QAbstractButton@@MAEXPAVQTimerEvent@@@Z 1000ec7c f   Qt5Widgets:Qt5Widgets.dll
 0001:0000dc82       ?timerEvent@QAbstractSpinBox@@MAEXPAVQTimerEvent@@@Z 1000ec82 f   Qt5Widgets:Qt5Widgets.dll
 0001:0000dc88       ?validate@QDoubleSpinBox@@UBE?AW4State@QValidator@@AAVQString@@AAH@Z 1000ec88 f   Qt5Widgets:Qt5Widgets.dll
 0001:0000dc8e       ?validate@QSpinBox@@MBE?AW4State@QValidator@@AAVQString@@AAH@Z 1000ec8e f   Qt5Widgets:Qt5Widgets.dll
 0001:0000dc94       ?valueFromText@QDoubleSpinBox@@UBENABVQString@@@Z 1000ec94 f   Qt5Widgets:Qt5Widgets.dll
 0001:0000dc9a       ?valueFromText@QSpinBox@@MBEHABVQString@@@Z 1000ec9a f   Qt5Widgets:Qt5Widgets.dll
 0001:0000dca0       ?wheelEvent@QAbstractSpinBox@@MAEXPAVQWheelEvent@@@Z 1000eca0 f   Qt5Widgets:Qt5Widgets.dll
 0001:0000dca6       ?wheelEvent@QWidget@@MAEXPAVQWheelEvent@@@Z 1000eca6 f   Qt5Widgets:Qt5Widgets.dll
 0001:0000dcac       ?widget@QLayoutItem@@UAEPAVQWidget@@XZ 1000ecac f   Qt5Widgets:Qt5Widgets.dll
 0001:0000dcb2       ?event@QAction@@MAE_NPAVQEvent@@@Z 1000ecb2 f   Qt5Widgets:Qt5Widgets.dll
 0001:0000dcb8       ?qt_metacast@QDialog@@UAEPAXPBD@Z 1000ecb8 f   Qt5Widgets:Qt5Widgets.dll
 0001:0000dcbe       ?qt_metacall@QDialog@@UAEHW4Call@QMetaObject@@HPAPAX@Z 1000ecbe f   Qt5Widgets:Qt5Widgets.dll
 0001:0000dcc4       ??0QIcon@@QAE@ABVQString@@@Z 1000ecc4 f   Qt5Gui:Qt5Gui.dll
 0001:0000dcca       ??1QIcon@@QAE@XZ           1000ecca f   Qt5Gui:Qt5Gui.dll
 0001:0000dcd0       ??1QByteArray@@QAE@XZ      1000ecd0 f   Qt5Core:Qt5Core.dll
 0001:0000dcd6       ?tr@QMetaObject@@QBE?AVQString@@PBD0H@Z 1000ecd6 f   Qt5Core:Qt5Core.dll
 0001:0000dcdc       ?connectSlotsByName@QMetaObject@@SAXPAVQObject@@@Z 1000ecdc f   Qt5Core:Qt5Core.dll
 0001:0000dce2       ??1Connection@QMetaObject@@QAE@XZ 1000ece2 f   Qt5Core:Qt5Core.dll
 0001:0000dce8       ??0QString@@QAE@XZ         1000ece8 f   Qt5Core:Qt5Core.dll
 0001:0000dcee       ??0QString@@QAE@ABV0@@Z    1000ecee f   Qt5Core:Qt5Core.dll
 0001:0000dcf4       ??1QString@@QAE@XZ         1000ecf4 f   Qt5Core:Qt5Core.dll
 0001:0000dcfa       ??4QString@@QAEAAV0@PBD@Z  1000ecfa f   Qt5Core:Qt5Core.dll
 0001:0000dd00       ?fromAscii_helper@QString@@CAPAU?$QTypedArrayData@G@@PBDH@Z 1000ed00 f   Qt5Core:Qt5Core.dll
 0001:0000dd06       ?objectName@QObject@@QBE?AVQString@@XZ 1000ed06 f   Qt5Core:Qt5Core.dll
 0001:0000dd0c       ?setObjectName@QObject@@QAEXABVQString@@@Z 1000ed0c f   Qt5Core:Qt5Core.dll
 0001:0000dd12       ?connect@QObject@@SA?AVConnection@QMetaObject@@PBV1@PBD01W4ConnectionType@Qt@@@Z 1000ed12 f   Qt5Core:Qt5Core.dll
 0001:0000dd18       ?connect@QObject@@QBE?AVConnection@QMetaObject@@PBV1@PBD1W4ConnectionType@Qt@@@Z 1000ed18 f   Qt5Core:Qt5Core.dll
 0001:0000dd1e       ?translate@QCoreApplication@@SA?AVQString@@PBD00H@Z 1000ed1e f   Qt5Core:Qt5Core.dll
 0001:0000dd24       ?childEvent@QObject@@MAEXPAVQChildEvent@@@Z 1000ed24 f   Qt5Core:Qt5Core.dll
 0001:0000dd2a       ?connectNotify@QObject@@MAEXABVQMetaMethod@@@Z 1000ed2a f   Qt5Core:Qt5Core.dll
 0001:0000dd30       ?customEvent@QObject@@MAEXPAVQEvent@@@Z 1000ed30 f   Qt5Core:Qt5Core.dll
 0001:0000dd36       ?disconnectNotify@QObject@@MAEXABVQMetaMethod@@@Z 1000ed36 f   Qt5Core:Qt5Core.dll
 0001:0000dd3c       ?event@QObject@@UAE_NPAVQEvent@@@Z 1000ed3c f   Qt5Core:Qt5Core.dll
 0001:0000dd42       ?eventFilter@QObject@@UAE_NPAV1@PAVQEvent@@@Z 1000ed42 f   Qt5Core:Qt5Core.dll
 0001:0000dd48       ?timerEvent@QObject@@MAEXPAVQTimerEvent@@@Z 1000ed48 f   Qt5Core:Qt5Core.dll
 0001:0000dd4e       ??8@YA_NABVQString@@0@Z    1000ed4e f   Qt5Core:Qt5Core.dll
 0001:0000dd54       ?detach_grow@QListData@@QAEPAUData@1@PAHH@Z 1000ed54 f   Qt5Core:Qt5Core.dll
 0001:0000dd5a       ?dispose@QListData@@SAXPAUData@1@@Z 1000ed5a f   Qt5Core:Qt5Core.dll
 0001:0000dd60       ?append@QListData@@QAEPAPAXXZ 1000ed60 f   Qt5Core:Qt5Core.dll
 0001:0000dd66       ?freeTree@QMapDataBase@@QAEXPAUQMapNodeBase@@H@Z 1000ed66 f   Qt5Core:Qt5Core.dll
 0001:0000dd6c       ?freeData@QMapDataBase@@SAXPAU1@@Z 1000ed6c f   Qt5Core:Qt5Core.dll
 0001:0000dd72       ?qBadAlloc@@YAXXZ          1000ed72 f   Qt5Core:Qt5Core.dll
 0001:0000dd78       ?data@QArrayData@@QAEPAXXZ 1000ed78 f   Qt5Core:Qt5Core.dll
 0001:0000dd7e       ?allocate@QArrayData@@SAPAU1@IIIV?$QFlags@W4AllocationOption@QArrayData@@@@@Z 1000ed7e f   Qt5Core:Qt5Core.dll
 0001:0000dd84       ?deallocate@QArrayData@@SAXPAU1@II@Z 1000ed84 f   Qt5Core:Qt5Core.dll
 0001:0000dd8a       ??AQByteArray@@QBEDH@Z     1000ed8a f   Qt5Core:Qt5Core.dll
 0001:0000dd90       ?cast@QMetaObject@@QBEPAVQObject@@PAV2@@Z 1000ed90 f   Qt5Core:Qt5Core.dll
 0001:0000dd96       ??0QChar@@QAE@UQLatin1Char@@@Z 1000ed96 f   Qt5Core:Qt5Core.dll
 0001:0000dd9c       ?arg@QString@@QBE?AV1@HHHVQChar@@@Z 1000ed9c f   Qt5Core:Qt5Core.dll
 0001:0000dda2       ?arg@QString@@QBE?AV1@ABV1@HVQChar@@@Z 1000eda2 f   Qt5Core:Qt5Core.dll
 0001:0000dda8       ?detach@QListData@@QAEPAUData@1@H@Z 1000eda8 f   Qt5Core:Qt5Core.dll
 0001:0000ddae       ?sender@QObject@@IBEPAV1@XZ 1000edae f   Qt5Core:Qt5Core.dll
 0001:0000ddb4       ?getAndRef@ExternalRefCountData@QtSharedPointer@@SAPAU12@PBVQObject@@@Z 1000edb4 f   Qt5Core:Qt5Core.dll
 0001:0000ddba       ??4QString@@QAEAAV0@ABV0@@Z 1000edba f   Qt5Core:Qt5Core.dll
 0001:0000ddc0       ?number@QString@@SA?AV1@HH@Z 1000edc0 f   Qt5Core:Qt5Core.dll
 0001:0000ddc6       ?number@QString@@SA?AV1@NDH@Z 1000edc6 f   Qt5Core:Qt5Core.dll
 0001:0000ddcc       ??0QByteArray@@QAE@ABV0@@Z 1000edcc f   Qt5Core:Qt5Core.dll
 0001:0000ddd2       ?append@QString@@QAEAAV1@ABV1@@Z 1000edd2 f   Qt5Core:Qt5Core.dll
 0001:0000ddd8       ?fromUtf8@QString@@SA?AV1@PBDH@Z 1000edd8 f   Qt5Core:Qt5Core.dll
 0001:0000ddde       ?tr@QObject@@SA?AVQString@@PBD0H@Z 1000edde f   Qt5Core:Qt5Core.dll
 0001:0000dde4       ??1QVariant@@QAE@XZ        1000ede4 f   Qt5Core:Qt5Core.dll
 0001:0000ddea       ??0QVariant@@QAE@H@Z       1000edea f   Qt5Core:Qt5Core.dll
 0001:0000ddf0       ??0QVariant@@QAE@N@Z       1000edf0 f   Qt5Core:Qt5Core.dll
 0001:0000ddf6       ?toInt@QVariant@@QBEHPA_N@Z 1000edf6 f   Qt5Core:Qt5Core.dll
 0001:0000ddfc       ?toDouble@QVariant@@QBENPA_N@Z 1000edfc f   Qt5Core:Qt5Core.dll
 0001:0000de02       ?dynamicMetaObject@QObjectData@@QBEPAUQMetaObject@@XZ 1000ee02 f   Qt5Core:Qt5Core.dll
 0001:0000de08       ?qt_metacast@QObject@@UAEPAXPBD@Z 1000ee08 f   Qt5Core:Qt5Core.dll
 0001:0000de0e       ?qt_metacall@QObject@@UAEHW4Call@QMetaObject@@HPAPAX@Z 1000ee0e f   Qt5Core:Qt5Core.dll
 0001:0000de14       ??0QByteArray@@QAE@XZ      1000ee14 f   Qt5Core:Qt5Core.dll
 0001:0000de1a       ?reserve@QByteArray@@QAEXH@Z 1000ee1a f   Qt5Core:Qt5Core.dll
 0001:0000de20       ?append@QByteArray@@QAEAAV1@D@Z 1000ee20 f   Qt5Core:Qt5Core.dll
 0001:0000de26       ?append@QByteArray@@QAEAAV1@PBD@Z 1000ee26 f   Qt5Core:Qt5Core.dll
 0001:0000de2c       ?className@QMetaObject@@QBEPBDXZ 1000ee2c f   Qt5Core:Qt5Core.dll
 0001:0000de32       ?registerNormalizedType@QMetaType@@SAHABVQByteArray@@P6AXPAX@ZP6APAXPBX@Z2P6APAX13@ZHV?$QFlags@W4TypeFlag@QMetaType@@@@PBUQMetaObject@@@Z 1000ee32 f   Qt5Core:Qt5Core.dll
 0001:0000de38       ?registerNormalizedTypedef@QMetaType@@SAHABVQByteArray@@H@Z 1000ee38 f   Qt5Core:Qt5Core.dll
 0001:0000de3e       ?qRegisterResourceData@@YA_NHPBE00@Z 1000ee3e f   Qt5Core:Qt5Core.dll
 0001:0000de44       ?qUnregisterResourceData@@YA_NHPBE00@Z 1000ee44 f   Qt5Core:Qt5Core.dll
 0001:0000de4a       ?_Xbad_alloc@std@@YAXXZ    1000ee4a f   msvcprt:MSVCP120.dll
 0001:0000de50       ?_Xlength_error@std@@YAXPBD@Z 1000ee50 f   msvcprt:MSVCP120.dll
 0001:0000de56       ?_Xout_of_range@std@@YAXPBD@Z 1000ee56 f   msvcprt:MSVCP120.dll
 0001:0000de5c       ?_Syserror_map@std@@YAPBDH@Z 1000ee5c f   msvcprt:MSVCP120.dll
 0001:0000de62       ?_Winerror_map@std@@YAPBDH@Z 1000ee62 f   msvcprt:MSVCP120.dll
 0001:0000de68       __purecall                 1000ee68 f   MSVCRT:MSVCR120.dll
 0001:0000de6e       ??2@YAPAXI@Z               1000ee6e f   MSVCRT:MSVCR120.dll
 0001:0000de74       ??3@YAXPAX@Z               1000ee74 f   MSVCRT:MSVCR120.dll
 0001:0000de7a       ___atonexitinit            1000ee7a f   MSVCRT:atonexit.obj
 0001:0000deb6       __onexit                   1000eeb6 f   MSVCRT:atonexit.obj
 0001:0000df5f       _atexit                    1000ef5f f   MSVCRT:atonexit.obj
 0001:0000df74       _memmove                   1000ef74 f   MSVCRT:MSVCR120.dll
 0001:0000df7a       __hypot                    1000ef7a f   MSVCRT:MSVCR120.dll
 0001:0000df80       @__security_check_cookie@4 1000ef80 f   MSVCRT:secchk.obj
 0001:0000df90       __CxxThrowException@8      1000ef90 f   MSVCRT:MSVCR120.dll
 0001:0000df96       ___CxxFrameHandler3        1000ef96 f   MSVCRT:MSVCR120.dll
 0001:0000df9c       _memcpy                    1000ef9c f   MSVCRT:MSVCR120.dll
 0001:0000dfa2       ??0type_info@@AAE@ABV0@@Z  1000efa2 f   MSVCRT:ti_inst.obj
 0001:0000dfad       ??4type_info@@AAEAAV0@ABV0@@Z 1000efad f   MSVCRT:ti_inst.obj
 0001:0000dfb2       ??_Etype_info@@UAEPAXI@Z   1000efb2 f i MSVCRT:ti_inst.obj
 0001:0000e000       _memset                    1000f000 f   MSVCRT:MSVCR120.dll
 0001:0000e052       _NtCurrentTeb              1000f052 f i MSVCRT:crtdll.obj
 0001:0000e059       __CRT_INIT@12              1000f059 f   MSVCRT:crtdll.obj
 0001:0000e250       __DllMainCRTStartup@12     1000f250 f   MSVCRT:crtdll.obj
 0001:0000e3a6       __lock                     1000f3a6 f   MSVCRT:MSVCR120.dll
 0001:0000e3ac       __unlock                   1000f3ac f   MSVCRT:MSVCR120.dll
 0001:0000e3b2       __calloc_crt               1000f3b2 f   MSVCRT:MSVCR120.dll
 0001:0000e3b8       ___dllonexit               1000f3b8 f   MSVCRT:MSVCR120.dll
 0001:0000e3c0       __SEH_prolog4              1000f3c0 f   MSVCRT:sehprolg4.obj
 0001:0000e405       __SEH_epilog4              1000f405 f   MSVCRT:sehprolg4.obj
 0001:0000e419       __except_handler4          1000f419 f   MSVCRT:chandler4gs.obj
 0001:0000e43c       ___raise_securityfailure   1000f43c f   MSVCRT:gs_report.obj
 0001:0000e479       ___report_gsfailure        1000f479 f   MSVCRT:gs_report.obj
 0001:0000e574       ___report_rangecheckfailure 1000f574 f   MSVCRT:gs_report.obj
 0001:0000e580       ___report_securityfailure  1000f580 f   MSVCRT:gs_report.obj
 0001:0000e650       ___report_securityfailureEx 1000f650 f   MSVCRT:gs_report.obj
 0001:0000e766       ??_M@YGXPAXIHP6EX0@Z@Z     1000f766 f   MSVCRT:ehvecdtr.obj
 0001:0000e7ee       ?__ArrayUnwind@@YGXPAXIHP6EX0@Z@Z 1000f7ee f   MSVCRT:ehvecdtr.obj
 0001:0000e84c       ??1type_info@@UAE@XZ       1000f84c f   MSVCRT:MSVCR120.dll
 0001:0000e852       ___CppXcptFilter           1000f852 f   MSVCRT:MSVCR120.dll
 0001:0000e858       __amsg_exit                1000f858 f   MSVCRT:MSVCR120.dll
 0001:0000e860       __FindPESection            1000f860 f   MSVCRT:pesect.obj
 0001:0000e8b0       __IsNonwritableInCurrentImage 1000f8b0 f   MSVCRT:pesect.obj
 0001:0000e970       __ValidateImageBase        1000f970 f   MSVCRT:pesect.obj
 0001:0000e9a2       _free                      1000f9a2 f   MSVCRT:MSVCR120.dll
 0001:0000e9a8       ___security_init_cookie    1000f9a8 f   MSVCRT:gs_support.obj
 0001:0000ea44       _DllMain@12                1000fa44 f   MSVCRT:dllmain.obj
 0001:0000ea66       __malloc_crt               1000fa66 f   MSVCRT:MSVCR120.dll
 0001:0000ea6c       __RTC_Initialize           1000fa6c f   MSVCRT:initsect.obj
 0001:0000ea8c       __RTC_Terminate            1000fa8c f   MSVCRT:initsect.obj
 0001:0000eaac       __initterm                 1000faac f   MSVCRT:MSVCR120.dll
 0001:0000eab2       __initterm_e               1000fab2 f   MSVCRT:MSVCR120.dll
 0001:0000eab8       ___clean_type_info_names   1000fab8 f   MSVCRT:tncleanup.obj
 0001:0000eac4       __except_handler4_common   1000fac4 f   MSVCRT:MSVCR120.dll
 0001:0000eaca       __crt_debugger_hook        1000faca f   MSVCRT:MSVCR120.dll
 0001:0000ead0       ___crtUnhandledException   1000fad0 f   MSVCRT:MSVCR120.dll
 0001:0000ead6       ___crtTerminateProcess     1000fad6 f   MSVCRT:MSVCR120.dll
 0001:0000eadc       ?terminate@@YAXXZ          1000fadc f   MSVCRT:MSVCR120.dll
 0001:0000eae2       ___clean_type_info_names_internal 1000fae2 f   MSVCRT:MSVCR120.dll
 0001:0000eae8       _EncodePointer@4           1000fae8 f   kernel32:KERNEL32.dll
 0001:0000eaee       _DecodePointer@4           1000faee f   kernel32:KERNEL32.dll
 0001:0000eaf4       _IsDebuggerPresent@0       1000faf4 f   kernel32:KERNEL32.dll
 0001:0000eafa       _IsProcessorFeaturePresent@4 1000fafa f   kernel32:KERNEL32.dll
 0001:0000eb00       _QueryPerformanceCounter@4 1000fb00 f   kernel32:KERNEL32.dll
 0001:0000eb06       _GetCurrentProcessId@0     1000fb06 f   kernel32:KERNEL32.dll
 0001:0000eb0c       _GetCurrentThreadId@0      1000fb0c f   kernel32:KERNEL32.dll
 0001:0000eb12       _GetSystemTimeAsFileTime@4 1000fb12 f   kernel32:KERNEL32.dll
 0001:0000eb18       _DisableThreadLibraryCalls@4 1000fb18 f   kernel32:KERNEL32.dll
 0002:00000000       __imp__DisableThreadLibraryCalls@4 10013000     kernel32:KERNEL32.dll
 0002:00000004       __imp__GetSystemTimeAsFileTime@4 10013004     kernel32:KERNEL32.dll
 0002:00000008       __imp__GetCurrentThreadId@0 10013008     kernel32:KERNEL32.dll
 0002:0000000c       __imp__GetCurrentProcessId@0 1001300c     kernel32:KERNEL32.dll
 0002:00000010       __imp__QueryPerformanceCounter@4 10013010     kernel32:KERNEL32.dll
 0002:00000014       __imp__IsProcessorFeaturePresent@4 10013014     kernel32:KERNEL32.dll
 0002:00000018       __imp__IsDebuggerPresent@0 10013018     kernel32:KERNEL32.dll
 0002:0000001c       __imp__DecodePointer@4     1001301c     kernel32:KERNEL32.dll
 0002:00000020       __imp__EncodePointer@4     10013020     kernel32:KERNEL32.dll
 0002:00000024       \177KERNEL32_NULL_THUNK_DATA 10013024     kernel32:KERNEL32.dll
 0002:00000028       __imp_?_Xlength_error@std@@YAXPBD@Z 10013028     msvcprt:MSVCP120.dll
 0002:0000002c       __imp_?_Xout_of_range@std@@YAXPBD@Z 1001302c     msvcprt:MSVCP120.dll
 0002:00000030       __imp_?_Syserror_map@std@@YAPBDH@Z 10013030     msvcprt:MSVCP120.dll
 0002:00000034       __imp_?_Winerror_map@std@@YAPBDH@Z 10013034     msvcprt:MSVCP120.dll
 0002:00000038       __imp_?_Xbad_alloc@std@@YAXXZ 10013038     msvcprt:MSVCP120.dll
 0002:0000003c       \177MSVCP120_NULL_THUNK_DATA 1001303c     msvcprt:MSVCP120.dll
 0002:00000040       __imp___initterm_e         10013040     MSVCRT:MSVCR120.dll
 0002:00000044       __imp___initterm           10013044     MSVCRT:MSVCR120.dll
 0002:00000048       __imp___malloc_crt         10013048     MSVCRT:MSVCR120.dll
 0002:0000004c       __imp__free                1001304c     MSVCRT:MSVCR120.dll
 0002:00000050       __imp___amsg_exit          10013050     MSVCRT:MSVCR120.dll
 0002:00000054       __imp___except_handler4_common 10013054     MSVCRT:MSVCR120.dll
 0002:00000058       __imp_??1type_info@@UAE@XZ 10013058     MSVCRT:MSVCR120.dll
 0002:0000005c       __imp___onexit             1001305c     MSVCRT:MSVCR120.dll
 0002:00000060       __imp____dllonexit         10013060     MSVCRT:MSVCR120.dll
 0002:00000064       __imp___calloc_crt         10013064     MSVCRT:MSVCR120.dll
 0002:00000068       __imp___unlock             10013068     MSVCRT:MSVCR120.dll
 0002:0000006c       __imp___lock               1001306c     MSVCRT:MSVCR120.dll
 0002:00000070       __imp__memset              10013070     MSVCRT:MSVCR120.dll
 0002:00000074       __imp__memcpy              10013074     MSVCRT:MSVCR120.dll
 0002:00000078       __imp____CxxFrameHandler3  10013078     MSVCRT:MSVCR120.dll
 0002:0000007c       __imp___CxxThrowException@8 1001307c     MSVCRT:MSVCR120.dll
 0002:00000080       __imp___hypot              10013080     MSVCRT:MSVCR120.dll
 0002:00000084       __imp__memmove             10013084     MSVCRT:MSVCR120.dll
 0002:00000088       __imp_??3@YAXPAX@Z         10013088     MSVCRT:MSVCR120.dll
 0002:0000008c       __imp_??2@YAPAXI@Z         1001308c     MSVCRT:MSVCR120.dll
 0002:00000090       __imp___purecall           10013090     MSVCRT:MSVCR120.dll
 0002:00000094       __imp___crt_debugger_hook  10013094     MSVCRT:MSVCR120.dll
 0002:00000098       __imp____crtUnhandledException 10013098     MSVCRT:MSVCR120.dll
 0002:0000009c       __imp____crtTerminateProcess 1001309c     MSVCRT:MSVCR120.dll
 0002:000000a0       __imp_?terminate@@YAXXZ    100130a0     MSVCRT:MSVCR120.dll
 0002:000000a4       __imp____clean_type_info_names_internal 100130a4     MSVCRT:MSVCR120.dll
 0002:000000a8       __imp____CppXcptFilter     100130a8     MSVCRT:MSVCR120.dll
 0002:000000ac       \177MSVCR120_NULL_THUNK_DATA 100130ac     MSVCRT:MSVCR120.dll
 0002:000000b0       __imp_?qUnregisterResourceData@@YA_NHPBE00@Z 100130b0     Qt5Core:Qt5Core.dll
 0002:000000b4       __imp_?qRegisterResourceData@@YA_NHPBE00@Z 100130b4     Qt5Core:Qt5Core.dll
 0002:000000b8       __imp_?registerNormalizedTypedef@QMetaType@@SAHABVQByteArray@@H@Z 100130b8     Qt5Core:Qt5Core.dll
 0002:000000bc       __imp_?registerNormalizedType@QMetaType@@SAHABVQByteArray@@P6AXPAX@ZP6APAXPBX@Z2P6APAX13@ZHV?$QFlags@W4TypeFlag@QMetaType@@@@PBUQMetaObject@@@Z 100130bc     Qt5Core:Qt5Core.dll
 0002:000000c0       __imp_?className@QMetaObject@@QBEPBDXZ 100130c0     Qt5Core:Qt5Core.dll
 0002:000000c4       __imp_?append@QByteArray@@QAEAAV1@PBD@Z 100130c4     Qt5Core:Qt5Core.dll
 0002:000000c8       __imp_?append@QByteArray@@QAEAAV1@D@Z 100130c8     Qt5Core:Qt5Core.dll
 0002:000000cc       __imp_?reserve@QByteArray@@QAEXH@Z 100130cc     Qt5Core:Qt5Core.dll
 0002:000000d0       __imp_??0QByteArray@@QAE@XZ 100130d0     Qt5Core:Qt5Core.dll
 0002:000000d4       __imp_?staticMetaObject@QObject@@2UQMetaObject@@B 100130d4     Qt5Core:Qt5Core.dll
 0002:000000d8       __imp_?qt_metacall@QObject@@UAEHW4Call@QMetaObject@@HPAPAX@Z 100130d8     Qt5Core:Qt5Core.dll
 0002:000000dc       __imp_?qt_metacast@QObject@@UAEPAXPBD@Z 100130dc     Qt5Core:Qt5Core.dll
 0002:000000e0       __imp_?dynamicMetaObject@QObjectData@@QBEPAUQMetaObject@@XZ 100130e0     Qt5Core:Qt5Core.dll
 0002:000000e4       __imp_?toDouble@QVariant@@QBENPA_N@Z 100130e4     Qt5Core:Qt5Core.dll
 0002:000000e8       __imp_?toInt@QVariant@@QBEHPA_N@Z 100130e8     Qt5Core:Qt5Core.dll
 0002:000000ec       __imp_??0QVariant@@QAE@N@Z 100130ec     Qt5Core:Qt5Core.dll
 0002:000000f0       __imp_??0QVariant@@QAE@H@Z 100130f0     Qt5Core:Qt5Core.dll
 0002:000000f4       __imp_??1QVariant@@QAE@XZ  100130f4     Qt5Core:Qt5Core.dll
 0002:000000f8       __imp_?tr@QObject@@SA?AVQString@@PBD0H@Z 100130f8     Qt5Core:Qt5Core.dll
 0002:000000fc       __imp_?fromUtf8@QString@@SA?AV1@PBDH@Z 100130fc     Qt5Core:Qt5Core.dll
 0002:00000100       __imp_?append@QString@@QAEAAV1@ABV1@@Z 10013100     Qt5Core:Qt5Core.dll
 0002:00000104       __imp_??0QByteArray@@QAE@ABV0@@Z 10013104     Qt5Core:Qt5Core.dll
 0002:00000108       __imp_?number@QString@@SA?AV1@NDH@Z 10013108     Qt5Core:Qt5Core.dll
 0002:0000010c       __imp_?number@QString@@SA?AV1@HH@Z 1001310c     Qt5Core:Qt5Core.dll
 0002:00000110       __imp_??4QString@@QAEAAV0@ABV0@@Z 10013110     Qt5Core:Qt5Core.dll
 0002:00000114       __imp_?getAndRef@ExternalRefCountData@QtSharedPointer@@SAPAU12@PBVQObject@@@Z 10013114     Qt5Core:Qt5Core.dll
 0002:00000118       __imp_?sender@QObject@@IBEPAV1@XZ 10013118     Qt5Core:Qt5Core.dll
 0002:0000011c       __imp_?detach@QListData@@QAEPAUData@1@H@Z 1001311c     Qt5Core:Qt5Core.dll
 0002:00000120       __imp_?arg@QString@@QBE?AV1@ABV1@HVQChar@@@Z 10013120     Qt5Core:Qt5Core.dll
 0002:00000124       __imp_?arg@QString@@QBE?AV1@HHHVQChar@@@Z 10013124     Qt5Core:Qt5Core.dll
 0002:00000128       __imp_??0QChar@@QAE@UQLatin1Char@@@Z 10013128     Qt5Core:Qt5Core.dll
 0002:0000012c       __imp_?cast@QMetaObject@@QBEPAVQObject@@PAV2@@Z 1001312c     Qt5Core:Qt5Core.dll
 0002:00000130       __imp_?shared_null@QArrayData@@2QBU1@B 10013130     Qt5Core:Qt5Core.dll
 0002:00000134       __imp_??AQByteArray@@QBEDH@Z 10013134     Qt5Core:Qt5Core.dll
 0002:00000138       __imp_?deallocate@QArrayData@@SAXPAU1@II@Z 10013138     Qt5Core:Qt5Core.dll
 0002:0000013c       __imp_?allocate@QArrayData@@SAPAU1@IIIV?$QFlags@W4AllocationOption@QArrayData@@@@@Z 1001313c     Qt5Core:Qt5Core.dll
 0002:00000140       __imp_?data@QArrayData@@QAEPAXXZ 10013140     Qt5Core:Qt5Core.dll
 0002:00000144       __imp_?qBadAlloc@@YAXXZ    10013144     Qt5Core:Qt5Core.dll
 0002:00000148       __imp_?shared_null@QMapDataBase@@2U1@B 10013148     Qt5Core:Qt5Core.dll
 0002:0000014c       __imp_?shared_null@QListData@@2UData@1@B 1001314c     Qt5Core:Qt5Core.dll
 0002:00000150       __imp_?freeData@QMapDataBase@@SAXPAU1@@Z 10013150     Qt5Core:Qt5Core.dll
 0002:00000154       __imp_?freeTree@QMapDataBase@@QAEXPAUQMapNodeBase@@H@Z 10013154     Qt5Core:Qt5Core.dll
 0002:00000158       __imp_?append@QListData@@QAEPAPAXXZ 10013158     Qt5Core:Qt5Core.dll
 0002:0000015c       __imp_?dispose@QListData@@SAXPAUData@1@@Z 1001315c     Qt5Core:Qt5Core.dll
 0002:00000160       __imp_?detach_grow@QListData@@QAEPAUData@1@PAHH@Z 10013160     Qt5Core:Qt5Core.dll
 0002:00000164       __imp_??8@YA_NABVQString@@0@Z 10013164     Qt5Core:Qt5Core.dll
 0002:00000168       __imp_?timerEvent@QObject@@MAEXPAVQTimerEvent@@@Z 10013168     Qt5Core:Qt5Core.dll
 0002:0000016c       __imp_?eventFilter@QObject@@UAE_NPAV1@PAVQEvent@@@Z 1001316c     Qt5Core:Qt5Core.dll
 0002:00000170       __imp_?event@QObject@@UAE_NPAVQEvent@@@Z 10013170     Qt5Core:Qt5Core.dll
 0002:00000174       __imp_?disconnectNotify@QObject@@MAEXABVQMetaMethod@@@Z 10013174     Qt5Core:Qt5Core.dll
 0002:00000178       __imp_?customEvent@QObject@@MAEXPAVQEvent@@@Z 10013178     Qt5Core:Qt5Core.dll
 0002:0000017c       __imp_?connectNotify@QObject@@MAEXABVQMetaMethod@@@Z 1001317c     Qt5Core:Qt5Core.dll
 0002:00000180       __imp_?childEvent@QObject@@MAEXPAVQChildEvent@@@Z 10013180     Qt5Core:Qt5Core.dll
 0002:00000184       __imp_?translate@QCoreApplication@@SA?AVQString@@PBD00H@Z 10013184     Qt5Core:Qt5Core.dll
 0002:00000188       __imp_?connect@QObject@@QBE?AVConnection@QMetaObject@@PBV1@PBD1W4ConnectionType@Qt@@@Z 10013188     Qt5Core:Qt5Core.dll
 0002:0000018c       __imp_?connect@QObject@@SA?AVConnection@QMetaObject@@PBV1@PBD01W4ConnectionType@Qt@@@Z 1001318c     Qt5Core:Qt5Core.dll
 0002:00000190       __imp_?setObjectName@QObject@@QAEXABVQString@@@Z 10013190     Qt5Core:Qt5Core.dll
 0002:00000194       __imp_?objectName@QObject@@QBE?AVQString@@XZ 10013194     Qt5Core:Qt5Core.dll
 0002:00000198       __imp_?fromAscii_helper@QString@@CAPAU?$QTypedArrayData@G@@PBDH@Z 10013198     Qt5Core:Qt5Core.dll
 0002:0000019c       __imp_??4QString@@QAEAAV0@PBD@Z 1001319c     Qt5Core:Qt5Core.dll
 0002:000001a0       __imp_??1QString@@QAE@XZ   100131a0     Qt5Core:Qt5Core.dll
 0002:000001a4       __imp_??0QString@@QAE@ABV0@@Z 100131a4     Qt5Core:Qt5Core.dll
 0002:000001a8       __imp_??0QString@@QAE@XZ   100131a8     Qt5Core:Qt5Core.dll
 0002:000001ac       __imp_??1Connection@QMetaObject@@QAE@XZ 100131ac     Qt5Core:Qt5Core.dll
 0002:000001b0       __imp_?connectSlotsByName@QMetaObject@@SAXPAVQObject@@@Z 100131b0     Qt5Core:Qt5Core.dll
 0002:000001b4       __imp_?tr@QMetaObject@@QBE?AVQString@@PBD0H@Z 100131b4     Qt5Core:Qt5Core.dll
 0002:000001b8       __imp_??1QByteArray@@QAE@XZ 100131b8     Qt5Core:Qt5Core.dll
 0002:000001bc       \177Qt5Core_NULL_THUNK_DATA 100131bc     Qt5Core:Qt5Core.dll
 0002:000001c0       __imp_??1QIcon@@QAE@XZ     100131c0     Qt5Gui:Qt5Gui.dll
 0002:000001c4       __imp_??0QIcon@@QAE@ABVQString@@@Z 100131c4     Qt5Gui:Qt5Gui.dll
 0002:000001c8       \177Qt5Gui_NULL_THUNK_DATA 100131c8     Qt5Gui:Qt5Gui.dll
 0002:000001cc       __imp_?staticMetaObject@QDialog@@2UQMetaObject@@B 100131cc     Qt5Widgets:Qt5Widgets.dll
 0002:000001d0       __imp_?qt_metacall@QDialog@@UAEHW4Call@QMetaObject@@HPAPAX@Z 100131d0     Qt5Widgets:Qt5Widgets.dll
 0002:000001d4       __imp_?qt_metacast@QDialog@@UAEPAXPBD@Z 100131d4     Qt5Widgets:Qt5Widgets.dll
 0002:000001d8       __imp_?event@QAction@@MAE_NPAVQEvent@@@Z 100131d8     Qt5Widgets:Qt5Widgets.dll
 0002:000001dc       __imp_?widget@QLayoutItem@@UAEPAVQWidget@@XZ 100131dc     Qt5Widgets:Qt5Widgets.dll
 0002:000001e0       __imp_?wheelEvent@QWidget@@MAEXPAVQWheelEvent@@@Z 100131e0     Qt5Widgets:Qt5Widgets.dll
 0002:000001e4       __imp_?wheelEvent@QAbstractSpinBox@@MAEXPAVQWheelEvent@@@Z 100131e4     Qt5Widgets:Qt5Widgets.dll
 0002:000001e8       __imp_?valueFromText@QSpinBox@@MBEHABVQString@@@Z 100131e8     Qt5Widgets:Qt5Widgets.dll
 0002:000001ec       __imp_?valueFromText@QDoubleSpinBox@@UBENABVQString@@@Z 100131ec     Qt5Widgets:Qt5Widgets.dll
 0002:000001f0       __imp_?validate@QSpinBox@@MBE?AW4State@QValidator@@AAVQString@@AAH@Z 100131f0     Qt5Widgets:Qt5Widgets.dll
 0002:000001f4       __imp_?validate@QDoubleSpinBox@@UBE?AW4State@QValidator@@AAVQString@@AAH@Z 100131f4     Qt5Widgets:Qt5Widgets.dll
 0002:000001f8       __imp_?timerEvent@QAbstractSpinBox@@MAEXPAVQTimerEvent@@@Z 100131f8     Qt5Widgets:Qt5Widgets.dll
 0002:000001fc       __imp_?timerEvent@QAbstractButton@@MAEXPAVQTimerEvent@@@Z 100131fc     Qt5Widgets:Qt5Widgets.dll
 0002:00000200       __imp_?textFromValue@QSpinBox@@MBE?AVQString@@H@Z 10013200     Qt5Widgets:Qt5Widgets.dll
 0002:00000204       __imp_?textFromValue@QDoubleSpinBox@@UBE?AVQString@@N@Z 10013204     Qt5Widgets:Qt5Widgets.dll
 0002:00000208       __imp_?takeAt@QGridLayout@@UAEPAVQLayoutItem@@H@Z 10013208     Qt5Widgets:Qt5Widgets.dll
 0002:0000020c       __imp_?takeAt@QBoxLayout@@UAEPAVQLayoutItem@@H@Z 1001320c     Qt5Widgets:Qt5Widgets.dll
 0002:00000210       __imp_?tabletEvent@QWidget@@MAEXPAVQTabletEvent@@@Z 10013210     Qt5Widgets:Qt5Widgets.dll
 0002:00000214       __imp_?tabRemoved@QTabWidget@@MAEXH@Z 10013214     Qt5Widgets:Qt5Widgets.dll
 0002:00000218       __imp_?tabInserted@QTabWidget@@MAEXH@Z 10013218     Qt5Widgets:Qt5Widgets.dll
 0002:0000021c       __imp_?stepEnabled@QAbstractSpinBox@@MBE?AV?$QFlags@W4StepEnabledFlag@QAbstractSpinBox@@@@XZ 1001321c     Qt5Widgets:Qt5Widgets.dll
 0002:00000220       __imp_?stepBy@QAbstractSpinBox@@UAEXH@Z 10013220     Qt5Widgets:Qt5Widgets.dll
 0002:00000224       __imp_?spacerItem@QSpacerItem@@UAEPAV1@XZ 10013224     Qt5Widgets:Qt5Widgets.dll
 0002:00000228       __imp_?spacerItem@QLayoutItem@@UAEPAVQSpacerItem@@XZ 10013228     Qt5Widgets:Qt5Widgets.dll
 0002:0000022c       __imp_?sizeHint@QWidget@@UBE?AVQSize@@XZ 1001322c     Qt5Widgets:Qt5Widgets.dll
 0002:00000230       __imp_?sizeHint@QTabWidget@@UBE?AVQSize@@XZ 10013230     Qt5Widgets:Qt5Widgets.dll
 0002:00000234       __imp_?sizeHint@QSpacerItem@@UBE?AVQSize@@XZ 10013234     Qt5Widgets:Qt5Widgets.dll
 0002:00000238       __imp_?sizeHint@QPushButton@@UBE?AVQSize@@XZ 10013238     Qt5Widgets:Qt5Widgets.dll
 0002:0000023c       __imp_?sizeHint@QLabel@@UBE?AVQSize@@XZ 1001323c     Qt5Widgets:Qt5Widgets.dll
 0002:00000240       __imp_?sizeHint@QGridLayout@@UBE?AVQSize@@XZ 10013240     Qt5Widgets:Qt5Widgets.dll
 0002:00000244       __imp_?sizeHint@QDialog@@UBE?AVQSize@@XZ 10013244     Qt5Widgets:Qt5Widgets.dll
 0002:00000248       __imp_?sizeHint@QBoxLayout@@UBE?AVQSize@@XZ 10013248     Qt5Widgets:Qt5Widgets.dll
 0002:0000024c       __imp_?sizeHint@QAbstractSpinBox@@UBE?AVQSize@@XZ 1001324c     Qt5Widgets:Qt5Widgets.dll
 0002:00000250       __imp_?showEvent@QWidget@@MAEXPAVQShowEvent@@@Z 10013250     Qt5Widgets:Qt5Widgets.dll
 0002:00000254       __imp_??0QSizePolicy@@QAE@W4Policy@0@0W4ControlType@0@@Z 10013254     Qt5Widgets:Qt5Widgets.dll
 0002:00000258       __imp_?setHorizontalStretch@QSizePolicy@@QAEXH@Z 10013258     Qt5Widgets:Qt5Widgets.dll
 0002:0000025c       __imp_?setVerticalStretch@QSizePolicy@@QAEXH@Z 1001325c     Qt5Widgets:Qt5Widgets.dll
 0002:00000260       __imp_??0QWidget@@QAE@PAV0@V?$QFlags@W4WindowType@Qt@@@@@Z 10013260     Qt5Widgets:Qt5Widgets.dll
 0002:00000264       __imp_??1QWidget@@UAE@XZ   10013264     Qt5Widgets:Qt5Widgets.dll
 0002:00000268       __imp_?setMinimumSize@QWidget@@QAEXHH@Z 10013268     Qt5Widgets:Qt5Widgets.dll
 0002:0000026c       __imp_?setWindowTitle@QWidget@@QAEXABVQString@@@Z 1001326c     Qt5Widgets:Qt5Widgets.dll
 0002:00000270       __imp_?setWindowIcon@QWidget@@QAEXABVQIcon@@@Z 10013270     Qt5Widgets:Qt5Widgets.dll
 0002:00000274       __imp_?setStatusTip@QWidget@@QAEXABVQString@@@Z 10013274     Qt5Widgets:Qt5Widgets.dll
 0002:00000278       __imp_?setWhatsThis@QWidget@@QAEXABVQString@@@Z 10013278     Qt5Widgets:Qt5Widgets.dll
 0002:0000027c       __imp_?resize@QWidget@@QAEXABVQSize@@@Z 1001327c     Qt5Widgets:Qt5Widgets.dll
 0002:00000280       __imp_?adjustSize@QWidget@@QAEXXZ 10013280     Qt5Widgets:Qt5Widgets.dll
 0002:00000284       __imp_?sizePolicy@QWidget@@QBE?AVQSizePolicy@@XZ 10013284     Qt5Widgets:Qt5Widgets.dll
 0002:00000288       __imp_?setSizePolicy@QWidget@@QAEXVQSizePolicy@@@Z 10013288     Qt5Widgets:Qt5Widgets.dll
 0002:0000028c       __imp_?layout@QWidget@@QBEPAVQLayout@@XZ 1001328c     Qt5Widgets:Qt5Widgets.dll
 0002:00000290       __imp_??0QDialog@@QAE@PAVQWidget@@V?$QFlags@W4WindowType@Qt@@@@@Z 10013290     Qt5Widgets:Qt5Widgets.dll
 0002:00000294       __imp_??1QDialog@@UAE@XZ   10013294     Qt5Widgets:Qt5Widgets.dll
 0002:00000298       __imp_?accept@QDialog@@UAEXXZ 10013298     Qt5Widgets:Qt5Widgets.dll
 0002:0000029c       __imp_??0QDialogButtonBox@@QAE@PAVQWidget@@@Z 1001329c     Qt5Widgets:Qt5Widgets.dll
 0002:000002a0       __imp_??1QDialogButtonBox@@UAE@XZ 100132a0     Qt5Widgets:Qt5Widgets.dll
 0002:000002a4       __imp_?setStandardButtons@QDialogButtonBox@@QAEXV?$QFlags@W4StandardButton@QDialogButtonBox@@@@@Z 100132a4     Qt5Widgets:Qt5Widgets.dll
 0002:000002a8       __imp_?button@QDialogButtonBox@@QBEPAVQPushButton@@W4StandardButton@1@@Z 100132a8     Qt5Widgets:Qt5Widgets.dll
 0002:000002ac       __imp_??0QSpinBox@@QAE@PAVQWidget@@@Z 100132ac     Qt5Widgets:Qt5Widgets.dll
 0002:000002b0       __imp_??1QSpinBox@@UAE@XZ  100132b0     Qt5Widgets:Qt5Widgets.dll
 0002:000002b4       __imp_?setMinimum@QSpinBox@@QAEXH@Z 100132b4     Qt5Widgets:Qt5Widgets.dll
 0002:000002b8       __imp_?setMaximum@QSpinBox@@QAEXH@Z 100132b8     Qt5Widgets:Qt5Widgets.dll
 0002:000002bc       __imp_?setValue@QSpinBox@@QAEXH@Z 100132bc     Qt5Widgets:Qt5Widgets.dll
 0002:000002c0       __imp_??0QDoubleSpinBox@@QAE@PAVQWidget@@@Z 100132c0     Qt5Widgets:Qt5Widgets.dll
 0002:000002c4       __imp_??1QDoubleSpinBox@@UAE@XZ 100132c4     Qt5Widgets:Qt5Widgets.dll
 0002:000002c8       __imp_?setSingleStep@QDoubleSpinBox@@QAEXN@Z 100132c8     Qt5Widgets:Qt5Widgets.dll
 0002:000002cc       __imp_?setMaximum@QDoubleSpinBox@@QAEXN@Z 100132cc     Qt5Widgets:Qt5Widgets.dll
 0002:000002d0       __imp_?setDecimals@QDoubleSpinBox@@QAEXH@Z 100132d0     Qt5Widgets:Qt5Widgets.dll
 0002:000002d4       __imp_?setValue@QDoubleSpinBox@@QAEXN@Z 100132d4     Qt5Widgets:Qt5Widgets.dll
 0002:000002d8       __imp_??0QSpacerItem@@QAE@HHW4Policy@QSizePolicy@@0@Z 100132d8     Qt5Widgets:Qt5Widgets.dll
 0002:000002dc       __imp_??1QSpacerItem@@UAE@XZ 100132dc     Qt5Widgets:Qt5Widgets.dll
 0002:000002e0       __imp_?addWidget@QLayout@@QAEXPAVQWidget@@@Z 100132e0     Qt5Widgets:Qt5Widgets.dll
 0002:000002e4       __imp_?addWidget@QBoxLayout@@QAEXPAVQWidget@@HV?$QFlags@W4AlignmentFlag@Qt@@@@@Z 100132e4     Qt5Widgets:Qt5Widgets.dll
 0002:000002e8       __imp_?addLayout@QBoxLayout@@QAEXPAVQLayout@@H@Z 100132e8     Qt5Widgets:Qt5Widgets.dll
 0002:000002ec       __imp_??0QHBoxLayout@@QAE@PAVQWidget@@@Z 100132ec     Qt5Widgets:Qt5Widgets.dll
 0002:000002f0       __imp_??1QHBoxLayout@@UAE@XZ 100132f0     Qt5Widgets:Qt5Widgets.dll
 0002:000002f4       __imp_??0QVBoxLayout@@QAE@PAVQWidget@@@Z 100132f4     Qt5Widgets:Qt5Widgets.dll
 0002:000002f8       __imp_??1QVBoxLayout@@UAE@XZ 100132f8     Qt5Widgets:Qt5Widgets.dll
 0002:000002fc       __imp_??0QGridLayout@@QAE@XZ 100132fc     Qt5Widgets:Qt5Widgets.dll
 0002:00000300       __imp_??1QGridLayout@@UAE@XZ 10013300     Qt5Widgets:Qt5Widgets.dll
 0002:00000304       __imp_?addWidget@QGridLayout@@QAEXPAVQWidget@@HHHHV?$QFlags@W4AlignmentFlag@Qt@@@@@Z 10013304     Qt5Widgets:Qt5Widgets.dll
 0002:00000308       __imp_??0QGroupBox@@QAE@PAVQWidget@@@Z 10013308     Qt5Widgets:Qt5Widgets.dll
 0002:0000030c       __imp_??1QGroupBox@@UAE@XZ 1001330c     Qt5Widgets:Qt5Widgets.dll
 0002:00000310       __imp_?setTitle@QGroupBox@@QAEXABVQString@@@Z 10013310     Qt5Widgets:Qt5Widgets.dll
 0002:00000314       __imp_??0QTabWidget@@QAE@PAVQWidget@@@Z 10013314     Qt5Widgets:Qt5Widgets.dll
 0002:00000318       __imp_??1QTabWidget@@UAE@XZ 10013318     Qt5Widgets:Qt5Widgets.dll
 0002:0000031c       __imp_?addTab@QTabWidget@@QAEHPAVQWidget@@ABVQString@@@Z 1001331c     Qt5Widgets:Qt5Widgets.dll
 0002:00000320       __imp_?setTabText@QTabWidget@@QAEXHABVQString@@@Z 10013320     Qt5Widgets:Qt5Widgets.dll
 0002:00000324       __imp_?currentWidget@QTabWidget@@QBEPAVQWidget@@XZ 10013324     Qt5Widgets:Qt5Widgets.dll
 0002:00000328       __imp_?widget@QTabWidget@@QBEPAVQWidget@@H@Z 10013328     Qt5Widgets:Qt5Widgets.dll
 0002:0000032c       __imp_?indexOf@QTabWidget@@QBEHPAVQWidget@@@Z 1001332c     Qt5Widgets:Qt5Widgets.dll
 0002:00000330       __imp_?count@QTabWidget@@QBEHXZ 10013330     Qt5Widgets:Qt5Widgets.dll
 0002:00000334       __imp_?setTabShape@QTabWidget@@QAEXW4TabShape@1@@Z 10013334     Qt5Widgets:Qt5Widgets.dll
 0002:00000338       __imp_?setCurrentIndex@QTabWidget@@QAEXH@Z 10013338     Qt5Widgets:Qt5Widgets.dll
 0002:0000033c       __imp_??0QLabel@@QAE@PAVQWidget@@V?$QFlags@W4WindowType@Qt@@@@@Z 1001333c     Qt5Widgets:Qt5Widgets.dll
 0002:00000340       __imp_??1QLabel@@UAE@XZ    10013340     Qt5Widgets:Qt5Widgets.dll
 0002:00000344       __imp_?setIndent@QLabel@@QAEXH@Z 10013344     Qt5Widgets:Qt5Widgets.dll
 0002:00000348       __imp_?setText@QLabel@@QAEXABVQString@@@Z 10013348     Qt5Widgets:Qt5Widgets.dll
 0002:0000034c       __imp_?setText@QAbstractButton@@QAEXABVQString@@@Z 1001334c     Qt5Widgets:Qt5Widgets.dll
 0002:00000350       __imp_??0QPushButton@@QAE@PAVQWidget@@@Z 10013350     Qt5Widgets:Qt5Widgets.dll
 0002:00000354       __imp_??1QPushButton@@UAE@XZ 10013354     Qt5Widgets:Qt5Widgets.dll
 0002:00000358       __imp_?warning@QMessageBox@@SA?AW4StandardButton@1@PAVQWidget@@ABVQString@@1V?$QFlags@W4StandardButton@QMessageBox@@@@W421@@Z 10013358     Qt5Widgets:Qt5Widgets.dll
 0002:0000035c       __imp_?critical@QMessageBox@@SA?AW4StandardButton@1@PAVQWidget@@ABVQString@@1V?$QFlags@W4StandardButton@QMessageBox@@@@W421@@Z 1001335c     Qt5Widgets:Qt5Widgets.dll
 0002:00000360       __imp_?actionEvent@QWidget@@MAEXPAVQActionEvent@@@Z 10013360     Qt5Widgets:Qt5Widgets.dll
 0002:00000364       __imp_?addItem@QBoxLayout@@UAEXPAVQLayoutItem@@@Z 10013364     Qt5Widgets:Qt5Widgets.dll
 0002:00000368       __imp_?addItem@QGridLayout@@MAEXPAVQLayoutItem@@@Z 10013368     Qt5Widgets:Qt5Widgets.dll
 0002:0000036c       __imp_?changeEvent@QAbstractButton@@MAEXPAVQEvent@@@Z 1001336c     Qt5Widgets:Qt5Widgets.dll
 0002:00000370       __imp_?changeEvent@QAbstractSpinBox@@MAEXPAVQEvent@@@Z 10013370     Qt5Widgets:Qt5Widgets.dll
 0002:00000374       __imp_?changeEvent@QDialogButtonBox@@MAEXPAVQEvent@@@Z 10013374     Qt5Widgets:Qt5Widgets.dll
 0002:00000378       __imp_?changeEvent@QGroupBox@@MAEXPAVQEvent@@@Z 10013378     Qt5Widgets:Qt5Widgets.dll
 0002:0000037c       __imp_?changeEvent@QLabel@@MAEXPAVQEvent@@@Z 1001337c     Qt5Widgets:Qt5Widgets.dll
 0002:00000380       __imp_?changeEvent@QTabWidget@@MAEXPAVQEvent@@@Z 10013380     Qt5Widgets:Qt5Widgets.dll
 0002:00000384       __imp_?changeEvent@QWidget@@MAEXPAVQEvent@@@Z 10013384     Qt5Widgets:Qt5Widgets.dll
 0002:00000388       __imp_?checkStateSet@QAbstractButton@@MAEXXZ 10013388     Qt5Widgets:Qt5Widgets.dll
 0002:0000038c       __imp_?childEvent@QGroupBox@@MAEXPAVQChildEvent@@@Z 1001338c     Qt5Widgets:Qt5Widgets.dll
 0002:00000390       __imp_?childEvent@QLayout@@MAEXPAVQChildEvent@@@Z 10013390     Qt5Widgets:Qt5Widgets.dll
 0002:00000394       __imp_?clear@QAbstractSpinBox@@UAEXXZ 10013394     Qt5Widgets:Qt5Widgets.dll
 0002:00000398       __imp_?closeEvent@QAbstractSpinBox@@MAEXPAVQCloseEvent@@@Z 10013398     Qt5Widgets:Qt5Widgets.dll
 0002:0000039c       __imp_?closeEvent@QDialog@@MAEXPAVQCloseEvent@@@Z 1001339c     Qt5Widgets:Qt5Widgets.dll
 0002:000003a0       __imp_?closeEvent@QWidget@@MAEXPAVQCloseEvent@@@Z 100133a0     Qt5Widgets:Qt5Widgets.dll
 0002:000003a4       __imp_?contextMenuEvent@QAbstractSpinBox@@MAEXPAVQContextMenuEvent@@@Z 100133a4     Qt5Widgets:Qt5Widgets.dll
 0002:000003a8       __imp_?contextMenuEvent@QDialog@@MAEXPAVQContextMenuEvent@@@Z 100133a8     Qt5Widgets:Qt5Widgets.dll
 0002:000003ac       __imp_?contextMenuEvent@QLabel@@MAEXPAVQContextMenuEvent@@@Z 100133ac     Qt5Widgets:Qt5Widgets.dll
 0002:000003b0       __imp_?contextMenuEvent@QWidget@@MAEXPAVQContextMenuEvent@@@Z 100133b0     Qt5Widgets:Qt5Widgets.dll
 0002:000003b4       __imp_?controlTypes@QLayout@@UBE?AV?$QFlags@W4ControlType@QSizePolicy@@@@XZ 100133b4     Qt5Widgets:Qt5Widgets.dll
 0002:000003b8       __imp_?controlTypes@QLayoutItem@@UBE?AV?$QFlags@W4ControlType@QSizePolicy@@@@XZ 100133b8     Qt5Widgets:Qt5Widgets.dll
 0002:000003bc       __imp_?count@QBoxLayout@@UBEHXZ 100133bc     Qt5Widgets:Qt5Widgets.dll
 0002:000003c0       __imp_?count@QGridLayout@@UBEHXZ 100133c0     Qt5Widgets:Qt5Widgets.dll
 0002:000003c4       __imp_?devType@QWidget@@UBEHXZ 100133c4     Qt5Widgets:Qt5Widgets.dll
 0002:000003c8       __imp_?done@QDialog@@UAEXH@Z 100133c8     Qt5Widgets:Qt5Widgets.dll
 0002:000003cc       __imp_?dragEnterEvent@QWidget@@MAEXPAVQDragEnterEvent@@@Z 100133cc     Qt5Widgets:Qt5Widgets.dll
 0002:000003d0       __imp_?dragLeaveEvent@QWidget@@MAEXPAVQDragLeaveEvent@@@Z 100133d0     Qt5Widgets:Qt5Widgets.dll
 0002:000003d4       __imp_?dragMoveEvent@QWidget@@MAEXPAVQDragMoveEvent@@@Z 100133d4     Qt5Widgets:Qt5Widgets.dll
 0002:000003d8       __imp_?dropEvent@QWidget@@MAEXPAVQDropEvent@@@Z 100133d8     Qt5Widgets:Qt5Widgets.dll
 0002:000003dc       __imp_?enterEvent@QWidget@@MAEXPAVQEvent@@@Z 100133dc     Qt5Widgets:Qt5Widgets.dll
 0002:000003e0       __imp_?event@QAbstractSpinBox@@UAE_NPAVQEvent@@@Z 100133e0     Qt5Widgets:Qt5Widgets.dll
 0002:000003e4       __imp_?event@QDialogButtonBox@@MAE_NPAVQEvent@@@Z 100133e4     Qt5Widgets:Qt5Widgets.dll
 0002:000003e8       __imp_?event@QGroupBox@@MAE_NPAVQEvent@@@Z 100133e8     Qt5Widgets:Qt5Widgets.dll
 0002:000003ec       __imp_?event@QLabel@@MAE_NPAVQEvent@@@Z 100133ec     Qt5Widgets:Qt5Widgets.dll
 0002:000003f0       __imp_?event@QPushButton@@MAE_NPAVQEvent@@@Z 100133f0     Qt5Widgets:Qt5Widgets.dll
 0002:000003f4       __imp_?event@QSpinBox@@MAE_NPAVQEvent@@@Z 100133f4     Qt5Widgets:Qt5Widgets.dll
 0002:000003f8       __imp_?event@QTabWidget@@MAE_NPAVQEvent@@@Z 100133f8     Qt5Widgets:Qt5Widgets.dll
 0002:000003fc       __imp_?event@QWidget@@MAE_NPAVQEvent@@@Z 100133fc     Qt5Widgets:Qt5Widgets.dll
 0002:00000400       __imp_?eventFilter@QDialog@@MAE_NPAVQObject@@PAVQEvent@@@Z 10013400     Qt5Widgets:Qt5Widgets.dll
 0002:00000404       __imp_?exec@QDialog@@UAEHXZ 10013404     Qt5Widgets:Qt5Widgets.dll
 0002:00000408       __imp_?expandingDirections@QBoxLayout@@UBE?AV?$QFlags@W4Orientation@Qt@@@@XZ 10013408     Qt5Widgets:Qt5Widgets.dll
 0002:0000040c       __imp_?expandingDirections@QGridLayout@@UBE?AV?$QFlags@W4Orientation@Qt@@@@XZ 1001340c     Qt5Widgets:Qt5Widgets.dll
 0002:00000410       __imp_?expandingDirections@QSpacerItem@@UBE?AV?$QFlags@W4Orientation@Qt@@@@XZ 10013410     Qt5Widgets:Qt5Widgets.dll
 0002:00000414       __imp_?fixup@QDoubleSpinBox@@UBEXAAVQString@@@Z 10013414     Qt5Widgets:Qt5Widgets.dll
 0002:00000418       __imp_?fixup@QSpinBox@@MBEXAAVQString@@@Z 10013418     Qt5Widgets:Qt5Widgets.dll
 0002:0000041c       __imp_?focusInEvent@QAbstractSpinBox@@MAEXPAVQFocusEvent@@@Z 1001341c     Qt5Widgets:Qt5Widgets.dll
 0002:00000420       __imp_?focusInEvent@QGroupBox@@MAEXPAVQFocusEvent@@@Z 10013420     Qt5Widgets:Qt5Widgets.dll
 0002:00000424       __imp_?focusInEvent@QLabel@@MAEXPAVQFocusEvent@@@Z 10013424     Qt5Widgets:Qt5Widgets.dll
 0002:00000428       __imp_?focusInEvent@QPushButton@@MAEXPAVQFocusEvent@@@Z 10013428     Qt5Widgets:Qt5Widgets.dll
 0002:0000042c       __imp_?focusInEvent@QWidget@@MAEXPAVQFocusEvent@@@Z 1001342c     Qt5Widgets:Qt5Widgets.dll
 0002:00000430       __imp_?focusNextPrevChild@QLabel@@MAE_N_N@Z 10013430     Qt5Widgets:Qt5Widgets.dll
 0002:00000434       __imp_?focusNextPrevChild@QWidget@@MAE_N_N@Z 10013434     Qt5Widgets:Qt5Widgets.dll
 0002:00000438       __imp_?focusOutEvent@QAbstractSpinBox@@MAEXPAVQFocusEvent@@@Z 10013438     Qt5Widgets:Qt5Widgets.dll
 0002:0000043c       __imp_?focusOutEvent@QLabel@@MAEXPAVQFocusEvent@@@Z 1001343c     Qt5Widgets:Qt5Widgets.dll
 0002:00000440       __imp_?focusOutEvent@QPushButton@@MAEXPAVQFocusEvent@@@Z 10013440     Qt5Widgets:Qt5Widgets.dll
 0002:00000444       __imp_?focusOutEvent@QWidget@@MAEXPAVQFocusEvent@@@Z 10013444     Qt5Widgets:Qt5Widgets.dll
 0002:00000448       __imp_?geometry@QLayout@@UBE?AVQRect@@XZ 10013448     Qt5Widgets:Qt5Widgets.dll
 0002:0000044c       __imp_?geometry@QSpacerItem@@UBE?AVQRect@@XZ 1001344c     Qt5Widgets:Qt5Widgets.dll
 0002:00000450       __imp_?hasHeightForWidth@QBoxLayout@@UBE_NXZ 10013450     Qt5Widgets:Qt5Widgets.dll
 0002:00000454       __imp_?hasHeightForWidth@QGridLayout@@UBE_NXZ 10013454     Qt5Widgets:Qt5Widgets.dll
 0002:00000458       __imp_?hasHeightForWidth@QLayoutItem@@UBE_NXZ 10013458     Qt5Widgets:Qt5Widgets.dll
 0002:0000045c       __imp_?hasHeightForWidth@QTabWidget@@UBE_NXZ 1001345c     Qt5Widgets:Qt5Widgets.dll
 0002:00000460       __imp_?hasHeightForWidth@QWidget@@UBE_NXZ 10013460     Qt5Widgets:Qt5Widgets.dll
 0002:00000464       __imp_?heightForWidth@QBoxLayout@@UBEHH@Z 10013464     Qt5Widgets:Qt5Widgets.dll
 0002:00000468       __imp_?heightForWidth@QGridLayout@@UBEHH@Z 10013468     Qt5Widgets:Qt5Widgets.dll
 0002:0000046c       __imp_?heightForWidth@QLabel@@UBEHH@Z 1001346c     Qt5Widgets:Qt5Widgets.dll
 0002:00000470       __imp_?heightForWidth@QLayoutItem@@UBEHH@Z 10013470     Qt5Widgets:Qt5Widgets.dll
 0002:00000474       __imp_?heightForWidth@QTabWidget@@UBEHH@Z 10013474     Qt5Widgets:Qt5Widgets.dll
 0002:00000478       __imp_?heightForWidth@QWidget@@UBEHH@Z 10013478     Qt5Widgets:Qt5Widgets.dll
 0002:0000047c       __imp_?hideEvent@QAbstractSpinBox@@MAEXPAVQHideEvent@@@Z 1001347c     Qt5Widgets:Qt5Widgets.dll
 0002:00000480       __imp_?hideEvent@QWidget@@MAEXPAVQHideEvent@@@Z 10013480     Qt5Widgets:Qt5Widgets.dll
 0002:00000484       __imp_?hitButton@QAbstractButton@@MBE_NABVQPoint@@@Z 10013484     Qt5Widgets:Qt5Widgets.dll
 0002:00000488       __imp_?indexOf@QLayout@@UBEHPAVQWidget@@@Z 10013488     Qt5Widgets:Qt5Widgets.dll
 0002:0000048c       __imp_?initPainter@QWidget@@MBEXPAVQPainter@@@Z 1001348c     Qt5Widgets:Qt5Widgets.dll
 0002:00000490       __imp_?inputMethodEvent@QWidget@@MAEXPAVQInputMethodEvent@@@Z 10013490     Qt5Widgets:Qt5Widgets.dll
 0002:00000494       __imp_?inputMethodQuery@QAbstractSpinBox@@UBE?AVQVariant@@W4InputMethodQuery@Qt@@@Z 10013494     Qt5Widgets:Qt5Widgets.dll
 0002:00000498       __imp_?inputMethodQuery@QWidget@@UBE?AVQVariant@@W4InputMethodQuery@Qt@@@Z 10013498     Qt5Widgets:Qt5Widgets.dll
 0002:0000049c       __imp_?invalidate@QBoxLayout@@UAEXXZ 1001349c     Qt5Widgets:Qt5Widgets.dll
 0002:000004a0       __imp_?invalidate@QGridLayout@@UAEXXZ 100134a0     Qt5Widgets:Qt5Widgets.dll
 0002:000004a4       __imp_?invalidate@QLayoutItem@@UAEXXZ 100134a4     Qt5Widgets:Qt5Widgets.dll
 0002:000004a8       __imp_?isEmpty@QLayout@@UBE_NXZ 100134a8     Qt5Widgets:Qt5Widgets.dll
 0002:000004ac       __imp_?isEmpty@QSpacerItem@@UBE_NXZ 100134ac     Qt5Widgets:Qt5Widgets.dll
 0002:000004b0       __imp_?itemAt@QBoxLayout@@UBEPAVQLayoutItem@@H@Z 100134b0     Qt5Widgets:Qt5Widgets.dll
 0002:000004b4       __imp_?itemAt@QGridLayout@@UBEPAVQLayoutItem@@H@Z 100134b4     Qt5Widgets:Qt5Widgets.dll
 0002:000004b8       __imp_?keyPressEvent@QAbstractSpinBox@@MAEXPAVQKeyEvent@@@Z 100134b8     Qt5Widgets:Qt5Widgets.dll
 0002:000004bc       __imp_?keyPressEvent@QDialog@@MAEXPAVQKeyEvent@@@Z 100134bc     Qt5Widgets:Qt5Widgets.dll
 0002:000004c0       __imp_?keyPressEvent@QLabel@@MAEXPAVQKeyEvent@@@Z 100134c0     Qt5Widgets:Qt5Widgets.dll
 0002:000004c4       __imp_?keyPressEvent@QPushButton@@MAEXPAVQKeyEvent@@@Z 100134c4     Qt5Widgets:Qt5Widgets.dll
 0002:000004c8       __imp_?keyPressEvent@QTabWidget@@MAEXPAVQKeyEvent@@@Z 100134c8     Qt5Widgets:Qt5Widgets.dll
 0002:000004cc       __imp_?keyPressEvent@QWidget@@MAEXPAVQKeyEvent@@@Z 100134cc     Qt5Widgets:Qt5Widgets.dll
 0002:000004d0       __imp_?keyReleaseEvent@QAbstractButton@@MAEXPAVQKeyEvent@@@Z 100134d0     Qt5Widgets:Qt5Widgets.dll
 0002:000004d4       __imp_?keyReleaseEvent@QAbstractSpinBox@@MAEXPAVQKeyEvent@@@Z 100134d4     Qt5Widgets:Qt5Widgets.dll
 0002:000004d8       __imp_?keyReleaseEvent@QWidget@@MAEXPAVQKeyEvent@@@Z 100134d8     Qt5Widgets:Qt5Widgets.dll
 0002:000004dc       __imp_?layout@QLayout@@UAEPAV1@XZ 100134dc     Qt5Widgets:Qt5Widgets.dll
 0002:000004e0       __imp_?layout@QLayoutItem@@UAEPAVQLayout@@XZ 100134e0     Qt5Widgets:Qt5Widgets.dll
 0002:000004e4       __imp_?leaveEvent@QWidget@@MAEXPAVQEvent@@@Z 100134e4     Qt5Widgets:Qt5Widgets.dll
 0002:000004e8       __imp_?maximumSize@QBoxLayout@@UBE?AVQSize@@XZ 100134e8     Qt5Widgets:Qt5Widgets.dll
 0002:000004ec       __imp_?maximumSize@QGridLayout@@UBE?AVQSize@@XZ 100134ec     Qt5Widgets:Qt5Widgets.dll
 0002:000004f0       __imp_?maximumSize@QSpacerItem@@UBE?AVQSize@@XZ 100134f0     Qt5Widgets:Qt5Widgets.dll
 0002:000004f4       __imp_?metaObject@QDialogButtonBox@@UBEPBUQMetaObject@@XZ 100134f4     Qt5Widgets:Qt5Widgets.dll
 0002:000004f8       __imp_?metaObject@QDoubleSpinBox@@UBEPBUQMetaObject@@XZ 100134f8     Qt5Widgets:Qt5Widgets.dll
 0002:000004fc       __imp_?metaObject@QGridLayout@@UBEPBUQMetaObject@@XZ 100134fc     Qt5Widgets:Qt5Widgets.dll
 0002:00000500       __imp_?metaObject@QGroupBox@@UBEPBUQMetaObject@@XZ 10013500     Qt5Widgets:Qt5Widgets.dll
 0002:00000504       __imp_?metaObject@QHBoxLayout@@UBEPBUQMetaObject@@XZ 10013504     Qt5Widgets:Qt5Widgets.dll
 0002:00000508       __imp_?metaObject@QLabel@@UBEPBUQMetaObject@@XZ 10013508     Qt5Widgets:Qt5Widgets.dll
 0002:0000050c       __imp_?metaObject@QPushButton@@UBEPBUQMetaObject@@XZ 1001350c     Qt5Widgets:Qt5Widgets.dll
 0002:00000510       __imp_?metaObject@QSpinBox@@UBEPBUQMetaObject@@XZ 10013510     Qt5Widgets:Qt5Widgets.dll
 0002:00000514       __imp_?metaObject@QTabWidget@@UBEPBUQMetaObject@@XZ 10013514     Qt5Widgets:Qt5Widgets.dll
 0002:00000518       __imp_?metaObject@QVBoxLayout@@UBEPBUQMetaObject@@XZ 10013518     Qt5Widgets:Qt5Widgets.dll
 0002:0000051c       __imp_?metaObject@QWidget@@UBEPBUQMetaObject@@XZ 1001351c     Qt5Widgets:Qt5Widgets.dll
 0002:00000520       __imp_?metric@QWidget@@MBEHW4PaintDeviceMetric@QPaintDevice@@@Z 10013520     Qt5Widgets:Qt5Widgets.dll
 0002:00000524       __imp_?minimumHeightForWidth@QBoxLayout@@UBEHH@Z 10013524     Qt5Widgets:Qt5Widgets.dll
 0002:00000528       __imp_?minimumHeightForWidth@QGridLayout@@UBEHH@Z 10013528     Qt5Widgets:Qt5Widgets.dll
 0002:0000052c       __imp_?minimumHeightForWidth@QLayoutItem@@UBEHH@Z 1001352c     Qt5Widgets:Qt5Widgets.dll
 0002:00000530       __imp_?minimumSize@QBoxLayout@@UBE?AVQSize@@XZ 10013530     Qt5Widgets:Qt5Widgets.dll
 0002:00000534       __imp_?minimumSize@QGridLayout@@UBE?AVQSize@@XZ 10013534     Qt5Widgets:Qt5Widgets.dll
 0002:00000538       __imp_?minimumSize@QSpacerItem@@UBE?AVQSize@@XZ 10013538     Qt5Widgets:Qt5Widgets.dll
 0002:0000053c       __imp_?minimumSizeHint@QAbstractSpinBox@@UBE?AVQSize@@XZ 1001353c     Qt5Widgets:Qt5Widgets.dll
 0002:00000540       __imp_?minimumSizeHint@QDialog@@UBE?AVQSize@@XZ 10013540     Qt5Widgets:Qt5Widgets.dll
 0002:00000544       __imp_?minimumSizeHint@QGroupBox@@UBE?AVQSize@@XZ 10013544     Qt5Widgets:Qt5Widgets.dll
 0002:00000548       __imp_?minimumSizeHint@QLabel@@UBE?AVQSize@@XZ 10013548     Qt5Widgets:Qt5Widgets.dll
 0002:0000054c       __imp_?minimumSizeHint@QPushButton@@UBE?AVQSize@@XZ 1001354c     Qt5Widgets:Qt5Widgets.dll
 0002:00000550       __imp_?minimumSizeHint@QTabWidget@@UBE?AVQSize@@XZ 10013550     Qt5Widgets:Qt5Widgets.dll
 0002:00000554       __imp_?minimumSizeHint@QWidget@@UBE?AVQSize@@XZ 10013554     Qt5Widgets:Qt5Widgets.dll
 0002:00000558       __imp_?mouseDoubleClickEvent@QWidget@@MAEXPAVQMouseEvent@@@Z 10013558     Qt5Widgets:Qt5Widgets.dll
 0002:0000055c       __imp_?mouseMoveEvent@QAbstractButton@@MAEXPAVQMouseEvent@@@Z 1001355c     Qt5Widgets:Qt5Widgets.dll
 0002:00000560       __imp_?mouseMoveEvent@QAbstractSpinBox@@MAEXPAVQMouseEvent@@@Z 10013560     Qt5Widgets:Qt5Widgets.dll
 0002:00000564       __imp_?mouseMoveEvent@QGroupBox@@MAEXPAVQMouseEvent@@@Z 10013564     Qt5Widgets:Qt5Widgets.dll
 0002:00000568       __imp_?mouseMoveEvent@QLabel@@MAEXPAVQMouseEvent@@@Z 10013568     Qt5Widgets:Qt5Widgets.dll
 0002:0000056c       __imp_?mouseMoveEvent@QWidget@@MAEXPAVQMouseEvent@@@Z 1001356c     Qt5Widgets:Qt5Widgets.dll
 0002:00000570       __imp_?mousePressEvent@QAbstractButton@@MAEXPAVQMouseEvent@@@Z 10013570     Qt5Widgets:Qt5Widgets.dll
 0002:00000574       __imp_?mousePressEvent@QAbstractSpinBox@@MAEXPAVQMouseEvent@@@Z 10013574     Qt5Widgets:Qt5Widgets.dll
 0002:00000578       __imp_?mousePressEvent@QGroupBox@@MAEXPAVQMouseEvent@@@Z 10013578     Qt5Widgets:Qt5Widgets.dll
 0002:0000057c       __imp_?mousePressEvent@QLabel@@MAEXPAVQMouseEvent@@@Z 1001357c     Qt5Widgets:Qt5Widgets.dll
 0002:00000580       __imp_?mousePressEvent@QWidget@@MAEXPAVQMouseEvent@@@Z 10013580     Qt5Widgets:Qt5Widgets.dll
 0002:00000584       __imp_?mouseReleaseEvent@QAbstractButton@@MAEXPAVQMouseEvent@@@Z 10013584     Qt5Widgets:Qt5Widgets.dll
 0002:00000588       __imp_?mouseReleaseEvent@QAbstractSpinBox@@MAEXPAVQMouseEvent@@@Z 10013588     Qt5Widgets:Qt5Widgets.dll
 0002:0000058c       __imp_?mouseReleaseEvent@QGroupBox@@MAEXPAVQMouseEvent@@@Z 1001358c     Qt5Widgets:Qt5Widgets.dll
 0002:00000590       __imp_?mouseReleaseEvent@QLabel@@MAEXPAVQMouseEvent@@@Z 10013590     Qt5Widgets:Qt5Widgets.dll
 0002:00000594       __imp_?mouseReleaseEvent@QWidget@@MAEXPAVQMouseEvent@@@Z 10013594     Qt5Widgets:Qt5Widgets.dll
 0002:00000598       __imp_?moveEvent@QWidget@@MAEXPAVQMoveEvent@@@Z 10013598     Qt5Widgets:Qt5Widgets.dll
 0002:0000059c       __imp_?nativeEvent@QWidget@@MAE_NABVQByteArray@@PAXPAJ@Z 1001359c     Qt5Widgets:Qt5Widgets.dll
 0002:000005a0       __imp_?nextCheckState@QAbstractButton@@MAEXXZ 100135a0     Qt5Widgets:Qt5Widgets.dll
 0002:000005a4       __imp_?open@QDialog@@UAEXXZ 100135a4     Qt5Widgets:Qt5Widgets.dll
 0002:000005a8       __imp_?paintEngine@QWidget@@UBEPAVQPaintEngine@@XZ 100135a8     Qt5Widgets:Qt5Widgets.dll
 0002:000005ac       __imp_?paintEvent@QAbstractSpinBox@@MAEXPAVQPaintEvent@@@Z 100135ac     Qt5Widgets:Qt5Widgets.dll
 0002:000005b0       __imp_?paintEvent@QGroupBox@@MAEXPAVQPaintEvent@@@Z 100135b0     Qt5Widgets:Qt5Widgets.dll
 0002:000005b4       __imp_?paintEvent@QLabel@@MAEXPAVQPaintEvent@@@Z 100135b4     Qt5Widgets:Qt5Widgets.dll
 0002:000005b8       __imp_?paintEvent@QPushButton@@MAEXPAVQPaintEvent@@@Z 100135b8     Qt5Widgets:Qt5Widgets.dll
 0002:000005bc       __imp_?paintEvent@QTabWidget@@MAEXPAVQPaintEvent@@@Z 100135bc     Qt5Widgets:Qt5Widgets.dll
 0002:000005c0       __imp_?paintEvent@QWidget@@MAEXPAVQPaintEvent@@@Z 100135c0     Qt5Widgets:Qt5Widgets.dll
 0002:000005c4       __imp_?qt_metacall@QDialogButtonBox@@UAEHW4Call@QMetaObject@@HPAPAX@Z 100135c4     Qt5Widgets:Qt5Widgets.dll
 0002:000005c8       __imp_?qt_metacall@QDoubleSpinBox@@UAEHW4Call@QMetaObject@@HPAPAX@Z 100135c8     Qt5Widgets:Qt5Widgets.dll
 0002:000005cc       __imp_?qt_metacall@QGridLayout@@UAEHW4Call@QMetaObject@@HPAPAX@Z 100135cc     Qt5Widgets:Qt5Widgets.dll
 0002:000005d0       __imp_?qt_metacall@QGroupBox@@UAEHW4Call@QMetaObject@@HPAPAX@Z 100135d0     Qt5Widgets:Qt5Widgets.dll
 0002:000005d4       __imp_?qt_metacall@QHBoxLayout@@UAEHW4Call@QMetaObject@@HPAPAX@Z 100135d4     Qt5Widgets:Qt5Widgets.dll
 0002:000005d8       __imp_?qt_metacall@QLabel@@UAEHW4Call@QMetaObject@@HPAPAX@Z 100135d8     Qt5Widgets:Qt5Widgets.dll
 0002:000005dc       __imp_?qt_metacall@QPushButton@@UAEHW4Call@QMetaObject@@HPAPAX@Z 100135dc     Qt5Widgets:Qt5Widgets.dll
 0002:000005e0       __imp_?qt_metacall@QSpinBox@@UAEHW4Call@QMetaObject@@HPAPAX@Z 100135e0     Qt5Widgets:Qt5Widgets.dll
 0002:000005e4       __imp_?qt_metacall@QTabWidget@@UAEHW4Call@QMetaObject@@HPAPAX@Z 100135e4     Qt5Widgets:Qt5Widgets.dll
 0002:000005e8       __imp_?qt_metacall@QVBoxLayout@@UAEHW4Call@QMetaObject@@HPAPAX@Z 100135e8     Qt5Widgets:Qt5Widgets.dll
 0002:000005ec       __imp_?qt_metacall@QWidget@@UAEHW4Call@QMetaObject@@HPAPAX@Z 100135ec     Qt5Widgets:Qt5Widgets.dll
 0002:000005f0       __imp_?qt_metacast@QDialogButtonBox@@UAEPAXPBD@Z 100135f0     Qt5Widgets:Qt5Widgets.dll
 0002:000005f4       __imp_?qt_metacast@QDoubleSpinBox@@UAEPAXPBD@Z 100135f4     Qt5Widgets:Qt5Widgets.dll
 0002:000005f8       __imp_?qt_metacast@QGridLayout@@UAEPAXPBD@Z 100135f8     Qt5Widgets:Qt5Widgets.dll
 0002:000005fc       __imp_?qt_metacast@QGroupBox@@UAEPAXPBD@Z 100135fc     Qt5Widgets:Qt5Widgets.dll
 0002:00000600       __imp_?qt_metacast@QHBoxLayout@@UAEPAXPBD@Z 10013600     Qt5Widgets:Qt5Widgets.dll
 0002:00000604       __imp_?qt_metacast@QLabel@@UAEPAXPBD@Z 10013604     Qt5Widgets:Qt5Widgets.dll
 0002:00000608       __imp_?qt_metacast@QPushButton@@UAEPAXPBD@Z 10013608     Qt5Widgets:Qt5Widgets.dll
 0002:0000060c       __imp_?qt_metacast@QSpinBox@@UAEPAXPBD@Z 1001360c     Qt5Widgets:Qt5Widgets.dll
 0002:00000610       __imp_?qt_metacast@QTabWidget@@UAEPAXPBD@Z 10013610     Qt5Widgets:Qt5Widgets.dll
 0002:00000614       __imp_?qt_metacast@QVBoxLayout@@UAEPAXPBD@Z 10013614     Qt5Widgets:Qt5Widgets.dll
 0002:00000618       __imp_?qt_metacast@QWidget@@UAEPAXPBD@Z 10013618     Qt5Widgets:Qt5Widgets.dll
 0002:0000061c       __imp_?redirected@QWidget@@MBEPAVQPaintDevice@@PAVQPoint@@@Z 1001361c     Qt5Widgets:Qt5Widgets.dll
 0002:00000620       __imp_?reject@QDialog@@UAEXXZ 10013620     Qt5Widgets:Qt5Widgets.dll
 0002:00000624       __imp_?resizeEvent@QAbstractSpinBox@@MAEXPAVQResizeEvent@@@Z 10013624     Qt5Widgets:Qt5Widgets.dll
 0002:00000628       __imp_?resizeEvent@QDialog@@MAEXPAVQResizeEvent@@@Z 10013628     Qt5Widgets:Qt5Widgets.dll
 0002:0000062c       __imp_?resizeEvent@QGroupBox@@MAEXPAVQResizeEvent@@@Z 1001362c     Qt5Widgets:Qt5Widgets.dll
 0002:00000630       __imp_?resizeEvent@QTabWidget@@MAEXPAVQResizeEvent@@@Z 10013630     Qt5Widgets:Qt5Widgets.dll
 0002:00000634       __imp_?resizeEvent@QWidget@@MAEXPAVQResizeEvent@@@Z 10013634     Qt5Widgets:Qt5Widgets.dll
 0002:00000638       __imp_?setGeometry@QBoxLayout@@UAEXABVQRect@@@Z 10013638     Qt5Widgets:Qt5Widgets.dll
 0002:0000063c       __imp_?setGeometry@QGridLayout@@UAEXABVQRect@@@Z 1001363c     Qt5Widgets:Qt5Widgets.dll
 0002:00000640       __imp_?setGeometry@QSpacerItem@@UAEXABVQRect@@@Z 10013640     Qt5Widgets:Qt5Widgets.dll
 0002:00000644       __imp_?setVisible@QDialog@@UAEX_N@Z 10013644     Qt5Widgets:Qt5Widgets.dll
 0002:00000648       __imp_?setVisible@QWidget@@UAEX_N@Z 10013648     Qt5Widgets:Qt5Widgets.dll
 0002:0000064c       __imp_?sharedPainter@QWidget@@MBEPAVQPainter@@XZ 1001364c     Qt5Widgets:Qt5Widgets.dll
 0002:00000650       __imp_?showEvent@QAbstractSpinBox@@MAEXPAVQShowEvent@@@Z 10013650     Qt5Widgets:Qt5Widgets.dll
 0002:00000654       __imp_?showEvent@QDialog@@MAEXPAVQShowEvent@@@Z 10013654     Qt5Widgets:Qt5Widgets.dll
 0002:00000658       __imp_?showEvent@QTabWidget@@MAEXPAVQShowEvent@@@Z 10013658     Qt5Widgets:Qt5Widgets.dll
 0002:0000065c       \177Qt5Widgets_NULL_THUNK_DATA 1001365c     Qt5Widgets:Qt5Widgets.dll
 0002:00000660       __imp_??1Logger@U2@@UAE@XZ 10013660     U2Core:U2Core.dll
 0002:00000664       __imp_?isCoR@U2OpStatus@U2@@UBE_NXZ 10013664     U2Core:U2Core.dll
 0002:00000668       __imp_??0GObjectReference@U2@@QAE@PBVGObject@1@_N@Z 10013668     U2Core:U2Core.dll
 0002:0000066c       __imp_??1GObjectReference@U2@@QAE@XZ 1001366c     U2Core:U2Core.dll
 0002:00000670       __imp_??4GObjectReference@U2@@QAEAAV01@ABV01@@Z 10013670     U2Core:U2Core.dll
 0002:00000674       __imp_??0DNASequence@U2@@QAE@ABVQByteArray@@PBVDNAAlphabet@1@@Z 10013674     U2Core:U2Core.dll
 0002:00000678       __imp_??1DNASequence@U2@@QAE@XZ 10013678     U2Core:U2Core.dll
 0002:0000067c       __imp_??1AnnotationData@U2@@QAE@XZ 1001367c     U2Core:U2Core.dll
 0002:00000680       __imp_??0AnnotationData@U2@@QAE@ABV01@@Z 10013680     U2Core:U2Core.dll
 0002:00000684       __imp_?getTaskScheduler@AppContext@U2@@SAPAVTaskScheduler@2@XZ 10013684     U2Core:U2Core.dll
 0002:00000688       __imp_?getSequenceLength@U2SequenceObject@U2@@QBE_JXZ 10013688     U2Core:U2Core.dll
 0002:0000068c       __imp_?getWholeSequenceData@U2SequenceObject@U2@@QBE?AVQByteArray@@AAVU2OpStatus@2@@Z 1001368c     U2Core:U2Core.dll
 0002:00000690       __imp_??0U2OpStatusImpl@U2@@QAE@XZ 10013690     U2Core:U2Core.dll
 0002:00000694       __imp_?getError@U2OpStatusImpl@U2@@UBE?AVQString@@XZ 10013694     U2Core:U2Core.dll
 0002:00000698       __imp_??1U2OpStatusImpl@U2@@UAE@XZ 10013698     U2Core:U2Core.dll
 0002:0000069c       __imp_?errorTitle@L10N@U2@@SA?AVQString@@XZ 1001369c     U2Core:U2Core.dll
 0002:000006a0       __imp_?getAlphabet@U2SequenceObject@U2@@QBEPBVDNAAlphabet@2@XZ 100136a0     U2Core:U2Core.dll
 0002:000006a4       __imp_?NUCL_DNA_DEFAULT@BaseDNAAlphabetIds@U2@@SA?BVQString@@XZ 100136a4     U2Core:U2Core.dll
 0002:000006a8       __imp_?getMainWindow@AppContext@U2@@SAPAVMainWindow@2@XZ 100136a8     U2Core:U2Core.dll
 0002:000006ac       __imp_?error@Logger@U2@@QAEXABVQString@@@Z 100136ac     U2Core:U2Core.dll
 0002:000006b0       __imp_??0Plugin@U2@@QAE@ABVQString@@0_NW4PluginState@1@@Z 100136b0     U2Core:U2Core.dll
 0002:000006b4       __imp_??1Plugin@U2@@UAE@XZ 100136b4     U2Core:U2Core.dll
 0002:000006b8       __imp_??CU2Location@U2@@QAEPAVU2LocationData@1@XZ 100136b8     U2Core:U2Core.dll
 0002:000006bc       __imp_??0U2Qualifier@U2@@QAE@XZ 100136bc     U2Core:U2Core.dll
 0002:000006c0       __imp_??0U2Qualifier@U2@@QAE@ABVQString@@0@Z 100136c0     U2Core:U2Core.dll
 0002:000006c4       __imp_??1U2Qualifier@U2@@QAE@XZ 100136c4     U2Core:U2Core.dll
 0002:000006c8       __imp_??0U2Qualifier@U2@@QAE@ABV01@@Z 100136c8     U2Core:U2Core.dll
 0002:000006cc       __imp_??0AnnotationData@U2@@QAE@XZ 100136cc     U2Core:U2Core.dll
 0002:000006d0       __imp_??0Task@U2@@QAE@ABVQString@@V?$QFlags@W4TaskFlag@U2@@@@@Z 100136d0     U2Core:U2Core.dll
 0002:000006d4       __imp_?addSubTask@Task@U2@@QAEXPAV12@@Z 100136d4     U2Core:U2Core.dll
 0002:000006d8       __imp_?hasError@Task@U2@@QBE_NXZ 100136d8     U2Core:U2Core.dll
 0002:000006dc       __imp_?getError@Task@U2@@QBE?AVQString@@XZ 100136dc     U2Core:U2Core.dll
 0002:000006e0       __imp_??1Task@U2@@UAE@XZ   100136e0     U2Core:U2Core.dll
 0002:000006e4       __imp_??0CreateAnnotationsTask@U2@@QAE@PAVAnnotationTableObject@1@ABV?$QList@V?$QSharedDataPointer@VAnnotationData@U2@@@@@@ABVQString@@@Z 100136e4     U2Core:U2Core.dll
 0002:000006e8       __imp_??1CreateAnnotationsTask@U2@@UAE@XZ 100136e8     U2Core:U2Core.dll
 0002:000006ec       __imp_??0DNASequence@U2@@QAE@ABV01@@Z 100136ec     U2Core:U2Core.dll
 0002:000006f0       __imp_?addDescriptionQualifier@U1AnnotationUtils@U2@@SAXAAV?$QSharedDataPointer@VAnnotationData@U2@@@@ABVQString@@@Z 100136f0     U2Core:U2Core.dll
 0002:000006f4       __imp_?cleanup@Task@U2@@UAEXXZ 100136f4     U2Core:U2Core.dll
 0002:000006f8       __imp_?generateReport@Task@U2@@UBE?AVQString@@XZ 100136f8     U2Core:U2Core.dll
 0002:000006fc       __imp_?getNumParallelSubtasks@Task@U2@@UBEHXZ 100136fc     U2Core:U2Core.dll
 0002:00000700       __imp_?getParentTask@Task@U2@@UBEPAV12@XZ 10013700     U2Core:U2Core.dll
 0002:00000704       __imp_?getSubtaskWithErrors@Task@U2@@UBEPAV12@XZ 10013704     U2Core:U2Core.dll
 0002:00000708       __imp_?getTaskId@Task@U2@@UBE_JXZ 10013708     U2Core:U2Core.dll
 0002:0000070c       __imp_?getTopLevelParentTask@Task@U2@@UAEPAV12@XZ 1001370c     U2Core:U2Core.dll
 0002:00000710       __imp_?getWarnings@Task@U2@@UBE?AVQStringList@@XZ 10013710     U2Core:U2Core.dll
 0002:00000714       __imp_?hasSubtasksWithErrors@Task@U2@@UBE_NXZ 10013714     U2Core:U2Core.dll
 0002:00000718       __imp_?hasWarning@Task@U2@@UBE_NXZ 10013718     U2Core:U2Core.dll
 0002:0000071c       __imp_?isNotificationReport@Task@U2@@UBE_NXZ 1001371c     U2Core:U2Core.dll
 0002:00000720       __imp_?isReportingEnabled@Task@U2@@UBE_NXZ 10013720     U2Core:U2Core.dll
 0002:00000724       __imp_?isReportingSupported@Task@U2@@UBE_NXZ 10013724     U2Core:U2Core.dll
 0002:00000728       __imp_?isTopLevelTask@Task@U2@@UBE_NXZ 10013728     U2Core:U2Core.dll
 0002:0000072c       __imp_?metaObject@CreateAnnotationsTask@U2@@UBEPBUQMetaObject@@XZ 1001372c     U2Core:U2Core.dll
 0002:00000730       __imp_?onSubTaskFinished@Task@U2@@MAE?AV?$QList@PAVTask@U2@@@@PAV12@@Z 10013730     U2Core:U2Core.dll
 0002:00000734       __imp_?prepare@Task@U2@@UAEXXZ 10013734     U2Core:U2Core.dll
 0002:00000738       __imp_?propagateSubtaskError@Task@U2@@UAE_NXZ 10013738     U2Core:U2Core.dll
 0002:0000073c       __imp_?qt_metacall@CreateAnnotationsTask@U2@@UAEHW4Call@QMetaObject@@HPAPAX@Z 1001373c     U2Core:U2Core.dll
 0002:00000740       __imp_?qt_metacast@CreateAnnotationsTask@U2@@UAEPAXPBD@Z 10013740     U2Core:U2Core.dll
 0002:00000744       __imp_?report@CreateAnnotationsTask@U2@@UAE?AW4ReportResult@Task@2@XZ 10013744     U2Core:U2Core.dll
 0002:00000748       __imp_?report@Task@U2@@UAE?AW4ReportResult@12@XZ 10013748     U2Core:U2Core.dll
 0002:0000074c       __imp_?run@CreateAnnotationsTask@U2@@UAEXXZ 1001374c     U2Core:U2Core.dll
 0002:00000750       __imp_?run@Task@U2@@UAEXXZ 10013750     U2Core:U2Core.dll
 0002:00000754       __imp_?setCollectChildrensWarningsFlag@Task@U2@@UAEX_N@Z 10013754     U2Core:U2Core.dll
 0002:00000758       __imp_?setNoAutoDelete@Task@U2@@UAEX_N@Z 10013758     U2Core:U2Core.dll
 0002:0000075c       __imp_?setNotificationReport@Task@U2@@UAEX_N@Z 1001375c     U2Core:U2Core.dll
 0002:00000760       __imp_?setReportingEnabled@Task@U2@@UAEX_N@Z 10013760     U2Core:U2Core.dll
 0002:00000764       __imp_?setReportingSupported@Task@U2@@UAEX_N@Z 10013764     U2Core:U2Core.dll
 0002:00000768       __imp_?getSettings@AppContext@U2@@SAPAVSettings@2@XZ 10013768     U2Core:U2Core.dll
 0002:0000076c       __imp_?qt_metacast@Plugin@U2@@UAEPAXPBD@Z 1001376c     U2Core:U2Core.dll
 0002:00000770       __imp_?qt_metacall@Plugin@U2@@UAEHW4Call@QMetaObject@@HPAPAX@Z 10013770     U2Core:U2Core.dll
 0002:00000774       __imp_?staticMetaObject@Plugin@U2@@2UQMetaObject@@B 10013774     U2Core:U2Core.dll
 0002:00000778       __imp_?qt_metacast@Task@U2@@UAEPAXPBD@Z 10013778     U2Core:U2Core.dll
 0002:0000077c       __imp_?qt_metacall@Task@U2@@UAEHW4Call@QMetaObject@@HPAPAX@Z 1001377c     U2Core:U2Core.dll
 0002:00000780       __imp_?staticMetaObject@Task@U2@@2UQMetaObject@@B 10013780     U2Core:U2Core.dll
 0002:00000784       __imp_??0Logger@U2@@QAE@ABVQString@@@Z 10013784     U2Core:U2Core.dll
 0002:00000788       \177U2Core_NULL_THUNK_DATA 10013788     U2Core:U2Core.dll
 0002:0000078c       __imp_??0CreateAnnotationModel@U2@@QAE@XZ 1001378c     U2Gui:U2Gui.dll
 0002:00000790       __imp_?getAnnotationObject@CreateAnnotationModel@U2@@QBEPAVAnnotationTableObject@2@XZ 10013790     U2Gui:U2Gui.dll
 0002:00000794       __imp_??1CreateAnnotationModel@U2@@QAE@XZ 10013794     U2Gui:U2Gui.dll
 0002:00000798       __imp_??0CreateAnnotationWidgetController@U2@@QAE@ABVCreateAnnotationModel@1@PAVQObject@@W4AnnotationWidgetMode@01@@Z 10013798     U2Gui:U2Gui.dll
 0002:0000079c       __imp_?validate@CreateAnnotationWidgetController@U2@@QAE?AVQString@@XZ 1001379c     U2Gui:U2Gui.dll
 0002:000007a0       __imp_?prepareAnnotationObject@CreateAnnotationWidgetController@U2@@QAE_NXZ 100137a0     U2Gui:U2Gui.dll
 0002:000007a4       __imp_?getWidget@CreateAnnotationWidgetController@U2@@QBEPAVQWidget@@XZ 100137a4     U2Gui:U2Gui.dll
 0002:000007a8       __imp_??1CreateAnnotationWidgetController@U2@@UAE@XZ 100137a8     U2Gui:U2Gui.dll
 0002:000007ac       __imp_??0HelpButton@U2@@QAE@PAVQObject@@PAVQDialogButtonBox@@ABVQString@@@Z 100137ac     U2Gui:U2Gui.dll
 0002:000007b0       __imp_??1HelpButton@U2@@UAE@XZ 100137b0     U2Gui:U2Gui.dll
 0002:000007b4       __imp_?getWidget@GObjectView@U2@@QAEPAVQWidget@@XZ 100137b4     U2Gui:U2Gui.dll
 0002:000007b8       __imp_?metaObject@CreateAnnotationWidgetController@U2@@UBEPBUQMetaObject@@XZ 100137b8     U2Gui:U2Gui.dll
 0002:000007bc       __imp_?metaObject@HelpButton@U2@@UBEPBUQMetaObject@@XZ 100137bc     U2Gui:U2Gui.dll
 0002:000007c0       __imp_?qt_metacall@CreateAnnotationWidgetController@U2@@UAEHW4Call@QMetaObject@@HPAPAX@Z 100137c0     U2Gui:U2Gui.dll
 0002:000007c4       __imp_?qt_metacall@HelpButton@U2@@UAEHW4Call@QMetaObject@@HPAPAX@Z 100137c4     U2Gui:U2Gui.dll
 0002:000007c8       __imp_?qt_metacast@CreateAnnotationWidgetController@U2@@UAEPAXPBD@Z 100137c8     U2Gui:U2Gui.dll
 0002:000007cc       __imp_?qt_metacast@HelpButton@U2@@UAEPAXPBD@Z 100137cc     U2Gui:U2Gui.dll
 0002:000007d0       __imp_?sl_buttonClicked@HelpButton@U2@@MAEXXZ 100137d0     U2Gui:U2Gui.dll
 0002:000007d4       __imp_?getObjectView@GObjectViewAction@U2@@QBEPAVGObjectView@2@XZ 100137d4     U2Gui:U2Gui.dll
 0002:000007d8       __imp_??0GObjectViewWindowContext@U2@@QAE@PAVQObject@@ABVGObjectViewFactoryId@1@@Z 100137d8     U2Gui:U2Gui.dll
 0002:000007dc       __imp_??1GObjectViewWindowContext@U2@@UAE@XZ 100137dc     U2Gui:U2Gui.dll
 0002:000007e0       __imp_?buildMenu@GObjectViewWindowContext@U2@@MAEXPAVGObjectView@2@PAVQMenu@@@Z 100137e0     U2Gui:U2Gui.dll
 0002:000007e4       __imp_?canHandle@GObjectViewObjectHandler@U2@@UAE_NPAVGObjectView@2@PAVGObject@2@@Z 100137e4     U2Gui:U2Gui.dll
 0002:000007e8       __imp_?disconnectView@GObjectViewWindowContext@U2@@MAEXPAVGObjectView@2@@Z 100137e8     U2Gui:U2Gui.dll
 0002:000007ec       __imp_?init@GObjectViewWindowContext@U2@@UAEXXZ 100137ec     U2Gui:U2Gui.dll
 0002:000007f0       __imp_?onObjectAdded@GObjectViewObjectHandler@U2@@UAEXPAVGObjectView@2@PAVGObject@2@@Z 100137f0     U2Gui:U2Gui.dll
 0002:000007f4       __imp_?onObjectRemoved@GObjectViewWindowContext@U2@@UAEXPAVGObjectView@2@PAVGObject@2@@Z 100137f4     U2Gui:U2Gui.dll
 0002:000007f8       __imp_?sl_buildContextMenu@GObjectViewWindowContext@U2@@MAEXPAVGObjectView@2@PAVQMenu@@@Z 100137f8     U2Gui:U2Gui.dll
 0002:000007fc       __imp_?sl_buildStaticMenu@GObjectViewWindowContext@U2@@MAEXPAVGObjectView@2@PAVQMenu@@@Z 100137fc     U2Gui:U2Gui.dll
 0002:00000800       __imp_?sl_windowAdded@GObjectViewWindowContext@U2@@MAEXPAVMWMDIWindow@2@@Z 10013800     U2Gui:U2Gui.dll
 0002:00000804       __imp_?sl_windowClosing@GObjectViewWindowContext@U2@@MAEXPAVMWMDIWindow@2@@Z 10013804     U2Gui:U2Gui.dll
 0002:00000808       __imp_?staticMetaObject@GObjectViewAction@U2@@2UQMetaObject@@B 10013808     U2Gui:U2Gui.dll
 0002:0000080c       __imp_?qt_metacast@GObjectViewWindowContext@U2@@UAEPAXPBD@Z 1001380c     U2Gui:U2Gui.dll
 0002:00000810       __imp_?qt_metacall@GObjectViewWindowContext@U2@@UAEHW4Call@QMetaObject@@HPAPAX@Z 10013810     U2Gui:U2Gui.dll
 0002:00000814       __imp_?staticMetaObject@GObjectViewWindowContext@U2@@2UQMetaObject@@B 10013814     U2Gui:U2Gui.dll
 0002:00000818       \177U2Gui_NULL_THUNK_DATA  10013818     U2Gui:U2Gui.dll
 0002:0000081c       __imp_?tryAddObject@AnnotatedDNAView@U2@@QAE?AVQString@@PAVGObject@2@@Z 1001381c     U2View:U2View.dll
 0002:00000820       __imp_??1GSequenceGraphWindowData@U2@@UAE@XZ 10013820     U2View:U2View.dll
 0002:00000824       __imp_??0GSequenceGraphDrawer@U2@@QAE@PAVGSequenceGraphView@1@ABVGSequenceGraphWindowData@1@V?$QMap@VQString@@VQColor@@@@@Z 10013824     U2View:U2View.dll
 0002:00000828       __imp_??1GSequenceGraphDrawer@U2@@UAE@XZ 10013828     U2View:U2View.dll
 0002:0000082c       __imp_??0GSequenceGraphData@U2@@QAE@ABVQString@@@Z 1001382c     U2View:U2View.dll
 0002:00000830       __imp_??1GSequenceGraphData@U2@@UAE@XZ 10013830     U2View:U2View.dll
 0002:00000834       __imp_??0GSequenceGraphFactory@U2@@QAE@ABVQString@@PAVQObject@@@Z 10013834     U2View:U2View.dll
 0002:00000838       __imp_??1GSequenceGraphFactory@U2@@UAE@XZ 10013838     U2View:U2View.dll
 0002:0000083c       __imp_?draw@GSequenceGraphDrawer@U2@@UAEXAAVQPainter@@ABV?$QList@V?$QSharedPointer@VGSequenceGraphData@U2@@@@@@ABVQRect@@@Z 1001383c     U2View:U2View.dll
 0002:00000840       __imp_?metaObject@GSequenceGraphDrawer@U2@@UBEPBUQMetaObject@@XZ 10013840     U2View:U2View.dll
 0002:00000844       __imp_?qt_metacall@GSequenceGraphDrawer@U2@@UAEHW4Call@QMetaObject@@HPAPAX@Z 10013844     U2View:U2View.dll
 0002:00000848       __imp_?qt_metacast@GSequenceGraphDrawer@U2@@UAEPAXPBD@Z 10013848     U2View:U2View.dll
 0002:0000084c       __imp_?showSettingsDialog@GSequenceGraphDrawer@U2@@UAEXXZ 1001384c     U2View:U2View.dll
 0002:00000850       __imp_??_7GSequenceGraphWindowData@U2@@6B@ 10013850     U2View:U2View.dll
 0002:00000854       __imp_??1GSequenceGraphAlgorithm@U2@@UAE@XZ 10013854     U2View:U2View.dll
 0002:00000858       __imp_??0GSequenceGraphAlgorithm@U2@@IAE@XZ 10013858     U2View:U2View.dll
 0002:0000085c       __imp_?getSequenceData@GSequenceGraphAlgorithm@U2@@IAEABVQByteArray@@PAVU2SequenceObject@2@AAVU2OpStatus@2@@Z 1001385c     U2View:U2View.dll
 0002:00000860       __imp_?getNumSteps@GSequenceGraphUtils@U2@@SAHABVU2Region@2@HH@Z 10013860     U2View:U2View.dll
 0002:00000864       __imp_?getAlphabet@SequenceObjectContext@U2@@QBEPBVDNAAlphabet@2@XZ 10013864     U2View:U2View.dll
 0002:00000868       __imp_??0ADVGlobalAction@U2@@QAE@PAVAnnotatedDNAView@1@ABVQIcon@@ABVQString@@HV?$QFlags@W4ADVGlobalActionFlag@U2@@@@@Z 10013868     U2View:U2View.dll
 0002:0000086c       __imp_?addAlphabetFilter@ADVGlobalAction@U2@@QAEXW4DNAAlphabetType@@@Z 1001386c     U2View:U2View.dll
 0002:00000870       __imp_??1ADVGlobalAction@U2@@UAE@XZ 10013870     U2View:U2View.dll
 0002:00000874       __imp_?getSequenceWidgets@AnnotatedDNAView@U2@@QBE?BV?$QList@PAVADVSequenceWidget@U2@@@@XZ 10013874     U2View:U2View.dll
 0002:00000878       __imp_?getSequenceInFocus@AnnotatedDNAView@U2@@QBEPAVADVSequenceObjectContext@2@XZ 10013878     U2View:U2View.dll
 0002:0000087c       __imp_?getSequenceContext@ADVSingleSequenceWidget@U2@@QBEPAVADVSequenceObjectContext@2@XZ 1001387c     U2View:U2View.dll
 0002:00000880       __imp_?getSequenceObject@ADVSingleSequenceWidget@U2@@QBEPAVU2SequenceObject@2@XZ 10013880     U2View:U2View.dll
 0002:00000884       __imp_??0GraphAction@U2@@QAE@PAVGSequenceGraphFactory@1@@Z 10013884     U2View:U2View.dll
 0002:00000888       __imp_??1GraphAction@U2@@UAE@XZ 10013888     U2View:U2View.dll
 0002:0000088c       __imp_?addGraphAction@GraphMenuAction@U2@@SAXPAVADVSequenceObjectContext@2@PAVGraphAction@2@@Z 1001388c     U2View:U2View.dll
 0002:00000890       __imp_?metaObject@ADVGlobalAction@U2@@UBEPBUQMetaObject@@XZ 10013890     U2View:U2View.dll
 0002:00000894       __imp_?metaObject@GraphAction@U2@@UBEPBUQMetaObject@@XZ 10013894     U2View:U2View.dll
 0002:00000898       __imp_?qt_metacall@ADVGlobalAction@U2@@UAEHW4Call@QMetaObject@@HPAPAX@Z 10013898     U2View:U2View.dll
 0002:0000089c       __imp_?qt_metacall@GraphAction@U2@@UAEHW4Call@QMetaObject@@HPAPAX@Z 1001389c     U2View:U2View.dll
 0002:000008a0       __imp_?qt_metacast@ADVGlobalAction@U2@@UAEPAXPBD@Z 100138a0     U2View:U2View.dll
 0002:000008a4       __imp_?qt_metacast@GraphAction@U2@@UAEPAXPBD@Z 100138a4     U2View:U2View.dll
 0002:000008a8       __imp_?staticMetaObject@AnnotatedDNAView@U2@@2UQMetaObject@@B 100138a8     U2View:U2View.dll
 0002:000008ac       __imp_?staticMetaObject@ADVSingleSequenceWidget@U2@@2UQMetaObject@@B 100138ac     U2View:U2View.dll
 0002:000008b0       __imp_?staticMetaObject@ADVSequenceWidget@U2@@2UQMetaObject@@B 100138b0     U2View:U2View.dll
 0002:000008b4       \177U2View_NULL_THUNK_DATA 100138b4     U2View:U2View.dll
 0002:000008b8       ___xc_a                    100138b8     MSVCRT:cinitexe.obj
 0002:00000bdc       ___xc_z                    10013bdc     MSVCRT:cinitexe.obj
 0002:00000be0       ___xi_a                    10013be0     MSVCRT:cinitexe.obj
 0002:00000bec       ___xi_z                    10013bec     MSVCRT:cinitexe.obj
 0002:00000c2c       ??_7error_category@std@@6B@ 10013c2c     DNAFlexDialog.obj
 0002:00000c48       ??_7_Generic_error_category@std@@6B@ 10013c48     DNAFlexDialog.obj
 0002:00000c60       ??_C@_07DCLBNMLN@generic?$AA@ 10013c60     DNAFlexDialog.obj
 0002:00000c68       ??_C@_0O@BFJCFAAK@unknown?5error?$AA@ 10013c68     DNAFlexDialog.obj
 0002:00000c7c       ??_7_Iostream_error_category@std@@6B@ 10013c7c     DNAFlexDialog.obj
 0002:00000c94       ??_C@_08LLGCOLLL@iostream?$AA@ 10013c94     DNAFlexDialog.obj
 0002:00000ca0       ??_C@_0BG@PADBLCHM@iostream?5stream?5error?$AA@ 10013ca0     DNAFlexDialog.obj
 0002:00000cbc       ??_7_System_error_category@std@@6B@ 10013cbc     DNAFlexDialog.obj
 0002:00000cd4       ??_C@_06FHFOAHML@system?$AA@ 10013cd4     DNAFlexDialog.obj
 0002:00000ce4       ??_SQWidget@@6BQObject@@@  10013ce4     DNAFlexDialog.obj
 0002:00000d9c       ??_SQWidget@@6BQPaintDevice@@@ 10013d9c     DNAFlexDialog.obj
 0002:00000dbc       ??_SQDialogButtonBox@@6BQObject@@@ 10013dbc     DNAFlexDialog.obj
 0002:00000e74       ??_SQDialogButtonBox@@6BQPaintDevice@@@ 10013e74     DNAFlexDialog.obj
 0002:00000e94       ??_SQSpinBox@@6BQObject@@@ 10013e94     DNAFlexDialog.obj
 0002:00000f68       ??_SQSpinBox@@6BQPaintDevice@@@ 10013f68     DNAFlexDialog.obj
 0002:00000f8c       ??_SQDoubleSpinBox@@6BQObject@@@ 10013f8c     DNAFlexDialog.obj
 0002:00001060       ??_SQDoubleSpinBox@@6BQPaintDevice@@@ 10014060     DNAFlexDialog.obj
 0002:00001084       ??_SQSpacerItem@@6B@       10014084     DNAFlexDialog.obj
 0002:000010cc       ??_SQHBoxLayout@@6BQObject@@@ 100140cc     DNAFlexDialog.obj
 0002:00001114       ??_SQHBoxLayout@@6BQLayoutItem@@@ 10014114     DNAFlexDialog.obj
 0002:0000115c       ??_SQVBoxLayout@@6BQObject@@@ 1001415c     DNAFlexDialog.obj
 0002:000011a4       ??_SQVBoxLayout@@6BQLayoutItem@@@ 100141a4     DNAFlexDialog.obj
 0002:000011ec       ??_SQGridLayout@@6BQObject@@@ 100141ec     DNAFlexDialog.obj
 0002:00001234       ??_SQGridLayout@@6BQLayoutItem@@@ 10014234     DNAFlexDialog.obj
 0002:0000127c       ??_SQGroupBox@@6BQObject@@@ 1001427c     DNAFlexDialog.obj
 0002:00001334       ??_SQGroupBox@@6BQPaintDevice@@@ 10014334     DNAFlexDialog.obj
 0002:00001354       ??_SQTabWidget@@6BQObject@@@ 10014354     DNAFlexDialog.obj
 0002:00001414       ??_SQTabWidget@@6BQPaintDevice@@@ 10014414     DNAFlexDialog.obj
 0002:00001434       ??_SQLabel@@6BQObject@@@   10014434     DNAFlexDialog.obj
 0002:000014ec       ??_SQLabel@@6BQPaintDevice@@@ 100144ec     DNAFlexDialog.obj
 0002:0000150c       ??_SQPushButton@@6BQObject@@@ 1001450c     DNAFlexDialog.obj
 0002:000015d0       ??_SQPushButton@@6BQPaintDevice@@@ 100145d0     DNAFlexDialog.obj
 0002:000015ec       ??_C@_09DMINLBG@1accept?$CI?$CJ?$AA@ 100145ec     DNAFlexDialog.obj
 0002:000015f8       ??_C@_0M@MBACPLBI@2accepted?$CI?$CJ?$AA@ 100145f8     DNAFlexDialog.obj
 0002:00001604       ??_C@_09OCDCAEKE@1reject?$CI?$CJ?$AA@ 10014604     DNAFlexDialog.obj
 0002:00001610       ??_C@_0M@BJNBJJN@2rejected?$CI?$CJ?$AA@ 10014610     DNAFlexDialog.obj
 0002:0000161c       ??_C@_0BA@BDPBBAID@DNA?5Flexibility?$AA@ 1001461c     DNAFlexDialog.obj
 0002:0000162c       ??_C@_0O@CFLBIJAJ@DNAFlexDialog?$AA@ 1001462c     DNAFlexDialog.obj
 0002:00001640       ??_C@_0EO@HABLBFDO@The?5DNA?5Flexibility?5plugin?5allow@ 10014640     DNAFlexDialog.obj
 0002:00001690       ??_C@_0CG@KLJMPHCO@High?5DNA?5Flexibility?5Regions?5Set@ 10014690     DNAFlexDialog.obj
 0002:000016b8       ??_C@_0M@LHOJMPLD@Window?5size?$AA@ 100146b8     DNAFlexDialog.obj
 0002:000016c4       ??_C@_0M@DFFFECKI@Window?5step?$AA@ 100146c4     DNAFlexDialog.obj
 0002:000016d0       ??_C@_09HLCHFPPJ@Threshold?$AA@ 100146d0     DNAFlexDialog.obj
 0002:000016dc       ??_C@_0BC@JOJMJBPP@Remember?5Settings?$AA@ 100146dc     DNAFlexDialog.obj
 0002:000016f0       ??_C@_0BB@KHHOADPF@Restore?5Defaults?$AA@ 100146f0     DNAFlexDialog.obj
 0002:00001704       ??_C@_0BA@OPIBFEIO@Search?5Settings?$AA@ 10014704     DNAFlexDialog.obj
 0002:00001714       ??_C@_06PFDLEJLJ@Output?$AA@ 10014714     DNAFlexDialog.obj
 0002:00001a98       ??_7DNAFlexDialog@U2@@6BQObject@@@ 10014a98     DNAFlexDialog.obj
 0002:00001b64       ??_7DNAFlexDialog@U2@@6BQPaintDevice@@@ 10014b64     DNAFlexDialog.obj
 0002:00001b84       ??_7?$AbstractId@H@U2@@6B@ 10014b84     DNAFlexDialog.obj
 0002:00001b90       ??_7AbstractInt32Id@U2@@6B@ 10014b90     DNAFlexDialog.obj
 0002:00001b9c       ??_7ServiceType@U2@@6B@    10014b9c     DNAFlexDialog.obj
 0002:00001ba4       ??_C@_0L@JLHNEGIN@Algorithms?$AA@ 10014ba4     DNAFlexDialog.obj
 0002:00001bb0       ??_C@_07PGLPGHFC@Console?$AA@ 10014bb0     DNAFlexDialog.obj
 0002:00001bb8       ??_C@_0O@BOFHOPCF@Core?5Services?$AA@ 10014bb8     DNAFlexDialog.obj
 0002:00001bc8       ??_C@_0N@PPADAKBM@Input?1Output?$AA@ 10014bc8     DNAFlexDialog.obj
 0002:00001bd8       ??_C@_0M@KPPBKPKK@Performance?$AA@ 10014bd8     DNAFlexDialog.obj
 0002:00001be4       ??_C@_07BFDHHBBI@Scripts?$AA@ 10014be4     DNAFlexDialog.obj
 0002:00001bec       ??_C@_05EEGKELMG@Tasks?$AA@ 10014bec     DNAFlexDialog.obj
 0002:00001bf4       ??_C@_0P@NIIOBHGA@User?5Interface?$AA@ 10014bf4     DNAFlexDialog.obj
 0002:00001c04       ??_C@_0N@JINCGGMN@User?5Actions?$AA@ 10014c04     DNAFlexDialog.obj
 0002:00001c18       ??_SCreateAnnotationWidgetController@U2@@6B@ 10014c18     DNAFlexDialog.obj
 0002:00001c48       ??_SHelpButton@U2@@6B@     10014c48     DNAFlexDialog.obj
 0002:00001c78       ??_C@_08CCGADMHE@23331160?$AA@ 10014c78     DNAFlexDialog.obj
 0002:00001c84       ??_C@_06KKEGOPHO@Search?$AA@ 10014c84     DNAFlexDialog.obj
 0002:00001c8c       ??_C@_06FMBNCPDL@Cancel?$AA@ 10014c8c     DNAFlexDialog.obj
 0002:00001c94       ??_C@_08MDHJEEGA@dna_flex?$AA@ 10014c94     DNAFlexDialog.obj
 0002:00001ca0       ??_C@_0BM@CABIODPE@?3?1ugene?1images?1ugene_16?4png?$AA@ 10014ca0     DNAFlexDialog.obj
 0002:00001cbc       ??_C@_0BP@HHOAHIGB@1sl_spinWindowSizeChanged?$CIint?$CJ?$AA@ 10014cbc     DNAFlexDialog.obj
 0002:00001cdc       ??_C@_0BD@OIBDOPAP@2valueChanged?$CIint?$CJ?$AA@ 10014cdc     DNAFlexDialog.obj
 0002:00001cf0       ??_C@_0BP@GKHGAKHF@1sl_spinWindowStepChanged?$CIint?$CJ?$AA@ 10014cf0     DNAFlexDialog.obj
 0002:00001d10       ??_C@_0CB@LDKCGKCJ@1sl_spinThresholdChanged?$CIdouble?$CJ@ 10014d10     DNAFlexDialog.obj
 0002:00001d34       ??_C@_0BG@PEKDJDCL@2valueChanged?$CIdouble?$CJ?$AA@ 10014d34     DNAFlexDialog.obj
 0002:00001d4c       ??_C@_0BH@EANHGBNK@1sl_rememberSettings?$CI?$CJ?$AA@ 10014d4c     DNAFlexDialog.obj
 0002:00001d64       ??_C@_0L@OELOHDKG@2clicked?$CI?$CJ?$AA@ 10014d64     DNAFlexDialog.obj
 0002:00001d70       ??_C@_0BG@KLMBGOPJ@1sl_defaultSettings?$CI?$CJ?$AA@ 10014d70     DNAFlexDialog.obj
 0002:00001d88       ??_C@_0BF@HHBALMNJ@1sl_updateSizes?$CIint?$CJ?$AA@ 10014d88     DNAFlexDialog.obj
 0002:00001da0       ??_C@_0BF@DPFPPAJM@2currentChanged?$CIint?$CJ?$AA@ 10014da0     DNAFlexDialog.obj
 0002:00001db8       ??_C@_05NAOIJFC@Error?$AA@ 10014db8     DNAFlexDialog.obj
 0002:00001dc0       ??_C@_0DK@NFDOGBNG@Cannot?5create?5an?5annotation?5obje@ 10014dc0     DNAFlexDialog.obj
 0002:00001dfc       ??_C@_0BA@JFNIOLAK@string?5too?5long?$AA@ 10014dfc     DNAFlexDialog.obj
 0002:00001e0c       ??_C@_0BI@CFPLBAOH@invalid?5string?5position?$AA@ 10014e0c     DNAFlexDialog.obj
 0002:00001e28       __real@3fb999999999999a    10014e28     DNAFlexDialog.obj
 0002:00001e30       __real@402b666666666666    10014e30     DNAFlexDialog.obj
 0002:00001e38       __real@40f86a0000000000    10014e38     DNAFlexDialog.obj
 0002:00001e40       ?DEFAULT_WINDOW_SIZE@DNAFlexGraphFactory@U2@@0_JB 10014e40     DNAFlexGraph.obj
 0002:00001e48       ?DEFAULT_WINDOW_STEP@DNAFlexGraphFactory@U2@@0HB 10014e48     DNAFlexGraph.obj
 0002:00001e50       ??_SGSequenceGraphDrawer@U2@@6B@ 10014e50     DNAFlexGraph.obj
 0002:00001e88       ??_SGSequenceGraphData@U2@@6B@ 10014e88     DNAFlexGraph.obj
 0002:00001e90       ??_7DNAFlexGraphFactory@U2@@6B@ 10014e90     DNAFlexGraph.obj
 0002:00001ecc       ??_7DNAFlexGraphAlgorithm@U2@@6B@ 10014ecc     DNAFlexGraphAlgorithm.obj
 0002:00001ed8       ??_C@_0KM@JMOEOFJH@UGENE?5ran?5out?5of?5memory?5during?5t@ 10014ed8     DNAFlexGraphAlgorithm.obj
 0002:00001f88       ??_C@_0EA@LDCPCFPO@Internal?5error?5occurred?5during?5t@ 10014f88     DNAFlexGraphAlgorithm.obj
 0002:00001fcc       ??_SADVGlobalAction@U2@@6B@ 10014fcc     DNAFlexPlugin.obj
 0002:00001ffc       ??_SGraphAction@U2@@6B@    10014ffc     DNAFlexPlugin.obj
 0002:0000202c       ??_7DNAFlexPlugin@U2@@6B@  1001502c     DNAFlexPlugin.obj
 0002:0000205c       ??_7DNAFlexViewContext@U2@@6BQObject@@@ 1001505c     DNAFlexPlugin.obj
 0002:000020ac       ??_7DNAFlexViewContext@U2@@6BGObjectViewObjectHandler@1@@ 100150ac     DNAFlexPlugin.obj
 0002:000020c0       ??_C@_0ED@PPEFEIIH@Searches?5a?5DNA?5sequence?5for?5regi@ 100150c0     DNAFlexPlugin.obj
 0002:00002104       ??_C@_0BB@JDMPMKOK@AnnotatedDNAView?$AA@ 10015104     DNAFlexPlugin.obj
 0002:00002118       ??_C@_0CK@IGBIANDN@Trying?5to?5recover?5from?5error?3?5?$CF1@ 10015118     DNAFlexPlugin.obj
 0002:00002144       ??_C@_0CD@BCNPNFBL@no?5sequence?5to?5perform?5flex?5sear@ 10015144     DNAFlexPlugin.obj
 0002:00002168       ??_C@_0BG@PGEOMCED@src?2DNAFlexPlugin?4cpp?$AA@ 10015168     DNAFlexPlugin.obj
 0002:00002180       ??_C@_0DN@JINBBPKK@alphabet?5is?5not?5nucleic?0?5dialog?5@ 10015180     DNAFlexPlugin.obj
 0002:000021c0       ??_C@_0EH@KNNEIBDB@Unsupported?5sequence?5alphabet?0?5o@ 100151c0     DNAFlexPlugin.obj
 0002:00002208       ??_C@_0CM@JOICIJIL@1sl_sequenceWidgetAdded?$CIADVSeque@ 10015208     DNAFlexPlugin.obj
 0002:00002234       ??_C@_0CM@KILGFMLI@2si_sequenceWidgetAdded?$CIADVSeque@ 10015234     DNAFlexPlugin.obj
 0002:00002260       ??_C@_0CF@KLKCAPJF@Find?5high?5DNA?5flexibility?5region@ 10015260     DNAFlexPlugin.obj
 0002:00002288       ??_C@_0CI@JBJGADIE@?3dna_flexibility?1images?1flexibil@ 10015288     DNAFlexPlugin.obj
 0002:000022b0       ??_C@_0BI@LBDHJHP@1sl_showDNAFlexDialog?$CI?$CJ?$AA@ 100152b0     DNAFlexPlugin.obj
 0002:000022c8       ??_C@_0N@NBJIAFIH@2triggered?$CI?$CJ?$AA@ 100152c8     DNAFlexPlugin.obj
 0002:000022d8       ??_C@_0DN@LGKKGEKM@1sl_updateGraphView?$CIconst?5QStrin@ 100152d8     DNAFlexPlugin.obj
 0002:00002318       ??_C@_0DN@CHPAKHJJ@2si_updateGraphView?$CIconst?5QStrin@ 10015318     DNAFlexPlugin.obj
 0002:0000235c       ??_SCreateAnnotationsTask@U2@@6B@ 1001535c     DNAFlexTask.obj
 0002:000023ec       ??_7DNAFlexTask@U2@@6B@    100153ec     DNAFlexTask.obj
 0002:00002478       ??_C@_0BF@CLGMHCJC@DNA?5Flexibility?5task?$AA@ 10015478     DNAFlexTask.obj
 0002:00002490       ??_C@_0CJ@IJAHNBBN@The?5annotations?5object?5is?5not?5av@ 10015490     DNAFlexTask.obj
 0002:000024bc       ??_C@_0CJ@OPLDJMEN@Failed?5to?5cast?5FindHighFlexRegio@ 100154bc     DNAFlexTask.obj
 0002:000024e8       ??_C@_0BE@BLMFFGOI@src?2DNAFlexTask?4cpp?$AA@ 100154e8     DNAFlexTask.obj
 0002:000024fc       ??_C@_0BC@KPNFEHNH@average_threshold?$AA@ 100154fc     DNAFlexTask.obj
 0002:00002510       ??_C@_0P@PJNEAPDK@windows_number?$AA@ 10015510     DNAFlexTask.obj
 0002:00002520       ??_C@_0BA@MABCDBAE@total_threshold?$AA@ 10015520     DNAFlexTask.obj
 0002:00002534       ??_7FindHighFlexRegionsListener@U2@@6B@ 10015534     FindHighFlexRegions.obj
 0002:00002540       ??_7FindHighFlexRegions@U2@@6BTask@1@@ 10015540     FindHighFlexRegions.obj
 0002:000025d0       ??_7FindHighFlexRegions@U2@@6BFindHighFlexRegionsListener@1@@ 100155d0     FindHighFlexRegions.obj
 0002:000025d8       ??_C@_0CO@DHEOMNIA@Searching?5for?5regions?5of?5high?5DN@ 100155d8     FindHighFlexRegions.obj
 0002:00002608       ??_C@_0EA@NCFDHEHA@Internal?5error?3?5a?5user?5is?5not?5al@ 10015608     FindHighFlexRegionsAlgorithm.obj
 0002:00002648       ??_C@_0CF@CMKALEHM@src?2FindHighFlexRegionsAlgorithm@ 10015648     FindHighFlexRegionsAlgorithm.obj
 0002:00002670       ??_C@_0EA@FAOPPJGL@Internal?5error?3?5a?5user?5is?5not?5al@ 10015670     FindHighFlexRegionsAlgorithm.obj
 0002:000026b0       ??_C@_0FB@DICBKBMH@Illegal?5combination?5of?5nucleotid@ 100156b0     FindHighFlexRegionsAlgorithm.obj
 0002:00002704       ??_C@_0CO@OENHKIHA@FindHighFlexRegionsListener?5is?5n@ 10015704     FindHighFlexRegionsAlgorithm.obj
 0002:00002738       __real@0000000000000000    10015738     FindHighFlexRegionsAlgorithm.obj
 0002:00002740       __real@401ccccccccccccd    10015740     FindHighFlexRegionsAlgorithm.obj
 0002:00002748       __real@401e666666666666    10015748     FindHighFlexRegionsAlgorithm.obj
 0002:00002750       __real@4020666666666666    10015750     FindHighFlexRegionsAlgorithm.obj
 0002:00002758       __real@402199999999999a    10015758     FindHighFlexRegionsAlgorithm.obj
 0002:00002760       __real@4021cccccccccccd    10015760     FindHighFlexRegionsAlgorithm.obj
 0002:00002768       __real@4025cccccccccccd    10015768     FindHighFlexRegionsAlgorithm.obj
 0002:00002770       __real@4026333333333333    10015770     FindHighFlexRegionsAlgorithm.obj
 0002:00002778       __real@4029000000000000    10015778     FindHighFlexRegionsAlgorithm.obj
 0002:00002780       __real@402d333333333333    10015780     FindHighFlexRegionsAlgorithm.obj
 0002:00002788       __real@4039000000000000    10015788     FindHighFlexRegionsAlgorithm.obj
 0002:00002790       ?DEFAULT_THRESHOLD@HighFlexSettings@U2@@0NB 10015790     HighFlexSettings.obj
 0002:00002798       ??_C@_0BD@BIJPCFFL@high_flex_settings?$AA@ 10015798     HighFlexSettings.obj
 0002:000027ac       ??_C@_0M@FFKMKLFP@window_size?$AA@ 100157ac     HighFlexSettings.obj
 0002:000027b8       ??_C@_0M@NHBACGEE@window_step?$AA@ 100157b8     HighFlexSettings.obj
 0002:000027c4       ??_C@_09DEHKFMCJ@threshold?$AA@ 100157c4     HighFlexSettings.obj
 0002:000027d0       ??_C@_01KMDKNFGN@?1?$AA@   100157d0     HighFlexSettings.obj
 0002:000027d8       ??_C@_0EN@JHPMHDE@Invalid?5high?5flex?5setting?5window@ 100157d8     HighFlexSettings.obj
 0002:00002828       ??_C@_0EN@BJPOACCB@Invalid?5high?5flex?5setting?5window@ 10015828     HighFlexSettings.obj
 0002:00002878       ??_C@_0EL@DEIJCEFI@Invalid?5high?5flex?5setting?5thresh@ 10015878     HighFlexSettings.obj
 0002:00002acc       ??_C@_0BB@LNHHLFIA@Ui_DNAFlexDialog?$AA@ 10015acc     moc_DNAFlexDialog.obj
 0002:00002d84       ??_C@_0BM@LOIBHFBJ@FindHighFlexRegionsListener?$AA@ 10015d84     moc_FindHighFlexRegions.obj
 0002:0000301c       ?value@?$integral_constant@_N$0A@@std@@2_NB 1001601c     MSVCRT:ti_inst.obj
 0002:0000301d       ?value@?$integral_constant@_N$00@std@@2_NB 1001601d     MSVCRT:ti_inst.obj
 0002:00003024       ??_7type_info@@6B@         10016024     MSVCRT:ti_inst.obj
 0002:00003028       __pDefaultRawDllMain       10016028     MSVCRT:crtdll.obj
 0002:00003028       __pRawDllMain              10016028     MSVCRT:crtdll.obj
 0002:00003034       ?ProcessDetach@NativeDll@<CrtImplementationDetails>@@0IB 10016034     MSVCRT:initsect.obj
 0002:00003038       ?ProcessAttach@NativeDll@<CrtImplementationDetails>@@0IB 10016038     MSVCRT:initsect.obj
 0002:0000303c       ?ThreadAttach@NativeDll@<CrtImplementationDetails>@@0IB 1001603c     MSVCRT:initsect.obj
 0002:00003040       ?ThreadDetach@NativeDll@<CrtImplementationDetails>@@0IB 10016040     MSVCRT:initsect.obj
 0002:00003044       ?ProcessVerifier@NativeDll@<CrtImplementationDetails>@@0IB 10016044     MSVCRT:initsect.obj
 0002:00003048       __load_config_used         10016048     MSVCRT:loadcfg.obj
 0002:00003108       ??_R4error_category@std@@6B@ 10016108     DNAFlexDialog.obj
 0002:0000311c       ??_R3error_category@std@@8 1001611c     DNAFlexDialog.obj
 0002:0000312c       ??_R2error_category@std@@8 1001612c     DNAFlexDialog.obj
 0002:00003134       ??_R1A@?0A@EA@error_category@std@@8 10016134     DNAFlexDialog.obj
 0002:00003150       ??_R4_Generic_error_category@std@@6B@ 10016150     DNAFlexDialog.obj
 0002:00003164       ??_R3_Generic_error_category@std@@8 10016164     DNAFlexDialog.obj
 0002:00003174       ??_R2_Generic_error_category@std@@8 10016174     DNAFlexDialog.obj
 0002:00003180       ??_R1A@?0A@EA@_Generic_error_category@std@@8 10016180     DNAFlexDialog.obj
 0002:0000319c       ??_R4_Iostream_error_category@std@@6B@ 1001619c     DNAFlexDialog.obj
 0002:000031b0       ??_R3_Iostream_error_category@std@@8 100161b0     DNAFlexDialog.obj
 0002:000031c0       ??_R2_Iostream_error_category@std@@8 100161c0     DNAFlexDialog.obj
 0002:000031d0       ??_R1A@?0A@EA@_Iostream_error_category@std@@8 100161d0     DNAFlexDialog.obj
 0002:000031ec       ??_R4_System_error_category@std@@6B@ 100161ec     DNAFlexDialog.obj
 0002:00003200       ??_R3_System_error_category@std@@8 10016200     DNAFlexDialog.obj
 0002:00003210       ??_R2_System_error_category@std@@8 10016210     DNAFlexDialog.obj
 0002:00003220       ??_R1A@?0A@EA@_System_error_category@std@@8 10016220     DNAFlexDialog.obj
 0002:0000323c       ??_R4QWidget@@6BQObject@@@ 1001623c     DNAFlexDialog.obj
 0002:00003250       ??_R3QWidget@@8            10016250     DNAFlexDialog.obj
 0002:00003260       ??_R2QWidget@@8            10016260     DNAFlexDialog.obj
 0002:00003270       ??_R1A@?0A@EA@QWidget@@8   10016270     DNAFlexDialog.obj
 0002:0000328c       ??_R1A@?0A@EA@QObject@@8   1001628c     DNAFlexDialog.obj
 0002:000032a8       ??_R3QObject@@8            100162a8     DNAFlexDialog.obj
 0002:000032b8       ??_R2QObject@@8            100162b8     DNAFlexDialog.obj
 0002:000032c0       ??_R17?0A@EA@QPaintDevice@@8 100162c0     DNAFlexDialog.obj
 0002:000032dc       ??_R3QPaintDevice@@8       100162dc     DNAFlexDialog.obj
 0002:000032ec       ??_R2QPaintDevice@@8       100162ec     DNAFlexDialog.obj
 0002:000032f4       ??_R1A@?0A@EA@QPaintDevice@@8 100162f4     DNAFlexDialog.obj
 0002:00003310       ??_R4QWidget@@6BQPaintDevice@@@ 10016310     DNAFlexDialog.obj
 0002:00003324       ??_R4QPushButton@@6BQObject@@@ 10016324     DNAFlexDialog.obj
 0002:00003338       ??_R3QPushButton@@8        10016338     DNAFlexDialog.obj
 0002:00003348       ??_R2QPushButton@@8        10016348     DNAFlexDialog.obj
 0002:00003360       ??_R1A@?0A@EA@QPushButton@@8 10016360     DNAFlexDialog.obj
 0002:0000337c       ??_R1A@?0A@EA@QAbstractButton@@8 1001637c     DNAFlexDialog.obj
 0002:00003398       ??_R3QAbstractButton@@8    10016398     DNAFlexDialog.obj
 0002:000033a8       ??_R2QAbstractButton@@8    100163a8     DNAFlexDialog.obj
 0002:000033bc       ??_R4QPushButton@@6BQPaintDevice@@@ 100163bc     DNAFlexDialog.obj
 0002:000033d0       ??_R4QDialogButtonBox@@6BQObject@@@ 100163d0     DNAFlexDialog.obj
 0002:000033e4       ??_R3QDialogButtonBox@@8   100163e4     DNAFlexDialog.obj
 0002:000033f4       ??_R2QDialogButtonBox@@8   100163f4     DNAFlexDialog.obj
 0002:00003408       ??_R1A@?0A@EA@QDialogButtonBox@@8 10016408     DNAFlexDialog.obj
 0002:00003424       ??_R4QDialogButtonBox@@6BQPaintDevice@@@ 10016424     DNAFlexDialog.obj
 0002:00003438       ??_R4QSpinBox@@6BQObject@@@ 10016438     DNAFlexDialog.obj
 0002:0000344c       ??_R3QSpinBox@@8           1001644c     DNAFlexDialog.obj
 0002:0000345c       ??_R2QSpinBox@@8           1001645c     DNAFlexDialog.obj
 0002:00003474       ??_R1A@?0A@EA@QSpinBox@@8  10016474     DNAFlexDialog.obj
 0002:00003490       ??_R1A@?0A@EA@QAbstractSpinBox@@8 10016490     DNAFlexDialog.obj
 0002:000034ac       ??_R3QAbstractSpinBox@@8   100164ac     DNAFlexDialog.obj
 0002:000034bc       ??_R2QAbstractSpinBox@@8   100164bc     DNAFlexDialog.obj
 0002:000034d0       ??_R4QSpinBox@@6BQPaintDevice@@@ 100164d0     DNAFlexDialog.obj
 0002:000034e4       ??_R4QDoubleSpinBox@@6BQObject@@@ 100164e4     DNAFlexDialog.obj
 0002:000034f8       ??_R3QDoubleSpinBox@@8     100164f8     DNAFlexDialog.obj
 0002:00003508       ??_R2QDoubleSpinBox@@8     10016508     DNAFlexDialog.obj
 0002:00003520       ??_R1A@?0A@EA@QDoubleSpinBox@@8 10016520     DNAFlexDialog.obj
 0002:0000353c       ??_R4QDoubleSpinBox@@6BQPaintDevice@@@ 1001653c     DNAFlexDialog.obj
 0002:00003550       ??_R4QSpacerItem@@6B@      10016550     DNAFlexDialog.obj
 0002:00003564       ??_R3QSpacerItem@@8        10016564     DNAFlexDialog.obj
 0002:00003574       ??_R2QSpacerItem@@8        10016574     DNAFlexDialog.obj
 0002:00003580       ??_R1A@?0A@EA@QSpacerItem@@8 10016580     DNAFlexDialog.obj
 0002:0000359c       ??_R1A@?0A@EA@QLayoutItem@@8 1001659c     DNAFlexDialog.obj
 0002:000035b8       ??_R3QLayoutItem@@8        100165b8     DNAFlexDialog.obj
 0002:000035c8       ??_R2QLayoutItem@@8        100165c8     DNAFlexDialog.obj
 0002:000035d0       ??_R4QHBoxLayout@@6BQObject@@@ 100165d0     DNAFlexDialog.obj
 0002:000035e4       ??_R3QHBoxLayout@@8        100165e4     DNAFlexDialog.obj
 0002:000035f4       ??_R2QHBoxLayout@@8        100165f4     DNAFlexDialog.obj
 0002:0000360c       ??_R1A@?0A@EA@QHBoxLayout@@8 1001660c     DNAFlexDialog.obj
 0002:00003628       ??_R1A@?0A@EA@QBoxLayout@@8 10016628     DNAFlexDialog.obj
 0002:00003644       ??_R3QBoxLayout@@8         10016644     DNAFlexDialog.obj
 0002:00003654       ??_R2QBoxLayout@@8         10016654     DNAFlexDialog.obj
 0002:00003668       ??_R1A@?0A@EA@QLayout@@8   10016668     DNAFlexDialog.obj
 0002:00003684       ??_R3QLayout@@8            10016684     DNAFlexDialog.obj
 0002:00003694       ??_R2QLayout@@8            10016694     DNAFlexDialog.obj
 0002:000036a4       ??_R17?0A@EA@QLayoutItem@@8 100166a4     DNAFlexDialog.obj
 0002:000036c0       ??_R4QHBoxLayout@@6BQLayoutItem@@@ 100166c0     DNAFlexDialog.obj
 0002:000036d4       ??_R4QVBoxLayout@@6BQObject@@@ 100166d4     DNAFlexDialog.obj
 0002:000036e8       ??_R3QVBoxLayout@@8        100166e8     DNAFlexDialog.obj
 0002:000036f8       ??_R2QVBoxLayout@@8        100166f8     DNAFlexDialog.obj
 0002:00003710       ??_R1A@?0A@EA@QVBoxLayout@@8 10016710     DNAFlexDialog.obj
 0002:0000372c       ??_R4QVBoxLayout@@6BQLayoutItem@@@ 1001672c     DNAFlexDialog.obj
 0002:00003740       ??_R4QGridLayout@@6BQObject@@@ 10016740     DNAFlexDialog.obj
 0002:00003754       ??_R3QGridLayout@@8        10016754     DNAFlexDialog.obj
 0002:00003764       ??_R2QGridLayout@@8        10016764     DNAFlexDialog.obj
 0002:00003778       ??_R1A@?0A@EA@QGridLayout@@8 10016778     DNAFlexDialog.obj
 0002:00003794       ??_R4QGridLayout@@6BQLayoutItem@@@ 10016794     DNAFlexDialog.obj
 0002:000037a8       ??_R4QGroupBox@@6BQObject@@@ 100167a8     DNAFlexDialog.obj
 0002:000037bc       ??_R3QGroupBox@@8          100167bc     DNAFlexDialog.obj
 0002:000037cc       ??_R2QGroupBox@@8          100167cc     DNAFlexDialog.obj
 0002:000037e0       ??_R1A@?0A@EA@QGroupBox@@8 100167e0     DNAFlexDialog.obj
 0002:000037fc       ??_R4QGroupBox@@6BQPaintDevice@@@ 100167fc     DNAFlexDialog.obj
 0002:00003810       ??_R4QTabWidget@@6BQObject@@@ 10016810     DNAFlexDialog.obj
 0002:00003824       ??_R3QTabWidget@@8         10016824     DNAFlexDialog.obj
 0002:00003834       ??_R2QTabWidget@@8         10016834     DNAFlexDialog.obj
 0002:00003848       ??_R1A@?0A@EA@QTabWidget@@8 10016848     DNAFlexDialog.obj
 0002:00003864       ??_R4QTabWidget@@6BQPaintDevice@@@ 10016864     DNAFlexDialog.obj
 0002:00003878       ??_R4QLabel@@6BQObject@@@  10016878     DNAFlexDialog.obj
 0002:0000388c       ??_R3QLabel@@8             1001688c     DNAFlexDialog.obj
 0002:0000389c       ??_R2QLabel@@8             1001689c     DNAFlexDialog.obj
 0002:000038b4       ??_R1A@?0A@EA@QLabel@@8    100168b4     DNAFlexDialog.obj
 0002:000038d0       ??_R1A@?0A@EA@QFrame@@8    100168d0     DNAFlexDialog.obj
 0002:000038ec       ??_R3QFrame@@8             100168ec     DNAFlexDialog.obj
 0002:000038fc       ??_R2QFrame@@8             100168fc     DNAFlexDialog.obj
 0002:00003910       ??_R4QLabel@@6BQPaintDevice@@@ 10016910     DNAFlexDialog.obj
 0002:00003924       ??_R4CreateAnnotationWidgetController@U2@@6B@ 10016924     DNAFlexDialog.obj
 0002:00003938       ??_R3CreateAnnotationWidgetController@U2@@8 10016938     DNAFlexDialog.obj
 0002:00003948       ??_R2CreateAnnotationWidgetController@U2@@8 10016948     DNAFlexDialog.obj
 0002:00003954       ??_R1A@?0A@EA@CreateAnnotationWidgetController@U2@@8 10016954     DNAFlexDialog.obj
 0002:00003970       ??_R4DNAFlexDialog@U2@@6BQObject@@@ 10016970     DNAFlexDialog.obj
 0002:00003984       ??_R3DNAFlexDialog@U2@@8   10016984     DNAFlexDialog.obj
 0002:00003994       ??_R2DNAFlexDialog@U2@@8   10016994     DNAFlexDialog.obj
 0002:000039b0       ??_R1A@?0A@EA@DNAFlexDialog@U2@@8 100169b0     DNAFlexDialog.obj
 0002:000039cc       ??_R1A@?0A@EA@QDialog@@8   100169cc     DNAFlexDialog.obj
 0002:000039e8       ??_R3QDialog@@8            100169e8     DNAFlexDialog.obj
 0002:000039f8       ??_R2QDialog@@8            100169f8     DNAFlexDialog.obj
 0002:00003a0c       ??_R1BI@?0A@EA@Ui_DNAFlexDialog@@8 10016a0c     DNAFlexDialog.obj
 0002:00003a28       ??_R3Ui_DNAFlexDialog@@8   10016a28     DNAFlexDialog.obj
 0002:00003a38       ??_R2Ui_DNAFlexDialog@@8   10016a38     DNAFlexDialog.obj
 0002:00003a40       ??_R1A@?0A@EA@Ui_DNAFlexDialog@@8 10016a40     DNAFlexDialog.obj
 0002:00003a5c       ??_R4DNAFlexDialog@U2@@6BQPaintDevice@@@ 10016a5c     DNAFlexDialog.obj
 0002:00003a70       ??_R4AbstractInt32Id@U2@@6B@ 10016a70     DNAFlexDialog.obj
 0002:00003a84       ??_R3AbstractInt32Id@U2@@8 10016a84     DNAFlexDialog.obj
 0002:00003a94       ??_R2AbstractInt32Id@U2@@8 10016a94     DNAFlexDialog.obj
 0002:00003aa0       ??_R1A@?0A@EA@AbstractInt32Id@U2@@8 10016aa0     DNAFlexDialog.obj
 0002:00003abc       ??_R1A@?0A@EA@?$AbstractId@H@U2@@8 10016abc     DNAFlexDialog.obj
 0002:00003ad8       ??_R3?$AbstractId@H@U2@@8  10016ad8     DNAFlexDialog.obj
 0002:00003ae8       ??_R2?$AbstractId@H@U2@@8  10016ae8     DNAFlexDialog.obj
 0002:00003af0       ??_R4?$AbstractId@H@U2@@6B@ 10016af0     DNAFlexDialog.obj
 0002:00003b04       ??_R4ServiceType@U2@@6B@   10016b04     DNAFlexDialog.obj
 0002:00003b18       ??_R3ServiceType@U2@@8     10016b18     DNAFlexDialog.obj
 0002:00003b28       ??_R2ServiceType@U2@@8     10016b28     DNAFlexDialog.obj
 0002:00003b38       ??_R1A@?0A@EA@ServiceType@U2@@8 10016b38     DNAFlexDialog.obj
 0002:00003b54       ??_R4HelpButton@U2@@6B@    10016b54     DNAFlexDialog.obj
 0002:00003b68       ??_R3HelpButton@U2@@8      10016b68     DNAFlexDialog.obj
 0002:00003b78       ??_R2HelpButton@U2@@8      10016b78     DNAFlexDialog.obj
 0002:00003b84       ??_R1A@?0A@EA@HelpButton@U2@@8 10016b84     DNAFlexDialog.obj
 0002:00003ba0       ??_R4GSequenceGraphData@U2@@6B@ 10016ba0     DNAFlexGraph.obj
 0002:00003bb4       ??_R3GSequenceGraphData@U2@@8 10016bb4     DNAFlexGraph.obj
 0002:00003bc4       ??_R2GSequenceGraphData@U2@@8 10016bc4     DNAFlexGraph.obj
 0002:00003bcc       ??_R1A@?0A@EA@GSequenceGraphData@U2@@8 10016bcc     DNAFlexGraph.obj
 0002:00003be8       ??_R4GSequenceGraphDrawer@U2@@6B@ 10016be8     DNAFlexGraph.obj
 0002:00003bfc       ??_R3GSequenceGraphDrawer@U2@@8 10016bfc     DNAFlexGraph.obj
 0002:00003c0c       ??_R2GSequenceGraphDrawer@U2@@8 10016c0c     DNAFlexGraph.obj
 0002:00003c18       ??_R1A@?0A@EA@GSequenceGraphDrawer@U2@@8 10016c18     DNAFlexGraph.obj
 0002:00003c34       ??_R4DNAFlexGraphFactory@U2@@6B@ 10016c34     DNAFlexGraph.obj
 0002:00003c48       ??_R3DNAFlexGraphFactory@U2@@8 10016c48     DNAFlexGraph.obj
 0002:00003c58       ??_R2DNAFlexGraphFactory@U2@@8 10016c58     DNAFlexGraph.obj
 0002:00003c68       ??_R1A@?0A@EA@DNAFlexGraphFactory@U2@@8 10016c68     DNAFlexGraph.obj
 0002:00003c84       ??_R1A@?0A@EA@GSequenceGraphFactory@U2@@8 10016c84     DNAFlexGraph.obj
 0002:00003ca0       ??_R3GSequenceGraphFactory@U2@@8 10016ca0     DNAFlexGraph.obj
 0002:00003cb0       ??_R2GSequenceGraphFactory@U2@@8 10016cb0     DNAFlexGraph.obj
 0002:00003cbc       ??_R4DNAFlexGraphAlgorithm@U2@@6B@ 10016cbc     DNAFlexGraphAlgorithm.obj
 0002:00003cd0       ??_R3DNAFlexGraphAlgorithm@U2@@8 10016cd0     DNAFlexGraphAlgorithm.obj
 0002:00003ce0       ??_R2DNAFlexGraphAlgorithm@U2@@8 10016ce0     DNAFlexGraphAlgorithm.obj
 0002:00003cec       ??_R1A@?0A@EA@DNAFlexGraphAlgorithm@U2@@8 10016cec     DNAFlexGraphAlgorithm.obj
 0002:00003d08       ??_R1A@?0A@EA@GSequenceGraphAlgorithm@U2@@8 10016d08     DNAFlexGraphAlgorithm.obj
 0002:00003d24       ??_R3GSequenceGraphAlgorithm@U2@@8 10016d24     DNAFlexGraphAlgorithm.obj
 0002:00003d34       ??_R2GSequenceGraphAlgorithm@U2@@8 10016d34     DNAFlexGraphAlgorithm.obj
 0002:00003d3c       ??_R4ADVGlobalAction@U2@@6B@ 10016d3c     DNAFlexPlugin.obj
 0002:00003d50       ??_R3ADVGlobalAction@U2@@8 10016d50     DNAFlexPlugin.obj
 0002:00003d60       ??_R2ADVGlobalAction@U2@@8 10016d60     DNAFlexPlugin.obj
 0002:00003d74       ??_R1A@?0A@EA@ADVGlobalAction@U2@@8 10016d74     DNAFlexPlugin.obj
 0002:00003d90       ??_R1A@?0A@EA@GObjectViewAction@U2@@8 10016d90     DNAFlexPlugin.obj
 0002:00003dac       ??_R3GObjectViewAction@U2@@8 10016dac     DNAFlexPlugin.obj
 0002:00003dbc       ??_R2GObjectViewAction@U2@@8 10016dbc     DNAFlexPlugin.obj
 0002:00003dcc       ??_R1A@?0A@EA@QAction@@8   10016dcc     DNAFlexPlugin.obj
 0002:00003de8       ??_R3QAction@@8            10016de8     DNAFlexPlugin.obj
 0002:00003df8       ??_R2QAction@@8            10016df8     DNAFlexPlugin.obj
 0002:00003e04       ??_R4GraphAction@U2@@6B@   10016e04     DNAFlexPlugin.obj
 0002:00003e18       ??_R3GraphAction@U2@@8     10016e18     DNAFlexPlugin.obj
 0002:00003e28       ??_R2GraphAction@U2@@8     10016e28     DNAFlexPlugin.obj
 0002:00003e38       ??_R1A@?0A@EA@GraphAction@U2@@8 10016e38     DNAFlexPlugin.obj
 0002:00003e54       ??_R4DNAFlexPlugin@U2@@6B@ 10016e54     DNAFlexPlugin.obj
 0002:00003e68       ??_R3DNAFlexPlugin@U2@@8   10016e68     DNAFlexPlugin.obj
 0002:00003e78       ??_R2DNAFlexPlugin@U2@@8   10016e78     DNAFlexPlugin.obj
 0002:00003e88       ??_R1A@?0A@EA@DNAFlexPlugin@U2@@8 10016e88     DNAFlexPlugin.obj
 0002:00003ea4       ??_R1A@?0A@EA@Plugin@U2@@8 10016ea4     DNAFlexPlugin.obj
 0002:00003ec0       ??_R3Plugin@U2@@8          10016ec0     DNAFlexPlugin.obj
 0002:00003ed0       ??_R2Plugin@U2@@8          10016ed0     DNAFlexPlugin.obj
 0002:00003edc       ??_R4DNAFlexViewContext@U2@@6BQObject@@@ 10016edc     DNAFlexPlugin.obj
 0002:00003ef0       ??_R3DNAFlexViewContext@U2@@8 10016ef0     DNAFlexPlugin.obj
 0002:00003f00       ??_R2DNAFlexViewContext@U2@@8 10016f00     DNAFlexPlugin.obj
 0002:00003f14       ??_R1A@?0A@EA@DNAFlexViewContext@U2@@8 10016f14     DNAFlexPlugin.obj
 0002:00003f30       ??_R1A@?0A@EA@GObjectViewWindowContext@U2@@8 10016f30     DNAFlexPlugin.obj
 0002:00003f4c       ??_R3GObjectViewWindowContext@U2@@8 10016f4c     DNAFlexPlugin.obj
 0002:00003f5c       ??_R2GObjectViewWindowContext@U2@@8 10016f5c     DNAFlexPlugin.obj
 0002:00003f6c       ??_R17?0A@EA@GObjectViewObjectHandler@U2@@8 10016f6c     DNAFlexPlugin.obj
 0002:00003f88       ??_R3GObjectViewObjectHandler@U2@@8 10016f88     DNAFlexPlugin.obj
 0002:00003f98       ??_R2GObjectViewObjectHandler@U2@@8 10016f98     DNAFlexPlugin.obj
 0002:00003fa0       ??_R1A@?0A@EA@GObjectViewObjectHandler@U2@@8 10016fa0     DNAFlexPlugin.obj
 0002:00003fbc       ??_R4DNAFlexViewContext@U2@@6BGObjectViewObjectHandler@1@@ 10016fbc     DNAFlexPlugin.obj
 0002:00003fd0       ??_R4CreateAnnotationsTask@U2@@6B@ 10016fd0     DNAFlexTask.obj
 0002:00003fe4       ??_R3CreateAnnotationsTask@U2@@8 10016fe4     DNAFlexTask.obj
 0002:00003ff4       ??_R2CreateAnnotationsTask@U2@@8 10016ff4     DNAFlexTask.obj
 0002:00004004       ??_R1A@?0A@EA@CreateAnnotationsTask@U2@@8 10017004     DNAFlexTask.obj
 0002:00004020       ??_R1A@?0A@EA@Task@U2@@8   10017020     DNAFlexTask.obj
 0002:0000403c       ??_R3Task@U2@@8            1001703c     DNAFlexTask.obj
 0002:0000404c       ??_R2Task@U2@@8            1001704c     DNAFlexTask.obj
 0002:00004058       ??_R4DNAFlexTask@U2@@6B@   10017058     DNAFlexTask.obj
 0002:0000406c       ??_R3DNAFlexTask@U2@@8     1001706c     DNAFlexTask.obj
 0002:0000407c       ??_R2DNAFlexTask@U2@@8     1001707c     DNAFlexTask.obj
 0002:0000408c       ??_R1A@?0A@EA@DNAFlexTask@U2@@8 1001708c     DNAFlexTask.obj
 0002:000040a8       ??_R4FindHighFlexRegionsListener@U2@@6B@ 100170a8     FindHighFlexRegions.obj
 0002:000040bc       ??_R3FindHighFlexRegionsListener@U2@@8 100170bc     FindHighFlexRegions.obj
 0002:000040cc       ??_R2FindHighFlexRegionsListener@U2@@8 100170cc     FindHighFlexRegions.obj
 0002:000040d4       ??_R1A@?0A@EA@FindHighFlexRegionsListener@U2@@8 100170d4     FindHighFlexRegions.obj
 0002:000040f0       ??_R4FindHighFlexRegions@U2@@6BTask@1@@ 100170f0     FindHighFlexRegions.obj
 0002:00004104       ??_R3FindHighFlexRegions@U2@@8 10017104     FindHighFlexRegions.obj
 0002:00004114       ??_R2FindHighFlexRegions@U2@@8 10017114     FindHighFlexRegions.obj
 0002:00004128       ??_R1A@?0A@EA@FindHighFlexRegions@U2@@8 10017128     FindHighFlexRegions.obj
 0002:00004144       ??_R1JA@?0A@EA@FindHighFlexRegionsListener@U2@@8 10017144     FindHighFlexRegions.obj
 0002:00004160       ??_R4FindHighFlexRegions@U2@@6BFindHighFlexRegionsListener@1@@ 10017160     FindHighFlexRegions.obj
 0002:00004174       ??_R4type_info@@6B@        10017174     MSVCRT:ti_inst.obj
 0002:00004188       ??_R3type_info@@8          10017188     MSVCRT:ti_inst.obj
 0002:00004198       ??_R2type_info@@8          10017198     MSVCRT:ti_inst.obj
 0002:000041a0       ??_R1A@?0A@EA@type_info@@8 100171a0     MSVCRT:ti_inst.obj
 0002:000041c0       ___safe_se_handler_table   100171c0     <linker-defined>
 0002:00004440       ___rtc_iaa                 10017440     MSVCRT:initsect.obj
 0002:00004444       ___rtc_izz                 10017444     MSVCRT:initsect.obj
 0002:00004448       ___rtc_taa                 10017448     MSVCRT:initsect.obj
 0002:0000444c       ___rtc_tzz                 1001744c     MSVCRT:initsect.obj
 0002:00006d18       __IMPORT_DESCRIPTOR_U2Core 10019d18     U2Core:U2Core.dll
 0002:00006d2c       __IMPORT_DESCRIPTOR_U2Gui  10019d2c     U2Gui:U2Gui.dll
 0002:00006d40       __IMPORT_DESCRIPTOR_U2View 10019d40     U2View:U2View.dll
 0002:00006d54       __IMPORT_DESCRIPTOR_Qt5Widgets 10019d54     Qt5Widgets:Qt5Widgets.dll
 0002:00006d68       __IMPORT_DESCRIPTOR_Qt5Gui 10019d68     Qt5Gui:Qt5Gui.dll
 0002:00006d7c       __IMPORT_DESCRIPTOR_Qt5Core 10019d7c     Qt5Core:Qt5Core.dll
 0002:00006d90       __IMPORT_DESCRIPTOR_MSVCP120 10019d90     msvcprt:MSVCP120.dll
 0002:00006da4       __IMPORT_DESCRIPTOR_MSVCR120 10019da4     MSVCRT:MSVCR120.dll
 0002:00006db8       __IMPORT_DESCRIPTOR_KERNEL32 10019db8     kernel32:KERNEL32.dll
 0002:00006dcc       __NULL_IMPORT_DESCRIPTOR   10019dcc     U2Core:U2Core.dll
 0003:00000000       ?_Generic_object@?$_Error_objects@H@std@@2V_Generic_error_category@2@A 10021000     DNAFlexDialog.obj
 0003:00000004       ?_Iostream_object@?$_Error_objects@H@std@@2V_Iostream_error_category@2@A 10021004     DNAFlexDialog.obj
 0003:00000008       ?_System_object@?$_Error_objects@H@std@@2V_System_error_category@2@A 10021008     DNAFlexDialog.obj
 0003:000001ac       ?staticMetaObject@DNAFlexDialog@U2@@2UQMetaObject@@B 100211ac     moc_DNAFlexDialog.obj
 0003:0000022c       ?staticMetaObject@DNAFlexGraphFactory@U2@@2UQMetaObject@@B 1002122c     moc_DNAFlexGraph.obj
 0003:000002ac       ?staticMetaObject@DNAFlexPlugin@U2@@2UQMetaObject@@B 100212ac     moc_DNAFlexPlugin.obj
 0003:000002c4       ?staticMetaObject@DNAFlexViewContext@U2@@2UQMetaObject@@B 100212c4     moc_DNAFlexPlugin.obj
 0003:000002dc       ?staticMetaObject@DNAFlexTask@U2@@2UQMetaObject@@B 100212dc     moc_DNAFlexTask.obj
 0003:000002f4       ?staticMetaObject@FindHighFlexRegions@U2@@2UQMetaObject@@B 100212f4     moc_FindHighFlexRegions.obj
 0003:0000030c       ___security_cookie         1002130c     MSVCRT:gs_cookie.obj
 0003:00000310       ___security_cookie_complement 10021310     MSVCRT:gs_cookie.obj
 0003:00000320       ___native_dllmain_reason   10021320     MSVCRT:natstart.obj
 0003:00000324       ??_R0?AVerror_category@std@@@8 10021324     DNAFlexDialog.obj
 0003:00000348       ??_R0?AV_Generic_error_category@std@@@8 10021348     DNAFlexDialog.obj
 0003:00000374       ??_R0?AV_Iostream_error_category@std@@@8 10021374     DNAFlexDialog.obj
 0003:000003a0       ??_R0?AV_System_error_category@std@@@8 100213a0     DNAFlexDialog.obj
 0003:000003cc       ??_R0?AVQWidget@@@8        100213cc     DNAFlexDialog.obj
 0003:000003e4       ??_R0?AVQObject@@@8        100213e4     DNAFlexDialog.obj
 0003:000003fc       ??_R0?AVQPaintDevice@@@8   100213fc     DNAFlexDialog.obj
 0003:00000418       ??_R0?AVQPushButton@@@8    10021418     DNAFlexDialog.obj
 0003:00000434       ??_R0?AVQAbstractButton@@@8 10021434     DNAFlexDialog.obj
 0003:00000454       ??_R0?AVQDialogButtonBox@@@8 10021454     DNAFlexDialog.obj
 0003:00000474       ??_R0?AVQSpinBox@@@8       10021474     DNAFlexDialog.obj
 0003:0000048c       ??_R0?AVQAbstractSpinBox@@@8 1002148c     DNAFlexDialog.obj
 0003:000004ac       ??_R0?AVQDoubleSpinBox@@@8 100214ac     DNAFlexDialog.obj
 0003:000004cc       ??_R0?AVQSpacerItem@@@8    100214cc     DNAFlexDialog.obj
 0003:000004e8       ??_R0?AVQLayoutItem@@@8    100214e8     DNAFlexDialog.obj
 0003:00000504       ??_R0?AVQHBoxLayout@@@8    10021504     DNAFlexDialog.obj
 0003:00000520       ??_R0?AVQBoxLayout@@@8     10021520     DNAFlexDialog.obj
 0003:0000053c       ??_R0?AVQLayout@@@8        1002153c     DNAFlexDialog.obj
 0003:00000554       ??_R0?AVQVBoxLayout@@@8    10021554     DNAFlexDialog.obj
 0003:00000570       ??_R0?AVQGridLayout@@@8    10021570     DNAFlexDialog.obj
 0003:0000058c       ??_R0?AVQGroupBox@@@8      1002158c     DNAFlexDialog.obj
 0003:000005a4       ??_R0?AVQTabWidget@@@8     100215a4     DNAFlexDialog.obj
 0003:000005c0       ??_R0?AVQLabel@@@8         100215c0     DNAFlexDialog.obj
 0003:000005d8       ??_R0?AVQFrame@@@8         100215d8     DNAFlexDialog.obj
 0003:000005f0       ??_R0?AVCreateAnnotationWidgetController@U2@@@8 100215f0     DNAFlexDialog.obj
 0003:00000624       ??_R0?AVDNAFlexDialog@U2@@@8 10021624     DNAFlexDialog.obj
 0003:00000644       ??_R0?AVQDialog@@@8        10021644     DNAFlexDialog.obj
 0003:0000065c       ??_R0?AVUi_DNAFlexDialog@@@8 1002165c     DNAFlexDialog.obj
 0003:0000067c       ??_R0?AVAbstractInt32Id@U2@@@8 1002167c     DNAFlexDialog.obj
 0003:000006a0       ??_R0?AV?$AbstractId@H@U2@@@8 100216a0     DNAFlexDialog.obj
 0003:000006c0       ??_R0?AVServiceType@U2@@@8 100216c0     DNAFlexDialog.obj
 0003:000006e0       ??_R0?AVHelpButton@U2@@@8  100216e0     DNAFlexDialog.obj
 0003:000006fc       ??_R0?AVGSequenceGraphData@U2@@@8 100216fc     DNAFlexGraph.obj
 0003:00000720       ??_R0?AVGSequenceGraphDrawer@U2@@@8 10021720     DNAFlexGraph.obj
 0003:00000748       ??_R0?AVDNAFlexGraphFactory@U2@@@8 10021748     DNAFlexGraph.obj
 0003:00000770       ??_R0?AVGSequenceGraphFactory@U2@@@8 10021770     DNAFlexGraph.obj
 0003:00000798       ??_R0?AVbad_alloc@std@@@8  10021798     DNAFlexGraphAlgorithm.obj
 0003:000007b4       ??_R0?AVDNAFlexGraphAlgorithm@U2@@@8 100217b4     DNAFlexGraphAlgorithm.obj
 0003:000007dc       ??_R0?AVGSequenceGraphAlgorithm@U2@@@8 100217dc     DNAFlexGraphAlgorithm.obj
 0003:00000808       ??_R0?AVADVGlobalAction@U2@@@8 10021808     DNAFlexPlugin.obj
 0003:0000082c       ??_R0?AVGObjectViewAction@U2@@@8 1002182c     DNAFlexPlugin.obj
 0003:00000850       ??_R0?AVQAction@@@8        10021850     DNAFlexPlugin.obj
 0003:00000868       ??_R0?AVGraphAction@U2@@@8 10021868     DNAFlexPlugin.obj
 0003:00000888       ??_R0?AVDNAFlexPlugin@U2@@@8 10021888     DNAFlexPlugin.obj
 0003:000008a8       ??_R0?AVPlugin@U2@@@8      100218a8     DNAFlexPlugin.obj
 0003:000008c0       ??_R0?AVDNAFlexViewContext@U2@@@8 100218c0     DNAFlexPlugin.obj
 0003:000008e4       ??_R0?AVGObjectViewWindowContext@U2@@@8 100218e4     DNAFlexPlugin.obj
 0003:00000910       ??_R0?AVGObjectViewObjectHandler@U2@@@8 10021910     DNAFlexPlugin.obj
 0003:0000093c       ??_R0?AVCreateAnnotationsTask@U2@@@8 1002193c     DNAFlexTask.obj
 0003:00000964       ??_R0?AVTask@U2@@@8        10021964     DNAFlexTask.obj
 0003:0000097c       ??_R0?AVDNAFlexTask@U2@@@8 1002197c     DNAFlexTask.obj
 0003:0000099c       ??_R0?AVFindHighFlexRegionsListener@U2@@@8 1002199c     FindHighFlexRegions.obj
 0003:000009cc       ??_R0?AVFindHighFlexRegions@U2@@@8 100219cc     FindHighFlexRegions.obj
 0003:000009f4       ??_R0?AVtype_info@@@8      100219f4     MSVCRT:ti_inst.obj
 0003:00000a5c       ?id@?$num_put@DV?$back_insert_iterator@V?$basic_string@DU?$char_traits@D@std@@V?$allocator@D@2@@std@@@std@@@std@@2V0locale@2@A 10021a5c     DNAFlexDialog.obj
 0003:00000a60       ?id@?$num_put@_WV?$back_insert_iterator@V?$basic_string@_WU?$char_traits@_W@std@@V?$allocator@_W@2@@std@@@std@@@std@@2V0locale@2@A 10021a60     DNAFlexDialog.obj
 0003:00000c40       ?SETTINGS_PATH@HighFlexSettings@U2@@0VQString@@B 10021c40     HighFlexSettings.obj
 0003:00000c6c       ?SETTING_WINDOW_STEP@HighFlexSettings@U2@@0VQString@@B 10021c6c     HighFlexSettings.obj
 0003:00000c78       ?SETTING_THRESHOLD@HighFlexSettings@U2@@0VQString@@B 10021c78     HighFlexSettings.obj
 0003:00000c84       ?SETTING_WINDOW_SIZE@HighFlexSettings@U2@@0VQString@@B 10021c84     HighFlexSettings.obj
 0003:00000d24       ?metatype_id@?1??qt_metatype_id@?$QMetaTypeIdQObject@PAVADVSequenceWidget@U2@@$00@@SAHXZ@4V?$QBasicAtomicInteger@H@@A 10021d24     moc_DNAFlexPlugin.obj
 0003:00000dc0       ?dummy@?A0xf1761197@@3Uinitializer@1@A 10021dc0     qrc_dna_flexibility.obj
 0003:000010e8       ?__type_info_root_node@@3U__type_info_node@@A 100220e8     MSVCRT:tncleanup.obj
 0003:000010f0       ___native_startup_lock     100220f0     <common>
 0003:000010f4       ___native_startup_state    100220f4     <common>
 0003:000010f8       ___dyn_tls_init_callback   100220f8     <common>
 0003:000010fc       ___onexitend               100220fc     <common>
 0003:00001100       ___onexitbegin             10022100     <common>

 entry point at        0001:0000e250

 Static symbols

 0000:fffd8000       .debug$S                   10000000     MSVCRT:MSVCR120.dll
 0000:fffd8000       .debug$S                   10000000     MSVCRT:MSVCR120.dll
 0000:fffd8000       .debug$S                   10000000     MSVCRT:MSVCR120.dll
 0000:fffd8000       .debug$S                   10000000     MSVCRT:MSVCR120.dll
 0000:fffd8000       .debug$S                   10000000     MSVCRT:MSVCR120.dll
 0000:fffd8000       .debug$S                   10000000     MSVCRT:MSVCR120.dll
 0000:fffd8000       .debug$S                   10000000     MSVCRT:MSVCR120.dll
 0000:fffd8000       .debug$S                   10000000     MSVCRT:MSVCR120.dll
 0000:fffd8000       .debug$S                   10000000     MSVCRT:MSVCR120.dll
 0000:fffd8000       .debug$S                   10000000     MSVCRT:MSVCR120.dll
 0002:fffed000       ?_Iostream_object$initializer$@?$_Error_objects@H@std@@2P6AXXZA 10000000     DNAFlexTask.obj
 0000:fffd8000       .debug$S                   10000000     MSVCRT:MSVCR120.dll
 0000:fffd8000       .debug$S                   10000000     MSVCRT:MSVCR120.dll
 0000:fffd8000       .debug$S                   10000000     MSVCRT:MSVCR120.dll
 0000:fffd8000       .debug$S                   10000000     MSVCRT:MSVCR120.dll
 0002:fffed000       ?_System_object$initializer$@?$_Error_objects@H@std@@2P6AXXZA 10000000     DNAFlexTask.obj
 0000:fffd8000       .debug$S                   10000000     MSVCRT:MSVCR120.dll
 0001:fffff000       __ehhandler$?_Copy@?$basic_string@DU?$char_traits@D@std@@V?$allocator@D@2@@std@@QAEXII@Z 10000000 f   DNAFlexPlugin.obj
 0000:fffd8000       .debug$S                   10000000     MSVCRT:MSVCR120.dll
 0002:fffed000       __catchsym$?_Copy@?$basic_string@DU?$char_traits@D@std@@V?$allocator@D@2@@std@@QAEXII@Z$5 10000000     DNAFlexPlugin.obj
 0000:fffd8000       .debug$S                   10000000     MSVCRT:MSVCR120.dll
 0002:fffed000       ?_Generic_object$initializer$@?$_Error_objects@H@std@@2P6AXXZA 10000000     DNAFlexPlugin.obj
 0000:fffd8000       .debug$S                   10000000     MSVCRT:MSVCR120.dll
 0002:fffed000       ?_Iostream_object$initializer$@?$_Error_objects@H@std@@2P6AXXZA 10000000     DNAFlexPlugin.obj
 0000:fffd8000       .debug$S                   10000000     MSVCRT:MSVCR120.dll
 0002:fffed000       ?_System_object$initializer$@?$_Error_objects@H@std@@2P6AXXZA 10000000     DNAFlexPlugin.obj
 0000:fffd8000       .debug$S                   10000000     MSVCRT:MSVCR120.dll
 0002:fffed000       __unwindtable$?detach_helper@?$QSharedDataPointer@VAnnotationData@U2@@@@AAEXXZ 10000000     DNAFlexTask.obj
 0000:fffd8000       .debug$S                   10000000     MSVCRT:MSVCR120.dll
 0002:fffed000       __unwindtable$?clone@?$QSharedDataPointer@VAnnotationData@U2@@@@IAEPAVAnnotationData@U2@@XZ 10000000     DNAFlexTask.obj
 0000:fffd8000       .debug$S                   10000000     MSVCRT:MSVCR120.dll
 0002:fffed000       __catchsym$?_Copy@?$basic_string@DU?$char_traits@D@std@@V?$allocator@D@2@@std@@QAEXII@Z$5 10000000     DNAFlexTask.obj
 0000:fffd8000       .debug$S                   10000000     MSVCRT:MSVCR120.dll
 0001:fffff000       __ehhandler$?_Copy@?$basic_string@DU?$char_traits@D@std@@V?$allocator@D@2@@std@@QAEXII@Z 10000000 f   DNAFlexGraphAlgorithm.obj
 0002:fffed000       __catchsym$?_Copy@?$basic_string@DU?$char_traits@D@std@@V?$allocator@D@2@@std@@QAEXII@Z$5 10000000     DNAFlexGraphAlgorithm.obj
 0000:fffd8000       .debug$S                   10000000     MSVCRT:MSVCR120.dll
 0002:fffed000       ?_Generic_object$initializer$@?$_Error_objects@H@std@@2P6AXXZA 10000000     DNAFlexGraphAlgorithm.obj
 0000:fffd8000       .debug$S                   10000000     MSVCRT:MSVCR120.dll
 0002:fffed000       ?_Iostream_object$initializer$@?$_Error_objects@H@std@@2P6AXXZA 10000000     DNAFlexGraphAlgorithm.obj
 0000:fffd8000       .debug$S                   10000000     MSVCRT:MSVCR120.dll
 0001:fffff000       __ehhandler$?_Copy@?$basic_string@DU?$char_traits@D@std@@V?$allocator@D@2@@std@@QAEXII@Z 10000000 f   moc_FindHighFlexRegions.obj
 0002:fffed000       ?_System_object$initializer$@?$_Error_objects@H@std@@2P6AXXZA 10000000     DNAFlexGraphAlgorithm.obj
 0001:fffff000       __unwindfunclet$?detach_helper@?$QSharedDataPointer@VAnnotationData@U2@@@@AAEXXZ$0 10000000 f   DNAFlexTask.obj
 0000:fffd8000       .debug$S                   10000000     MSVCRT:MSVCR120.dll
 0001:fffff000       __unwindfunclet$?clone@?$QSharedDataPointer@VAnnotationData@U2@@@@IAEPAVAnnotationData@U2@@XZ$0 10000000 f   DNAFlexTask.obj
 0001:fffff000       __ehhandler$?_Copy@?$basic_string@DU?$char_traits@D@std@@V?$allocator@D@2@@std@@QAEXII@Z 10000000 f   DNAFlexGraph.obj
 0001:fffff000       __ehhandler$?_Copy@?$basic_string@DU?$char_traits@D@std@@V?$allocator@D@2@@std@@QAEXII@Z 10000000 f   DNAFlexTask.obj
 0002:fffed000       ?_System_object$initializer$@?$_Error_objects@H@std@@2P6AXXZA 10000000     FindHighFlexRegions.obj
 0000:fffd8000       .debug$S                   10000000     msvcprt:MSVCP120.dll
 0000:fffd8000       .debug$S                   10000000     msvcprt:MSVCP120.dll
 0000:fffd8000       .debug$S                   10000000     msvcprt:MSVCP120.dll
 0000:fffd8000       .debug$S                   10000000     msvcprt:MSVCP120.dll
 0000:fffd8000       .debug$S                   10000000     msvcprt:MSVCP120.dll
 0000:fffd8000       .debug$S                   10000000     kernel32:KERNEL32.dll
 0000:fffd8000       .debug$S                   10000000     kernel32:KERNEL32.dll
 0000:fffd8000       .debug$S                   10000000     kernel32:KERNEL32.dll
 0000:fffd8000       .debug$S                   10000000     kernel32:KERNEL32.dll
 0000:fffd8000       .debug$S                   10000000     kernel32:KERNEL32.dll
 0000:fffd8000       .debug$S                   10000000     kernel32:KERNEL32.dll
 0000:fffd8000       .debug$S                   10000000     kernel32:KERNEL32.dll
 0000:fffd8000       .debug$S                   10000000     kernel32:KERNEL32.dll
 0002:fffed000       ?_Iostream_object$initializer$@?$_Error_objects@H@std@@2P6AXXZA 10000000     FindHighFlexRegions.obj
 0002:fffed000       ?_Generic_object$initializer$@?$_Error_objects@H@std@@2P6AXXZA 10000000     FindHighFlexRegions.obj
 0002:fffed000       __catchsym$?node_copy@?$QList@VHighFlexResult@U2@@@@AAEXPAUNode@1@00@Z$4 10000000     FindHighFlexRegions.obj
 0002:fffed000       __catchsym$?_Copy@?$basic_string@DU?$char_traits@D@std@@V?$allocator@D@2@@std@@QAEXII@Z$5 10000000     DNAFlexGraph.obj
 0002:fffed000       __catchsym$?_Copy@?$basic_string@DU?$char_traits@D@std@@V?$allocator@D@2@@std@@QAEXII@Z$5 10000000     moc_FindHighFlexRegions.obj
 0000:fffd8000       .debug$S                   10000000     kernel32:KERNEL32.dll
 0000:fffd8000       .debug$S                   10000000     Qt5Core:Qt5Core.dll
 0000:fffd8000       .debug$S                   10000000     Qt5Core:Qt5Core.dll
 0000:fffd8000       .debug$S                   10000000     Qt5Core:Qt5Core.dll
 0000:fffd8000       .debug$S                   10000000     Qt5Core:Qt5Core.dll
 0000:fffd8000       .debug$S                   10000000     Qt5Core:Qt5Core.dll
 0000:fffd8000       .debug$S                   10000000     Qt5Core:Qt5Core.dll
 0000:fffd8000       .debug$S                   10000000     Qt5Core:Qt5Core.dll
 0000:fffd8000       .debug$S                   10000000     Qt5Core:Qt5Core.dll
 0000:fffd8000       .debug$S                   10000000     Qt5Core:Qt5Core.dll
 0000:fffd8000       .debug$S                   10000000     Qt5Core:Qt5Core.dll
 0000:fffd8000       .debug$S                   10000000     Qt5Core:Qt5Core.dll
 0000:fffd8000       .debug$S                   10000000     Qt5Core:Qt5Core.dll
 0000:fffd8000       .debug$S                   10000000     Qt5Core:Qt5Core.dll
 0000:fffd8000       .debug$S                   10000000     Qt5Core:Qt5Core.dll
 0000:fffd8000       .debug$S                   10000000     Qt5Core:Qt5Core.dll
 0000:fffd8000       .debug$S                   10000000     Qt5Core:Qt5Core.dll
 0000:fffd8000       .debug$S                   10000000     Qt5Core:Qt5Core.dll
 0000:fffd8000       .debug$S                   10000000     Qt5Core:Qt5Core.dll
 0000:fffd8000       .debug$S                   10000000     Qt5Core:Qt5Core.dll
 0000:fffd8000       .debug$S                   10000000     Qt5Core:Qt5Core.dll
 0000:fffd8000       .debug$S                   10000000     Qt5Core:Qt5Core.dll
 0000:fffd8000       .debug$S                   10000000     Qt5Core:Qt5Core.dll
 0000:fffd8000       .debug$S                   10000000     Qt5Core:Qt5Core.dll
 0000:fffd8000       .debug$S                   10000000     Qt5Core:Qt5Core.dll
 0000:fffd8000       .debug$S                   10000000     Qt5Core:Qt5Core.dll
 0000:fffd8000       .debug$S                   10000000     Qt5Core:Qt5Core.dll
 0000:fffd8000       .debug$S                   10000000     Qt5Core:Qt5Core.dll
 0000:fffd8000       .debug$S                   10000000     Qt5Core:Qt5Core.dll
 0000:fffd8000       .debug$S                   10000000     Qt5Core:Qt5Core.dll
 0000:fffd8000       .debug$S                   10000000     Qt5Core:Qt5Core.dll
 0000:fffd8000       .debug$S                   10000000     Qt5Core:Qt5Core.dll
 0000:fffd8000       .debug$S                   10000000     Qt5Core:Qt5Core.dll
 0000:fffd8000       .debug$S                   10000000     Qt5Core:Qt5Core.dll
 0000:fffd8000       .debug$S                   10000000     Qt5Core:Qt5Core.dll
 0000:fffd8000       .debug$S                   10000000     Qt5Core:Qt5Core.dll
 0000:fffd8000       .debug$S                   10000000     Qt5Core:Qt5Core.dll
 0000:fffd8000       .debug$S                   10000000     Qt5Core:Qt5Core.dll
 0000:fffd8000       .debug$S                   10000000     Qt5Core:Qt5Core.dll
 0000:fffd8000       .debug$S                   10000000     Qt5Core:Qt5Core.dll
 0000:fffd8000       .debug$S                   10000000     Qt5Core:Qt5Core.dll
 0002:fffed000       ?_Generic_object$initializer$@?$_Error_objects@H@std@@2P6AXXZA 10000000     moc_FindHighFlexRegions.obj
 0002:fffed000       ?_Iostream_object$initializer$@?$_Error_objects@H@std@@2P6AXXZA 10000000     moc_FindHighFlexRegions.obj
 0002:fffed000       ?_System_object$initializer$@?$_Error_objects@H@std@@2P6AXXZA 10000000     moc_FindHighFlexRegions.obj
 0000:fffd8000       .debug$S                   10000000     Qt5Core:Qt5Core.dll
 0000:fffd8000       .debug$S                   10000000     Qt5Core:Qt5Core.dll
 0002:fffed000       ?_Generic_object$initializer$@?$_Error_objects@H@std@@2P6AXXZA 10000000     DNAFlexGraph.obj
 0000:fffd8000       .debug$S                   10000000     Qt5Core:Qt5Core.dll
 0002:fffed000       ?_Iostream_object$initializer$@?$_Error_objects@H@std@@2P6AXXZA 10000000     DNAFlexGraph.obj
 0000:fffd8000       .debug$S                   10000000     Qt5Core:Qt5Core.dll
 0002:fffed000       ?_System_object$initializer$@?$_Error_objects@H@std@@2P6AXXZA 10000000     DNAFlexGraph.obj
 0000:fffd8000       .debug$S                   10000000     Qt5Core:Qt5Core.dll
 0002:fffed000       __catchsym$??0?$QList@VHighFlexResult@U2@@@@QAE@ABV0@@Z$2 10000000     FindHighFlexRegions.obj
 0000:fffd8000       .debug$S                   10000000     Qt5Core:Qt5Core.dll
 0002:fffed000       __catchsym$?_Copy@?$basic_string@DU?$char_traits@D@std@@V?$allocator@D@2@@std@@QAEXII@Z$5 10000000     FindHighFlexRegions.obj
 0000:fffd8000       .debug$S                   10000000     Qt5Core:Qt5Core.dll
 0001:fffff000       __ehhandler$?node_copy@?$QList@VHighFlexResult@U2@@@@AAEXPAUNode@1@00@Z 10000000 f   FindHighFlexRegions.obj
 0000:fffd8000       .debug$S                   10000000     Qt5Core:Qt5Core.dll
 0001:fffff000       __ehhandler$??0?$QList@VHighFlexResult@U2@@@@QAE@ABV0@@Z 10000000 f   FindHighFlexRegions.obj
 0000:fffd8000       .debug$S                   10000000     Qt5Core:Qt5Core.dll
 0001:fffff000       __ehhandler$?_Copy@?$basic_string@DU?$char_traits@D@std@@V?$allocator@D@2@@std@@QAEXII@Z 10000000 f   FindHighFlexRegions.obj
 0000:fffd8000       .debug$S                   10000000     Qt5Core:Qt5Core.dll
 0002:fffed000       ?_System_object$initializer$@?$_Error_objects@H@std@@2P6AXXZA 10000000     FindHighFlexRegionsAlgorithm.obj
 0000:fffd8000       .debug$S                   10000000     Qt5Core:Qt5Core.dll
 0002:fffed000       ?_Iostream_object$initializer$@?$_Error_objects@H@std@@2P6AXXZA 10000000     FindHighFlexRegionsAlgorithm.obj
 0002:fffed000       ?_Generic_object$initializer$@?$_Error_objects@H@std@@2P6AXXZA 10000000     FindHighFlexRegionsAlgorithm.obj
 0000:fffd8000       .debug$S                   10000000     Qt5Core:Qt5Core.dll
 0002:fffed000       __catchsym$?_Copy@?$basic_string@DU?$char_traits@D@std@@V?$allocator@D@2@@std@@QAEXII@Z$5 10000000     FindHighFlexRegionsAlgorithm.obj
 0000:fffd8000       .debug$S                   10000000     Qt5Core:Qt5Core.dll
 0000:fffd8000       .debug$S                   10000000     U2Core:U2Core.dll
 0000:fffd8000       .debug$S                   10000000     Qt5Core:Qt5Core.dll
 0001:fffff000       __ehhandler$?_Copy@?$basic_string@DU?$char_traits@D@std@@V?$allocator@D@2@@std@@QAEXII@Z 10000000 f   moc_DNAFlexTask.obj
 0000:fffd8000       .debug$S                   10000000     U2Core:U2Core.dll
 0000:fffd8000       .debug$S                   10000000     U2Core:U2Core.dll
 0000:fffd8000       .debug$S                   10000000     Qt5Core:Qt5Core.dll
 0000:fffd8000       .debug$S                   10000000     Qt5Core:Qt5Core.dll
 0000:fffd8000       .debug$S                   10000000     Qt5Core:Qt5Core.dll
 0000:fffd8000       .debug$S                   10000000     Qt5Core:Qt5Core.dll
 0000:fffd8000       .debug$S                   10000000     Qt5Core:Qt5Core.dll
 0000:fffd8000       .debug$S                   10000000     Qt5Core:Qt5Core.dll
 0000:fffd8000       .debug$S                   10000000     Qt5Core:Qt5Core.dll
 0000:fffd8000       .debug$S                   10000000     Qt5Core:Qt5Core.dll
 0000:fffd8000       .debug$S                   10000000     Qt5Core:Qt5Core.dll
 0000:fffd8000       .debug$S                   10000000     Qt5Core:Qt5Core.dll
 0000:fffd8000       .debug$S                   10000000     Qt5Core:Qt5Core.dll
 0000:fffd8000       .debug$S                   10000000     Qt5Core:Qt5Core.dll
 0000:fffd8000       .debug$S                   10000000     Qt5Core:Qt5Core.dll
 0000:fffd8000       .debug$S                   10000000     Qt5Gui:Qt5Gui.dll
 0000:fffd8000       .debug$S                   10000000     Qt5Gui:Qt5Gui.dll
 0000:fffd8000       .debug$S                   10000000     Qt5Widgets:Qt5Widgets.dll
 0000:fffd8000       .debug$S                   10000000     Qt5Widgets:Qt5Widgets.dll
 0000:fffd8000       .debug$S                   10000000     Qt5Widgets:Qt5Widgets.dll
 0000:fffd8000       .debug$S                   10000000     U2Core:U2Core.dll
 0000:fffd8000       .debug$S                   10000000     U2Core:U2Core.dll
 0000:fffd8000       .debug$S                   10000000     U2Core:U2Core.dll
 0000:fffd8000       .debug$S                   10000000     U2Core:U2Core.dll
 0002:fffed000       __catchsym$?_Copy@?$basic_string@DU?$char_traits@D@std@@V?$allocator@D@2@@std@@QAEXII@Z$5 10000000     moc_DNAFlexTask.obj
 0000:fffd8000       .debug$S                   10000000     Qt5Widgets:Qt5Widgets.dll
 0000:fffd8000       .debug$S                   10000000     Qt5Widgets:Qt5Widgets.dll
 0000:fffd8000       .debug$S                   10000000     Qt5Widgets:Qt5Widgets.dll
 0000:fffd8000       .debug$S                   10000000     Qt5Widgets:Qt5Widgets.dll
 0000:fffd8000       .debug$S                   10000000     Qt5Widgets:Qt5Widgets.dll
 0000:fffd8000       .debug$S                   10000000     Qt5Widgets:Qt5Widgets.dll
 0000:fffd8000       .debug$S                   10000000     Qt5Widgets:Qt5Widgets.dll
 0000:fffd8000       .debug$S                   10000000     Qt5Widgets:Qt5Widgets.dll
 0000:fffd8000       .debug$S                   10000000     Qt5Widgets:Qt5Widgets.dll
 0000:fffd8000       .debug$S                   10000000     Qt5Widgets:Qt5Widgets.dll
 0000:fffd8000       .debug$S                   10000000     Qt5Widgets:Qt5Widgets.dll
 0000:fffd8000       .debug$S                   10000000     Qt5Widgets:Qt5Widgets.dll
 0000:fffd8000       .debug$S                   10000000     Qt5Widgets:Qt5Widgets.dll
 0000:fffd8000       .debug$S                   10000000     Qt5Widgets:Qt5Widgets.dll
 0000:fffd8000       .debug$S                   10000000     Qt5Widgets:Qt5Widgets.dll
 0000:fffd8000       .debug$S                   10000000     Qt5Widgets:Qt5Widgets.dll
 0000:fffd8000       .debug$S                   10000000     Qt5Widgets:Qt5Widgets.dll
 0000:fffd8000       .debug$S                   10000000     Qt5Widgets:Qt5Widgets.dll
 0000:fffd8000       .debug$S                   10000000     Qt5Widgets:Qt5Widgets.dll
 0000:fffd8000       .debug$S                   10000000     Qt5Widgets:Qt5Widgets.dll
 0000:fffd8000       .debug$S                   10000000     Qt5Widgets:Qt5Widgets.dll
 0000:fffd8000       .debug$S                   10000000     Qt5Widgets:Qt5Widgets.dll
 0000:fffd8000       .debug$S                   10000000     Qt5Widgets:Qt5Widgets.dll
 0000:fffd8000       .debug$S                   10000000     Qt5Widgets:Qt5Widgets.dll
 0000:fffd8000       .debug$S                   10000000     Qt5Widgets:Qt5Widgets.dll
 0000:fffd8000       .debug$S                   10000000     Qt5Widgets:Qt5Widgets.dll
 0000:fffd8000       .debug$S                   10000000     Qt5Widgets:Qt5Widgets.dll
 0000:fffd8000       .debug$S                   10000000     Qt5Widgets:Qt5Widgets.dll
 0000:fffd8000       .debug$S                   10000000     Qt5Widgets:Qt5Widgets.dll
 0000:fffd8000       .debug$S                   10000000     Qt5Widgets:Qt5Widgets.dll
 0000:fffd8000       .debug$S                   10000000     Qt5Widgets:Qt5Widgets.dll
 0000:fffd8000       .debug$S                   10000000     Qt5Widgets:Qt5Widgets.dll
 0000:fffd8000       .debug$S                   10000000     Qt5Widgets:Qt5Widgets.dll
 0000:fffd8000       .debug$S                   10000000     Qt5Widgets:Qt5Widgets.dll
 0000:fffd8000       .debug$S                   10000000     Qt5Widgets:Qt5Widgets.dll
 0000:fffd8000       .debug$S                   10000000     Qt5Widgets:Qt5Widgets.dll
 0000:fffd8000       .debug$S                   10000000     Qt5Widgets:Qt5Widgets.dll
 0000:fffd8000       .debug$S                   10000000     Qt5Widgets:Qt5Widgets.dll
 0000:fffd8000       .debug$S                   10000000     Qt5Widgets:Qt5Widgets.dll
 0000:fffd8000       .debug$S                   10000000     Qt5Widgets:Qt5Widgets.dll
 0000:fffd8000       .debug$S                   10000000     Qt5Widgets:Qt5Widgets.dll
 0002:fffed000       ?_Generic_object$initializer$@?$_Error_objects@H@std@@2P6AXXZA 10000000     moc_DNAFlexTask.obj
 0002:fffed000       ?_Iostream_object$initializer$@?$_Error_objects@H@std@@2P6AXXZA 10000000     moc_DNAFlexTask.obj
 0002:fffed000       ?_System_object$initializer$@?$_Error_objects@H@std@@2P6AXXZA 10000000     moc_DNAFlexTask.obj
 0000:fffd8000       .debug$S                   10000000     Qt5Widgets:Qt5Widgets.dll
 0000:fffd8000       .debug$S                   10000000     Qt5Widgets:Qt5Widgets.dll
 0000:fffd8000       .debug$S                   10000000     Qt5Widgets:Qt5Widgets.dll
 0000:fffd8000       .debug$S                   10000000     Qt5Widgets:Qt5Widgets.dll
 0000:fffd8000       .debug$S                   10000000     U2Core:U2Core.dll
 0000:fffd8000       .debug$S                   10000000     Qt5Widgets:Qt5Widgets.dll
 0000:fffd8000       .debug$S                   10000000     U2Core:U2Core.dll
 0000:fffd8000       .debug$S                   10000000     Qt5Widgets:Qt5Widgets.dll
 0000:fffd8000       .debug$S                   10000000     U2Core:U2Core.dll
 0000:fffd8000       .debug$S                   10000000     Qt5Widgets:Qt5Widgets.dll
 0000:fffd8000       .debug$S                   10000000     U2Core:U2Core.dll
 0000:fffd8000       .debug$S                   10000000     Qt5Widgets:Qt5Widgets.dll
 0000:fffd8000       .debug$S                   10000000     U2Core:U2Core.dll
 0000:fffd8000       .debug$S                   10000000     Qt5Widgets:Qt5Widgets.dll
 0000:fffd8000       .debug$S                   10000000     U2Core:U2Core.dll
 0000:fffd8000       .debug$S                   10000000     Qt5Widgets:Qt5Widgets.dll
 0000:fffd8000       .debug$S                   10000000     U2Core:U2Core.dll
 0000:fffd8000       .debug$S                   10000000     Qt5Widgets:Qt5Widgets.dll
 0000:fffd8000       .debug$S                   10000000     U2Core:U2Core.dll
 0000:fffd8000       .debug$S                   10000000     Qt5Widgets:Qt5Widgets.dll
 0000:fffd8000       .debug$S                   10000000     U2Core:U2Core.dll
 0000:fffd8000       .debug$S                   10000000     Qt5Widgets:Qt5Widgets.dll
 0001:fffff000       __ehhandler$?_Copy@?$basic_string@DU?$char_traits@D@std@@V?$allocator@D@2@@std@@QAEXII@Z 10000000 f   FindHighFlexRegionsAlgorithm.obj
 0000:fffd8000       .debug$S                   10000000     Qt5Widgets:Qt5Widgets.dll
 0000:fffd8000       .debug$S                   10000000     U2Core:U2Core.dll
 0000:fffd8000       .debug$S                   10000000     Qt5Widgets:Qt5Widgets.dll
 0000:fffd8000       .debug$S                   10000000     U2Core:U2Core.dll
 0000:fffd8000       .debug$S                   10000000     Qt5Widgets:Qt5Widgets.dll
 0000:fffd8000       .debug$S                   10000000     U2Core:U2Core.dll
 0000:fffd8000       .debug$S                   10000000     Qt5Widgets:Qt5Widgets.dll
 0000:fffd8000       .debug$S                   10000000     U2Core:U2Core.dll
 0000:fffd8000       .debug$S                   10000000     Qt5Widgets:Qt5Widgets.dll
 0000:fffd8000       .debug$S                   10000000     U2Core:U2Core.dll
 0000:fffd8000       .debug$S                   10000000     Qt5Widgets:Qt5Widgets.dll
 0000:fffd8000       .debug$S                   10000000     U2Core:U2Core.dll
 0000:fffd8000       .debug$S                   10000000     Qt5Widgets:Qt5Widgets.dll
 0000:fffd8000       .debug$S                   10000000     U2Core:U2Core.dll
 0000:fffd8000       .debug$S                   10000000     Qt5Widgets:Qt5Widgets.dll
 0000:fffd8000       .debug$S                   10000000     U2Core:U2Core.dll
 0000:fffd8000       .debug$S                   10000000     Qt5Widgets:Qt5Widgets.dll
 0000:fffd8000       .debug$S                   10000000     U2Core:U2Core.dll
 0000:fffd8000       .debug$S                   10000000     Qt5Widgets:Qt5Widgets.dll
 0000:fffd8000       .debug$S                   10000000     U2Core:U2Core.dll
 0000:fffd8000       .debug$S                   10000000     Qt5Widgets:Qt5Widgets.dll
 0000:fffd8000       .debug$S                   10000000     U2Core:U2Core.dll
 0000:fffd8000       .debug$S                   10000000     Qt5Widgets:Qt5Widgets.dll
 0000:fffd8000       .debug$S                   10000000     U2Core:U2Core.dll
 0000:fffd8000       .debug$S                   10000000     Qt5Widgets:Qt5Widgets.dll
 0002:fffed000       ?_System_object$initializer$@?$_Error_objects@H@std@@2P6AXXZA 10000000     HighFlexSettings.obj
 0002:fffed000       ?_Iostream_object$initializer$@?$_Error_objects@H@std@@2P6AXXZA 10000000     HighFlexSettings.obj
 0002:fffed000       ?_Generic_object$initializer$@?$_Error_objects@H@std@@2P6AXXZA 10000000     HighFlexSettings.obj
 0000:fffd8000       .debug$S                   10000000     Qt5Widgets:Qt5Widgets.dll
 0000:fffd8000       .debug$S                   10000000     U2Core:U2Core.dll
 0000:fffd8000       .debug$S                   10000000     Qt5Widgets:Qt5Widgets.dll
 0000:fffd8000       .debug$S                   10000000     U2Core:U2Core.dll
 0000:fffd8000       .debug$S                   10000000     Qt5Widgets:Qt5Widgets.dll
 0001:fffff000       __ehhandler$?_Copy@?$basic_string@DU?$char_traits@D@std@@V?$allocator@D@2@@std@@QAEXII@Z 10000000 f   moc_DNAFlexPlugin.obj
 0000:fffd8000       .debug$S                   10000000     U2Core:U2Core.dll
 0000:fffd8000       .debug$S                   10000000     U2Core:U2Core.dll
 0000:fffd8000       .debug$S                   10000000     Qt5Widgets:Qt5Widgets.dll
 0000:fffd8000       .debug$S                   10000000     Qt5Widgets:Qt5Widgets.dll
 0000:fffd8000       .debug$S                   10000000     Qt5Widgets:Qt5Widgets.dll
 0000:fffd8000       .debug$S                   10000000     Qt5Widgets:Qt5Widgets.dll
 0000:fffd8000       .debug$S                   10000000     Qt5Widgets:Qt5Widgets.dll
 0000:fffd8000       .debug$S                   10000000     Qt5Widgets:Qt5Widgets.dll
 0000:fffd8000       .debug$S                   10000000     Qt5Widgets:Qt5Widgets.dll
 0000:fffd8000       .debug$S                   10000000     Qt5Widgets:Qt5Widgets.dll
 0000:fffd8000       .debug$S                   10000000     Qt5Widgets:Qt5Widgets.dll
 0000:fffd8000       .debug$S                   10000000     Qt5Widgets:Qt5Widgets.dll
 0000:fffd8000       .debug$S                   10000000     Qt5Widgets:Qt5Widgets.dll
 0000:fffd8000       .debug$S                   10000000     Qt5Widgets:Qt5Widgets.dll
 0000:fffd8000       .debug$S                   10000000     Qt5Widgets:Qt5Widgets.dll
 0000:fffd8000       .debug$S                   10000000     Qt5Widgets:Qt5Widgets.dll
 0000:fffd8000       .debug$S                   10000000     Qt5Widgets:Qt5Widgets.dll
 0000:fffd8000       .debug$S                   10000000     Qt5Widgets:Qt5Widgets.dll
 0000:fffd8000       .debug$S                   10000000     Qt5Widgets:Qt5Widgets.dll
 0000:fffd8000       .debug$S                   10000000     Qt5Widgets:Qt5Widgets.dll
 0000:fffd8000       .debug$S                   10000000     Qt5Widgets:Qt5Widgets.dll
 0000:fffd8000       .debug$S                   10000000     Qt5Widgets:Qt5Widgets.dll
 0000:fffd8000       .debug$S                   10000000     U2Core:U2Core.dll
 0000:fffd8000       .debug$S                   10000000     U2Core:U2Core.dll
 0000:fffd8000       .debug$S                   10000000     U2Core:U2Core.dll
 0000:fffd8000       .debug$S                   10000000     U2Core:U2Core.dll
 0002:fffed000       __catchsym$?_Copy@?$basic_string@DU?$char_traits@D@std@@V?$allocator@D@2@@std@@QAEXII@Z$5 10000000     moc_DNAFlexPlugin.obj
 0000:fffd8000       .debug$S                   10000000     Qt5Widgets:Qt5Widgets.dll
 0000:fffd8000       .debug$S                   10000000     Qt5Widgets:Qt5Widgets.dll
 0000:fffd8000       .debug$S                   10000000     Qt5Widgets:Qt5Widgets.dll
 0000:fffd8000       .debug$S                   10000000     Qt5Widgets:Qt5Widgets.dll
 0000:fffd8000       .debug$S                   10000000     Qt5Widgets:Qt5Widgets.dll
 0000:fffd8000       .debug$S                   10000000     Qt5Widgets:Qt5Widgets.dll
 0000:fffd8000       .debug$S                   10000000     Qt5Widgets:Qt5Widgets.dll
 0000:fffd8000       .debug$S                   10000000     Qt5Widgets:Qt5Widgets.dll
 0000:fffd8000       .debug$S                   10000000     Qt5Widgets:Qt5Widgets.dll
 0000:fffd8000       .debug$S                   10000000     Qt5Widgets:Qt5Widgets.dll
 0000:fffd8000       .debug$S                   10000000     Qt5Widgets:Qt5Widgets.dll
 0000:fffd8000       .debug$S                   10000000     Qt5Widgets:Qt5Widgets.dll
 0000:fffd8000       .debug$S                   10000000     Qt5Widgets:Qt5Widgets.dll
 0000:fffd8000       .debug$S                   10000000     Qt5Widgets:Qt5Widgets.dll
 0000:fffd8000       .debug$S                   10000000     Qt5Widgets:Qt5Widgets.dll
 0000:fffd8000       .debug$S                   10000000     Qt5Widgets:Qt5Widgets.dll
 0000:fffd8000       .debug$S                   10000000     Qt5Widgets:Qt5Widgets.dll
 0000:fffd8000       .debug$S                   10000000     Qt5Widgets:Qt5Widgets.dll
 0000:fffd8000       .debug$S                   10000000     Qt5Widgets:Qt5Widgets.dll
 0000:fffd8000       .debug$S                   10000000     Qt5Widgets:Qt5Widgets.dll
 0000:fffd8000       .debug$S                   10000000     Qt5Widgets:Qt5Widgets.dll
 0000:fffd8000       .debug$S                   10000000     Qt5Widgets:Qt5Widgets.dll
 0000:fffd8000       .debug$S                   10000000     Qt5Widgets:Qt5Widgets.dll
 0000:fffd8000       .debug$S                   10000000     Qt5Widgets:Qt5Widgets.dll
 0000:fffd8000       .debug$S                   10000000     Qt5Widgets:Qt5Widgets.dll
 0000:fffd8000       .debug$S                   10000000     Qt5Widgets:Qt5Widgets.dll
 0000:fffd8000       .debug$S                   10000000     Qt5Widgets:Qt5Widgets.dll
 0000:fffd8000       .debug$S                   10000000     Qt5Widgets:Qt5Widgets.dll
 0000:fffd8000       .debug$S                   10000000     Qt5Widgets:Qt5Widgets.dll
 0000:fffd8000       .debug$S                   10000000     Qt5Widgets:Qt5Widgets.dll
 0000:fffd8000       .debug$S                   10000000     Qt5Widgets:Qt5Widgets.dll
 0000:fffd8000       .debug$S                   10000000     Qt5Widgets:Qt5Widgets.dll
 0000:fffd8000       .debug$S                   10000000     Qt5Widgets:Qt5Widgets.dll
 0000:fffd8000       .debug$S                   10000000     Qt5Widgets:Qt5Widgets.dll
 0000:fffd8000       .debug$S                   10000000     Qt5Widgets:Qt5Widgets.dll
 0000:fffd8000       .debug$S                   10000000     Qt5Widgets:Qt5Widgets.dll
 0000:fffd8000       .debug$S                   10000000     Qt5Widgets:Qt5Widgets.dll
 0000:fffd8000       .debug$S                   10000000     Qt5Widgets:Qt5Widgets.dll
 0000:fffd8000       .debug$S                   10000000     Qt5Widgets:Qt5Widgets.dll
 0000:fffd8000       .debug$S                   10000000     Qt5Widgets:Qt5Widgets.dll
 0000:fffd8000       .debug$S                   10000000     Qt5Widgets:Qt5Widgets.dll
 0000:fffd8000       .debug$S                   10000000     Qt5Widgets:Qt5Widgets.dll
 0000:fffd8000       .debug$S                   10000000     Qt5Widgets:Qt5Widgets.dll
 0000:fffd8000       .debug$S                   10000000     Qt5Widgets:Qt5Widgets.dll
 0000:fffd8000       .debug$S                   10000000     Qt5Widgets:Qt5Widgets.dll
 0000:fffd8000       .debug$S                   10000000     Qt5Widgets:Qt5Widgets.dll
 0000:fffd8000       .debug$S                   10000000     Qt5Widgets:Qt5Widgets.dll
 0000:fffd8000       .debug$S                   10000000     Qt5Widgets:Qt5Widgets.dll
 0000:fffd8000       .debug$S                   10000000     Qt5Widgets:Qt5Widgets.dll
 0000:fffd8000       .debug$S                   10000000     Qt5Widgets:Qt5Widgets.dll
 0000:fffd8000       .debug$S                   10000000     Qt5Widgets:Qt5Widgets.dll
 0000:fffd8000       .debug$S                   10000000     Qt5Widgets:Qt5Widgets.dll
 0000:fffd8000       .debug$S                   10000000     Qt5Widgets:Qt5Widgets.dll
 0000:fffd8000       .debug$S                   10000000     Qt5Widgets:Qt5Widgets.dll
 0000:fffd8000       .debug$S                   10000000     Qt5Widgets:Qt5Widgets.dll
 0000:fffd8000       .debug$S                   10000000     Qt5Widgets:Qt5Widgets.dll
 0000:fffd8000       .debug$S                   10000000     Qt5Widgets:Qt5Widgets.dll
 0000:fffd8000       .debug$S                   10000000     Qt5Widgets:Qt5Widgets.dll
 0000:fffd8000       .debug$S                   10000000     Qt5Widgets:Qt5Widgets.dll
 0000:fffd8000       .debug$S                   10000000     Qt5Widgets:Qt5Widgets.dll
 0000:fffd8000       .debug$S                   10000000     Qt5Widgets:Qt5Widgets.dll
 0000:fffd8000       .debug$S                   10000000     Qt5Widgets:Qt5Widgets.dll
 0000:fffd8000       .debug$S                   10000000     Qt5Widgets:Qt5Widgets.dll
 0000:fffd8000       .debug$S                   10000000     Qt5Widgets:Qt5Widgets.dll
 0000:fffd8000       .debug$S                   10000000     Qt5Widgets:Qt5Widgets.dll
 0000:fffd8000       .debug$S                   10000000     Qt5Widgets:Qt5Widgets.dll
 0000:fffd8000       .debug$S                   10000000     Qt5Widgets:Qt5Widgets.dll
 0000:fffd8000       .debug$S                   10000000     Qt5Widgets:Qt5Widgets.dll
 0000:fffd8000       .debug$S                   10000000     Qt5Widgets:Qt5Widgets.dll
 0000:fffd8000       .debug$S                   10000000     Qt5Widgets:Qt5Widgets.dll
 0002:fffed000       ?_Generic_object$initializer$@?$_Error_objects@H@std@@2P6AXXZA 10000000     moc_DNAFlexPlugin.obj
 0002:fffed000       ?_Iostream_object$initializer$@?$_Error_objects@H@std@@2P6AXXZA 10000000     moc_DNAFlexPlugin.obj
 0002:fffed000       ?_System_object$initializer$@?$_Error_objects@H@std@@2P6AXXZA 10000000     moc_DNAFlexPlugin.obj
 0000:fffd8000       .debug$S                   10000000     Qt5Widgets:Qt5Widgets.dll
 0000:fffd8000       .debug$S                   10000000     Qt5Widgets:Qt5Widgets.dll
 0000:fffd8000       .debug$S                   10000000     U2Core:U2Core.dll
 0000:fffd8000       .debug$S                   10000000     Qt5Widgets:Qt5Widgets.dll
 0000:fffd8000       .debug$S                   10000000     U2Core:U2Core.dll
 0000:fffd8000       .debug$S                   10000000     Qt5Widgets:Qt5Widgets.dll
 0000:fffd8000       .debug$S                   10000000     U2Core:U2Core.dll
 0000:fffd8000       .debug$S                   10000000     Qt5Widgets:Qt5Widgets.dll
 0000:fffd8000       .debug$S                   10000000     U2Core:U2Core.dll
 0000:fffd8000       .debug$S                   10000000     Qt5Widgets:Qt5Widgets.dll
 0000:fffd8000       .debug$S                   10000000     U2Core:U2Core.dll
 0000:fffd8000       .debug$S                   10000000     Qt5Widgets:Qt5Widgets.dll
 0000:fffd8000       .debug$S                   10000000     U2Core:U2Core.dll
 0000:fffd8000       .debug$S                   10000000     Qt5Widgets:Qt5Widgets.dll
 0000:fffd8000       .debug$S                   10000000     U2Core:U2Core.dll
 0000:fffd8000       .debug$S                   10000000     Qt5Widgets:Qt5Widgets.dll
 0000:fffd8000       .debug$S                   10000000     U2Core:U2Core.dll
 0000:fffd8000       .debug$S                   10000000     Qt5Widgets:Qt5Widgets.dll
 0000:fffd8000       .debug$S                   10000000     U2Core:U2Core.dll
 0000:fffd8000       .debug$S                   10000000     Qt5Widgets:Qt5Widgets.dll
 0000:fffd8000       .debug$S                   10000000     U2Core:U2Core.dll
 0000:fffd8000       .debug$S                   10000000     Qt5Widgets:Qt5Widgets.dll
 0000:fffd8000       .debug$S                   10000000     U2Core:U2Core.dll
 0000:fffd8000       .debug$S                   10000000     Qt5Widgets:Qt5Widgets.dll
 0000:fffd8000       .debug$S                   10000000     U2Core:U2Core.dll
 0000:fffd8000       .debug$S                   10000000     Qt5Widgets:Qt5Widgets.dll
 0000:fffd8000       .debug$S                   10000000     U2Core:U2Core.dll
 0000:fffd8000       .debug$S                   10000000     Qt5Widgets:Qt5Widgets.dll
 0000:fffd8000       .debug$S                   10000000     U2Core:U2Core.dll
 0000:fffd8000       .debug$S                   10000000     Qt5Widgets:Qt5Widgets.dll
 0000:fffd8000       .debug$S                   10000000     U2Core:U2Core.dll
 0000:fffd8000       .debug$S                   10000000     Qt5Widgets:Qt5Widgets.dll
 0000:fffd8000       .debug$S                   10000000     U2Core:U2Core.dll
 0000:fffd8000       .debug$S                   10000000     Qt5Widgets:Qt5Widgets.dll
 0000:fffd8000       .debug$S                   10000000     U2Core:U2Core.dll
 0000:fffd8000       .debug$S                   10000000     Qt5Widgets:Qt5Widgets.dll
 0000:fffd8000       .debug$S                   10000000     U2Core:U2Core.dll
 0000:fffd8000       .debug$S                   10000000     Qt5Widgets:Qt5Widgets.dll
 0000:fffd8000       .debug$S                   10000000     U2Core:U2Core.dll
 0000:fffd8000       .debug$S                   10000000     Qt5Widgets:Qt5Widgets.dll
 0000:fffd8000       .debug$S                   10000000     U2Core:U2Core.dll
 0000:fffd8000       .debug$S                   10000000     Qt5Widgets:Qt5Widgets.dll
 0000:fffd8000       .debug$S                   10000000     U2Core:U2Core.dll
 0000:fffd8000       .debug$S                   10000000     Qt5Widgets:Qt5Widgets.dll
 0000:fffd8000       .debug$S                   10000000     U2Core:U2Core.dll
 0000:fffd8000       .debug$S                   10000000     Qt5Widgets:Qt5Widgets.dll
 0000:fffd8000       .debug$S                   10000000     U2Core:U2Core.dll
 0000:fffd8000       .debug$S                   10000000     U2Core:U2Core.dll
 0000:fffd8000       .debug$S                   10000000     Qt5Widgets:Qt5Widgets.dll
 0000:fffd8000       .debug$S                   10000000     U2Core:U2Core.dll
 0000:fffd8000       .debug$S                   10000000     Qt5Widgets:Qt5Widgets.dll
 0000:fffd8000       .debug$S                   10000000     U2Core:U2Core.dll
 0000:fffd8000       .debug$S                   10000000     Qt5Widgets:Qt5Widgets.dll
 0001:fffff000       __ehhandler$?_Copy@?$basic_string@DU?$char_traits@D@std@@V?$allocator@D@2@@std@@QAEXII@Z 10000000 f   moc_DNAFlexGraph.obj
 0000:fffd8000       .debug$S                   10000000     U2Core:U2Core.dll
 0000:fffd8000       .debug$S                   10000000     U2Core:U2Core.dll
 0000:fffd8000       .debug$S                   10000000     Qt5Widgets:Qt5Widgets.dll
 0000:fffd8000       .debug$S                   10000000     Qt5Widgets:Qt5Widgets.dll
 0000:fffd8000       .debug$S                   10000000     Qt5Widgets:Qt5Widgets.dll
 0000:fffd8000       .debug$S                   10000000     Qt5Widgets:Qt5Widgets.dll
 0000:fffd8000       .debug$S                   10000000     Qt5Widgets:Qt5Widgets.dll
 0000:fffd8000       .debug$S                   10000000     Qt5Widgets:Qt5Widgets.dll
 0000:fffd8000       .debug$S                   10000000     Qt5Widgets:Qt5Widgets.dll
 0000:fffd8000       .debug$S                   10000000     Qt5Widgets:Qt5Widgets.dll
 0000:fffd8000       .debug$S                   10000000     Qt5Widgets:Qt5Widgets.dll
 0000:fffd8000       .debug$S                   10000000     Qt5Widgets:Qt5Widgets.dll
 0000:fffd8000       .debug$S                   10000000     Qt5Widgets:Qt5Widgets.dll
 0000:fffd8000       .debug$S                   10000000     Qt5Widgets:Qt5Widgets.dll
 0000:fffd8000       .debug$S                   10000000     Qt5Widgets:Qt5Widgets.dll
 0000:fffd8000       .debug$S                   10000000     Qt5Widgets:Qt5Widgets.dll
 0000:fffd8000       .debug$S                   10000000     Qt5Widgets:Qt5Widgets.dll
 0000:fffd8000       .debug$S                   10000000     Qt5Widgets:Qt5Widgets.dll
 0000:fffd8000       .debug$S                   10000000     Qt5Widgets:Qt5Widgets.dll
 0000:fffd8000       .debug$S                   10000000     Qt5Widgets:Qt5Widgets.dll
 0000:fffd8000       .debug$S                   10000000     U2Core:U2Core.dll
 0000:fffd8000       .debug$S                   10000000     U2Core:U2Core.dll
 0000:fffd8000       .debug$S                   10000000     U2Core:U2Core.dll
 0000:fffd8000       .debug$S                   10000000     U2Core:U2Core.dll
 0002:fffed000       __catchsym$?_Copy@?$basic_string@DU?$char_traits@D@std@@V?$allocator@D@2@@std@@QAEXII@Z$5 10000000     moc_DNAFlexGraph.obj
 0000:fffd8000       .debug$S                   10000000     Qt5Widgets:Qt5Widgets.dll
 0000:fffd8000       .debug$S                   10000000     Qt5Widgets:Qt5Widgets.dll
 0000:fffd8000       .debug$S                   10000000     Qt5Widgets:Qt5Widgets.dll
 0000:fffd8000       .debug$S                   10000000     Qt5Widgets:Qt5Widgets.dll
 0000:fffd8000       .debug$S                   10000000     Qt5Widgets:Qt5Widgets.dll
 0000:fffd8000       .debug$S                   10000000     Qt5Widgets:Qt5Widgets.dll
 0000:fffd8000       .debug$S                   10000000     Qt5Widgets:Qt5Widgets.dll
 0000:fffd8000       .debug$S                   10000000     Qt5Widgets:Qt5Widgets.dll
 0000:fffd8000       .debug$S                   10000000     Qt5Widgets:Qt5Widgets.dll
 0000:fffd8000       .debug$S                   10000000     Qt5Widgets:Qt5Widgets.dll
 0000:fffd8000       .debug$S                   10000000     Qt5Widgets:Qt5Widgets.dll
 0000:fffd8000       .debug$S                   10000000     Qt5Widgets:Qt5Widgets.dll
 0000:fffd8000       .debug$S                   10000000     Qt5Widgets:Qt5Widgets.dll
 0000:fffd8000       .debug$S                   10000000     Qt5Widgets:Qt5Widgets.dll
 0000:fffd8000       .debug$S                   10000000     Qt5Widgets:Qt5Widgets.dll
 0000:fffd8000       .debug$S                   10000000     Qt5Widgets:Qt5Widgets.dll
 0000:fffd8000       .debug$S                   10000000     Qt5Widgets:Qt5Widgets.dll
 0000:fffd8000       .debug$S                   10000000     Qt5Widgets:Qt5Widgets.dll
 0000:fffd8000       .debug$S                   10000000     Qt5Widgets:Qt5Widgets.dll
 0000:fffd8000       .debug$S                   10000000     Qt5Widgets:Qt5Widgets.dll
 0000:fffd8000       .debug$S                   10000000     Qt5Widgets:Qt5Widgets.dll
 0000:fffd8000       .debug$S                   10000000     Qt5Widgets:Qt5Widgets.dll
 0000:fffd8000       .debug$S                   10000000     Qt5Widgets:Qt5Widgets.dll
 0000:fffd8000       .debug$S                   10000000     Qt5Widgets:Qt5Widgets.dll
 0000:fffd8000       .debug$S                   10000000     Qt5Widgets:Qt5Widgets.dll
 0000:fffd8000       .debug$S                   10000000     Qt5Widgets:Qt5Widgets.dll
 0000:fffd8000       .debug$S                   10000000     Qt5Widgets:Qt5Widgets.dll
 0000:fffd8000       .debug$S                   10000000     Qt5Widgets:Qt5Widgets.dll
 0000:fffd8000       .debug$S                   10000000     Qt5Widgets:Qt5Widgets.dll
 0000:fffd8000       .debug$S                   10000000     Qt5Widgets:Qt5Widgets.dll
 0000:fffd8000       .debug$S                   10000000     Qt5Widgets:Qt5Widgets.dll
 0000:fffd8000       .debug$S                   10000000     Qt5Widgets:Qt5Widgets.dll
 0000:fffd8000       .debug$S                   10000000     Qt5Widgets:Qt5Widgets.dll
 0000:fffd8000       .debug$S                   10000000     Qt5Widgets:Qt5Widgets.dll
 0000:fffd8000       .debug$S                   10000000     Qt5Widgets:Qt5Widgets.dll
 0000:fffd8000       .debug$S                   10000000     Qt5Widgets:Qt5Widgets.dll
 0000:fffd8000       .debug$S                   10000000     Qt5Widgets:Qt5Widgets.dll
 0000:fffd8000       .debug$S                   10000000     Qt5Widgets:Qt5Widgets.dll
 0000:fffd8000       .debug$S                   10000000     Qt5Widgets:Qt5Widgets.dll
 0000:fffd8000       .debug$S                   10000000     Qt5Widgets:Qt5Widgets.dll
 0000:fffd8000       .debug$S                   10000000     Qt5Widgets:Qt5Widgets.dll
 0000:fffd8000       .debug$S                   10000000     Qt5Widgets:Qt5Widgets.dll
 0000:fffd8000       .debug$S                   10000000     Qt5Widgets:Qt5Widgets.dll
 0000:fffd8000       .debug$S                   10000000     Qt5Widgets:Qt5Widgets.dll
 0000:fffd8000       .debug$S                   10000000     Qt5Widgets:Qt5Widgets.dll
 0000:fffd8000       .debug$S                   10000000     Qt5Widgets:Qt5Widgets.dll
 0000:fffd8000       .debug$S                   10000000     Qt5Widgets:Qt5Widgets.dll
 0000:fffd8000       .debug$S                   10000000     Qt5Widgets:Qt5Widgets.dll
 0000:fffd8000       .debug$S                   10000000     Qt5Widgets:Qt5Widgets.dll
 0000:fffd8000       .debug$S                   10000000     Qt5Widgets:Qt5Widgets.dll
 0000:fffd8000       .debug$S                   10000000     Qt5Widgets:Qt5Widgets.dll
 0000:fffd8000       .debug$S                   10000000     Qt5Widgets:Qt5Widgets.dll
 0000:fffd8000       .debug$S                   10000000     Qt5Widgets:Qt5Widgets.dll
 0000:fffd8000       .debug$S                   10000000     Qt5Widgets:Qt5Widgets.dll
 0000:fffd8000       .debug$S                   10000000     Qt5Widgets:Qt5Widgets.dll
 0000:fffd8000       .debug$S                   10000000     Qt5Widgets:Qt5Widgets.dll
 0000:fffd8000       .debug$S                   10000000     Qt5Widgets:Qt5Widgets.dll
 0000:fffd8000       .debug$S                   10000000     Qt5Widgets:Qt5Widgets.dll
 0000:fffd8000       .debug$S                   10000000     Qt5Widgets:Qt5Widgets.dll
 0000:fffd8000       .debug$S                   10000000     Qt5Widgets:Qt5Widgets.dll
 0000:fffd8000       .debug$S                   10000000     Qt5Widgets:Qt5Widgets.dll
 0000:fffd8000       .debug$S                   10000000     Qt5Widgets:Qt5Widgets.dll
 0000:fffd8000       .debug$S                   10000000     Qt5Widgets:Qt5Widgets.dll
 0000:fffd8000       .debug$S                   10000000     Qt5Widgets:Qt5Widgets.dll
 0000:fffd8000       .debug$S                   10000000     Qt5Widgets:Qt5Widgets.dll
 0000:fffd8000       .debug$S                   10000000     Qt5Widgets:Qt5Widgets.dll
 0000:fffd8000       .debug$S                   10000000     Qt5Widgets:Qt5Widgets.dll
 0002:fffed000       ?_Generic_object$initializer$@?$_Error_objects@H@std@@2P6AXXZA 10000000     moc_DNAFlexGraph.obj
 0002:fffed000       ?_Iostream_object$initializer$@?$_Error_objects@H@std@@2P6AXXZA 10000000     moc_DNAFlexGraph.obj
 0002:fffed000       ?_System_object$initializer$@?$_Error_objects@H@std@@2P6AXXZA 10000000     moc_DNAFlexGraph.obj
 0000:fffd8000       .debug$S                   10000000     Qt5Widgets:Qt5Widgets.dll
 0000:fffd8000       .debug$S                   10000000     Qt5Widgets:Qt5Widgets.dll
 0000:fffd8000       .debug$S                   10000000     U2Core:U2Core.dll
 0000:fffd8000       .debug$S                   10000000     U2Core:U2Core.dll
 0000:fffd8000       .debug$S                   10000000     Qt5Widgets:Qt5Widgets.dll
 0000:fffd8000       .debug$S                   10000000     U2Core:U2Core.dll
 0000:fffd8000       .debug$S                   10000000     Qt5Widgets:Qt5Widgets.dll
 0000:fffd8000       .debug$S                   10000000     U2Core:U2Core.dll
 0000:fffd8000       .debug$S                   10000000     Qt5Widgets:Qt5Widgets.dll
 0001:fffff000       __ehhandler$?_Copy@?$basic_string@DU?$char_traits@D@std@@V?$allocator@D@2@@std@@QAEXII@Z 10000000 f   moc_DNAFlexDialog.obj
 0000:fffd8000       .debug$S                   10000000     U2Core:U2Core.dll
 0000:fffd8000       .debug$S                   10000000     U2Core:U2Core.dll
 0000:fffd8000       .debug$S                   10000000     U2Gui:U2Gui.dll
 0000:fffd8000       .debug$S                   10000000     U2Gui:U2Gui.dll
 0000:fffd8000       .debug$S                   10000000     U2Gui:U2Gui.dll
 0000:fffd8000       .debug$S                   10000000     U2Gui:U2Gui.dll
 0000:fffd8000       .debug$S                   10000000     U2Gui:U2Gui.dll
 0002:fffed000       __catchsym$?_Copy@?$basic_string@DU?$char_traits@D@std@@V?$allocator@D@2@@std@@QAEXII@Z$5 10000000     moc_DNAFlexDialog.obj
 0000:fffd8000       .debug$S                   10000000     Qt5Widgets:Qt5Widgets.dll
 0000:fffd8000       .debug$S                   10000000     Qt5Widgets:Qt5Widgets.dll
 0000:fffd8000       .debug$S                   10000000     Qt5Widgets:Qt5Widgets.dll
 0000:fffd8000       .debug$S                   10000000     Qt5Widgets:Qt5Widgets.dll
 0000:fffd8000       .debug$S                   10000000     Qt5Widgets:Qt5Widgets.dll
 0002:fffed000       ?_Generic_object$initializer$@?$_Error_objects@H@std@@2P6AXXZA 10000000     moc_DNAFlexDialog.obj
 0002:fffed000       ?_Iostream_object$initializer$@?$_Error_objects@H@std@@2P6AXXZA 10000000     moc_DNAFlexDialog.obj
 0002:fffed000       ?_System_object$initializer$@?$_Error_objects@H@std@@2P6AXXZA 10000000     moc_DNAFlexDialog.obj
 0000:fffd8000       .debug$S                   10000000     U2Gui:U2Gui.dll
 0000:fffd8000       .debug$S                   10000000     Qt5Widgets:Qt5Widgets.dll
 0000:fffd8000       .debug$S                   10000000     U2Gui:U2Gui.dll
 0000:fffd8000       .debug$S                   10000000     Qt5Widgets:Qt5Widgets.dll
 0000:fffd8000       .debug$S                   10000000     U2Gui:U2Gui.dll
 0000:fffd8000       .debug$S                   10000000     Qt5Widgets:Qt5Widgets.dll
 0002:fffed000       __catchsym$?_Copy@?$basic_string@DU?$char_traits@D@std@@V?$allocator@D@2@@std@@QAEXII@Z$5 10000000     HighFlexSettings.obj
 0000:fffd8000       .debug$S                   10000000     Qt5Widgets:Qt5Widgets.dll
 0000:fffd8000       .debug$S                   10000000     U2Gui:U2Gui.dll
 0000:fffd8000       .debug$S                   10000000     Qt5Widgets:Qt5Widgets.dll
 0000:fffd8000       .debug$S                   10000000     U2Gui:U2Gui.dll
 0000:fffd8000       .debug$S                   10000000     Qt5Widgets:Qt5Widgets.dll
 0000:fffd8000       .debug$S                   10000000     U2Gui:U2Gui.dll
 0000:fffd8000       .debug$S                   10000000     Qt5Widgets:Qt5Widgets.dll
 0000:fffd8000       .debug$S                   10000000     U2Gui:U2Gui.dll
 0000:fffd8000       .debug$S                   10000000     U2View:U2View.dll
 0000:fffd8000       .debug$S                   10000000     U2Gui:U2Gui.dll
 0000:fffd8000       .debug$S                   10000000     U2View:U2View.dll
 0000:fffd8000       .debug$S                   10000000     U2Gui:U2Gui.dll
 0000:fffd8000       .debug$S                   10000000     U2View:U2View.dll
 0000:fffd8000       .debug$S                   10000000     U2Gui:U2Gui.dll
 0000:fffd8000       .debug$S                   10000000     U2View:U2View.dll
 0000:fffd8000       .debug$S                   10000000     U2Gui:U2Gui.dll
 0000:fffd8000       .debug$S                   10000000     U2View:U2View.dll
 0000:fffd8000       .debug$S                   10000000     U2Gui:U2Gui.dll
 0000:fffd8000       .debug$S                   10000000     U2View:U2View.dll
 0000:fffd8000       .debug$S                   10000000     U2Gui:U2Gui.dll
 0000:fffd8000       .debug$S                   10000000     U2View:U2View.dll
 0000:fffd8000       .debug$S                   10000000     U2Gui:U2Gui.dll
 0000:fffd8000       .debug$S                   10000000     U2View:U2View.dll
 0000:fffd8000       .debug$S                   10000000     U2Gui:U2Gui.dll
 0000:fffd8000       .debug$S                   10000000     U2View:U2View.dll
 0001:fffff000       __ehhandler$?_Copy@?$basic_string@DU?$char_traits@D@std@@V?$allocator@D@2@@std@@QAEXII@Z 10000000 f   HighFlexSettings.obj
 0000:fffd8000       .debug$S                   10000000     U2Gui:U2Gui.dll
 0000:fffd8000       .debug$S                   10000000     U2Gui:U2Gui.dll
 0000:fffd8000       .debug$S                   10000000     U2View:U2View.dll
 0000:fffd8000       .debug$S                   10000000     U2View:U2View.dll
 0000:fffd8000       .debug$S                   10000000     U2View:U2View.dll
 0000:fffd8000       .debug$S                   10000000     U2View:U2View.dll
 0000:fffd8000       .debug$S                   10000000     U2View:U2View.dll
 0000:fffd8000       .debug$S                   10000000     U2View:U2View.dll
 0000:fffd8000       .debug$S                   10000000     U2View:U2View.dll
 0000:fffd8000       .debug$S                   10000000     U2View:U2View.dll
 0000:fffd8000       .debug$S                   10000000     U2View:U2View.dll
 0000:fffd8000       .debug$S                   10000000     U2View:U2View.dll
 0000:fffd8000       .debug$S                   10000000     U2View:U2View.dll
 0000:fffd8000       .debug$S                   10000000     U2View:U2View.dll
 0000:fffd8000       .debug$S                   10000000     U2View:U2View.dll
 0000:fffd8000       .debug$S                   10000000     U2View:U2View.dll
 0000:fffd8000       .debug$S                   10000000     U2View:U2View.dll
 0000:fffd8000       .debug$S                   10000000     U2View:U2View.dll
 0000:fffd8000       .debug$S                   10000000     U2View:U2View.dll
 0000:fffd8000       .debug$S                   10000000     U2View:U2View.dll
 0000:fffd8000       .debug$S                   10000000     U2View:U2View.dll
 0000:fffd8000       .debug$S                   10000000     U2View:U2View.dll
 0000:fffd8000       .debug$S                   10000000     U2View:U2View.dll
 0000:fffd8000       .debug$S                   10000000     U2View:U2View.dll
 0000:fffd8000       .debug$S                   10000000     U2View:U2View.dll
 0000:fffd8000       .debug$S                   10000000     U2View:U2View.dll
 0000:fffd8000       .debug$S                   10000000     U2View:U2View.dll
 0000:fffd8000       .debug$S                   10000000     U2View:U2View.dll
 0000:fffd8000       .debug$S                   10000000     U2View:U2View.dll
 0000:fffd8000       .debug$S                   10000000     U2View:U2View.dll
 0000:fffd8000       .debug$S                   10000000     U2View:U2View.dll
 0000:fffd8000       .debug$S                   10000000     U2Gui:U2Gui.dll
 0000:fffd8000       .debug$S                   10000000     U2Gui:U2Gui.dll
 0000:fffd8000       .debug$S                   10000000     U2Gui:U2Gui.dll
 0000:fffd8000       .debug$S                   10000000     U2Gui:U2Gui.dll
 0000:fffd8000       .debug$S                   10000000     U2Gui:U2Gui.dll
 0000:fffd8000       .debug$S                   10000000     U2Gui:U2Gui.dll
 0000:fffd8000       .debug$S                   10000000     U2Gui:U2Gui.dll
 0000:fffd8000       .debug$S                   10000000     U2Gui:U2Gui.dll
 0000:fffd8000       .debug$S                   10000000     U2Gui:U2Gui.dll
 0000:fffd8000       .debug$S                   10000000     U2Gui:U2Gui.dll
 0000:fffd8000       .debug$S                   10000000     U2Gui:U2Gui.dll
 0000:fffd8000       .debug$S                   10000000     U2Gui:U2Gui.dll
 0000:fffd8000       .debug$S                   10000000     U2Gui:U2Gui.dll
 0002:fffed000       ?_Generic_object$initializer$@?$_Error_objects@H@std@@2P6AXXZA 10000000     DNAFlexTask.obj
 0002:fffed008       __ehfuncinfo$?clone@?$QSharedDataPointer@VAnnotationData@U2@@@@IAEPAVAnnotationData@U2@@XZ 10000008     DNAFlexTask.obj
 0002:fffed008       __ehfuncinfo$?detach_helper@?$QSharedDataPointer@VAnnotationData@U2@@@@AAEXXZ 10000008     DNAFlexTask.obj
 0001:fffff00b       __ehhandler$?clone@?$QSharedDataPointer@VAnnotationData@U2@@@@IAEPAVAnnotationData@U2@@XZ 1000000b f   DNAFlexTask.obj
 0001:fffff00b       __ehhandler$?detach_helper@?$QSharedDataPointer@VAnnotationData@U2@@@@AAEXXZ 1000000b f   DNAFlexTask.obj
 0002:fffed010       __catchsym$?_Copy@?$basic_string@DU?$char_traits@D@std@@V?$allocator@D@2@@std@@QAEXII@Z$4 10000010     DNAFlexPlugin.obj
 0002:fffed010       __catchsym$?_Copy@?$basic_string@DU?$char_traits@D@std@@V?$allocator@D@2@@std@@QAEXII@Z$4 10000010     DNAFlexTask.obj
 0002:fffed010       __catchsym$?_Copy@?$basic_string@DU?$char_traits@D@std@@V?$allocator@D@2@@std@@QAEXII@Z$4 10000010     FindHighFlexRegionsAlgorithm.obj
 0002:fffed010       __catchsym$?_Copy@?$basic_string@DU?$char_traits@D@std@@V?$allocator@D@2@@std@@QAEXII@Z$4 10000010     FindHighFlexRegions.obj
 0002:fffed010       __unwindtable$??0?$QList@VHighFlexResult@U2@@@@QAE@ABV0@@Z 10000010     FindHighFlexRegions.obj
 0002:fffed010       __catchsym$?_Copy@?$basic_string@DU?$char_traits@D@std@@V?$allocator@D@2@@std@@QAEXII@Z$4 10000010     moc_FindHighFlexRegions.obj
 0002:fffed010       __catchsym$?_Copy@?$basic_string@DU?$char_traits@D@std@@V?$allocator@D@2@@std@@QAEXII@Z$4 10000010     DNAFlexGraphAlgorithm.obj
 0002:fffed010       __catchsym$?_Copy@?$basic_string@DU?$char_traits@D@std@@V?$allocator@D@2@@std@@QAEXII@Z$4 10000010     moc_DNAFlexTask.obj
 0002:fffed010       __catchsym$?_Copy@?$basic_string@DU?$char_traits@D@std@@V?$allocator@D@2@@std@@QAEXII@Z$4 10000010     moc_DNAFlexGraph.obj
 0002:fffed010       __tryblocktable$?node_copy@?$QList@VHighFlexResult@U2@@@@AAEXPAUNode@1@00@Z 10000010     FindHighFlexRegions.obj
 0002:fffed010       __catchsym$?_Copy@?$basic_string@DU?$char_traits@D@std@@V?$allocator@D@2@@std@@QAEXII@Z$4 10000010     moc_DNAFlexDialog.obj
 0002:fffed010       __catchsym$?_Copy@?$basic_string@DU?$char_traits@D@std@@V?$allocator@D@2@@std@@QAEXII@Z$4 10000010     DNAFlexGraph.obj
 0002:fffed010       __catchsym$?_Copy@?$basic_string@DU?$char_traits@D@std@@V?$allocator@D@2@@std@@QAEXII@Z$4 10000010     HighFlexSettings.obj
 0002:fffed010       __catchsym$?_Copy@?$basic_string@DU?$char_traits@D@std@@V?$allocator@D@2@@std@@QAEXII@Z$4 10000010     moc_DNAFlexPlugin.obj
 0002:fffed020       __unwindtable$?_Copy@?$basic_string@DU?$char_traits@D@std@@V?$allocator@D@2@@std@@QAEXII@Z 10000020     moc_DNAFlexPlugin.obj
 0002:fffed020       __unwindtable$?_Copy@?$basic_string@DU?$char_traits@D@std@@V?$allocator@D@2@@std@@QAEXII@Z 10000020     DNAFlexGraph.obj
 0002:fffed020       __unwindtable$?_Copy@?$basic_string@DU?$char_traits@D@std@@V?$allocator@D@2@@std@@QAEXII@Z 10000020     moc_DNAFlexTask.obj
 0002:fffed020       __unwindtable$?_Copy@?$basic_string@DU?$char_traits@D@std@@V?$allocator@D@2@@std@@QAEXII@Z 10000020     HighFlexSettings.obj
 0002:fffed020       __unwindtable$?_Copy@?$basic_string@DU?$char_traits@D@std@@V?$allocator@D@2@@std@@QAEXII@Z 10000020     FindHighFlexRegionsAlgorithm.obj
 0002:fffed020       __unwindtable$?_Copy@?$basic_string@DU?$char_traits@D@std@@V?$allocator@D@2@@std@@QAEXII@Z 10000020     moc_DNAFlexDialog.obj
 0002:fffed020       __unwindtable$?_Copy@?$basic_string@DU?$char_traits@D@std@@V?$allocator@D@2@@std@@QAEXII@Z 10000020     DNAFlexPlugin.obj
 0002:fffed020       __unwindtable$?_Copy@?$basic_string@DU?$char_traits@D@std@@V?$allocator@D@2@@std@@QAEXII@Z 10000020     moc_DNAFlexGraph.obj
 0002:fffed020       __unwindtable$?_Copy@?$basic_string@DU?$char_traits@D@std@@V?$allocator@D@2@@std@@QAEXII@Z 10000020     DNAFlexGraphAlgorithm.obj
 0002:fffed020       __tryblocktable$??0?$QList@VHighFlexResult@U2@@@@QAE@ABV0@@Z 10000020     FindHighFlexRegions.obj
 0002:fffed020       __unwindtable$?_Copy@?$basic_string@DU?$char_traits@D@std@@V?$allocator@D@2@@std@@QAEXII@Z 10000020     DNAFlexTask.obj
 0002:fffed020       __unwindtable$?_Copy@?$basic_string@DU?$char_traits@D@std@@V?$allocator@D@2@@std@@QAEXII@Z 10000020     FindHighFlexRegions.obj
 0002:fffed020       __unwindtable$?_Copy@?$basic_string@DU?$char_traits@D@std@@V?$allocator@D@2@@std@@QAEXII@Z 10000020     moc_FindHighFlexRegions.obj
 0002:fffed024       __unwindtable$?node_copy@?$QList@VHighFlexResult@U2@@@@AAEXPAUNode@1@00@Z 10000024     FindHighFlexRegions.obj
 0002:fffed034       __ehfuncinfo$??0?$QList@VHighFlexResult@U2@@@@QAE@ABV0@@Z 10000034     FindHighFlexRegions.obj
 0002:fffed040       __ehfuncinfo$?_Copy@?$basic_string@DU?$char_traits@D@std@@V?$allocator@D@2@@std@@QAEXII@Z 10000040     FindHighFlexRegions.obj
 0002:fffed040       __ehfuncinfo$?_Copy@?$basic_string@DU?$char_traits@D@std@@V?$allocator@D@2@@std@@QAEXII@Z 10000040     DNAFlexGraphAlgorithm.obj
 0002:fffed040       __ehfuncinfo$?_Copy@?$basic_string@DU?$char_traits@D@std@@V?$allocator@D@2@@std@@QAEXII@Z 10000040     moc_DNAFlexGraph.obj
 0002:fffed040       __ehfuncinfo$?_Copy@?$basic_string@DU?$char_traits@D@std@@V?$allocator@D@2@@std@@QAEXII@Z 10000040     moc_DNAFlexDialog.obj
 0002:fffed040       __ehfuncinfo$?_Copy@?$basic_string@DU?$char_traits@D@std@@V?$allocator@D@2@@std@@QAEXII@Z 10000040     HighFlexSettings.obj
 0002:fffed040       __ehfuncinfo$?_Copy@?$basic_string@DU?$char_traits@D@std@@V?$allocator@D@2@@std@@QAEXII@Z 10000040     FindHighFlexRegionsAlgorithm.obj
 0002:fffed040       __ehfuncinfo$?_Copy@?$basic_string@DU?$char_traits@D@std@@V?$allocator@D@2@@std@@QAEXII@Z 10000040     moc_DNAFlexTask.obj
 0002:fffed040       __ehfuncinfo$?_Copy@?$basic_string@DU?$char_traits@D@std@@V?$allocator@D@2@@std@@QAEXII@Z 10000040     moc_FindHighFlexRegions.obj
 0002:fffed040       __ehfuncinfo$?_Copy@?$basic_string@DU?$char_traits@D@std@@V?$allocator@D@2@@std@@QAEXII@Z 10000040     DNAFlexPlugin.obj
 0002:fffed040       __ehfuncinfo$?_Copy@?$basic_string@DU?$char_traits@D@std@@V?$allocator@D@2@@std@@QAEXII@Z 10000040     moc_DNAFlexPlugin.obj
 0002:fffed040       __ehfuncinfo$?_Copy@?$basic_string@DU?$char_traits@D@std@@V?$allocator@D@2@@std@@QAEXII@Z 10000040     DNAFlexGraph.obj
 0002:fffed040       __ehfuncinfo$?_Copy@?$basic_string@DU?$char_traits@D@std@@V?$allocator@D@2@@std@@QAEXII@Z 10000040     DNAFlexTask.obj
 0002:fffed044       __ehfuncinfo$?node_copy@?$QList@VHighFlexResult@U2@@@@AAEXPAUNode@1@00@Z 10000044     FindHighFlexRegions.obj
 0002:fffed064       __tryblocktable$?_Copy@?$basic_string@DU?$char_traits@D@std@@V?$allocator@D@2@@std@@QAEXII@Z 10000064     DNAFlexGraphAlgorithm.obj
 0002:fffed064       __tryblocktable$?_Copy@?$basic_string@DU?$char_traits@D@std@@V?$allocator@D@2@@std@@QAEXII@Z 10000064     moc_DNAFlexPlugin.obj
 0002:fffed064       __tryblocktable$?_Copy@?$basic_string@DU?$char_traits@D@std@@V?$allocator@D@2@@std@@QAEXII@Z 10000064     moc_DNAFlexGraph.obj
 0002:fffed064       __tryblocktable$?_Copy@?$basic_string@DU?$char_traits@D@std@@V?$allocator@D@2@@std@@QAEXII@Z 10000064     FindHighFlexRegions.obj
 0002:fffed064       __tryblocktable$?_Copy@?$basic_string@DU?$char_traits@D@std@@V?$allocator@D@2@@std@@QAEXII@Z 10000064     DNAFlexTask.obj
 0002:fffed064       __tryblocktable$?_Copy@?$basic_string@DU?$char_traits@D@std@@V?$allocator@D@2@@std@@QAEXII@Z 10000064     moc_DNAFlexTask.obj
 0002:fffed064       __tryblocktable$?_Copy@?$basic_string@DU?$char_traits@D@std@@V?$allocator@D@2@@std@@QAEXII@Z 10000064     HighFlexSettings.obj
 0002:fffed064       __tryblocktable$?_Copy@?$basic_string@DU?$char_traits@D@std@@V?$allocator@D@2@@std@@QAEXII@Z 10000064     DNAFlexPlugin.obj
 0002:fffed064       __tryblocktable$?_Copy@?$basic_string@DU?$char_traits@D@std@@V?$allocator@D@2@@std@@QAEXII@Z 10000064     DNAFlexGraph.obj
 0002:fffed064       __tryblocktable$?_Copy@?$basic_string@DU?$char_traits@D@std@@V?$allocator@D@2@@std@@QAEXII@Z 10000064     moc_DNAFlexDialog.obj
 0002:fffed064       __tryblocktable$?_Copy@?$basic_string@DU?$char_traits@D@std@@V?$allocator@D@2@@std@@QAEXII@Z 10000064     moc_FindHighFlexRegions.obj
 0002:fffed064       __tryblocktable$?_Copy@?$basic_string@DU?$char_traits@D@std@@V?$allocator@D@2@@std@@QAEXII@Z 10000064     FindHighFlexRegionsAlgorithm.obj
 0001:fffff084       __catch$?node_copy@?$QList@VHighFlexResult@U2@@@@AAEXPAUNode@1@00@Z$0 10000084 f   FindHighFlexRegions.obj
 0001:fffff096       __catch$?_Copy@?$basic_string@DU?$char_traits@D@std@@V?$allocator@D@2@@std@@QAEXII@Z$0 10000096 f   DNAFlexTask.obj
 0001:fffff096       __catch$?_Copy@?$basic_string@DU?$char_traits@D@std@@V?$allocator@D@2@@std@@QAEXII@Z$0 10000096 f   FindHighFlexRegions.obj
 0001:fffff096       __catch$?_Copy@?$basic_string@DU?$char_traits@D@std@@V?$allocator@D@2@@std@@QAEXII@Z$0 10000096 f   moc_DNAFlexTask.obj
 0001:fffff096       __catch$?_Copy@?$basic_string@DU?$char_traits@D@std@@V?$allocator@D@2@@std@@QAEXII@Z$0 10000096 f   DNAFlexGraph.obj
 0001:fffff096       __catch$?_Copy@?$basic_string@DU?$char_traits@D@std@@V?$allocator@D@2@@std@@QAEXII@Z$0 10000096 f   HighFlexSettings.obj
 0001:fffff096       __catch$?_Copy@?$basic_string@DU?$char_traits@D@std@@V?$allocator@D@2@@std@@QAEXII@Z$0 10000096 f   FindHighFlexRegionsAlgorithm.obj
 0001:fffff096       __catch$?_Copy@?$basic_string@DU?$char_traits@D@std@@V?$allocator@D@2@@std@@QAEXII@Z$0 10000096 f   DNAFlexPlugin.obj
 0001:fffff096       __catch$?_Copy@?$basic_string@DU?$char_traits@D@std@@V?$allocator@D@2@@std@@QAEXII@Z$0 10000096 f   moc_DNAFlexDialog.obj
 0001:fffff096       __catch$?_Copy@?$basic_string@DU?$char_traits@D@std@@V?$allocator@D@2@@std@@QAEXII@Z$0 10000096 f   moc_DNAFlexGraph.obj
 0001:fffff096       __catch$?_Copy@?$basic_string@DU?$char_traits@D@std@@V?$allocator@D@2@@std@@QAEXII@Z$0 10000096 f   moc_FindHighFlexRegions.obj
 0001:fffff096       __catch$?_Copy@?$basic_string@DU?$char_traits@D@std@@V?$allocator@D@2@@std@@QAEXII@Z$0 10000096 f   moc_DNAFlexPlugin.obj
 0001:fffff096       __catch$?_Copy@?$basic_string@DU?$char_traits@D@std@@V?$allocator@D@2@@std@@QAEXII@Z$0 10000096 f   DNAFlexGraphAlgorithm.obj
 0001:fffff09e       __catch$??0?$QList@VHighFlexResult@U2@@@@QAE@ABV0@@Z$0 1000009e f   FindHighFlexRegions.obj
 0001:fffff0d3       __catch$?_Copy@?$basic_string@DU?$char_traits@D@std@@V?$allocator@D@2@@std@@QAEXII@Z$1 100000d3 f   moc_DNAFlexPlugin.obj
 0001:fffff0d3       __catch$?_Copy@?$basic_string@DU?$char_traits@D@std@@V?$allocator@D@2@@std@@QAEXII@Z$1 100000d3 f   DNAFlexGraphAlgorithm.obj
 0001:fffff0d3       __catch$?_Copy@?$basic_string@DU?$char_traits@D@std@@V?$allocator@D@2@@std@@QAEXII@Z$1 100000d3 f   moc_FindHighFlexRegions.obj
 0001:fffff0d3       __catch$?_Copy@?$basic_string@DU?$char_traits@D@std@@V?$allocator@D@2@@std@@QAEXII@Z$1 100000d3 f   DNAFlexGraph.obj
 0001:fffff0d3       __catch$?_Copy@?$basic_string@DU?$char_traits@D@std@@V?$allocator@D@2@@std@@QAEXII@Z$1 100000d3 f   moc_DNAFlexTask.obj
 0001:fffff0d3       __catch$?_Copy@?$basic_string@DU?$char_traits@D@std@@V?$allocator@D@2@@std@@QAEXII@Z$1 100000d3 f   DNAFlexTask.obj
 0001:fffff0d3       __catch$?_Copy@?$basic_string@DU?$char_traits@D@std@@V?$allocator@D@2@@std@@QAEXII@Z$1 100000d3 f   moc_DNAFlexDialog.obj
 0001:fffff0d3       __catch$?_Copy@?$basic_string@DU?$char_traits@D@std@@V?$allocator@D@2@@std@@QAEXII@Z$1 100000d3 f   FindHighFlexRegions.obj
 0001:fffff0d3       __catch$?_Copy@?$basic_string@DU?$char_traits@D@std@@V?$allocator@D@2@@std@@QAEXII@Z$1 100000d3 f   DNAFlexPlugin.obj
 0001:fffff0d3       __catch$?_Copy@?$basic_string@DU?$char_traits@D@std@@V?$allocator@D@2@@std@@QAEXII@Z$1 100000d3 f   moc_DNAFlexGraph.obj
 0001:fffff0d3       __catch$?_Copy@?$basic_string@DU?$char_traits@D@std@@V?$allocator@D@2@@std@@QAEXII@Z$1 100000d3 f   FindHighFlexRegionsAlgorithm.obj
 0001:fffff0d3       __catch$?_Copy@?$basic_string@DU?$char_traits@D@std@@V?$allocator@D@2@@std@@QAEXII@Z$1 100000d3 f   HighFlexSettings.obj
 0001:00000000       ??__E?_Generic_object@?$_Error_objects@H@std@@2V_Generic_error_category@2@A@@YAXXZ 10001000 f   DNAFlexDialog.obj
 0001:00000010       ??__E?_Iostream_object@?$_Error_objects@H@std@@2V_Iostream_error_category@2@A@@YAXXZ 10001010 f   DNAFlexDialog.obj
 0001:00000020       ??__E?_System_object@?$_Error_objects@H@std@@2V_System_error_category@2@A@@YAXXZ 10001020 f   DNAFlexDialog.obj
 0001:00000030       ??__EService_DNAExport@U2@@YAXXZ 10001030 f   DNAFlexDialog.obj
 0001:00000040       ??__EService_DNAGraphPack@U2@@YAXXZ 10001040 f   DNAFlexDialog.obj
 0001:00000050       ??__EService_ExternalToolSupport@U2@@YAXXZ 10001050 f   DNAFlexDialog.obj
 0001:00000060       ??__EService_GUITesting@U2@@YAXXZ 10001060 f   DNAFlexDialog.obj
 0001:00000070       ??__EService_MaxCoreServiceId@U2@@YAXXZ 10001070 f   DNAFlexDialog.obj
 0001:00000080       ??__EService_MinCoreServiceId@U2@@YAXXZ 10001080 f   DNAFlexDialog.obj
 0001:00000090       ??__EService_PluginViewer@U2@@YAXXZ 10001090 f   DNAFlexDialog.obj
 0001:000000a0       ??__EService_Project@U2@@YAXXZ 100010a0 f   DNAFlexDialog.obj
 0001:000000b0       ??__EService_ProjectView@U2@@YAXXZ 100010b0 f   DNAFlexDialog.obj
 0001:000000c0       ??__EService_QueryDesigner@U2@@YAXXZ 100010c0 f   DNAFlexDialog.obj
 0001:000000d0       ??__EService_ScriptRegistry@U2@@YAXXZ 100010d0 f   DNAFlexDialog.obj
 0001:000000e0       ??__EService_TestRunner@U2@@YAXXZ 100010e0 f   DNAFlexDialog.obj
 0001:000000f0       ??__EService_WorkflowDesigner@U2@@YAXXZ 100010f0 f   DNAFlexDialog.obj
 0001:00000100       ??__EalgoLog@U2@@YAXXZ     10001100 f   DNAFlexDialog.obj
 0001:00000180       ??__EcmdLog@U2@@YAXXZ      10001180 f   DNAFlexDialog.obj
 0001:00000200       ??__EcoreLog@U2@@YAXXZ     10001200 f   DNAFlexDialog.obj
 0001:00000280       ??__EioLog@U2@@YAXXZ       10001280 f   DNAFlexDialog.obj
 0001:00000300       ??__EperfLog@U2@@YAXXZ     10001300 f   DNAFlexDialog.obj
 0001:00000380       ??__EscriptLog@U2@@YAXXZ   10001380 f   DNAFlexDialog.obj
 0001:00000400       ??__EtaskLog@U2@@YAXXZ     10001400 f   DNAFlexDialog.obj
 0001:00000480       ??__EuiLog@U2@@YAXXZ       10001480 f   DNAFlexDialog.obj
 0001:00000500       ??__EuserActLog@U2@@YAXXZ  10001500 f   DNAFlexDialog.obj
 0001:00000580       ??__E?_Generic_object@?$_Error_objects@H@std@@2V_Generic_error_category@2@A@@YAXXZ 10001580 f   DNAFlexGraph.obj
 0001:00000590       ??__E?_Iostream_object@?$_Error_objects@H@std@@2V_Iostream_error_category@2@A@@YAXXZ 10001590 f   DNAFlexGraph.obj
 0001:000005a0       ??__E?_System_object@?$_Error_objects@H@std@@2V_System_error_category@2@A@@YAXXZ 100015a0 f   DNAFlexGraph.obj
 0001:000005b0       ??__EService_DNAExport@U2@@YAXXZ 100015b0 f   DNAFlexGraph.obj
 0001:000005c0       ??__EService_DNAGraphPack@U2@@YAXXZ 100015c0 f   DNAFlexGraph.obj
 0001:000005d0       ??__EService_ExternalToolSupport@U2@@YAXXZ 100015d0 f   DNAFlexGraph.obj
 0001:000005e0       ??__EService_GUITesting@U2@@YAXXZ 100015e0 f   DNAFlexGraph.obj
 0001:000005f0       ??__EService_MaxCoreServiceId@U2@@YAXXZ 100015f0 f   DNAFlexGraph.obj
 0001:00000600       ??__EService_MinCoreServiceId@U2@@YAXXZ 10001600 f   DNAFlexGraph.obj
 0001:00000610       ??__EService_PluginViewer@U2@@YAXXZ 10001610 f   DNAFlexGraph.obj
 0001:00000620       ??__EService_Project@U2@@YAXXZ 10001620 f   DNAFlexGraph.obj
 0001:00000630       ??__EService_ProjectView@U2@@YAXXZ 10001630 f   DNAFlexGraph.obj
 0001:00000640       ??__EService_QueryDesigner@U2@@YAXXZ 10001640 f   DNAFlexGraph.obj
 0001:00000650       ??__EService_ScriptRegistry@U2@@YAXXZ 10001650 f   DNAFlexGraph.obj
 0001:00000660       ??__EService_TestRunner@U2@@YAXXZ 10001660 f   DNAFlexGraph.obj
 0001:00000670       ??__EService_WorkflowDesigner@U2@@YAXXZ 10001670 f   DNAFlexGraph.obj
 0001:00000680       ??__EalgoLog@U2@@YAXXZ     10001680 f   DNAFlexGraph.obj
 0001:00000700       ??__EcmdLog@U2@@YAXXZ      10001700 f   DNAFlexGraph.obj
 0001:00000780       ??__EcoreLog@U2@@YAXXZ     10001780 f   DNAFlexGraph.obj
 0001:00000800       ??__EioLog@U2@@YAXXZ       10001800 f   DNAFlexGraph.obj
 0001:00000880       ??__EperfLog@U2@@YAXXZ     10001880 f   DNAFlexGraph.obj
 0001:00000900       ??__EscriptLog@U2@@YAXXZ   10001900 f   DNAFlexGraph.obj
 0001:00000980       ??__EtaskLog@U2@@YAXXZ     10001980 f   DNAFlexGraph.obj
 0001:00000a00       ??__EuiLog@U2@@YAXXZ       10001a00 f   DNAFlexGraph.obj
 0001:00000a80       ??__EuserActLog@U2@@YAXXZ  10001a80 f   DNAFlexGraph.obj
 0001:00000b00       ??__E?_Generic_object@?$_Error_objects@H@std@@2V_Generic_error_category@2@A@@YAXXZ 10001b00 f   DNAFlexGraphAlgorithm.obj
 0001:00000b10       ??__E?_Iostream_object@?$_Error_objects@H@std@@2V_Iostream_error_category@2@A@@YAXXZ 10001b10 f   DNAFlexGraphAlgorithm.obj
 0001:00000b20       ??__E?_System_object@?$_Error_objects@H@std@@2V_System_error_category@2@A@@YAXXZ 10001b20 f   DNAFlexGraphAlgorithm.obj
 0001:00000b30       ??__EService_DNAExport@U2@@YAXXZ 10001b30 f   DNAFlexGraphAlgorithm.obj
 0001:00000b40       ??__EService_DNAGraphPack@U2@@YAXXZ 10001b40 f   DNAFlexGraphAlgorithm.obj
 0001:00000b50       ??__EService_ExternalToolSupport@U2@@YAXXZ 10001b50 f   DNAFlexGraphAlgorithm.obj
 0001:00000b60       ??__EService_GUITesting@U2@@YAXXZ 10001b60 f   DNAFlexGraphAlgorithm.obj
 0001:00000b70       ??__EService_MaxCoreServiceId@U2@@YAXXZ 10001b70 f   DNAFlexGraphAlgorithm.obj
 0001:00000b80       ??__EService_MinCoreServiceId@U2@@YAXXZ 10001b80 f   DNAFlexGraphAlgorithm.obj
 0001:00000b90       ??__EService_PluginViewer@U2@@YAXXZ 10001b90 f   DNAFlexGraphAlgorithm.obj
 0001:00000ba0       ??__EService_Project@U2@@YAXXZ 10001ba0 f   DNAFlexGraphAlgorithm.obj
 0001:00000bb0       ??__EService_ProjectView@U2@@YAXXZ 10001bb0 f   DNAFlexGraphAlgorithm.obj
 0001:00000bc0       ??__EService_QueryDesigner@U2@@YAXXZ 10001bc0 f   DNAFlexGraphAlgorithm.obj
 0001:00000bd0       ??__EService_ScriptRegistry@U2@@YAXXZ 10001bd0 f   DNAFlexGraphAlgorithm.obj
 0001:00000be0       ??__EService_TestRunner@U2@@YAXXZ 10001be0 f   DNAFlexGraphAlgorithm.obj
 0001:00000bf0       ??__EService_WorkflowDesigner@U2@@YAXXZ 10001bf0 f   DNAFlexGraphAlgorithm.obj
 0001:00000c00       ??__EalgoLog@U2@@YAXXZ     10001c00 f   DNAFlexGraphAlgorithm.obj
 0001:00000c80       ??__EcmdLog@U2@@YAXXZ      10001c80 f   DNAFlexGraphAlgorithm.obj
 0001:00000d00       ??__EcoreLog@U2@@YAXXZ     10001d00 f   DNAFlexGraphAlgorithm.obj
 0001:00000d80       ??__EioLog@U2@@YAXXZ       10001d80 f   DNAFlexGraphAlgorithm.obj
 0001:00000e00       ??__EperfLog@U2@@YAXXZ     10001e00 f   DNAFlexGraphAlgorithm.obj
 0001:00000e80       ??__EscriptLog@U2@@YAXXZ   10001e80 f   DNAFlexGraphAlgorithm.obj
 0001:00000f00       ??__EtaskLog@U2@@YAXXZ     10001f00 f   DNAFlexGraphAlgorithm.obj
 0001:00000f80       ??__EuiLog@U2@@YAXXZ       10001f80 f   DNAFlexGraphAlgorithm.obj
 0001:00001000       ??__EuserActLog@U2@@YAXXZ  10002000 f   DNAFlexGraphAlgorithm.obj
 0001:00001080       ??__E?_Generic_object@?$_Error_objects@H@std@@2V_Generic_error_category@2@A@@YAXXZ 10002080 f   DNAFlexPlugin.obj
 0001:00001090       ??__E?_Iostream_object@?$_Error_objects@H@std@@2V_Iostream_error_category@2@A@@YAXXZ 10002090 f   DNAFlexPlugin.obj
 0001:000010a0       ??__E?_System_object@?$_Error_objects@H@std@@2V_System_error_category@2@A@@YAXXZ 100020a0 f   DNAFlexPlugin.obj
 0001:000010b0       ??__EService_DNAExport@U2@@YAXXZ 100020b0 f   DNAFlexPlugin.obj
 0001:000010c0       ??__EService_DNAGraphPack@U2@@YAXXZ 100020c0 f   DNAFlexPlugin.obj
 0001:000010d0       ??__EService_ExternalToolSupport@U2@@YAXXZ 100020d0 f   DNAFlexPlugin.obj
 0001:000010e0       ??__EService_GUITesting@U2@@YAXXZ 100020e0 f   DNAFlexPlugin.obj
 0001:000010f0       ??__EService_MaxCoreServiceId@U2@@YAXXZ 100020f0 f   DNAFlexPlugin.obj
 0001:00001100       ??__EService_MinCoreServiceId@U2@@YAXXZ 10002100 f   DNAFlexPlugin.obj
 0001:00001110       ??__EService_PluginViewer@U2@@YAXXZ 10002110 f   DNAFlexPlugin.obj
 0001:00001120       ??__EService_Project@U2@@YAXXZ 10002120 f   DNAFlexPlugin.obj
 0001:00001130       ??__EService_ProjectView@U2@@YAXXZ 10002130 f   DNAFlexPlugin.obj
 0001:00001140       ??__EService_QueryDesigner@U2@@YAXXZ 10002140 f   DNAFlexPlugin.obj
 0001:00001150       ??__EService_ScriptRegistry@U2@@YAXXZ 10002150 f   DNAFlexPlugin.obj
 0001:00001160       ??__EService_TestRunner@U2@@YAXXZ 10002160 f   DNAFlexPlugin.obj
 0001:00001170       ??__EService_WorkflowDesigner@U2@@YAXXZ 10002170 f   DNAFlexPlugin.obj
 0001:00001180       ??__EalgoLog@U2@@YAXXZ     10002180 f   DNAFlexPlugin.obj
 0001:00001200       ??__EcmdLog@U2@@YAXXZ      10002200 f   DNAFlexPlugin.obj
 0001:00001280       ??__EcoreLog@U2@@YAXXZ     10002280 f   DNAFlexPlugin.obj
 0001:00001300       ??__EioLog@U2@@YAXXZ       10002300 f   DNAFlexPlugin.obj
 0001:00001380       ??__EperfLog@U2@@YAXXZ     10002380 f   DNAFlexPlugin.obj
 0001:00001400       ??__EscriptLog@U2@@YAXXZ   10002400 f   DNAFlexPlugin.obj
 0001:00001480       ??__EtaskLog@U2@@YAXXZ     10002480 f   DNAFlexPlugin.obj
 0001:00001500       ??__EuiLog@U2@@YAXXZ       10002500 f   DNAFlexPlugin.obj
 0001:00001580       ??__EuserActLog@U2@@YAXXZ  10002580 f   DNAFlexPlugin.obj
 0001:00001600       ??__E?_Generic_object@?$_Error_objects@H@std@@2V_Generic_error_category@2@A@@YAXXZ 10002600 f   DNAFlexTask.obj
 0001:00001610       ??__E?_Iostream_object@?$_Error_objects@H@std@@2V_Iostream_error_category@2@A@@YAXXZ 10002610 f   DNAFlexTask.obj
 0001:00001620       ??__E?_System_object@?$_Error_objects@H@std@@2V_System_error_category@2@A@@YAXXZ 10002620 f   DNAFlexTask.obj
 0001:00001630       ??__EalgoLog@U2@@YAXXZ     10002630 f   DNAFlexTask.obj
 0001:000016b0       ??__EcmdLog@U2@@YAXXZ      100026b0 f   DNAFlexTask.obj
 0001:00001730       ??__EcoreLog@U2@@YAXXZ     10002730 f   DNAFlexTask.obj
 0001:000017b0       ??__EioLog@U2@@YAXXZ       100027b0 f   DNAFlexTask.obj
 0001:00001830       ??__EperfLog@U2@@YAXXZ     10002830 f   DNAFlexTask.obj
 0001:000018b0       ??__EscriptLog@U2@@YAXXZ   100028b0 f   DNAFlexTask.obj
 0001:00001930       ??__EtaskLog@U2@@YAXXZ     10002930 f   DNAFlexTask.obj
 0001:000019b0       ??__EuiLog@U2@@YAXXZ       100029b0 f   DNAFlexTask.obj
 0001:00001a30       ??__EuserActLog@U2@@YAXXZ  10002a30 f   DNAFlexTask.obj
 0001:00001ab0       ??__E?_Generic_object@?$_Error_objects@H@std@@2V_Generic_error_category@2@A@@YAXXZ 10002ab0 f   FindHighFlexRegions.obj
 0001:00001ac0       ??__E?_Iostream_object@?$_Error_objects@H@std@@2V_Iostream_error_category@2@A@@YAXXZ 10002ac0 f   FindHighFlexRegions.obj
 0001:00001ad0       ??__E?_System_object@?$_Error_objects@H@std@@2V_System_error_category@2@A@@YAXXZ 10002ad0 f   FindHighFlexRegions.obj
 0001:00001ae0       ??__EalgoLog@U2@@YAXXZ     10002ae0 f   FindHighFlexRegions.obj
 0001:00001b60       ??__EcmdLog@U2@@YAXXZ      10002b60 f   FindHighFlexRegions.obj
 0001:00001be0       ??__EcoreLog@U2@@YAXXZ     10002be0 f   FindHighFlexRegions.obj
 0001:00001c60       ??__EioLog@U2@@YAXXZ       10002c60 f   FindHighFlexRegions.obj
 0001:00001ce0       ??__EperfLog@U2@@YAXXZ     10002ce0 f   FindHighFlexRegions.obj
 0001:00001d60       ??__EscriptLog@U2@@YAXXZ   10002d60 f   FindHighFlexRegions.obj
 0001:00001de0       ??__EtaskLog@U2@@YAXXZ     10002de0 f   FindHighFlexRegions.obj
 0001:00001e60       ??__EuiLog@U2@@YAXXZ       10002e60 f   FindHighFlexRegions.obj
 0001:00001ee0       ??__EuserActLog@U2@@YAXXZ  10002ee0 f   FindHighFlexRegions.obj
 0001:00001f60       ??__E?_Generic_object@?$_Error_objects@H@std@@2V_Generic_error_category@2@A@@YAXXZ 10002f60 f   FindHighFlexRegionsAlgorithm.obj
 0001:00001f70       ??__E?_Iostream_object@?$_Error_objects@H@std@@2V_Iostream_error_category@2@A@@YAXXZ 10002f70 f   FindHighFlexRegionsAlgorithm.obj
 0001:00001f80       ??__E?_System_object@?$_Error_objects@H@std@@2V_System_error_category@2@A@@YAXXZ 10002f80 f   FindHighFlexRegionsAlgorithm.obj
 0001:00001f90       ??__EalgoLog@U2@@YAXXZ     10002f90 f   FindHighFlexRegionsAlgorithm.obj
 0001:00002010       ??__EcmdLog@U2@@YAXXZ      10003010 f   FindHighFlexRegionsAlgorithm.obj
 0001:00002090       ??__EcoreLog@U2@@YAXXZ     10003090 f   FindHighFlexRegionsAlgorithm.obj
 0001:00002110       ??__EioLog@U2@@YAXXZ       10003110 f   FindHighFlexRegionsAlgorithm.obj
 0001:00002190       ??__EperfLog@U2@@YAXXZ     10003190 f   FindHighFlexRegionsAlgorithm.obj
 0001:00002210       ??__EscriptLog@U2@@YAXXZ   10003210 f   FindHighFlexRegionsAlgorithm.obj
 0001:00002290       ??__EtaskLog@U2@@YAXXZ     10003290 f   FindHighFlexRegionsAlgorithm.obj
 0001:00002310       ??__EuiLog@U2@@YAXXZ       10003310 f   FindHighFlexRegionsAlgorithm.obj
 0001:00002390       ??__EuserActLog@U2@@YAXXZ  10003390 f   FindHighFlexRegionsAlgorithm.obj
 0001:00002410       ??__E?SETTINGS_PATH@HighFlexSettings@U2@@0VQString@@B@@YAXXZ 10003410 f   HighFlexSettings.obj
 0001:00002430       ??__E?SETTING_THRESHOLD@HighFlexSettings@U2@@0VQString@@B@@YAXXZ 10003430 f   HighFlexSettings.obj
 0001:00002450       ??__E?SETTING_WINDOW_SIZE@HighFlexSettings@U2@@0VQString@@B@@YAXXZ 10003450 f   HighFlexSettings.obj
 0001:00002470       ??__E?SETTING_WINDOW_STEP@HighFlexSettings@U2@@0VQString@@B@@YAXXZ 10003470 f   HighFlexSettings.obj
 0001:00002490       ??__E?_Generic_object@?$_Error_objects@H@std@@2V_Generic_error_category@2@A@@YAXXZ 10003490 f   HighFlexSettings.obj
 0001:000024a0       ??__E?_Iostream_object@?$_Error_objects@H@std@@2V_Iostream_error_category@2@A@@YAXXZ 100034a0 f   HighFlexSettings.obj
 0001:000024b0       ??__E?_System_object@?$_Error_objects@H@std@@2V_System_error_category@2@A@@YAXXZ 100034b0 f   HighFlexSettings.obj
 0001:000024c0       ??__EalgoLog@U2@@YAXXZ     100034c0 f   HighFlexSettings.obj
 0001:00002540       ??__EcmdLog@U2@@YAXXZ      10003540 f   HighFlexSettings.obj
 0001:000025c0       ??__EcoreLog@U2@@YAXXZ     100035c0 f   HighFlexSettings.obj
 0001:00002640       ??__EioLog@U2@@YAXXZ       10003640 f   HighFlexSettings.obj
 0001:000026c0       ??__EperfLog@U2@@YAXXZ     100036c0 f   HighFlexSettings.obj
 0001:00002740       ??__EscriptLog@U2@@YAXXZ   10003740 f   HighFlexSettings.obj
 0001:000027c0       ??__EtaskLog@U2@@YAXXZ     100037c0 f   HighFlexSettings.obj
 0001:00002840       ??__EuiLog@U2@@YAXXZ       10003840 f   HighFlexSettings.obj
 0001:000028c0       ??__EuserActLog@U2@@YAXXZ  100038c0 f   HighFlexSettings.obj
 0001:00002940       ??__E?_Generic_object@?$_Error_objects@H@std@@2V_Generic_error_category@2@A@@YAXXZ 10003940 f   moc_DNAFlexDialog.obj
 0001:00002950       ??__E?_Iostream_object@?$_Error_objects@H@std@@2V_Iostream_error_category@2@A@@YAXXZ 10003950 f   moc_DNAFlexDialog.obj
 0001:00002960       ??__E?_System_object@?$_Error_objects@H@std@@2V_System_error_category@2@A@@YAXXZ 10003960 f   moc_DNAFlexDialog.obj
 0001:00002970       ??__E?staticMetaObject@DNAFlexDialog@U2@@2UQMetaObject@@B@@YAXXZ 10003970 f   moc_DNAFlexDialog.obj
 0001:00002980       ??__E?_Generic_object@?$_Error_objects@H@std@@2V_Generic_error_category@2@A@@YAXXZ 10003980 f   moc_DNAFlexGraph.obj
 0001:00002990       ??__E?_Iostream_object@?$_Error_objects@H@std@@2V_Iostream_error_category@2@A@@YAXXZ 10003990 f   moc_DNAFlexGraph.obj
 0001:000029a0       ??__E?_System_object@?$_Error_objects@H@std@@2V_System_error_category@2@A@@YAXXZ 100039a0 f   moc_DNAFlexGraph.obj
 0001:000029b0       ??__E?staticMetaObject@DNAFlexGraphFactory@U2@@2UQMetaObject@@B@@YAXXZ 100039b0 f   moc_DNAFlexGraph.obj
 0001:000029c0       ??__EService_DNAExport@U2@@YAXXZ 100039c0 f   moc_DNAFlexGraph.obj
 0001:000029d0       ??__EService_DNAGraphPack@U2@@YAXXZ 100039d0 f   moc_DNAFlexGraph.obj
 0001:000029e0       ??__EService_ExternalToolSupport@U2@@YAXXZ 100039e0 f   moc_DNAFlexGraph.obj
 0001:000029f0       ??__EService_GUITesting@U2@@YAXXZ 100039f0 f   moc_DNAFlexGraph.obj
 0001:00002a00       ??__EService_MaxCoreServiceId@U2@@YAXXZ 10003a00 f   moc_DNAFlexGraph.obj
 0001:00002a10       ??__EService_MinCoreServiceId@U2@@YAXXZ 10003a10 f   moc_DNAFlexGraph.obj
 0001:00002a20       ??__EService_PluginViewer@U2@@YAXXZ 10003a20 f   moc_DNAFlexGraph.obj
 0001:00002a30       ??__EService_Project@U2@@YAXXZ 10003a30 f   moc_DNAFlexGraph.obj
 0001:00002a40       ??__EService_ProjectView@U2@@YAXXZ 10003a40 f   moc_DNAFlexGraph.obj
 0001:00002a50       ??__EService_QueryDesigner@U2@@YAXXZ 10003a50 f   moc_DNAFlexGraph.obj
 0001:00002a60       ??__EService_ScriptRegistry@U2@@YAXXZ 10003a60 f   moc_DNAFlexGraph.obj
 0001:00002a70       ??__EService_TestRunner@U2@@YAXXZ 10003a70 f   moc_DNAFlexGraph.obj
 0001:00002a80       ??__EService_WorkflowDesigner@U2@@YAXXZ 10003a80 f   moc_DNAFlexGraph.obj
 0001:00002a90       ??__EalgoLog@U2@@YAXXZ     10003a90 f   moc_DNAFlexGraph.obj
 0001:00002b10       ??__EcmdLog@U2@@YAXXZ      10003b10 f   moc_DNAFlexGraph.obj
 0001:00002b90       ??__EcoreLog@U2@@YAXXZ     10003b90 f   moc_DNAFlexGraph.obj
 0001:00002c10       ??__EioLog@U2@@YAXXZ       10003c10 f   moc_DNAFlexGraph.obj
 0001:00002c90       ??__EperfLog@U2@@YAXXZ     10003c90 f   moc_DNAFlexGraph.obj
 0001:00002d10       ??__EscriptLog@U2@@YAXXZ   10003d10 f   moc_DNAFlexGraph.obj
 0001:00002d90       ??__EtaskLog@U2@@YAXXZ     10003d90 f   moc_DNAFlexGraph.obj
 0001:00002e10       ??__EuiLog@U2@@YAXXZ       10003e10 f   moc_DNAFlexGraph.obj
 0001:00002e90       ??__EuserActLog@U2@@YAXXZ  10003e90 f   moc_DNAFlexGraph.obj
 0001:00002f10       ??__E?_Generic_object@?$_Error_objects@H@std@@2V_Generic_error_category@2@A@@YAXXZ 10003f10 f   moc_DNAFlexPlugin.obj
 0001:00002f20       ??__E?_Iostream_object@?$_Error_objects@H@std@@2V_Iostream_error_category@2@A@@YAXXZ 10003f20 f   moc_DNAFlexPlugin.obj
 0001:00002f30       ??__E?_System_object@?$_Error_objects@H@std@@2V_System_error_category@2@A@@YAXXZ 10003f30 f   moc_DNAFlexPlugin.obj
 0001:00002f40       ??__E?staticMetaObject@DNAFlexPlugin@U2@@2UQMetaObject@@B@@YAXXZ 10003f40 f   moc_DNAFlexPlugin.obj
 0001:00002f50       ??__E?staticMetaObject@DNAFlexViewContext@U2@@2UQMetaObject@@B@@YAXXZ 10003f50 f   moc_DNAFlexPlugin.obj
 0001:00002f60       ??__EService_DNAExport@U2@@YAXXZ 10003f60 f   moc_DNAFlexPlugin.obj
 0001:00002f70       ??__EService_DNAGraphPack@U2@@YAXXZ 10003f70 f   moc_DNAFlexPlugin.obj
 0001:00002f80       ??__EService_ExternalToolSupport@U2@@YAXXZ 10003f80 f   moc_DNAFlexPlugin.obj
 0001:00002f90       ??__EService_GUITesting@U2@@YAXXZ 10003f90 f   moc_DNAFlexPlugin.obj
 0001:00002fa0       ??__EService_MaxCoreServiceId@U2@@YAXXZ 10003fa0 f   moc_DNAFlexPlugin.obj
 0001:00002fb0       ??__EService_MinCoreServiceId@U2@@YAXXZ 10003fb0 f   moc_DNAFlexPlugin.obj
 0001:00002fc0       ??__EService_PluginViewer@U2@@YAXXZ 10003fc0 f   moc_DNAFlexPlugin.obj
 0001:00002fd0       ??__EService_Project@U2@@YAXXZ 10003fd0 f   moc_DNAFlexPlugin.obj
 0001:00002fe0       ??__EService_ProjectView@U2@@YAXXZ 10003fe0 f   moc_DNAFlexPlugin.obj
 0001:00002ff0       ??__EService_QueryDesigner@U2@@YAXXZ 10003ff0 f   moc_DNAFlexPlugin.obj
 0001:00003000       ??__EService_ScriptRegistry@U2@@YAXXZ 10004000 f   moc_DNAFlexPlugin.obj
 0001:00003010       ??__EService_TestRunner@U2@@YAXXZ 10004010 f   moc_DNAFlexPlugin.obj
 0001:00003020       ??__EService_WorkflowDesigner@U2@@YAXXZ 10004020 f   moc_DNAFlexPlugin.obj
 0001:00003030       ??__EalgoLog@U2@@YAXXZ     10004030 f   moc_DNAFlexPlugin.obj
 0001:000030b0       ??__EcmdLog@U2@@YAXXZ      100040b0 f   moc_DNAFlexPlugin.obj
 0001:00003130       ??__EcoreLog@U2@@YAXXZ     10004130 f   moc_DNAFlexPlugin.obj
 0001:000031b0       ??__EioLog@U2@@YAXXZ       100041b0 f   moc_DNAFlexPlugin.obj
 0001:00003230       ??__EperfLog@U2@@YAXXZ     10004230 f   moc_DNAFlexPlugin.obj
 0001:000032b0       ??__EscriptLog@U2@@YAXXZ   100042b0 f   moc_DNAFlexPlugin.obj
 0001:00003330       ??__EtaskLog@U2@@YAXXZ     10004330 f   moc_DNAFlexPlugin.obj
 0001:000033b0       ??__EuiLog@U2@@YAXXZ       100043b0 f   moc_DNAFlexPlugin.obj
 0001:00003430       ??__EuserActLog@U2@@YAXXZ  10004430 f   moc_DNAFlexPlugin.obj
 0001:000034b0       ??__E?_Generic_object@?$_Error_objects@H@std@@2V_Generic_error_category@2@A@@YAXXZ 100044b0 f   moc_DNAFlexTask.obj
 0001:000034c0       ??__E?_Iostream_object@?$_Error_objects@H@std@@2V_Iostream_error_category@2@A@@YAXXZ 100044c0 f   moc_DNAFlexTask.obj
 0001:000034d0       ??__E?_System_object@?$_Error_objects@H@std@@2V_System_error_category@2@A@@YAXXZ 100044d0 f   moc_DNAFlexTask.obj
 0001:000034e0       ??__E?staticMetaObject@DNAFlexTask@U2@@2UQMetaObject@@B@@YAXXZ 100044e0 f   moc_DNAFlexTask.obj
 0001:000034f0       ??__EalgoLog@U2@@YAXXZ     100044f0 f   moc_DNAFlexTask.obj
 0001:00003570       ??__EcmdLog@U2@@YAXXZ      10004570 f   moc_DNAFlexTask.obj
 0001:000035f0       ??__EcoreLog@U2@@YAXXZ     100045f0 f   moc_DNAFlexTask.obj
 0001:00003670       ??__EioLog@U2@@YAXXZ       10004670 f   moc_DNAFlexTask.obj
 0001:000036f0       ??__EperfLog@U2@@YAXXZ     100046f0 f   moc_DNAFlexTask.obj
 0001:00003770       ??__EscriptLog@U2@@YAXXZ   10004770 f   moc_DNAFlexTask.obj
 0001:000037f0       ??__EtaskLog@U2@@YAXXZ     100047f0 f   moc_DNAFlexTask.obj
 0001:00003870       ??__EuiLog@U2@@YAXXZ       10004870 f   moc_DNAFlexTask.obj
 0001:000038f0       ??__EuserActLog@U2@@YAXXZ  100048f0 f   moc_DNAFlexTask.obj
 0001:00003970       ??__E?_Generic_object@?$_Error_objects@H@std@@2V_Generic_error_category@2@A@@YAXXZ 10004970 f   moc_FindHighFlexRegions.obj
 0001:00003980       ??__E?_Iostream_object@?$_Error_objects@H@std@@2V_Iostream_error_category@2@A@@YAXXZ 10004980 f   moc_FindHighFlexRegions.obj
 0001:00003990       ??__E?_System_object@?$_Error_objects@H@std@@2V_System_error_category@2@A@@YAXXZ 10004990 f   moc_FindHighFlexRegions.obj
 0001:000039a0       ??__E?staticMetaObject@FindHighFlexRegions@U2@@2UQMetaObject@@B@@YAXXZ 100049a0 f   moc_FindHighFlexRegions.obj
 0001:000039b0       ??__EalgoLog@U2@@YAXXZ     100049b0 f   moc_FindHighFlexRegions.obj
 0001:00003a30       ??__EcmdLog@U2@@YAXXZ      10004a30 f   moc_FindHighFlexRegions.obj
 0001:00003ab0       ??__EcoreLog@U2@@YAXXZ     10004ab0 f   moc_FindHighFlexRegions.obj
 0001:00003b30       ??__EioLog@U2@@YAXXZ       10004b30 f   moc_FindHighFlexRegions.obj
 0001:00003bb0       ??__EperfLog@U2@@YAXXZ     10004bb0 f   moc_FindHighFlexRegions.obj
 0001:00003c30       ??__EscriptLog@U2@@YAXXZ   10004c30 f   moc_FindHighFlexRegions.obj
 0001:00003cb0       ??__EtaskLog@U2@@YAXXZ     10004cb0 f   moc_FindHighFlexRegions.obj
 0001:00003d30       ??__EuiLog@U2@@YAXXZ       10004d30 f   moc_FindHighFlexRegions.obj
 0001:00003db0       ??__EuserActLog@U2@@YAXXZ  10004db0 f   moc_FindHighFlexRegions.obj
 0001:00003e30       ??__Edummy@?A0xf1761197@@YAXXZ 10004e30 f   qrc_dna_flexibility.obj
 0001:000046a0       ??R<lambda_00118d359345adf794be5d433703ad4b>@@QBE?AVQString@@XZ 100056a0 f   DNAFlexDialog.obj
 0001:000046c0       ??R<lambda_17b0b2d6700668d280cd86f7b3fbe6a9>@@QBE?AVQString@@XZ 100056c0 f   DNAFlexDialog.obj
 0001:000046e0       ??R<lambda_1cfb2c5c4119324300889144faedee2e>@@QBE?AVQString@@XZ 100056e0 f   DNAFlexDialog.obj
 0001:00004700       ??R<lambda_1d1eaa33596ff48552c744a4378a660b>@@QBE?AVQString@@XZ 10005700 f   DNAFlexDialog.obj
 0001:00004720       ??R<lambda_2a848a472f6df9fe3550693bba86a84d>@@QBE?AVQString@@XZ 10005720 f   DNAFlexDialog.obj
 0001:00004740       ??R<lambda_458b0f23edea6d4478a012c5955cb606>@@QBE?AVQString@@XZ 10005740 f   DNAFlexDialog.obj
 0001:00004760       ??R<lambda_4717dcb402506f06d2b359e39d831609>@@QBE?AVQString@@XZ 10005760 f   DNAFlexDialog.obj
 0001:00004780       ??R<lambda_52ee9bd10a54360c0a60eb05b65cf928>@@QBE?AVQString@@XZ 10005780 f   DNAFlexDialog.obj
 0001:000047a0       ??R<lambda_57a051c781f8d8c95caf7ca077bc5f12>@@QBE?AVQString@@XZ 100057a0 f   DNAFlexDialog.obj
 0001:000047c0       ??R<lambda_5c6a044f2f458955f0d06defa39d488f>@@QBE?AVQString@@XZ 100057c0 f   DNAFlexDialog.obj
 0001:000047e0       ??R<lambda_60c36b2ba8f6ac249075d3447a06946a>@@QBE?AVQString@@XZ 100057e0 f   DNAFlexDialog.obj
 0001:00004800       ??R<lambda_707fe8b4ae45d9fe5ca46cd514e2687d>@@QBE?AVQString@@XZ 10005800 f   DNAFlexDialog.obj
 0001:00004820       ??R<lambda_7151c4947fd3098b290b8908712616f2>@@QBE?AVQString@@XZ 10005820 f   DNAFlexDialog.obj
 0001:00004840       ??R<lambda_821a87b4b859d3d71973b8c7c9ac2d25>@@QBE?AVQString@@XZ 10005840 f   DNAFlexDialog.obj
 0001:00004860       ??R<lambda_8dadecbf2ac41c19a976dc614914c4ce>@@QBE?AVQString@@XZ 10005860 f   DNAFlexDialog.obj
 0001:00004880       ??R<lambda_99cbfa8a2e2a089352d749da904ef1d2>@@QBE?AVQString@@XZ 10005880 f   DNAFlexDialog.obj
 0001:000048a0       ??R<lambda_c54a255dbb70683bcc9e7ac18dc46ed1>@@QBE?AVQString@@XZ 100058a0 f   DNAFlexDialog.obj
 0001:000048c0       ??R<lambda_eda4e94934f57365d954060c5e0ec9a8>@@QBE?AVQString@@XZ 100058c0 f   DNAFlexDialog.obj
 0001:000048e0       ??R<lambda_f5440838e2e94d9a157f8927169bbc41>@@QBE?AVQString@@XZ 100058e0 f   DNAFlexDialog.obj
 0001:00004e76       __catch$?_Copy@?$basic_string@DU?$char_traits@D@std@@V?$allocator@D@2@@std@@QAEXII@Z$0 10005e76 f i DNAFlexDialog.obj
 0001:00004eb3       __catch$?_Copy@?$basic_string@DU?$char_traits@D@std@@V?$allocator@D@2@@std@@QAEXII@Z$1 10005eb3 f i DNAFlexDialog.obj
 0001:0000730f       __catch$?append@?$QList@V?$QSharedPointer@VGSequenceGraphData@U2@@@@@@QAEXABV?$QSharedPointer@VGSequenceGraphData@U2@@@@@Z$2 1000830f f i DNAFlexGraph.obj
 0001:0000730f       __catch$?append@?$QList@V?$QSharedPointer@VGSequenceGraphData@U2@@@@@@QAEXABV?$QSharedPointer@VGSequenceGraphData@U2@@@@@Z$0 1000830f f i DNAFlexGraph.obj
 0001:0000773c       __catch$?detach_helper_grow@?$QList@V?$QSharedPointer@VGSequenceGraphData@U2@@@@@@AAEPAUNode@1@HH@Z$2 1000873c f i DNAFlexGraph.obj
 0001:00007777       __catch$?detach_helper_grow@?$QList@V?$QSharedPointer@VGSequenceGraphData@U2@@@@@@AAEPAUNode@1@HH@Z$0 10008777 f i DNAFlexGraph.obj
 0001:00007950       ?nameByType@U2@@YA?AVQString@@XZ 10008950 f   DNAFlexGraph.obj
 0001:00007a6e       __catch$?node_copy@?$QList@V?$QSharedPointer@VGSequenceGraphData@U2@@@@@@AAEXPAUNode@1@00@Z$0 10008a6e f i DNAFlexGraph.obj
 0001:00007e74       __catch$?calculate@DNAFlexGraphAlgorithm@U2@@UAEXAAV?$QVector@M@@PAVU2SequenceObject@2@ABVU2Region@2@PBVGSequenceGraphWindowData@2@AAVU2OpStatus@2@@Z$0 10008e74 f   DNAFlexGraphAlgorithm.obj
 0001:00007eba       __catch$?calculate@DNAFlexGraphAlgorithm@U2@@UAEXAAV?$QVector@M@@PAVU2SequenceObject@2@ABVU2Region@2@PBVGSequenceGraphWindowData@2@AAVU2OpStatus@2@@Z$1 10008eba f   DNAFlexGraphAlgorithm.obj
 0001:00008224       __catch$?reallocData@?$QVector@M@@AAEXHHV?$QFlags@W4AllocationOption@QArrayData@@@@@Z$0 10009224 f i DNAFlexGraphAlgorithm.obj
 0001:00008236       __catch$?reallocData@?$QVector@M@@AAEXHHV?$QFlags@W4AllocationOption@QArrayData@@@@@Z$2 10009236 f i DNAFlexGraphAlgorithm.obj
 0001:000084de       __catch$??0?$QList@PAVADVSequenceWidget@U2@@@@QAE@ABV0@@Z$0 100094de f i DNAFlexPlugin.obj
 0001:000094ee       __catch$??0?$QList@VHighFlexResult@U2@@@@QAE@ABV0@@Z$0 1000a4ee f i DNAFlexTask.obj
 0001:00009b25       __catch$?append@?$QList@PAVTask@U2@@@@QAEXABQAVTask@U2@@@Z$4 1000ab25 f i DNAFlexTask.obj
 0001:00009be2       __catch$?append@?$QList@V?$QSharedDataPointer@VAnnotationData@U2@@@@@@QAEXABV?$QSharedDataPointer@VAnnotationData@U2@@@@@Z$4 1000abe2 f i DNAFlexTask.obj
 0001:0000a071       __catch$?detach_helper_grow@?$QList@PAVTask@U2@@@@AAEPAUNode@1@HH@Z$2 1000b071 f i DNAFlexTask.obj
 0001:0000a071       __catch$?detach_helper_grow@?$QList@PAVTask@U2@@@@AAEPAUNode@1@HH@Z$0 1000b071 f i DNAFlexTask.obj
 0001:0000a19c       __catch$?detach_helper_grow@?$QList@V?$QSharedDataPointer@VAnnotationData@U2@@@@@@AAEPAUNode@1@HH@Z$2 1000b19c f i DNAFlexTask.obj
 0001:0000a1d7       __catch$?detach_helper_grow@?$QList@V?$QSharedDataPointer@VAnnotationData@U2@@@@@@AAEPAUNode@1@HH@Z$0 1000b1d7 f i DNAFlexTask.obj
 0001:0000aa74       __catch$?node_copy@?$QList@VHighFlexResult@U2@@@@AAEXPAUNode@1@00@Z$0 1000ba74 f i DNAFlexTask.obj
 0001:0000b08b       __catch$?reallocData@?$QVector@VU2Qualifier@U2@@@@AAEXHHV?$QFlags@W4AllocationOption@QArrayData@@@@@Z$0 1000c08b f i DNAFlexTask.obj
 0001:0000b0a9       __catch$?reallocData@?$QVector@VU2Qualifier@U2@@@@AAEXHHV?$QFlags@W4AllocationOption@QArrayData@@@@@Z$2 1000c0a9 f i DNAFlexTask.obj
 0001:0000b2b5       __catch$?reallocData@?$QVector@VU2Region@U2@@@@AAEXHHV?$QFlags@W4AllocationOption@QArrayData@@@@@Z$0 1000c2b5 f i DNAFlexTask.obj
 0001:0000b2c7       __catch$?reallocData@?$QVector@VU2Region@U2@@@@AAEXHHV?$QFlags@W4AllocationOption@QArrayData@@@@@Z$2 1000c2c7 f i DNAFlexTask.obj
 0001:0000b640       __catch$?append@?$QList@VHighFlexResult@U2@@@@QAEXABVHighFlexResult@U2@@@Z$0 1000c640 f i FindHighFlexRegions.obj
 0001:0000b640       __catch$?append@?$QList@VHighFlexResult@U2@@@@QAEXABVHighFlexResult@U2@@@Z$2 1000c640 f i FindHighFlexRegions.obj
 0001:0000b7d1       __catch$?detach_helper_grow@?$QList@VHighFlexResult@U2@@@@AAEPAUNode@1@HH@Z$2 1000c7d1 f i FindHighFlexRegions.obj
 0001:0000b80c       __catch$?detach_helper_grow@?$QList@VHighFlexResult@U2@@@@AAEPAUNode@1@HH@Z$0 1000c80c f i FindHighFlexRegions.obj
 0001:0000cb0c       $LN16                      1000db0c     moc_DNAFlexDialog.obj
 0001:0000e006       _pre_c_init                1000f006 f   MSVCRT:crtdll.obj
 0001:0000e273       ___DllMainCRTStartup       1000f273 f   MSVCRT:crtdll.obj
 0001:0000e3c0       $$000000                   1000f3c0     MSVCRT:sehprolg4.obj
 0001:0000e7d5       ?ArrayUnwindFilter@@YAHPAU_EXCEPTION_POINTERS@@@Z 1000f7d5 f   MSVCRT:ehvecdtr.obj
 0001:0000eb20       __unwindfunclet$??0DNAFlexDialog@U2@@QAE@PAVADVSequenceObjectContext@1@@Z$0 1000fb20 f   DNAFlexDialog.obj
 0001:0000eb29       __unwindfunclet$??0DNAFlexDialog@U2@@QAE@PAVADVSequenceObjectContext@1@@Z$1 1000fb29 f   DNAFlexDialog.obj
 0001:0000eb34       __unwindfunclet$??0DNAFlexDialog@U2@@QAE@PAVADVSequenceObjectContext@1@@Z$2 1000fb34 f   DNAFlexDialog.obj
 0001:0000eb4e       __unwindfunclet$??0DNAFlexDialog@U2@@QAE@PAVADVSequenceObjectContext@1@@Z$3 1000fb4e f   DNAFlexDialog.obj
 0001:0000eb57       __unwindfunclet$??0DNAFlexDialog@U2@@QAE@PAVADVSequenceObjectContext@1@@Z$4 1000fb57 f   DNAFlexDialog.obj
 0001:0000eb60       __unwindfunclet$??0DNAFlexDialog@U2@@QAE@PAVADVSequenceObjectContext@1@@Z$5 1000fb60 f   DNAFlexDialog.obj
 0001:0000eb6c       __unwindfunclet$??0DNAFlexDialog@U2@@QAE@PAVADVSequenceObjectContext@1@@Z$6 1000fb6c f   DNAFlexDialog.obj
 0001:0000eb78       __unwindfunclet$??0DNAFlexDialog@U2@@QAE@PAVADVSequenceObjectContext@1@@Z$7 1000fb78 f   DNAFlexDialog.obj
 0001:0000eb83       __unwindfunclet$??0DNAFlexDialog@U2@@QAE@PAVADVSequenceObjectContext@1@@Z$8 1000fb83 f   DNAFlexDialog.obj
 0001:0000eb8c       __unwindfunclet$??0DNAFlexDialog@U2@@QAE@PAVADVSequenceObjectContext@1@@Z$9 1000fb8c f   DNAFlexDialog.obj
 0001:0000eb95       __ehhandler$??0DNAFlexDialog@U2@@QAE@PAVADVSequenceObjectContext@1@@Z 1000fb95 f   DNAFlexDialog.obj
 0001:0000ebc0       __unwindfunclet$??__EalgoLog@U2@@YAXXZ$0 1000fbc0 f   DNAFlexDialog.obj
 0001:0000ebc9       __ehhandler$??__EalgoLog@U2@@YAXXZ 1000fbc9 f   DNAFlexDialog.obj
 0001:0000ebf0       __unwindfunclet$??__EcmdLog@U2@@YAXXZ$0 1000fbf0 f   DNAFlexDialog.obj
 0001:0000ebf9       __ehhandler$??__EcmdLog@U2@@YAXXZ 1000fbf9 f   DNAFlexDialog.obj
 0001:0000ec20       __unwindfunclet$??__EcoreLog@U2@@YAXXZ$0 1000fc20 f   DNAFlexDialog.obj
 0001:0000ec29       __ehhandler$??__EcoreLog@U2@@YAXXZ 1000fc29 f   DNAFlexDialog.obj
 0001:0000ec50       __unwindfunclet$??__EioLog@U2@@YAXXZ$0 1000fc50 f   DNAFlexDialog.obj
 0001:0000ec59       __ehhandler$??__EioLog@U2@@YAXXZ 1000fc59 f   DNAFlexDialog.obj
 0001:0000ec80       __unwindfunclet$??__EperfLog@U2@@YAXXZ$0 1000fc80 f   DNAFlexDialog.obj
 0001:0000ec89       __ehhandler$??__EperfLog@U2@@YAXXZ 1000fc89 f   DNAFlexDialog.obj
 0001:0000ecb0       __unwindfunclet$??__EscriptLog@U2@@YAXXZ$0 1000fcb0 f   DNAFlexDialog.obj
 0001:0000ecb9       __ehhandler$??__EscriptLog@U2@@YAXXZ 1000fcb9 f   DNAFlexDialog.obj
 0001:0000ece0       __unwindfunclet$??__EtaskLog@U2@@YAXXZ$0 1000fce0 f   DNAFlexDialog.obj
 0001:0000ece9       __ehhandler$??__EtaskLog@U2@@YAXXZ 1000fce9 f   DNAFlexDialog.obj
 0001:0000ed10       __unwindfunclet$??__EuiLog@U2@@YAXXZ$0 1000fd10 f   DNAFlexDialog.obj
 0001:0000ed19       __ehhandler$??__EuiLog@U2@@YAXXZ 1000fd19 f   DNAFlexDialog.obj
 0001:0000ed40       __unwindfunclet$??__EuserActLog@U2@@YAXXZ$0 1000fd40 f   DNAFlexDialog.obj
 0001:0000ed49       __ehhandler$??__EuserActLog@U2@@YAXXZ 1000fd49 f   DNAFlexDialog.obj
 0001:0000ed70       __ehhandler$?_Copy@?$basic_string@DU?$char_traits@D@std@@V?$allocator@D@2@@std@@QAEXII@Z 1000fd70 f   DNAFlexDialog.obj
 0001:0000ed90       __unwindfunclet$?accept@DNAFlexDialog@U2@@UAEXXZ$0 1000fd90 f   DNAFlexDialog.obj
 0001:0000ed99       __unwindfunclet$?accept@DNAFlexDialog@U2@@UAEXXZ$1 1000fd99 f   DNAFlexDialog.obj
 0001:0000eda2       __unwindfunclet$?accept@DNAFlexDialog@U2@@UAEXXZ$2 1000fda2 f   DNAFlexDialog.obj
 0001:0000edab       __unwindfunclet$?accept@DNAFlexDialog@U2@@UAEXXZ$3 1000fdab f   DNAFlexDialog.obj
 0001:0000edb4       __unwindfunclet$?accept@DNAFlexDialog@U2@@UAEXXZ$4 1000fdb4 f   DNAFlexDialog.obj
 0001:0000edbd       __unwindfunclet$?accept@DNAFlexDialog@U2@@UAEXXZ$5 1000fdbd f   DNAFlexDialog.obj
 0001:0000edc6       __unwindfunclet$?accept@DNAFlexDialog@U2@@UAEXXZ$7 1000fdc6 f   DNAFlexDialog.obj
 0001:0000edcf       __unwindfunclet$?accept@DNAFlexDialog@U2@@UAEXXZ$8 1000fdcf f   DNAFlexDialog.obj
 0001:0000edd8       __unwindfunclet$?accept@DNAFlexDialog@U2@@UAEXXZ$9 1000fdd8 f   DNAFlexDialog.obj
 0001:0000ede1       __unwindfunclet$?accept@DNAFlexDialog@U2@@UAEXXZ$10 1000fde1 f   DNAFlexDialog.obj
 0001:0000edea       __unwindfunclet$?accept@DNAFlexDialog@U2@@UAEXXZ$11 1000fdea f   DNAFlexDialog.obj
 0001:0000edf5       __unwindfunclet$?accept@DNAFlexDialog@U2@@UAEXXZ$12 1000fdf5 f   DNAFlexDialog.obj
 0001:0000ee0f       __ehhandler$?accept@DNAFlexDialog@U2@@UAEXXZ 1000fe0f f   DNAFlexDialog.obj
 0001:0000ee30       __unwindfunclet$?clone@?$QSharedDataPointer@VAnnotationData@U2@@@@IAEPAVAnnotationData@U2@@XZ$0 1000fe30 f   DNAFlexDialog.obj
 0001:0000ee3b       __ehhandler$?clone@?$QSharedDataPointer@VAnnotationData@U2@@@@IAEPAVAnnotationData@U2@@XZ 1000fe3b f   DNAFlexDialog.obj
 0001:0000ee60       __unwindfunclet$?detach_helper@?$QSharedDataPointer@VAnnotationData@U2@@@@AAEXXZ$0 1000fe60 f   DNAFlexDialog.obj
 0001:0000ee6b       __ehhandler$?detach_helper@?$QSharedDataPointer@VAnnotationData@U2@@@@AAEXXZ 1000fe6b f   DNAFlexDialog.obj
 0001:0000ee90       __unwindfunclet$?retranslateUi@Ui_DNAFlexDialog@@QAEXPAVQDialog@@@Z$0 1000fe90 f   DNAFlexDialog.obj
 0001:0000ee99       __unwindfunclet$?retranslateUi@Ui_DNAFlexDialog@@QAEXPAVQDialog@@@Z$1 1000fe99 f   DNAFlexDialog.obj
 0001:0000eea2       __unwindfunclet$?retranslateUi@Ui_DNAFlexDialog@@QAEXPAVQDialog@@@Z$2 1000fea2 f   DNAFlexDialog.obj
 0001:0000eeab       __unwindfunclet$?retranslateUi@Ui_DNAFlexDialog@@QAEXPAVQDialog@@@Z$3 1000feab f   DNAFlexDialog.obj
 0001:0000eeb4       __unwindfunclet$?retranslateUi@Ui_DNAFlexDialog@@QAEXPAVQDialog@@@Z$4 1000feb4 f   DNAFlexDialog.obj
 0001:0000eebd       __unwindfunclet$?retranslateUi@Ui_DNAFlexDialog@@QAEXPAVQDialog@@@Z$5 1000febd f   DNAFlexDialog.obj
 0001:0000eec6       __unwindfunclet$?retranslateUi@Ui_DNAFlexDialog@@QAEXPAVQDialog@@@Z$6 1000fec6 f   DNAFlexDialog.obj
 0001:0000eecf       __unwindfunclet$?retranslateUi@Ui_DNAFlexDialog@@QAEXPAVQDialog@@@Z$7 1000fecf f   DNAFlexDialog.obj
 0001:0000eed8       __unwindfunclet$?retranslateUi@Ui_DNAFlexDialog@@QAEXPAVQDialog@@@Z$8 1000fed8 f   DNAFlexDialog.obj
 0001:0000eee1       __unwindfunclet$?retranslateUi@Ui_DNAFlexDialog@@QAEXPAVQDialog@@@Z$9 1000fee1 f   DNAFlexDialog.obj
 0001:0000eeea       __unwindfunclet$?retranslateUi@Ui_DNAFlexDialog@@QAEXPAVQDialog@@@Z$10 1000feea f   DNAFlexDialog.obj
 0001:0000eef3       __ehhandler$?retranslateUi@Ui_DNAFlexDialog@@QAEXPAVQDialog@@@Z 1000fef3 f   DNAFlexDialog.obj
 0001:0000ef10       __unwindfunclet$?setupUi@Ui_DNAFlexDialog@@QAEXPAVQDialog@@@Z$1 1000ff10 f   DNAFlexDialog.obj
 0001:0000ef19       __unwindfunclet$?setupUi@Ui_DNAFlexDialog@@QAEXPAVQDialog@@@Z$2 1000ff19 f   DNAFlexDialog.obj
 0001:0000ef24       __unwindfunclet$?setupUi@Ui_DNAFlexDialog@@QAEXPAVQDialog@@@Z$3 1000ff24 f   DNAFlexDialog.obj
 0001:0000ef2d       __unwindfunclet$?setupUi@Ui_DNAFlexDialog@@QAEXPAVQDialog@@@Z$4 1000ff2d f   DNAFlexDialog.obj
 0001:0000ef38       __unwindfunclet$?setupUi@Ui_DNAFlexDialog@@QAEXPAVQDialog@@@Z$5 1000ff38 f   DNAFlexDialog.obj
 0001:0000ef41       __unwindfunclet$?setupUi@Ui_DNAFlexDialog@@QAEXPAVQDialog@@@Z$6 1000ff41 f   DNAFlexDialog.obj
 0001:0000ef4c       __unwindfunclet$?setupUi@Ui_DNAFlexDialog@@QAEXPAVQDialog@@@Z$7 1000ff4c f   DNAFlexDialog.obj
 0001:0000ef55       __unwindfunclet$?setupUi@Ui_DNAFlexDialog@@QAEXPAVQDialog@@@Z$8 1000ff55 f   DNAFlexDialog.obj
 0001:0000ef60       __unwindfunclet$?setupUi@Ui_DNAFlexDialog@@QAEXPAVQDialog@@@Z$9 1000ff60 f   DNAFlexDialog.obj
 0001:0000ef69       __unwindfunclet$?setupUi@Ui_DNAFlexDialog@@QAEXPAVQDialog@@@Z$10 1000ff69 f   DNAFlexDialog.obj
 0001:0000ef74       __unwindfunclet$?setupUi@Ui_DNAFlexDialog@@QAEXPAVQDialog@@@Z$11 1000ff74 f   DNAFlexDialog.obj
 0001:0000ef7d       __unwindfunclet$?setupUi@Ui_DNAFlexDialog@@QAEXPAVQDialog@@@Z$12 1000ff7d f   DNAFlexDialog.obj
 0001:0000ef88       __unwindfunclet$?setupUi@Ui_DNAFlexDialog@@QAEXPAVQDialog@@@Z$13 1000ff88 f   DNAFlexDialog.obj
 0001:0000ef91       __unwindfunclet$?setupUi@Ui_DNAFlexDialog@@QAEXPAVQDialog@@@Z$14 1000ff91 f   DNAFlexDialog.obj
 0001:0000ef9c       __unwindfunclet$?setupUi@Ui_DNAFlexDialog@@QAEXPAVQDialog@@@Z$15 1000ff9c f   DNAFlexDialog.obj
 0001:0000efa5       __unwindfunclet$?setupUi@Ui_DNAFlexDialog@@QAEXPAVQDialog@@@Z$16 1000ffa5 f   DNAFlexDialog.obj
 0001:0000efb0       __unwindfunclet$?setupUi@Ui_DNAFlexDialog@@QAEXPAVQDialog@@@Z$17 1000ffb0 f   DNAFlexDialog.obj
 0001:0000efb9       __unwindfunclet$?setupUi@Ui_DNAFlexDialog@@QAEXPAVQDialog@@@Z$18 1000ffb9 f   DNAFlexDialog.obj
 0001:0000efc4       __unwindfunclet$?setupUi@Ui_DNAFlexDialog@@QAEXPAVQDialog@@@Z$19 1000ffc4 f   DNAFlexDialog.obj
 0001:0000efcd       __unwindfunclet$?setupUi@Ui_DNAFlexDialog@@QAEXPAVQDialog@@@Z$20 1000ffcd f   DNAFlexDialog.obj
 0001:0000efd8       __unwindfunclet$?setupUi@Ui_DNAFlexDialog@@QAEXPAVQDialog@@@Z$21 1000ffd8 f   DNAFlexDialog.obj
 0001:0000efe1       __unwindfunclet$?setupUi@Ui_DNAFlexDialog@@QAEXPAVQDialog@@@Z$22 1000ffe1 f   DNAFlexDialog.obj
 0001:0000efec       __unwindfunclet$?setupUi@Ui_DNAFlexDialog@@QAEXPAVQDialog@@@Z$23 1000ffec f   DNAFlexDialog.obj
 0001:0000eff5       __unwindfunclet$?setupUi@Ui_DNAFlexDialog@@QAEXPAVQDialog@@@Z$24 1000fff5 f   DNAFlexDialog.obj
 0001:0000f000       __unwindfunclet$?setupUi@Ui_DNAFlexDialog@@QAEXPAVQDialog@@@Z$25 10010000 f   DNAFlexDialog.obj
 0001:0000f009       __unwindfunclet$?setupUi@Ui_DNAFlexDialog@@QAEXPAVQDialog@@@Z$26 10010009 f   DNAFlexDialog.obj
 0001:0000f014       __unwindfunclet$?setupUi@Ui_DNAFlexDialog@@QAEXPAVQDialog@@@Z$27 10010014 f   DNAFlexDialog.obj
 0001:0000f01d       __unwindfunclet$?setupUi@Ui_DNAFlexDialog@@QAEXPAVQDialog@@@Z$28 1001001d f   DNAFlexDialog.obj
 0001:0000f028       __unwindfunclet$?setupUi@Ui_DNAFlexDialog@@QAEXPAVQDialog@@@Z$29 10010028 f   DNAFlexDialog.obj
 0001:0000f031       __unwindfunclet$?setupUi@Ui_DNAFlexDialog@@QAEXPAVQDialog@@@Z$30 10010031 f   DNAFlexDialog.obj
 0001:0000f03c       __unwindfunclet$?setupUi@Ui_DNAFlexDialog@@QAEXPAVQDialog@@@Z$31 1001003c f   DNAFlexDialog.obj
 0001:0000f045       __unwindfunclet$?setupUi@Ui_DNAFlexDialog@@QAEXPAVQDialog@@@Z$32 10010045 f   DNAFlexDialog.obj
 0001:0000f04e       __unwindfunclet$?setupUi@Ui_DNAFlexDialog@@QAEXPAVQDialog@@@Z$33 1001004e f   DNAFlexDialog.obj
 0001:0000f059       __unwindfunclet$?setupUi@Ui_DNAFlexDialog@@QAEXPAVQDialog@@@Z$34 10010059 f   DNAFlexDialog.obj
 0001:0000f062       __unwindfunclet$?setupUi@Ui_DNAFlexDialog@@QAEXPAVQDialog@@@Z$35 10010062 f   DNAFlexDialog.obj
 0001:0000f06d       __unwindfunclet$?setupUi@Ui_DNAFlexDialog@@QAEXPAVQDialog@@@Z$36 1001006d f   DNAFlexDialog.obj
 0001:0000f076       __unwindfunclet$?setupUi@Ui_DNAFlexDialog@@QAEXPAVQDialog@@@Z$37 10010076 f   DNAFlexDialog.obj
 0001:0000f07f       __unwindfunclet$?setupUi@Ui_DNAFlexDialog@@QAEXPAVQDialog@@@Z$38 1001007f f   DNAFlexDialog.obj
 0001:0000f08a       __unwindfunclet$?setupUi@Ui_DNAFlexDialog@@QAEXPAVQDialog@@@Z$39 1001008a f   DNAFlexDialog.obj
 0001:0000f095       __unwindfunclet$?setupUi@Ui_DNAFlexDialog@@QAEXPAVQDialog@@@Z$40 10010095 f   DNAFlexDialog.obj
 0001:0000f09e       __ehhandler$?setupUi@Ui_DNAFlexDialog@@QAEXPAVQDialog@@@Z 1001009e f   DNAFlexDialog.obj
 0001:0000f0c0       __unwindfunclet$??0DNAFlexGraphFactory@U2@@QAE@PAVQObject@@@Z$0 100100c0 f   DNAFlexGraph.obj
 0001:0000f0c9       __unwindfunclet$??0DNAFlexGraphFactory@U2@@QAE@PAVQObject@@@Z$1 100100c9 f   DNAFlexGraph.obj
 0001:0000f0d2       __ehhandler$??0DNAFlexGraphFactory@U2@@QAE@PAVQObject@@@Z 100100d2 f   DNAFlexGraph.obj
 0001:0000f0f0       __unwindfunclet$??__EalgoLog@U2@@YAXXZ$0 100100f0 f   DNAFlexGraph.obj
 0001:0000f0f9       __ehhandler$??__EalgoLog@U2@@YAXXZ 100100f9 f   DNAFlexGraph.obj
 0001:0000f120       __unwindfunclet$??__EcmdLog@U2@@YAXXZ$0 10010120 f   DNAFlexGraph.obj
 0001:0000f129       __ehhandler$??__EcmdLog@U2@@YAXXZ 10010129 f   DNAFlexGraph.obj
 0001:0000f150       __unwindfunclet$??__EcoreLog@U2@@YAXXZ$0 10010150 f   DNAFlexGraph.obj
 0001:0000f159       __ehhandler$??__EcoreLog@U2@@YAXXZ 10010159 f   DNAFlexGraph.obj
 0001:0000f180       __unwindfunclet$??__EioLog@U2@@YAXXZ$0 10010180 f   DNAFlexGraph.obj
 0001:0000f189       __ehhandler$??__EioLog@U2@@YAXXZ 10010189 f   DNAFlexGraph.obj
 0001:0000f1b0       __unwindfunclet$??__EperfLog@U2@@YAXXZ$0 100101b0 f   DNAFlexGraph.obj
 0001:0000f1b9       __ehhandler$??__EperfLog@U2@@YAXXZ 100101b9 f   DNAFlexGraph.obj
 0001:0000f1e0       __unwindfunclet$??__EscriptLog@U2@@YAXXZ$0 100101e0 f   DNAFlexGraph.obj
 0001:0000f1e9       __ehhandler$??__EscriptLog@U2@@YAXXZ 100101e9 f   DNAFlexGraph.obj
 0001:0000f210       __unwindfunclet$??__EtaskLog@U2@@YAXXZ$0 10010210 f   DNAFlexGraph.obj
 0001:0000f219       __ehhandler$??__EtaskLog@U2@@YAXXZ 10010219 f   DNAFlexGraph.obj
 0001:0000f240       __unwindfunclet$??__EuiLog@U2@@YAXXZ$0 10010240 f   DNAFlexGraph.obj
 0001:0000f249       __ehhandler$??__EuiLog@U2@@YAXXZ 10010249 f   DNAFlexGraph.obj
 0001:0000f270       __unwindfunclet$??__EuserActLog@U2@@YAXXZ$0 10010270 f   DNAFlexGraph.obj
 0001:0000f279       __ehhandler$??__EuserActLog@U2@@YAXXZ 10010279 f   DNAFlexGraph.obj
 0001:0000f2a0       __ehhandler$?append@?$QList@V?$QSharedPointer@VGSequenceGraphData@U2@@@@@@QAEXABV?$QSharedPointer@VGSequenceGraphData@U2@@@@@Z 100102a0 f   DNAFlexGraph.obj
 0001:0000f2c0       __unwindfunclet$?createGraphs@DNAFlexGraphFactory@U2@@UAE?AV?$QList@V?$QSharedPointer@VGSequenceGraphData@U2@@@@@@PAVGSequenceGraphView@2@@Z$0 100102c0 f   DNAFlexGraph.obj
 0001:0000f2d9       __unwindfunclet$?createGraphs@DNAFlexGraphFactory@U2@@UAE?AV?$QList@V?$QSharedPointer@VGSequenceGraphData@U2@@@@@@PAVGSequenceGraphView@2@@Z$1 100102d9 f   DNAFlexGraph.obj
 0001:0000f2e4       __unwindfunclet$?createGraphs@DNAFlexGraphFactory@U2@@UAE?AV?$QList@V?$QSharedPointer@VGSequenceGraphData@U2@@@@@@PAVGSequenceGraphView@2@@Z$2 100102e4 f   DNAFlexGraph.obj
 0001:0000f2ec       __unwindfunclet$?createGraphs@DNAFlexGraphFactory@U2@@UAE?AV?$QList@V?$QSharedPointer@VGSequenceGraphData@U2@@@@@@PAVGSequenceGraphView@2@@Z$3 100102ec f   DNAFlexGraph.obj
 0001:0000f2f7       __ehhandler$?createGraphs@DNAFlexGraphFactory@U2@@UAE?AV?$QList@V?$QSharedPointer@VGSequenceGraphData@U2@@@@@@PAVGSequenceGraphView@2@@Z 100102f7 f   DNAFlexGraph.obj
 0001:0000f320       __ehhandler$?detach_helper_grow@?$QList@V?$QSharedPointer@VGSequenceGraphData@U2@@@@@@AAEPAUNode@1@HH@Z 10010320 f   DNAFlexGraph.obj
 0001:0000f340       __unwindfunclet$?getDrawer@DNAFlexGraphFactory@U2@@UAEPAVGSequenceGraphDrawer@2@PAVGSequenceGraphView@2@@Z$0 10010340 f   DNAFlexGraph.obj
 0001:0000f349       __unwindfunclet$?getDrawer@DNAFlexGraphFactory@U2@@UAEPAVGSequenceGraphDrawer@2@PAVGSequenceGraphView@2@@Z$1 10010349 f   DNAFlexGraph.obj
 0001:0000f354       __ehhandler$?getDrawer@DNAFlexGraphFactory@U2@@UAEPAVGSequenceGraphDrawer@2@PAVGSequenceGraphView@2@@Z 10010354 f   DNAFlexGraph.obj
 0001:0000f370       __unwindfunclet$?isEnabled@DNAFlexGraphFactory@U2@@UBE_NPBVU2SequenceObject@2@@Z$0 10010370 f   DNAFlexGraph.obj
 0001:0000f379       __ehhandler$?isEnabled@DNAFlexGraphFactory@U2@@UBE_NPBVU2SequenceObject@2@@Z 10010379 f   DNAFlexGraph.obj
 0001:0000f3a0       __ehhandler$?node_copy@?$QList@V?$QSharedPointer@VGSequenceGraphData@U2@@@@@@AAEXPAUNode@1@00@Z 100103a0 f   DNAFlexGraph.obj
 0001:0000f3c0       __unwindfunclet$??__EalgoLog@U2@@YAXXZ$0 100103c0 f   DNAFlexGraphAlgorithm.obj
 0001:0000f3c9       __ehhandler$??__EalgoLog@U2@@YAXXZ 100103c9 f   DNAFlexGraphAlgorithm.obj
 0001:0000f3f0       __unwindfunclet$??__EcmdLog@U2@@YAXXZ$0 100103f0 f   DNAFlexGraphAlgorithm.obj
 0001:0000f3f9       __ehhandler$??__EcmdLog@U2@@YAXXZ 100103f9 f   DNAFlexGraphAlgorithm.obj
 0001:0000f420       __unwindfunclet$??__EcoreLog@U2@@YAXXZ$0 10010420 f   DNAFlexGraphAlgorithm.obj
 0001:0000f429       __ehhandler$??__EcoreLog@U2@@YAXXZ 10010429 f   DNAFlexGraphAlgorithm.obj
 0001:0000f450       __unwindfunclet$??__EioLog@U2@@YAXXZ$0 10010450 f   DNAFlexGraphAlgorithm.obj
 0001:0000f459       __ehhandler$??__EioLog@U2@@YAXXZ 10010459 f   DNAFlexGraphAlgorithm.obj
 0001:0000f480       __unwindfunclet$??__EperfLog@U2@@YAXXZ$0 10010480 f   DNAFlexGraphAlgorithm.obj
 0001:0000f489       __ehhandler$??__EperfLog@U2@@YAXXZ 10010489 f   DNAFlexGraphAlgorithm.obj
 0001:0000f4b0       __unwindfunclet$??__EscriptLog@U2@@YAXXZ$0 100104b0 f   DNAFlexGraphAlgorithm.obj
 0001:0000f4b9       __ehhandler$??__EscriptLog@U2@@YAXXZ 100104b9 f   DNAFlexGraphAlgorithm.obj
 0001:0000f4e0       __unwindfunclet$??__EtaskLog@U2@@YAXXZ$0 100104e0 f   DNAFlexGraphAlgorithm.obj
 0001:0000f4e9       __ehhandler$??__EtaskLog@U2@@YAXXZ 100104e9 f   DNAFlexGraphAlgorithm.obj
 0001:0000f510       __unwindfunclet$??__EuiLog@U2@@YAXXZ$0 10010510 f   DNAFlexGraphAlgorithm.obj
 0001:0000f519       __ehhandler$??__EuiLog@U2@@YAXXZ 10010519 f   DNAFlexGraphAlgorithm.obj
 0001:0000f540       __unwindfunclet$??__EuserActLog@U2@@YAXXZ$0 10010540 f   DNAFlexGraphAlgorithm.obj
 0001:0000f549       __ehhandler$??__EuserActLog@U2@@YAXXZ 10010549 f   DNAFlexGraphAlgorithm.obj
 0001:0000f570       __unwindfunclet$?calculate@DNAFlexGraphAlgorithm@U2@@UAEXAAV?$QVector@M@@PAVU2SequenceObject@2@ABVU2Region@2@PBVGSequenceGraphWindowData@2@AAVU2OpStatus@2@@Z$3 10010570 f   DNAFlexGraphAlgorithm.obj
 0001:0000f579       __unwindfunclet$?calculate@DNAFlexGraphAlgorithm@U2@@UAEXAAV?$QVector@M@@PAVU2SequenceObject@2@ABVU2Region@2@PBVGSequenceGraphWindowData@2@AAVU2OpStatus@2@@Z$4 10010579 f   DNAFlexGraphAlgorithm.obj
 0001:0000f582       __ehhandler$?calculate@DNAFlexGraphAlgorithm@U2@@UAEXAAV?$QVector@M@@PAVU2SequenceObject@2@ABVU2Region@2@PBVGSequenceGraphWindowData@2@AAVU2OpStatus@2@@Z 10010582 f   DNAFlexGraphAlgorithm.obj
 0001:0000f5a0       __ehhandler$?reallocData@?$QVector@M@@AAEXHHV?$QFlags@W4AllocationOption@QArrayData@@@@@Z 100105a0 f   DNAFlexGraphAlgorithm.obj
 0001:0000f5c0       __ehhandler$??0?$QList@PAVADVSequenceWidget@U2@@@@QAE@ABV0@@Z 100105c0 f   DNAFlexPlugin.obj
 0001:0000f5e0       __unwindfunclet$??0DNAFlexPlugin@U2@@QAE@XZ$0 100105e0 f   DNAFlexPlugin.obj
 0001:0000f5e9       __unwindfunclet$??0DNAFlexPlugin@U2@@QAE@XZ$1 100105e9 f   DNAFlexPlugin.obj
 0001:0000f5f2       __unwindfunclet$??0DNAFlexPlugin@U2@@QAE@XZ$2 100105f2 f   DNAFlexPlugin.obj
 0001:0000f5fb       __unwindfunclet$??0DNAFlexPlugin@U2@@QAE@XZ$3 100105fb f   DNAFlexPlugin.obj
 0001:0000f606       __ehhandler$??0DNAFlexPlugin@U2@@QAE@XZ 10010606 f   DNAFlexPlugin.obj
 0001:0000f630       __unwindfunclet$??0DNAFlexViewContext@U2@@QAE@PAVQObject@@@Z$0 10010630 f   DNAFlexPlugin.obj
 0001:0000f638       __unwindfunclet$??0DNAFlexViewContext@U2@@QAE@PAVQObject@@@Z$1 10010638 f   DNAFlexPlugin.obj
 0001:0000f641       __unwindfunclet$??0DNAFlexViewContext@U2@@QAE@PAVQObject@@@Z$2 10010641 f   DNAFlexPlugin.obj
 0001:0000f64c       __ehhandler$??0DNAFlexViewContext@U2@@QAE@PAVQObject@@@Z 1001064c f   DNAFlexPlugin.obj
 0001:0000f670       __unwindfunclet$??1?$QObjectScopedPointer@VDNAFlexDialog@U2@@@U2@@QAE@XZ$0 10010670 f   DNAFlexPlugin.obj
 0001:0000f678       __ehhandler$??1?$QObjectScopedPointer@VDNAFlexDialog@U2@@@U2@@QAE@XZ 10010678 f   DNAFlexPlugin.obj
 0001:0000f6a0       __unwindfunclet$??__EalgoLog@U2@@YAXXZ$0 100106a0 f   DNAFlexPlugin.obj
 0001:0000f6a9       __ehhandler$??__EalgoLog@U2@@YAXXZ 100106a9 f   DNAFlexPlugin.obj
 0001:0000f6d0       __unwindfunclet$??__EcmdLog@U2@@YAXXZ$0 100106d0 f   DNAFlexPlugin.obj
 0001:0000f6d9       __ehhandler$??__EcmdLog@U2@@YAXXZ 100106d9 f   DNAFlexPlugin.obj
 0001:0000f700       __unwindfunclet$??__EcoreLog@U2@@YAXXZ$0 10010700 f   DNAFlexPlugin.obj
 0001:0000f709       __ehhandler$??__EcoreLog@U2@@YAXXZ 10010709 f   DNAFlexPlugin.obj
 0001:0000f730       __unwindfunclet$??__EioLog@U2@@YAXXZ$0 10010730 f   DNAFlexPlugin.obj
 0001:0000f739       __ehhandler$??__EioLog@U2@@YAXXZ 10010739 f   DNAFlexPlugin.obj
 0001:0000f760       __unwindfunclet$??__EperfLog@U2@@YAXXZ$0 10010760 f   DNAFlexPlugin.obj
 0001:0000f769       __ehhandler$??__EperfLog@U2@@YAXXZ 10010769 f   DNAFlexPlugin.obj
 0001:0000f790       __unwindfunclet$??__EscriptLog@U2@@YAXXZ$0 10010790 f   DNAFlexPlugin.obj
 0001:0000f799       __ehhandler$??__EscriptLog@U2@@YAXXZ 10010799 f   DNAFlexPlugin.obj
 0001:0000f7c0       __unwindfunclet$??__EtaskLog@U2@@YAXXZ$0 100107c0 f   DNAFlexPlugin.obj
 0001:0000f7c9       __ehhandler$??__EtaskLog@U2@@YAXXZ 100107c9 f   DNAFlexPlugin.obj
 0001:0000f7f0       __unwindfunclet$??__EuiLog@U2@@YAXXZ$0 100107f0 f   DNAFlexPlugin.obj
 0001:0000f7f9       __ehhandler$??__EuiLog@U2@@YAXXZ 100107f9 f   DNAFlexPlugin.obj
 0001:0000f820       __unwindfunclet$??__EuserActLog@U2@@YAXXZ$0 10010820 f   DNAFlexPlugin.obj
 0001:0000f829       __ehhandler$??__EuserActLog@U2@@YAXXZ 10010829 f   DNAFlexPlugin.obj
 0001:0000f850       __unwindfunclet$?initViewContext@DNAFlexViewContext@U2@@EAEXPAVGObjectView@2@@Z$1 10010850 f   DNAFlexPlugin.obj
 0001:0000f858       __unwindfunclet$?initViewContext@DNAFlexViewContext@U2@@EAEXPAVGObjectView@2@@Z$2 10010858 f   DNAFlexPlugin.obj
 0001:0000f860       __unwindfunclet$?initViewContext@DNAFlexViewContext@U2@@EAEXPAVGObjectView@2@@Z$3 10010860 f   DNAFlexPlugin.obj
 0001:0000f86b       __unwindfunclet$?initViewContext@DNAFlexViewContext@U2@@EAEXPAVGObjectView@2@@Z$4 1001086b f   DNAFlexPlugin.obj
 0001:0000f885       __unwindfunclet$?initViewContext@DNAFlexViewContext@U2@@EAEXPAVGObjectView@2@@Z$5 10010885 f   DNAFlexPlugin.obj
 0001:0000f89f       __unwindfunclet$?initViewContext@DNAFlexViewContext@U2@@EAEXPAVGObjectView@2@@Z$6 1001089f f   DNAFlexPlugin.obj
 0001:0000f8b9       __ehhandler$?initViewContext@DNAFlexViewContext@U2@@EAEXPAVGObjectView@2@@Z 100108b9 f   DNAFlexPlugin.obj
 0001:0000f8e0       __unwindfunclet$?sl_sequenceWidgetAdded@DNAFlexViewContext@U2@@AAEXPAVADVSequenceWidget@2@@Z$0 100108e0 f   DNAFlexPlugin.obj
 0001:0000f8e9       __unwindfunclet$?sl_sequenceWidgetAdded@DNAFlexViewContext@U2@@AAEXPAVADVSequenceWidget@2@@Z$1 100108e9 f   DNAFlexPlugin.obj
 0001:0000f8f4       __ehhandler$?sl_sequenceWidgetAdded@DNAFlexViewContext@U2@@AAEXPAVADVSequenceWidget@2@@Z 100108f4 f   DNAFlexPlugin.obj
 0001:0000f910       __unwindfunclet$?sl_showDNAFlexDialog@DNAFlexViewContext@U2@@AAEXXZ$0 10010910 f   DNAFlexPlugin.obj
 0001:0000f919       __unwindfunclet$?sl_showDNAFlexDialog@DNAFlexViewContext@U2@@AAEXXZ$1 10010919 f   DNAFlexPlugin.obj
 0001:0000f922       __unwindfunclet$?sl_showDNAFlexDialog@DNAFlexViewContext@U2@@AAEXXZ$2 10010922 f   DNAFlexPlugin.obj
 0001:0000f92b       __unwindfunclet$?sl_showDNAFlexDialog@DNAFlexViewContext@U2@@AAEXXZ$3 1001092b f   DNAFlexPlugin.obj
 0001:0000f934       __unwindfunclet$?sl_showDNAFlexDialog@DNAFlexViewContext@U2@@AAEXXZ$4 10010934 f   DNAFlexPlugin.obj
 0001:0000f93d       __unwindfunclet$?sl_showDNAFlexDialog@DNAFlexViewContext@U2@@AAEXXZ$5 1001093d f   DNAFlexPlugin.obj
 0001:0000f946       __unwindfunclet$?sl_showDNAFlexDialog@DNAFlexViewContext@U2@@AAEXXZ$6 10010946 f   DNAFlexPlugin.obj
 0001:0000f94f       __unwindfunclet$?sl_showDNAFlexDialog@DNAFlexViewContext@U2@@AAEXXZ$7 1001094f f   DNAFlexPlugin.obj
 0001:0000f958       __unwindfunclet$?sl_showDNAFlexDialog@DNAFlexViewContext@U2@@AAEXXZ$8 10010958 f   DNAFlexPlugin.obj
 0001:0000f961       __unwindfunclet$?sl_showDNAFlexDialog@DNAFlexViewContext@U2@@AAEXXZ$9 10010961 f   DNAFlexPlugin.obj
 0001:0000f96a       __unwindfunclet$?sl_showDNAFlexDialog@DNAFlexViewContext@U2@@AAEXXZ$10 1001096a f   DNAFlexPlugin.obj
 0001:0000f973       __unwindfunclet$?sl_showDNAFlexDialog@DNAFlexViewContext@U2@@AAEXXZ$11 10010973 f   DNAFlexPlugin.obj
 0001:0000f97c       __unwindfunclet$?sl_showDNAFlexDialog@DNAFlexViewContext@U2@@AAEXXZ$12 1001097c f   DNAFlexPlugin.obj
 0001:0000f985       __unwindfunclet$?sl_showDNAFlexDialog@DNAFlexViewContext@U2@@AAEXXZ$13 10010985 f   DNAFlexPlugin.obj
 0001:0000f990       __unwindfunclet$?sl_showDNAFlexDialog@DNAFlexViewContext@U2@@AAEXXZ$14 10010990 f   DNAFlexPlugin.obj
 0001:0000f998       __unwindfunclet$?sl_showDNAFlexDialog@DNAFlexViewContext@U2@@AAEXXZ$15 10010998 f   DNAFlexPlugin.obj
 0001:0000f9a1       __unwindfunclet$?sl_showDNAFlexDialog@DNAFlexViewContext@U2@@AAEXXZ$16 100109a1 f   DNAFlexPlugin.obj
 0001:0000f9aa       __ehhandler$?sl_showDNAFlexDialog@DNAFlexViewContext@U2@@AAEXXZ 100109aa f   DNAFlexPlugin.obj
 0001:0000f9d0       __ehhandler$??0?$QList@VHighFlexResult@U2@@@@QAE@ABV0@@Z 100109d0 f   DNAFlexTask.obj
 0001:0000f9f0       __unwindfunclet$??0DNAFlexTask@U2@@QAE@ABVHighFlexSettings@1@PAVAnnotationTableObject@1@ABVQString@@22ABVDNASequence@1@@Z$0 100109f0 f   DNAFlexTask.obj
 0001:0000f9f9       __unwindfunclet$??0DNAFlexTask@U2@@QAE@ABVHighFlexSettings@1@PAVAnnotationTableObject@1@ABVQString@@22ABVDNASequence@1@@Z$1 100109f9 f   DNAFlexTask.obj
 0001:0000fa02       __unwindfunclet$??0DNAFlexTask@U2@@QAE@ABVHighFlexSettings@1@PAVAnnotationTableObject@1@ABVQString@@22ABVDNASequence@1@@Z$2 10010a02 f   DNAFlexTask.obj
 0001:0000fa10       __unwindfunclet$??0DNAFlexTask@U2@@QAE@ABVHighFlexSettings@1@PAVAnnotationTableObject@1@ABVQString@@22ABVDNASequence@1@@Z$3 10010a10 f   DNAFlexTask.obj
 0001:0000fa1f       __unwindfunclet$??0DNAFlexTask@U2@@QAE@ABVHighFlexSettings@1@PAVAnnotationTableObject@1@ABVQString@@22ABVDNASequence@1@@Z$4 10010a1f f   DNAFlexTask.obj
 0001:0000fa2e       __unwindfunclet$??0DNAFlexTask@U2@@QAE@ABVHighFlexSettings@1@PAVAnnotationTableObject@1@ABVQString@@22ABVDNASequence@1@@Z$5 10010a2e f   DNAFlexTask.obj
 0001:0000fa3d       __unwindfunclet$??0DNAFlexTask@U2@@QAE@ABVHighFlexSettings@1@PAVAnnotationTableObject@1@ABVQString@@22ABVDNASequence@1@@Z$6 10010a3d f   DNAFlexTask.obj
 0001:0000fa4c       __unwindfunclet$??0DNAFlexTask@U2@@QAE@ABVHighFlexSettings@1@PAVAnnotationTableObject@1@ABVQString@@22ABVDNASequence@1@@Z$7 10010a4c f   DNAFlexTask.obj
 0001:0000fa57       __ehhandler$??0DNAFlexTask@U2@@QAE@ABVHighFlexSettings@1@PAVAnnotationTableObject@1@ABVQString@@22ABVDNASequence@1@@Z 10010a57 f   DNAFlexTask.obj
 0001:0000fa80       __unwindfunclet$??1DNAFlexTask@U2@@UAE@XZ$0 10010a80 f   DNAFlexTask.obj
 0001:0000fa89       __unwindfunclet$??1DNAFlexTask@U2@@UAE@XZ$1 10010a89 f   DNAFlexTask.obj
 0001:0000fa97       __unwindfunclet$??1DNAFlexTask@U2@@UAE@XZ$2 10010a97 f   DNAFlexTask.obj
 0001:0000faa6       __unwindfunclet$??1DNAFlexTask@U2@@UAE@XZ$3 10010aa6 f   DNAFlexTask.obj
 0001:0000fab5       __unwindfunclet$??1DNAFlexTask@U2@@UAE@XZ$4 10010ab5 f   DNAFlexTask.obj
 0001:0000fac4       __ehhandler$??1DNAFlexTask@U2@@UAE@XZ 10010ac4 f   DNAFlexTask.obj
 0001:0000fae0       __unwindfunclet$??__EalgoLog@U2@@YAXXZ$0 10010ae0 f   DNAFlexTask.obj
 0001:0000fae9       __ehhandler$??__EalgoLog@U2@@YAXXZ 10010ae9 f   DNAFlexTask.obj
 0001:0000fb10       __unwindfunclet$??__EcmdLog@U2@@YAXXZ$0 10010b10 f   DNAFlexTask.obj
 0001:0000fb19       __ehhandler$??__EcmdLog@U2@@YAXXZ 10010b19 f   DNAFlexTask.obj
 0001:0000fb40       __unwindfunclet$??__EcoreLog@U2@@YAXXZ$0 10010b40 f   DNAFlexTask.obj
 0001:0000fb49       __ehhandler$??__EcoreLog@U2@@YAXXZ 10010b49 f   DNAFlexTask.obj
 0001:0000fb70       __unwindfunclet$??__EioLog@U2@@YAXXZ$0 10010b70 f   DNAFlexTask.obj
 0001:0000fb79       __ehhandler$??__EioLog@U2@@YAXXZ 10010b79 f   DNAFlexTask.obj
 0001:0000fba0       __unwindfunclet$??__EperfLog@U2@@YAXXZ$0 10010ba0 f   DNAFlexTask.obj
 0001:0000fba9       __ehhandler$??__EperfLog@U2@@YAXXZ 10010ba9 f   DNAFlexTask.obj
 0001:0000fbd0       __unwindfunclet$??__EscriptLog@U2@@YAXXZ$0 10010bd0 f   DNAFlexTask.obj
 0001:0000fbd9       __ehhandler$??__EscriptLog@U2@@YAXXZ 10010bd9 f   DNAFlexTask.obj
 0001:0000fc00       __unwindfunclet$??__EtaskLog@U2@@YAXXZ$0 10010c00 f   DNAFlexTask.obj
 0001:0000fc09       __ehhandler$??__EtaskLog@U2@@YAXXZ 10010c09 f   DNAFlexTask.obj
 0001:0000fc30       __unwindfunclet$??__EuiLog@U2@@YAXXZ$0 10010c30 f   DNAFlexTask.obj
 0001:0000fc39       __ehhandler$??__EuiLog@U2@@YAXXZ 10010c39 f   DNAFlexTask.obj
 0001:0000fc60       __unwindfunclet$??__EuserActLog@U2@@YAXXZ$0 10010c60 f   DNAFlexTask.obj
 0001:0000fc69       __ehhandler$??__EuserActLog@U2@@YAXXZ 10010c69 f   DNAFlexTask.obj
 0001:0000fc90       __ehhandler$?append@?$QList@PAVTask@U2@@@@QAEXABQAVTask@U2@@@Z 10010c90 f   DNAFlexTask.obj
 0001:0000fcb0       __ehhandler$?append@?$QList@V?$QSharedDataPointer@VAnnotationData@U2@@@@@@QAEXABV?$QSharedDataPointer@VAnnotationData@U2@@@@@Z 10010cb0 f   DNAFlexTask.obj
 0001:0000fcd0       __unwindfunclet$?append@?$QVector@VU2Qualifier@U2@@@@QAEXABVU2Qualifier@U2@@@Z$0 10010cd0 f   DNAFlexTask.obj
 0001:0000fcd9       __unwindfunclet$?append@?$QVector@VU2Qualifier@U2@@@@QAEXABVU2Qualifier@U2@@@Z$1 10010cd9 f   DNAFlexTask.obj
 0001:0000fcea       __ehhandler$?append@?$QVector@VU2Qualifier@U2@@@@QAEXABVU2Qualifier@U2@@@Z 10010cea f   DNAFlexTask.obj
 0001:0000fd10       __unwindfunclet$?defaultConstruct@?$QVector@VU2Qualifier@U2@@@@AAEXPAVU2Qualifier@U2@@0@Z$0 10010d10 f   DNAFlexTask.obj
 0001:0000fd21       __ehhandler$?defaultConstruct@?$QVector@VU2Qualifier@U2@@@@AAEXPAVU2Qualifier@U2@@0@Z 10010d21 f   DNAFlexTask.obj
 0001:0000fd40       __ehhandler$?detach_helper_grow@?$QList@PAVTask@U2@@@@AAEPAUNode@1@HH@Z 10010d40 f   DNAFlexTask.obj
 0001:0000fd60       __ehhandler$?detach_helper_grow@?$QList@V?$QSharedDataPointer@VAnnotationData@U2@@@@@@AAEPAUNode@1@HH@Z 10010d60 f   DNAFlexTask.obj
 0001:0000fd80       __unwindfunclet$?getAnnotationsFromResults@DNAFlexTask@U2@@QAE?AV?$QList@V?$QSharedDataPointer@VAnnotationData@U2@@@@@@ABV?$QList@VHighFlexResult@U2@@@@@Z$0 10010d80 f   DNAFlexTask.obj
 0001:0000fd99       __unwindfunclet$?getAnnotationsFromResults@DNAFlexTask@U2@@QAE?AV?$QList@V?$QSharedDataPointer@VAnnotationData@U2@@@@@@ABV?$QList@VHighFlexResult@U2@@@@@Z$1 10010d99 f   DNAFlexTask.obj
 0001:0000fda1       __unwindfunclet$?getAnnotationsFromResults@DNAFlexTask@U2@@QAE?AV?$QList@V?$QSharedDataPointer@VAnnotationData@U2@@@@@@ABV?$QList@VHighFlexResult@U2@@@@@Z$2 10010da1 f   DNAFlexTask.obj
 0001:0000fdac       __unwindfunclet$?getAnnotationsFromResults@DNAFlexTask@U2@@QAE?AV?$QList@V?$QSharedDataPointer@VAnnotationData@U2@@@@@@ABV?$QList@VHighFlexResult@U2@@@@@Z$3 10010dac f   DNAFlexTask.obj
 0001:0000fdb4       __unwindfunclet$?getAnnotationsFromResults@DNAFlexTask@U2@@QAE?AV?$QList@V?$QSharedDataPointer@VAnnotationData@U2@@@@@@ABV?$QList@VHighFlexResult@U2@@@@@Z$14 10010db4 f   DNAFlexTask.obj
 0001:0000fdbf       __unwindfunclet$?getAnnotationsFromResults@DNAFlexTask@U2@@QAE?AV?$QList@V?$QSharedDataPointer@VAnnotationData@U2@@@@@@ABV?$QList@VHighFlexResult@U2@@@@@Z$15 10010dbf f   DNAFlexTask.obj
 0001:0000fdca       __unwindfunclet$?getAnnotationsFromResults@DNAFlexTask@U2@@QAE?AV?$QList@V?$QSharedDataPointer@VAnnotationData@U2@@@@@@ABV?$QList@VHighFlexResult@U2@@@@@Z$4 10010dca f   DNAFlexTask.obj
 0001:0000fdd3       __unwindfunclet$?getAnnotationsFromResults@DNAFlexTask@U2@@QAE?AV?$QList@V?$QSharedDataPointer@VAnnotationData@U2@@@@@@ABV?$QList@VHighFlexResult@U2@@@@@Z$5 10010dd3 f   DNAFlexTask.obj
 0001:0000fddc       __unwindfunclet$?getAnnotationsFromResults@DNAFlexTask@U2@@QAE?AV?$QList@V?$QSharedDataPointer@VAnnotationData@U2@@@@@@ABV?$QList@VHighFlexResult@U2@@@@@Z$6 10010ddc f   DNAFlexTask.obj
 0001:0000fde5       __unwindfunclet$?getAnnotationsFromResults@DNAFlexTask@U2@@QAE?AV?$QList@V?$QSharedDataPointer@VAnnotationData@U2@@@@@@ABV?$QList@VHighFlexResult@U2@@@@@Z$16 10010de5 f   DNAFlexTask.obj
 0001:0000fdf0       __unwindfunclet$?getAnnotationsFromResults@DNAFlexTask@U2@@QAE?AV?$QList@V?$QSharedDataPointer@VAnnotationData@U2@@@@@@ABV?$QList@VHighFlexResult@U2@@@@@Z$7 10010df0 f   DNAFlexTask.obj
 0001:0000fdf9       __unwindfunclet$?getAnnotationsFromResults@DNAFlexTask@U2@@QAE?AV?$QList@V?$QSharedDataPointer@VAnnotationData@U2@@@@@@ABV?$QList@VHighFlexResult@U2@@@@@Z$8 10010df9 f   DNAFlexTask.obj
 0001:0000fe02       __unwindfunclet$?getAnnotationsFromResults@DNAFlexTask@U2@@QAE?AV?$QList@V?$QSharedDataPointer@VAnnotationData@U2@@@@@@ABV?$QList@VHighFlexResult@U2@@@@@Z$9 10010e02 f   DNAFlexTask.obj
 0001:0000fe0b       __unwindfunclet$?getAnnotationsFromResults@DNAFlexTask@U2@@QAE?AV?$QList@V?$QSharedDataPointer@VAnnotationData@U2@@@@@@ABV?$QList@VHighFlexResult@U2@@@@@Z$17 10010e0b f   DNAFlexTask.obj
 0001:0000fe16       __unwindfunclet$?getAnnotationsFromResults@DNAFlexTask@U2@@QAE?AV?$QList@V?$QSharedDataPointer@VAnnotationData@U2@@@@@@ABV?$QList@VHighFlexResult@U2@@@@@Z$10 10010e16 f   DNAFlexTask.obj
 0001:0000fe1f       __unwindfunclet$?getAnnotationsFromResults@DNAFlexTask@U2@@QAE?AV?$QList@V?$QSharedDataPointer@VAnnotationData@U2@@@@@@ABV?$QList@VHighFlexResult@U2@@@@@Z$11 10010e1f f   DNAFlexTask.obj
 0001:0000fe28       __unwindfunclet$?getAnnotationsFromResults@DNAFlexTask@U2@@QAE?AV?$QList@V?$QSharedDataPointer@VAnnotationData@U2@@@@@@ABV?$QList@VHighFlexResult@U2@@@@@Z$12 10010e28 f   DNAFlexTask.obj
 0001:0000fe31       __unwindfunclet$?getAnnotationsFromResults@DNAFlexTask@U2@@QAE?AV?$QList@V?$QSharedDataPointer@VAnnotationData@U2@@@@@@ABV?$QList@VHighFlexResult@U2@@@@@Z$18 10010e31 f   DNAFlexTask.obj
 0001:0000fe3c       __ehhandler$?getAnnotationsFromResults@DNAFlexTask@U2@@QAE?AV?$QList@V?$QSharedDataPointer@VAnnotationData@U2@@@@@@ABV?$QList@VHighFlexResult@U2@@@@@Z 10010e3c f   DNAFlexTask.obj
 0001:0000fe60       __ehhandler$?node_copy@?$QList@VHighFlexResult@U2@@@@AAEXPAUNode@1@00@Z 10010e60 f   DNAFlexTask.obj
 0001:0000fe80       __unwindfunclet$?onSubTaskFinished@DNAFlexTask@U2@@UAE?AV?$QList@PAVTask@U2@@@@PAVTask@2@@Z$0 10010e80 f   DNAFlexTask.obj
 0001:0000fe88       __unwindfunclet$?onSubTaskFinished@DNAFlexTask@U2@@UAE?AV?$QList@PAVTask@U2@@@@PAVTask@2@@Z$1 10010e88 f   DNAFlexTask.obj
 0001:0000fe91       __unwindfunclet$?onSubTaskFinished@DNAFlexTask@U2@@UAE?AV?$QList@PAVTask@U2@@@@PAVTask@2@@Z$4 10010e91 f   DNAFlexTask.obj
 0001:0000fe9a       __unwindfunclet$?onSubTaskFinished@DNAFlexTask@U2@@UAE?AV?$QList@PAVTask@U2@@@@PAVTask@2@@Z$5 10010e9a f   DNAFlexTask.obj
 0001:0000fea3       __unwindfunclet$?onSubTaskFinished@DNAFlexTask@U2@@UAE?AV?$QList@PAVTask@U2@@@@PAVTask@2@@Z$6 10010ea3 f   DNAFlexTask.obj
 0001:0000feac       __unwindfunclet$?onSubTaskFinished@DNAFlexTask@U2@@UAE?AV?$QList@PAVTask@U2@@@@PAVTask@2@@Z$7 10010eac f   DNAFlexTask.obj
 0001:0000feb5       __unwindfunclet$?onSubTaskFinished@DNAFlexTask@U2@@UAE?AV?$QList@PAVTask@U2@@@@PAVTask@2@@Z$8 10010eb5 f   DNAFlexTask.obj
 0001:0000febe       __unwindfunclet$?onSubTaskFinished@DNAFlexTask@U2@@UAE?AV?$QList@PAVTask@U2@@@@PAVTask@2@@Z$9 10010ebe f   DNAFlexTask.obj
 0001:0000fec7       __unwindfunclet$?onSubTaskFinished@DNAFlexTask@U2@@UAE?AV?$QList@PAVTask@U2@@@@PAVTask@2@@Z$10 10010ec7 f   DNAFlexTask.obj
 0001:0000fecf       __unwindfunclet$?onSubTaskFinished@DNAFlexTask@U2@@UAE?AV?$QList@PAVTask@U2@@@@PAVTask@2@@Z$11 10010ecf f   DNAFlexTask.obj
 0001:0000fed7       __unwindfunclet$?onSubTaskFinished@DNAFlexTask@U2@@UAE?AV?$QList@PAVTask@U2@@@@PAVTask@2@@Z$12 10010ed7 f   DNAFlexTask.obj
 0001:0000fee2       __unwindfunclet$?onSubTaskFinished@DNAFlexTask@U2@@UAE?AV?$QList@PAVTask@U2@@@@PAVTask@2@@Z$3 10010ee2 f   DNAFlexTask.obj
 0001:0000feeb       __unwindfunclet$?onSubTaskFinished@DNAFlexTask@U2@@UAE?AV?$QList@PAVTask@U2@@@@PAVTask@2@@Z$2 10010eeb f   DNAFlexTask.obj
 0001:0000ff04       __ehhandler$?onSubTaskFinished@DNAFlexTask@U2@@UAE?AV?$QList@PAVTask@U2@@@@PAVTask@2@@Z 10010f04 f   DNAFlexTask.obj
 0001:0000ff20       __unwindfunclet$?reallocData@?$QVector@VU2Qualifier@U2@@@@AAEXHHV?$QFlags@W4AllocationOption@QArrayData@@@@@Z$4 10010f20 f   DNAFlexTask.obj
 0001:0000ff31       __ehhandler$?reallocData@?$QVector@VU2Qualifier@U2@@@@AAEXHHV?$QFlags@W4AllocationOption@QArrayData@@@@@Z 10010f31 f   DNAFlexTask.obj
 0001:0000ff50       __ehhandler$?reallocData@?$QVector@VU2Region@U2@@@@AAEXHHV?$QFlags@W4AllocationOption@QArrayData@@@@@Z 10010f50 f   DNAFlexTask.obj
 0001:0000ff70       __unwindfunclet$??0FindHighFlexRegions@U2@@QAE@ABVDNASequence@1@ABVHighFlexSettings@1@@Z$0 10010f70 f   FindHighFlexRegions.obj
 0001:0000ff79       __unwindfunclet$??0FindHighFlexRegions@U2@@QAE@ABVDNASequence@1@ABVHighFlexSettings@1@@Z$1 10010f79 f   FindHighFlexRegions.obj
 0001:0000ff82       __unwindfunclet$??0FindHighFlexRegions@U2@@QAE@ABVDNASequence@1@ABVHighFlexSettings@1@@Z$2 10010f82 f   FindHighFlexRegions.obj
 0001:0000ff90       __ehhandler$??0FindHighFlexRegions@U2@@QAE@ABVDNASequence@1@ABVHighFlexSettings@1@@Z 10010f90 f   FindHighFlexRegions.obj
 0001:0000ffb0       __unwindfunclet$??1FindHighFlexRegions@U2@@UAE@XZ$0 10010fb0 f   FindHighFlexRegions.obj
 0001:0000ffb9       __unwindfunclet$??1FindHighFlexRegions@U2@@UAE@XZ$1 10010fb9 f   FindHighFlexRegions.obj
 0001:0000ffc7       __unwindfunclet$??1FindHighFlexRegions@U2@@UAE@XZ$2 10010fc7 f   FindHighFlexRegions.obj
 0001:0000ffd6       __ehhandler$??1FindHighFlexRegions@U2@@UAE@XZ 10010fd6 f   FindHighFlexRegions.obj
 0001:00010000       __unwindfunclet$??_GFindHighFlexRegions@U2@@UAEPAXI@Z$0 10011000 f   FindHighFlexRegions.obj
 0001:00010009       __unwindfunclet$??_GFindHighFlexRegions@U2@@UAEPAXI@Z$1 10011009 f   FindHighFlexRegions.obj
 0001:00010017       __unwindfunclet$??_GFindHighFlexRegions@U2@@UAEPAXI@Z$2 10011017 f   FindHighFlexRegions.obj
 0001:00010026       __ehhandler$??_GFindHighFlexRegions@U2@@UAEPAXI@Z 10011026 f   FindHighFlexRegions.obj
 0001:00010050       __unwindfunclet$??__EalgoLog@U2@@YAXXZ$0 10011050 f   FindHighFlexRegions.obj
 0001:00010059       __ehhandler$??__EalgoLog@U2@@YAXXZ 10011059 f   FindHighFlexRegions.obj
 0001:00010080       __unwindfunclet$??__EcmdLog@U2@@YAXXZ$0 10011080 f   FindHighFlexRegions.obj
 0001:00010089       __ehhandler$??__EcmdLog@U2@@YAXXZ 10011089 f   FindHighFlexRegions.obj
 0001:000100b0       __unwindfunclet$??__EcoreLog@U2@@YAXXZ$0 100110b0 f   FindHighFlexRegions.obj
 0001:000100b9       __ehhandler$??__EcoreLog@U2@@YAXXZ 100110b9 f   FindHighFlexRegions.obj
 0001:000100e0       __unwindfunclet$??__EioLog@U2@@YAXXZ$0 100110e0 f   FindHighFlexRegions.obj
 0001:000100e9       __ehhandler$??__EioLog@U2@@YAXXZ 100110e9 f   FindHighFlexRegions.obj
 0001:00010110       __unwindfunclet$??__EperfLog@U2@@YAXXZ$0 10011110 f   FindHighFlexRegions.obj
 0001:00010119       __ehhandler$??__EperfLog@U2@@YAXXZ 10011119 f   FindHighFlexRegions.obj
 0001:00010140       __unwindfunclet$??__EscriptLog@U2@@YAXXZ$0 10011140 f   FindHighFlexRegions.obj
 0001:00010149       __ehhandler$??__EscriptLog@U2@@YAXXZ 10011149 f   FindHighFlexRegions.obj
 0001:00010170       __unwindfunclet$??__EtaskLog@U2@@YAXXZ$0 10011170 f   FindHighFlexRegions.obj
 0001:00010179       __ehhandler$??__EtaskLog@U2@@YAXXZ 10011179 f   FindHighFlexRegions.obj
 0001:000101a0       __unwindfunclet$??__EuiLog@U2@@YAXXZ$0 100111a0 f   FindHighFlexRegions.obj
 0001:000101a9       __ehhandler$??__EuiLog@U2@@YAXXZ 100111a9 f   FindHighFlexRegions.obj
 0001:000101d0       __unwindfunclet$??__EuserActLog@U2@@YAXXZ$0 100111d0 f   FindHighFlexRegions.obj
 0001:000101d9       __ehhandler$??__EuserActLog@U2@@YAXXZ 100111d9 f   FindHighFlexRegions.obj
 0001:00010200       __ehhandler$?append@?$QList@VHighFlexResult@U2@@@@QAEXABVHighFlexResult@U2@@@Z 10011200 f   FindHighFlexRegions.obj
 0001:00010220       __ehhandler$?detach_helper_grow@?$QList@VHighFlexResult@U2@@@@AAEPAUNode@1@HH@Z 10011220 f   FindHighFlexRegions.obj
 0001:00010240       __unwindfunclet$??__EalgoLog@U2@@YAXXZ$0 10011240 f   FindHighFlexRegionsAlgorithm.obj
 0001:00010249       __ehhandler$??__EalgoLog@U2@@YAXXZ 10011249 f   FindHighFlexRegionsAlgorithm.obj
 0001:00010270       __unwindfunclet$??__EcmdLog@U2@@YAXXZ$0 10011270 f   FindHighFlexRegionsAlgorithm.obj
 0001:00010279       __ehhandler$??__EcmdLog@U2@@YAXXZ 10011279 f   FindHighFlexRegionsAlgorithm.obj
 0001:000102a0       __unwindfunclet$??__EcoreLog@U2@@YAXXZ$0 100112a0 f   FindHighFlexRegionsAlgorithm.obj
 0001:000102a9       __ehhandler$??__EcoreLog@U2@@YAXXZ 100112a9 f   FindHighFlexRegionsAlgorithm.obj
 0001:000102d0       __unwindfunclet$??__EioLog@U2@@YAXXZ$0 100112d0 f   FindHighFlexRegionsAlgorithm.obj
 0001:000102d9       __ehhandler$??__EioLog@U2@@YAXXZ 100112d9 f   FindHighFlexRegionsAlgorithm.obj
 0001:00010300       __unwindfunclet$??__EperfLog@U2@@YAXXZ$0 10011300 f   FindHighFlexRegionsAlgorithm.obj
 0001:00010309       __ehhandler$??__EperfLog@U2@@YAXXZ 10011309 f   FindHighFlexRegionsAlgorithm.obj
 0001:00010330       __unwindfunclet$??__EscriptLog@U2@@YAXXZ$0 10011330 f   FindHighFlexRegionsAlgorithm.obj
 0001:00010339       __ehhandler$??__EscriptLog@U2@@YAXXZ 10011339 f   FindHighFlexRegionsAlgorithm.obj
 0001:00010360       __unwindfunclet$??__EtaskLog@U2@@YAXXZ$0 10011360 f   FindHighFlexRegionsAlgorithm.obj
 0001:00010369       __ehhandler$??__EtaskLog@U2@@YAXXZ 10011369 f   FindHighFlexRegionsAlgorithm.obj
 0001:00010390       __unwindfunclet$??__EuiLog@U2@@YAXXZ$0 10011390 f   FindHighFlexRegionsAlgorithm.obj
 0001:00010399       __ehhandler$??__EuiLog@U2@@YAXXZ 10011399 f   FindHighFlexRegionsAlgorithm.obj
 0001:000103c0       __unwindfunclet$??__EuserActLog@U2@@YAXXZ$0 100113c0 f   FindHighFlexRegionsAlgorithm.obj
 0001:000103c9       __ehhandler$??__EuserActLog@U2@@YAXXZ 100113c9 f   FindHighFlexRegionsAlgorithm.obj
 0001:000103f0       __unwindfunclet$?addToResults@FindHighFlexRegionsAlgorithm@U2@@CAXPAVFindHighFlexRegionsListener@2@ABVHighFlexResult@2@@Z$0 100113f0 f   FindHighFlexRegionsAlgorithm.obj
 0001:000103f9       __unwindfunclet$?addToResults@FindHighFlexRegionsAlgorithm@U2@@CAXPAVFindHighFlexRegionsListener@2@ABVHighFlexResult@2@@Z$1 100113f9 f   FindHighFlexRegionsAlgorithm.obj
 0001:00010402       __unwindfunclet$?addToResults@FindHighFlexRegionsAlgorithm@U2@@CAXPAVFindHighFlexRegionsListener@2@ABVHighFlexResult@2@@Z$2 10011402 f   FindHighFlexRegionsAlgorithm.obj
 0001:0001040b       __unwindfunclet$?addToResults@FindHighFlexRegionsAlgorithm@U2@@CAXPAVFindHighFlexRegionsListener@2@ABVHighFlexResult@2@@Z$3 1001140b f   FindHighFlexRegionsAlgorithm.obj
 0001:00010414       __unwindfunclet$?addToResults@FindHighFlexRegionsAlgorithm@U2@@CAXPAVFindHighFlexRegionsListener@2@ABVHighFlexResult@2@@Z$4 10011414 f   FindHighFlexRegionsAlgorithm.obj
 0001:0001041d       __unwindfunclet$?addToResults@FindHighFlexRegionsAlgorithm@U2@@CAXPAVFindHighFlexRegionsListener@2@ABVHighFlexResult@2@@Z$5 1001141d f   FindHighFlexRegionsAlgorithm.obj
 0001:00010426       __ehhandler$?addToResults@FindHighFlexRegionsAlgorithm@U2@@CAXPAVFindHighFlexRegionsListener@2@ABVHighFlexResult@2@@Z 10011426 f   FindHighFlexRegionsAlgorithm.obj
 0001:00010450       __unwindfunclet$?find@FindHighFlexRegionsAlgorithm@U2@@SAXPAVFindHighFlexRegionsListener@2@ABVHighFlexSettings@2@VQByteArray@@HAAH3@Z$0 10011450 f   FindHighFlexRegionsAlgorithm.obj
 0001:00010459       __unwindfunclet$?find@FindHighFlexRegionsAlgorithm@U2@@SAXPAVFindHighFlexRegionsListener@2@ABVHighFlexSettings@2@VQByteArray@@HAAH3@Z$1 10011459 f   FindHighFlexRegionsAlgorithm.obj
 0001:00010462       __unwindfunclet$?find@FindHighFlexRegionsAlgorithm@U2@@SAXPAVFindHighFlexRegionsListener@2@ABVHighFlexSettings@2@VQByteArray@@HAAH3@Z$2 10011462 f   FindHighFlexRegionsAlgorithm.obj
 0001:0001046b       __unwindfunclet$?find@FindHighFlexRegionsAlgorithm@U2@@SAXPAVFindHighFlexRegionsListener@2@ABVHighFlexSettings@2@VQByteArray@@HAAH3@Z$3 1001146b f   FindHighFlexRegionsAlgorithm.obj
 0001:00010474       __unwindfunclet$?find@FindHighFlexRegionsAlgorithm@U2@@SAXPAVFindHighFlexRegionsListener@2@ABVHighFlexSettings@2@VQByteArray@@HAAH3@Z$4 10011474 f   FindHighFlexRegionsAlgorithm.obj
 0001:0001047d       __unwindfunclet$?find@FindHighFlexRegionsAlgorithm@U2@@SAXPAVFindHighFlexRegionsListener@2@ABVHighFlexSettings@2@VQByteArray@@HAAH3@Z$5 1001147d f   FindHighFlexRegionsAlgorithm.obj
 0001:00010486       __unwindfunclet$?find@FindHighFlexRegionsAlgorithm@U2@@SAXPAVFindHighFlexRegionsListener@2@ABVHighFlexSettings@2@VQByteArray@@HAAH3@Z$6 10011486 f   FindHighFlexRegionsAlgorithm.obj
 0001:0001048f       __unwindfunclet$?find@FindHighFlexRegionsAlgorithm@U2@@SAXPAVFindHighFlexRegionsListener@2@ABVHighFlexSettings@2@VQByteArray@@HAAH3@Z$7 1001148f f   FindHighFlexRegionsAlgorithm.obj
 0001:00010498       __unwindfunclet$?find@FindHighFlexRegionsAlgorithm@U2@@SAXPAVFindHighFlexRegionsListener@2@ABVHighFlexSettings@2@VQByteArray@@HAAH3@Z$8 10011498 f   FindHighFlexRegionsAlgorithm.obj
 0001:000104a1       __unwindfunclet$?find@FindHighFlexRegionsAlgorithm@U2@@SAXPAVFindHighFlexRegionsListener@2@ABVHighFlexSettings@2@VQByteArray@@HAAH3@Z$9 100114a1 f   FindHighFlexRegionsAlgorithm.obj
 0001:000104aa       __unwindfunclet$?find@FindHighFlexRegionsAlgorithm@U2@@SAXPAVFindHighFlexRegionsListener@2@ABVHighFlexSettings@2@VQByteArray@@HAAH3@Z$10 100114aa f   FindHighFlexRegionsAlgorithm.obj
 0001:000104b3       __unwindfunclet$?find@FindHighFlexRegionsAlgorithm@U2@@SAXPAVFindHighFlexRegionsListener@2@ABVHighFlexSettings@2@VQByteArray@@HAAH3@Z$11 100114b3 f   FindHighFlexRegionsAlgorithm.obj
 0001:000104bc       __unwindfunclet$?find@FindHighFlexRegionsAlgorithm@U2@@SAXPAVFindHighFlexRegionsListener@2@ABVHighFlexSettings@2@VQByteArray@@HAAH3@Z$12 100114bc f   FindHighFlexRegionsAlgorithm.obj
 0001:000104c5       __ehhandler$?find@FindHighFlexRegionsAlgorithm@U2@@SAXPAVFindHighFlexRegionsListener@2@ABVHighFlexSettings@2@VQByteArray@@HAAH3@Z 100114c5 f   FindHighFlexRegionsAlgorithm.obj
 0001:000104e0       __unwindfunclet$?flexibilityAngle@FindHighFlexRegionsAlgorithm@U2@@SANDD@Z$0 100114e0 f   FindHighFlexRegionsAlgorithm.obj
 0001:000104e9       __unwindfunclet$?flexibilityAngle@FindHighFlexRegionsAlgorithm@U2@@SANDD@Z$1 100114e9 f   FindHighFlexRegionsAlgorithm.obj
 0001:000104f2       __unwindfunclet$?flexibilityAngle@FindHighFlexRegionsAlgorithm@U2@@SANDD@Z$2 100114f2 f   FindHighFlexRegionsAlgorithm.obj
 0001:000104fb       __unwindfunclet$?flexibilityAngle@FindHighFlexRegionsAlgorithm@U2@@SANDD@Z$3 100114fb f   FindHighFlexRegionsAlgorithm.obj
 0001:00010504       __unwindfunclet$?flexibilityAngle@FindHighFlexRegionsAlgorithm@U2@@SANDD@Z$4 10011504 f   FindHighFlexRegionsAlgorithm.obj
 0001:0001050d       __unwindfunclet$?flexibilityAngle@FindHighFlexRegionsAlgorithm@U2@@SANDD@Z$5 1001150d f   FindHighFlexRegionsAlgorithm.obj
 0001:00010516       __ehhandler$?flexibilityAngle@FindHighFlexRegionsAlgorithm@U2@@SANDD@Z 10011516 f   FindHighFlexRegionsAlgorithm.obj
 0001:00010540       __unwindfunclet$??H@YA?BVQString@@ABV0@0@Z$0 10011540 f   HighFlexSettings.obj
 0001:0001055a       __ehhandler$??H@YA?BVQString@@ABV0@0@Z 1001155a f   HighFlexSettings.obj
 0001:00010580       __unwindfunclet$??H@YA?BVQString@@ABV0@PBD@Z$0 10011580 f   HighFlexSettings.obj
 0001:0001059a       __unwindfunclet$??H@YA?BVQString@@ABV0@PBD@Z$1 1001159a f   HighFlexSettings.obj
 0001:000105a3       __ehhandler$??H@YA?BVQString@@ABV0@PBD@Z 100115a3 f   HighFlexSettings.obj
 0001:000105c0       __unwindfunclet$??__EalgoLog@U2@@YAXXZ$0 100115c0 f   HighFlexSettings.obj
 0001:000105c9       __ehhandler$??__EalgoLog@U2@@YAXXZ 100115c9 f   HighFlexSettings.obj
 0001:000105f0       __unwindfunclet$??__EcmdLog@U2@@YAXXZ$0 100115f0 f   HighFlexSettings.obj
 0001:000105f9       __ehhandler$??__EcmdLog@U2@@YAXXZ 100115f9 f   HighFlexSettings.obj
 0001:00010620       __unwindfunclet$??__EcoreLog@U2@@YAXXZ$0 10011620 f   HighFlexSettings.obj
 0001:00010629       __ehhandler$??__EcoreLog@U2@@YAXXZ 10011629 f   HighFlexSettings.obj
 0001:00010650       __unwindfunclet$??__EioLog@U2@@YAXXZ$0 10011650 f   HighFlexSettings.obj
 0001:00010659       __ehhandler$??__EioLog@U2@@YAXXZ 10011659 f   HighFlexSettings.obj
 0001:00010680       __unwindfunclet$??__EperfLog@U2@@YAXXZ$0 10011680 f   HighFlexSettings.obj
 0001:00010689       __ehhandler$??__EperfLog@U2@@YAXXZ 10011689 f   HighFlexSettings.obj
 0001:000106b0       __unwindfunclet$??__EscriptLog@U2@@YAXXZ$0 100116b0 f   HighFlexSettings.obj
 0001:000106b9       __ehhandler$??__EscriptLog@U2@@YAXXZ 100116b9 f   HighFlexSettings.obj
 0001:000106e0       __unwindfunclet$??__EtaskLog@U2@@YAXXZ$0 100116e0 f   HighFlexSettings.obj
 0001:000106e9       __ehhandler$??__EtaskLog@U2@@YAXXZ 100116e9 f   HighFlexSettings.obj
 0001:00010710       __unwindfunclet$??__EuiLog@U2@@YAXXZ$0 10011710 f   HighFlexSettings.obj
 0001:00010719       __ehhandler$??__EuiLog@U2@@YAXXZ 10011719 f   HighFlexSettings.obj
 0001:00010740       __unwindfunclet$??__EuserActLog@U2@@YAXXZ$0 10011740 f   HighFlexSettings.obj
 0001:00010749       __ehhandler$??__EuserActLog@U2@@YAXXZ 10011749 f   HighFlexSettings.obj
 0001:00010770       __unwindfunclet$?rememberSettings@HighFlexSettings@U2@@QAEXXZ$0 10011770 f   HighFlexSettings.obj
 0001:00010779       __unwindfunclet$?rememberSettings@HighFlexSettings@U2@@QAEXXZ$1 10011779 f   HighFlexSettings.obj
 0001:00010782       __unwindfunclet$?rememberSettings@HighFlexSettings@U2@@QAEXXZ$2 10011782 f   HighFlexSettings.obj
 0001:0001078b       __unwindfunclet$?rememberSettings@HighFlexSettings@U2@@QAEXXZ$3 1001178b f   HighFlexSettings.obj
 0001:00010794       __unwindfunclet$?rememberSettings@HighFlexSettings@U2@@QAEXXZ$4 10011794 f   HighFlexSettings.obj
 0001:0001079d       __unwindfunclet$?rememberSettings@HighFlexSettings@U2@@QAEXXZ$5 1001179d f   HighFlexSettings.obj
 0001:000107a6       __unwindfunclet$?rememberSettings@HighFlexSettings@U2@@QAEXXZ$6 100117a6 f   HighFlexSettings.obj
 0001:000107af       __unwindfunclet$?rememberSettings@HighFlexSettings@U2@@QAEXXZ$7 100117af f   HighFlexSettings.obj
 0001:000107b8       __unwindfunclet$?rememberSettings@HighFlexSettings@U2@@QAEXXZ$8 100117b8 f   HighFlexSettings.obj
 0001:000107c1       __ehhandler$?rememberSettings@HighFlexSettings@U2@@QAEXXZ 100117c1 f   HighFlexSettings.obj
 0001:000107e0       __unwindfunclet$?restoreDefaults@HighFlexSettings@U2@@QAEXXZ$0 100117e0 f   HighFlexSettings.obj
 0001:000107e9       __unwindfunclet$?restoreDefaults@HighFlexSettings@U2@@QAEXXZ$1 100117e9 f   HighFlexSettings.obj
 0001:000107f2       __unwindfunclet$?restoreDefaults@HighFlexSettings@U2@@QAEXXZ$2 100117f2 f   HighFlexSettings.obj
 0001:000107fb       __unwindfunclet$?restoreDefaults@HighFlexSettings@U2@@QAEXXZ$3 100117fb f   HighFlexSettings.obj
 0001:00010804       __unwindfunclet$?restoreDefaults@HighFlexSettings@U2@@QAEXXZ$4 10011804 f   HighFlexSettings.obj
 0001:0001080d       __unwindfunclet$?restoreDefaults@HighFlexSettings@U2@@QAEXXZ$5 1001180d f   HighFlexSettings.obj
 0001:00010816       __ehhandler$?restoreDefaults@HighFlexSettings@U2@@QAEXXZ 10011816 f   HighFlexSettings.obj
 0001:00010840       __unwindfunclet$?restoreRememberedSettings@HighFlexSettings@U2@@AAE_NXZ$0 10011840 f   HighFlexSettings.obj
 0001:00010849       __unwindfunclet$?restoreRememberedSettings@HighFlexSettings@U2@@AAE_NXZ$1 10011849 f   HighFlexSettings.obj
 0001:00010852       __unwindfunclet$?restoreRememberedSettings@HighFlexSettings@U2@@AAE_NXZ$2 10011852 f   HighFlexSettings.obj
 0001:0001085b       __unwindfunclet$?restoreRememberedSettings@HighFlexSettings@U2@@AAE_NXZ$3 1001185b f   HighFlexSettings.obj
 0001:00010867       __unwindfunclet$?restoreRememberedSettings@HighFlexSettings@U2@@AAE_NXZ$4 10011867 f   HighFlexSettings.obj
 0001:00010870       __unwindfunclet$?restoreRememberedSettings@HighFlexSettings@U2@@AAE_NXZ$5 10011870 f   HighFlexSettings.obj
 0001:00010879       __unwindfunclet$?restoreRememberedSettings@HighFlexSettings@U2@@AAE_NXZ$6 10011879 f   HighFlexSettings.obj
 0001:00010882       __unwindfunclet$?restoreRememberedSettings@HighFlexSettings@U2@@AAE_NXZ$7 10011882 f   HighFlexSettings.obj
 0001:0001088b       __unwindfunclet$?restoreRememberedSettings@HighFlexSettings@U2@@AAE_NXZ$8 1001188b f   HighFlexSettings.obj
 0001:00010894       __unwindfunclet$?restoreRememberedSettings@HighFlexSettings@U2@@AAE_NXZ$9 10011894 f   HighFlexSettings.obj
 0001:0001089d       __unwindfunclet$?restoreRememberedSettings@HighFlexSettings@U2@@AAE_NXZ$10 1001189d f   HighFlexSettings.obj
 0001:000108a6       __unwindfunclet$?restoreRememberedSettings@HighFlexSettings@U2@@AAE_NXZ$11 100118a6 f   HighFlexSettings.obj
 0001:000108af       __unwindfunclet$?restoreRememberedSettings@HighFlexSettings@U2@@AAE_NXZ$12 100118af f   HighFlexSettings.obj
 0001:000108b8       __unwindfunclet$?restoreRememberedSettings@HighFlexSettings@U2@@AAE_NXZ$13 100118b8 f   HighFlexSettings.obj
 0001:000108c1       __unwindfunclet$?restoreRememberedSettings@HighFlexSettings@U2@@AAE_NXZ$14 100118c1 f   HighFlexSettings.obj
 0001:000108ca       __ehhandler$?restoreRememberedSettings@HighFlexSettings@U2@@AAE_NXZ 100118ca f   HighFlexSettings.obj
 0001:000108f0       __unwindfunclet$??__EalgoLog@U2@@YAXXZ$0 100118f0 f   moc_DNAFlexGraph.obj
 0001:000108f9       __ehhandler$??__EalgoLog@U2@@YAXXZ 100118f9 f   moc_DNAFlexGraph.obj
 0001:00010920       __unwindfunclet$??__EcmdLog@U2@@YAXXZ$0 10011920 f   moc_DNAFlexGraph.obj
 0001:00010929       __ehhandler$??__EcmdLog@U2@@YAXXZ 10011929 f   moc_DNAFlexGraph.obj
 0001:00010950       __unwindfunclet$??__EcoreLog@U2@@YAXXZ$0 10011950 f   moc_DNAFlexGraph.obj
 0001:00010959       __ehhandler$??__EcoreLog@U2@@YAXXZ 10011959 f   moc_DNAFlexGraph.obj
 0001:00010980       __unwindfunclet$??__EioLog@U2@@YAXXZ$0 10011980 f   moc_DNAFlexGraph.obj
 0001:00010989       __ehhandler$??__EioLog@U2@@YAXXZ 10011989 f   moc_DNAFlexGraph.obj
 0001:000109b0       __unwindfunclet$??__EperfLog@U2@@YAXXZ$0 100119b0 f   moc_DNAFlexGraph.obj
 0001:000109b9       __ehhandler$??__EperfLog@U2@@YAXXZ 100119b9 f   moc_DNAFlexGraph.obj
 0001:000109e0       __unwindfunclet$??__EscriptLog@U2@@YAXXZ$0 100119e0 f   moc_DNAFlexGraph.obj
 0001:000109e9       __ehhandler$??__EscriptLog@U2@@YAXXZ 100119e9 f   moc_DNAFlexGraph.obj
 0001:00010a10       __unwindfunclet$??__EtaskLog@U2@@YAXXZ$0 10011a10 f   moc_DNAFlexGraph.obj
 0001:00010a19       __ehhandler$??__EtaskLog@U2@@YAXXZ 10011a19 f   moc_DNAFlexGraph.obj
 0001:00010a40       __unwindfunclet$??__EuiLog@U2@@YAXXZ$0 10011a40 f   moc_DNAFlexGraph.obj
 0001:00010a49       __ehhandler$??__EuiLog@U2@@YAXXZ 10011a49 f   moc_DNAFlexGraph.obj
 0001:00010a70       __unwindfunclet$??__EuserActLog@U2@@YAXXZ$0 10011a70 f   moc_DNAFlexGraph.obj
 0001:00010a79       __ehhandler$??__EuserActLog@U2@@YAXXZ 10011a79 f   moc_DNAFlexGraph.obj
 0001:00010aa0       __unwindfunclet$??__EalgoLog@U2@@YAXXZ$0 10011aa0 f   moc_DNAFlexPlugin.obj
 0001:00010aa9       __ehhandler$??__EalgoLog@U2@@YAXXZ 10011aa9 f   moc_DNAFlexPlugin.obj
 0001:00010ad0       __unwindfunclet$??__EcmdLog@U2@@YAXXZ$0 10011ad0 f   moc_DNAFlexPlugin.obj
 0001:00010ad9       __ehhandler$??__EcmdLog@U2@@YAXXZ 10011ad9 f   moc_DNAFlexPlugin.obj
 0001:00010b00       __unwindfunclet$??__EcoreLog@U2@@YAXXZ$0 10011b00 f   moc_DNAFlexPlugin.obj
 0001:00010b09       __ehhandler$??__EcoreLog@U2@@YAXXZ 10011b09 f   moc_DNAFlexPlugin.obj
 0001:00010b30       __unwindfunclet$??__EioLog@U2@@YAXXZ$0 10011b30 f   moc_DNAFlexPlugin.obj
 0001:00010b39       __ehhandler$??__EioLog@U2@@YAXXZ 10011b39 f   moc_DNAFlexPlugin.obj
 0001:00010b60       __unwindfunclet$??__EperfLog@U2@@YAXXZ$0 10011b60 f   moc_DNAFlexPlugin.obj
 0001:00010b69       __ehhandler$??__EperfLog@U2@@YAXXZ 10011b69 f   moc_DNAFlexPlugin.obj
 0001:00010b90       __unwindfunclet$??__EscriptLog@U2@@YAXXZ$0 10011b90 f   moc_DNAFlexPlugin.obj
 0001:00010b99       __ehhandler$??__EscriptLog@U2@@YAXXZ 10011b99 f   moc_DNAFlexPlugin.obj
 0001:00010bc0       __unwindfunclet$??__EtaskLog@U2@@YAXXZ$0 10011bc0 f   moc_DNAFlexPlugin.obj
 0001:00010bc9       __ehhandler$??__EtaskLog@U2@@YAXXZ 10011bc9 f   moc_DNAFlexPlugin.obj
 0001:00010bf0       __unwindfunclet$??__EuiLog@U2@@YAXXZ$0 10011bf0 f   moc_DNAFlexPlugin.obj
 0001:00010bf9       __ehhandler$??__EuiLog@U2@@YAXXZ 10011bf9 f   moc_DNAFlexPlugin.obj
 0001:00010c20       __unwindfunclet$??__EuserActLog@U2@@YAXXZ$0 10011c20 f   moc_DNAFlexPlugin.obj
 0001:00010c29       __ehhandler$??__EuserActLog@U2@@YAXXZ 10011c29 f   moc_DNAFlexPlugin.obj
 0001:00010c50       __unwindfunclet$?qt_metatype_id@?$QMetaTypeIdQObject@PAVADVSequenceWidget@U2@@$00@@SAHXZ$0 10011c50 f   moc_DNAFlexPlugin.obj
 0001:00010c59       __ehhandler$?qt_metatype_id@?$QMetaTypeIdQObject@PAVADVSequenceWidget@U2@@$00@@SAHXZ 10011c59 f   moc_DNAFlexPlugin.obj
 0001:00010c80       __unwindfunclet$??__EalgoLog@U2@@YAXXZ$0 10011c80 f   moc_DNAFlexTask.obj
 0001:00010c89       __ehhandler$??__EalgoLog@U2@@YAXXZ 10011c89 f   moc_DNAFlexTask.obj
 0001:00010cb0       __unwindfunclet$??__EcmdLog@U2@@YAXXZ$0 10011cb0 f   moc_DNAFlexTask.obj
 0001:00010cb9       __ehhandler$??__EcmdLog@U2@@YAXXZ 10011cb9 f   moc_DNAFlexTask.obj
 0001:00010ce0       __unwindfunclet$??__EcoreLog@U2@@YAXXZ$0 10011ce0 f   moc_DNAFlexTask.obj
 0001:00010ce9       __ehhandler$??__EcoreLog@U2@@YAXXZ 10011ce9 f   moc_DNAFlexTask.obj
 0001:00010d10       __unwindfunclet$??__EioLog@U2@@YAXXZ$0 10011d10 f   moc_DNAFlexTask.obj
 0001:00010d19       __ehhandler$??__EioLog@U2@@YAXXZ 10011d19 f   moc_DNAFlexTask.obj
 0001:00010d40       __unwindfunclet$??__EperfLog@U2@@YAXXZ$0 10011d40 f   moc_DNAFlexTask.obj
 0001:00010d49       __ehhandler$??__EperfLog@U2@@YAXXZ 10011d49 f   moc_DNAFlexTask.obj
 0001:00010d70       __unwindfunclet$??__EscriptLog@U2@@YAXXZ$0 10011d70 f   moc_DNAFlexTask.obj
 0001:00010d79       __ehhandler$??__EscriptLog@U2@@YAXXZ 10011d79 f   moc_DNAFlexTask.obj
 0001:00010da0       __unwindfunclet$??__EtaskLog@U2@@YAXXZ$0 10011da0 f   moc_DNAFlexTask.obj
 0001:00010da9       __ehhandler$??__EtaskLog@U2@@YAXXZ 10011da9 f   moc_DNAFlexTask.obj
 0001:00010dd0       __unwindfunclet$??__EuiLog@U2@@YAXXZ$0 10011dd0 f   moc_DNAFlexTask.obj
 0001:00010dd9       __ehhandler$??__EuiLog@U2@@YAXXZ 10011dd9 f   moc_DNAFlexTask.obj
 0001:00010e00       __unwindfunclet$??__EuserActLog@U2@@YAXXZ$0 10011e00 f   moc_DNAFlexTask.obj
 0001:00010e09       __ehhandler$??__EuserActLog@U2@@YAXXZ 10011e09 f   moc_DNAFlexTask.obj
 0001:00010e30       __unwindfunclet$??__EalgoLog@U2@@YAXXZ$0 10011e30 f   moc_FindHighFlexRegions.obj
 0001:00010e39       __ehhandler$??__EalgoLog@U2@@YAXXZ 10011e39 f   moc_FindHighFlexRegions.obj
 0001:00010e60       __unwindfunclet$??__EcmdLog@U2@@YAXXZ$0 10011e60 f   moc_FindHighFlexRegions.obj
 0001:00010e69       __ehhandler$??__EcmdLog@U2@@YAXXZ 10011e69 f   moc_FindHighFlexRegions.obj
 0001:00010e90       __unwindfunclet$??__EcoreLog@U2@@YAXXZ$0 10011e90 f   moc_FindHighFlexRegions.obj
 0001:00010e99       __ehhandler$??__EcoreLog@U2@@YAXXZ 10011e99 f   moc_FindHighFlexRegions.obj
 0001:00010ec0       __unwindfunclet$??__EioLog@U2@@YAXXZ$0 10011ec0 f   moc_FindHighFlexRegions.obj
 0001:00010ec9       __ehhandler$??__EioLog@U2@@YAXXZ 10011ec9 f   moc_FindHighFlexRegions.obj
 0001:00010ef0       __unwindfunclet$??__EperfLog@U2@@YAXXZ$0 10011ef0 f   moc_FindHighFlexRegions.obj
 0001:00010ef9       __ehhandler$??__EperfLog@U2@@YAXXZ 10011ef9 f   moc_FindHighFlexRegions.obj
 0001:00010f20       __unwindfunclet$??__EscriptLog@U2@@YAXXZ$0 10011f20 f   moc_FindHighFlexRegions.obj
 0001:00010f29       __ehhandler$??__EscriptLog@U2@@YAXXZ 10011f29 f   moc_FindHighFlexRegions.obj
 0001:00010f50       __unwindfunclet$??__EtaskLog@U2@@YAXXZ$0 10011f50 f   moc_FindHighFlexRegions.obj
 0001:00010f59       __ehhandler$??__EtaskLog@U2@@YAXXZ 10011f59 f   moc_FindHighFlexRegions.obj
 0001:00010f80       __unwindfunclet$??__EuiLog@U2@@YAXXZ$0 10011f80 f   moc_FindHighFlexRegions.obj
 0001:00010f89       __ehhandler$??__EuiLog@U2@@YAXXZ 10011f89 f   moc_FindHighFlexRegions.obj
 0001:00010fb0       __unwindfunclet$??__EuserActLog@U2@@YAXXZ$0 10011fb0 f   moc_FindHighFlexRegions.obj
 0001:00010fb9       __ehhandler$??__EuserActLog@U2@@YAXXZ 10011fb9 f   moc_FindHighFlexRegions.obj
 0001:00010fe0       ??__F?_Generic_object@?$_Error_objects@H@std@@2V_Generic_error_category@2@A@@YAXXZ 10011fe0 f   DNAFlexDialog.obj
 0001:00010ff0       ??__F?_Iostream_object@?$_Error_objects@H@std@@2V_Iostream_error_category@2@A@@YAXXZ 10011ff0 f   DNAFlexDialog.obj
 0001:00011000       ??__F?_System_object@?$_Error_objects@H@std@@2V_System_error_category@2@A@@YAXXZ 10012000 f   DNAFlexDialog.obj
 0001:00011010       ??__FService_DNAExport@U2@@YAXXZ 10012010 f   DNAFlexDialog.obj
 0001:00011020       ??__FService_DNAGraphPack@U2@@YAXXZ 10012020 f   DNAFlexDialog.obj
 0001:00011030       ??__FService_ExternalToolSupport@U2@@YAXXZ 10012030 f   DNAFlexDialog.obj
 0001:00011040       ??__FService_GUITesting@U2@@YAXXZ 10012040 f   DNAFlexDialog.obj
 0001:00011050       ??__FService_MaxCoreServiceId@U2@@YAXXZ 10012050 f   DNAFlexDialog.obj
 0001:00011060       ??__FService_MinCoreServiceId@U2@@YAXXZ 10012060 f   DNAFlexDialog.obj
 0001:00011070       ??__FService_PluginViewer@U2@@YAXXZ 10012070 f   DNAFlexDialog.obj
 0001:00011080       ??__FService_Project@U2@@YAXXZ 10012080 f   DNAFlexDialog.obj
 0001:00011090       ??__FService_ProjectView@U2@@YAXXZ 10012090 f   DNAFlexDialog.obj
 0001:000110a0       ??__FService_QueryDesigner@U2@@YAXXZ 100120a0 f   DNAFlexDialog.obj
 0001:000110b0       ??__FService_ScriptRegistry@U2@@YAXXZ 100120b0 f   DNAFlexDialog.obj
 0001:000110c0       ??__FService_TestRunner@U2@@YAXXZ 100120c0 f   DNAFlexDialog.obj
 0001:000110d0       ??__FService_WorkflowDesigner@U2@@YAXXZ 100120d0 f   DNAFlexDialog.obj
 0001:000110e0       ??__FalgoLog@U2@@YAXXZ     100120e0 f   DNAFlexDialog.obj
 0001:000110f0       ??__FcmdLog@U2@@YAXXZ      100120f0 f   DNAFlexDialog.obj
 0001:00011100       ??__FcoreLog@U2@@YAXXZ     10012100 f   DNAFlexDialog.obj
 0001:00011110       ??__FioLog@U2@@YAXXZ       10012110 f   DNAFlexDialog.obj
 0001:00011120       ??__FperfLog@U2@@YAXXZ     10012120 f   DNAFlexDialog.obj
 0001:00011130       ??__FscriptLog@U2@@YAXXZ   10012130 f   DNAFlexDialog.obj
 0001:00011140       ??__FtaskLog@U2@@YAXXZ     10012140 f   DNAFlexDialog.obj
 0001:00011150       ??__FuiLog@U2@@YAXXZ       10012150 f   DNAFlexDialog.obj
 0001:00011160       ??__FuserActLog@U2@@YAXXZ  10012160 f   DNAFlexDialog.obj
 0001:00011170       ??__F?_Generic_object@?$_Error_objects@H@std@@2V_Generic_error_category@2@A@@YAXXZ 10012170 f   DNAFlexGraph.obj
 0001:00011180       ??__F?_Iostream_object@?$_Error_objects@H@std@@2V_Iostream_error_category@2@A@@YAXXZ 10012180 f   DNAFlexGraph.obj
 0001:00011190       ??__F?_System_object@?$_Error_objects@H@std@@2V_System_error_category@2@A@@YAXXZ 10012190 f   DNAFlexGraph.obj
 0001:000111a0       ??__FService_DNAExport@U2@@YAXXZ 100121a0 f   DNAFlexGraph.obj
 0001:000111b0       ??__FService_DNAGraphPack@U2@@YAXXZ 100121b0 f   DNAFlexGraph.obj
 0001:000111c0       ??__FService_ExternalToolSupport@U2@@YAXXZ 100121c0 f   DNAFlexGraph.obj
 0001:000111d0       ??__FService_GUITesting@U2@@YAXXZ 100121d0 f   DNAFlexGraph.obj
 0001:000111e0       ??__FService_MaxCoreServiceId@U2@@YAXXZ 100121e0 f   DNAFlexGraph.obj
 0001:000111f0       ??__FService_MinCoreServiceId@U2@@YAXXZ 100121f0 f   DNAFlexGraph.obj
 0001:00011200       ??__FService_PluginViewer@U2@@YAXXZ 10012200 f   DNAFlexGraph.obj
 0001:00011210       ??__FService_Project@U2@@YAXXZ 10012210 f   DNAFlexGraph.obj
 0001:00011220       ??__FService_ProjectView@U2@@YAXXZ 10012220 f   DNAFlexGraph.obj
 0001:00011230       ??__FService_QueryDesigner@U2@@YAXXZ 10012230 f   DNAFlexGraph.obj
 0001:00011240       ??__FService_ScriptRegistry@U2@@YAXXZ 10012240 f   DNAFlexGraph.obj
 0001:00011250       ??__FService_TestRunner@U2@@YAXXZ 10012250 f   DNAFlexGraph.obj
 0001:00011260       ??__FService_WorkflowDesigner@U2@@YAXXZ 10012260 f   DNAFlexGraph.obj
 0001:00011270       ??__FalgoLog@U2@@YAXXZ     10012270 f   DNAFlexGraph.obj
 0001:00011280       ??__FcmdLog@U2@@YAXXZ      10012280 f   DNAFlexGraph.obj
 0001:00011290       ??__FcoreLog@U2@@YAXXZ     10012290 f   DNAFlexGraph.obj
 0001:000112a0       ??__FioLog@U2@@YAXXZ       100122a0 f   DNAFlexGraph.obj
 0001:000112b0       ??__FperfLog@U2@@YAXXZ     100122b0 f   DNAFlexGraph.obj
 0001:000112c0       ??__FscriptLog@U2@@YAXXZ   100122c0 f   DNAFlexGraph.obj
 0001:000112d0       ??__FtaskLog@U2@@YAXXZ     100122d0 f   DNAFlexGraph.obj
 0001:000112e0       ??__FuiLog@U2@@YAXXZ       100122e0 f   DNAFlexGraph.obj
 0001:000112f0       ??__FuserActLog@U2@@YAXXZ  100122f0 f   DNAFlexGraph.obj
 0001:00011300       ??__F?_Generic_object@?$_Error_objects@H@std@@2V_Generic_error_category@2@A@@YAXXZ 10012300 f   DNAFlexGraphAlgorithm.obj
 0001:00011310       ??__F?_Iostream_object@?$_Error_objects@H@std@@2V_Iostream_error_category@2@A@@YAXXZ 10012310 f   DNAFlexGraphAlgorithm.obj
 0001:00011320       ??__F?_System_object@?$_Error_objects@H@std@@2V_System_error_category@2@A@@YAXXZ 10012320 f   DNAFlexGraphAlgorithm.obj
 0001:00011330       ??__FService_DNAExport@U2@@YAXXZ 10012330 f   DNAFlexGraphAlgorithm.obj
 0001:00011340       ??__FService_DNAGraphPack@U2@@YAXXZ 10012340 f   DNAFlexGraphAlgorithm.obj
 0001:00011350       ??__FService_ExternalToolSupport@U2@@YAXXZ 10012350 f   DNAFlexGraphAlgorithm.obj
 0001:00011360       ??__FService_GUITesting@U2@@YAXXZ 10012360 f   DNAFlexGraphAlgorithm.obj
 0001:00011370       ??__FService_MaxCoreServiceId@U2@@YAXXZ 10012370 f   DNAFlexGraphAlgorithm.obj
 0001:00011380       ??__FService_MinCoreServiceId@U2@@YAXXZ 10012380 f   DNAFlexGraphAlgorithm.obj
 0001:00011390       ??__FService_PluginViewer@U2@@YAXXZ 10012390 f   DNAFlexGraphAlgorithm.obj
 0001:000113a0       ??__FService_Project@U2@@YAXXZ 100123a0 f   DNAFlexGraphAlgorithm.obj
 0001:000113b0       ??__FService_ProjectView@U2@@YAXXZ 100123b0 f   DNAFlexGraphAlgorithm.obj
 0001:000113c0       ??__FService_QueryDesigner@U2@@YAXXZ 100123c0 f   DNAFlexGraphAlgorithm.obj
 0001:000113d0       ??__FService_ScriptRegistry@U2@@YAXXZ 100123d0 f   DNAFlexGraphAlgorithm.obj
 0001:000113e0       ??__FService_TestRunner@U2@@YAXXZ 100123e0 f   DNAFlexGraphAlgorithm.obj
 0001:000113f0       ??__FService_WorkflowDesigner@U2@@YAXXZ 100123f0 f   DNAFlexGraphAlgorithm.obj
 0001:00011400       ??__FalgoLog@U2@@YAXXZ     10012400 f   DNAFlexGraphAlgorithm.obj
 0001:00011410       ??__FcmdLog@U2@@YAXXZ      10012410 f   DNAFlexGraphAlgorithm.obj
 0001:00011420       ??__FcoreLog@U2@@YAXXZ     10012420 f   DNAFlexGraphAlgorithm.obj
 0001:00011430       ??__FioLog@U2@@YAXXZ       10012430 f   DNAFlexGraphAlgorithm.obj
 0001:00011440       ??__FperfLog@U2@@YAXXZ     10012440 f   DNAFlexGraphAlgorithm.obj
 0001:00011450       ??__FscriptLog@U2@@YAXXZ   10012450 f   DNAFlexGraphAlgorithm.obj
 0001:00011460       ??__FtaskLog@U2@@YAXXZ     10012460 f   DNAFlexGraphAlgorithm.obj
 0001:00011470       ??__FuiLog@U2@@YAXXZ       10012470 f   DNAFlexGraphAlgorithm.obj
 0001:00011480       ??__FuserActLog@U2@@YAXXZ  10012480 f   DNAFlexGraphAlgorithm.obj
 0001:00011490       ??__F?_Generic_object@?$_Error_objects@H@std@@2V_Generic_error_category@2@A@@YAXXZ 10012490 f   DNAFlexPlugin.obj
 0001:000114a0       ??__F?_Iostream_object@?$_Error_objects@H@std@@2V_Iostream_error_category@2@A@@YAXXZ 100124a0 f   DNAFlexPlugin.obj
 0001:000114b0       ??__F?_System_object@?$_Error_objects@H@std@@2V_System_error_category@2@A@@YAXXZ 100124b0 f   DNAFlexPlugin.obj
 0001:000114c0       ??__FService_DNAExport@U2@@YAXXZ 100124c0 f   DNAFlexPlugin.obj
 0001:000114d0       ??__FService_DNAGraphPack@U2@@YAXXZ 100124d0 f   DNAFlexPlugin.obj
 0001:000114e0       ??__FService_ExternalToolSupport@U2@@YAXXZ 100124e0 f   DNAFlexPlugin.obj
 0001:000114f0       ??__FService_GUITesting@U2@@YAXXZ 100124f0 f   DNAFlexPlugin.obj
 0001:00011500       ??__FService_MaxCoreServiceId@U2@@YAXXZ 10012500 f   DNAFlexPlugin.obj
 0001:00011510       ??__FService_MinCoreServiceId@U2@@YAXXZ 10012510 f   DNAFlexPlugin.obj
 0001:00011520       ??__FService_PluginViewer@U2@@YAXXZ 10012520 f   DNAFlexPlugin.obj
 0001:00011530       ??__FService_Project@U2@@YAXXZ 10012530 f   DNAFlexPlugin.obj
 0001:00011540       ??__FService_ProjectView@U2@@YAXXZ 10012540 f   DNAFlexPlugin.obj
 0001:00011550       ??__FService_QueryDesigner@U2@@YAXXZ 10012550 f   DNAFlexPlugin.obj
 0001:00011560       ??__FService_ScriptRegistry@U2@@YAXXZ 10012560 f   DNAFlexPlugin.obj
 0001:00011570       ??__FService_TestRunner@U2@@YAXXZ 10012570 f   DNAFlexPlugin.obj
 0001:00011580       ??__FService_WorkflowDesigner@U2@@YAXXZ 10012580 f   DNAFlexPlugin.obj
 0001:00011590       ??__FalgoLog@U2@@YAXXZ     10012590 f   DNAFlexPlugin.obj
 0001:000115a0       ??__FcmdLog@U2@@YAXXZ      100125a0 f   DNAFlexPlugin.obj
 0001:000115b0       ??__FcoreLog@U2@@YAXXZ     100125b0 f   DNAFlexPlugin.obj
 0001:000115c0       ??__FioLog@U2@@YAXXZ       100125c0 f   DNAFlexPlugin.obj
 0001:000115d0       ??__FperfLog@U2@@YAXXZ     100125d0 f   DNAFlexPlugin.obj
 0001:000115e0       ??__FscriptLog@U2@@YAXXZ   100125e0 f   DNAFlexPlugin.obj
 0001:000115f0       ??__FtaskLog@U2@@YAXXZ     100125f0 f   DNAFlexPlugin.obj
 0001:00011600       ??__FuiLog@U2@@YAXXZ       10012600 f   DNAFlexPlugin.obj
 0001:00011610       ??__FuserActLog@U2@@YAXXZ  10012610 f   DNAFlexPlugin.obj
 0001:00011620       ??__F?_Generic_object@?$_Error_objects@H@std@@2V_Generic_error_category@2@A@@YAXXZ 10012620 f   DNAFlexTask.obj
 0001:00011630       ??__F?_Iostream_object@?$_Error_objects@H@std@@2V_Iostream_error_category@2@A@@YAXXZ 10012630 f   DNAFlexTask.obj
 0001:00011640       ??__F?_System_object@?$_Error_objects@H@std@@2V_System_error_category@2@A@@YAXXZ 10012640 f   DNAFlexTask.obj
 0001:00011650       ??__FalgoLog@U2@@YAXXZ     10012650 f   DNAFlexTask.obj
 0001:00011660       ??__FcmdLog@U2@@YAXXZ      10012660 f   DNAFlexTask.obj
 0001:00011670       ??__FcoreLog@U2@@YAXXZ     10012670 f   DNAFlexTask.obj
 0001:00011680       ??__FioLog@U2@@YAXXZ       10012680 f   DNAFlexTask.obj
 0001:00011690       ??__FperfLog@U2@@YAXXZ     10012690 f   DNAFlexTask.obj
 0001:000116a0       ??__FscriptLog@U2@@YAXXZ   100126a0 f   DNAFlexTask.obj
 0001:000116b0       ??__FtaskLog@U2@@YAXXZ     100126b0 f   DNAFlexTask.obj
 0001:000116c0       ??__FuiLog@U2@@YAXXZ       100126c0 f   DNAFlexTask.obj
 0001:000116d0       ??__FuserActLog@U2@@YAXXZ  100126d0 f   DNAFlexTask.obj
 0001:000116e0       ??__F?_Generic_object@?$_Error_objects@H@std@@2V_Generic_error_category@2@A@@YAXXZ 100126e0 f   FindHighFlexRegions.obj
 0001:000116f0       ??__F?_Iostream_object@?$_Error_objects@H@std@@2V_Iostream_error_category@2@A@@YAXXZ 100126f0 f   FindHighFlexRegions.obj
 0001:00011700       ??__F?_System_object@?$_Error_objects@H@std@@2V_System_error_category@2@A@@YAXXZ 10012700 f   FindHighFlexRegions.obj
 0001:00011710       ??__FalgoLog@U2@@YAXXZ     10012710 f   FindHighFlexRegions.obj
 0001:00011720       ??__FcmdLog@U2@@YAXXZ      10012720 f   FindHighFlexRegions.obj
 0001:00011730       ??__FcoreLog@U2@@YAXXZ     10012730 f   FindHighFlexRegions.obj
 0001:00011740       ??__FioLog@U2@@YAXXZ       10012740 f   FindHighFlexRegions.obj
 0001:00011750       ??__FperfLog@U2@@YAXXZ     10012750 f   FindHighFlexRegions.obj
 0001:00011760       ??__FscriptLog@U2@@YAXXZ   10012760 f   FindHighFlexRegions.obj
 0001:00011770       ??__FtaskLog@U2@@YAXXZ     10012770 f   FindHighFlexRegions.obj
 0001:00011780       ??__FuiLog@U2@@YAXXZ       10012780 f   FindHighFlexRegions.obj
 0001:00011790       ??__FuserActLog@U2@@YAXXZ  10012790 f   FindHighFlexRegions.obj
 0001:000117a0       ??__F?_Generic_object@?$_Error_objects@H@std@@2V_Generic_error_category@2@A@@YAXXZ 100127a0 f   FindHighFlexRegionsAlgorithm.obj
 0001:000117b0       ??__F?_Iostream_object@?$_Error_objects@H@std@@2V_Iostream_error_category@2@A@@YAXXZ 100127b0 f   FindHighFlexRegionsAlgorithm.obj
 0001:000117c0       ??__F?_System_object@?$_Error_objects@H@std@@2V_System_error_category@2@A@@YAXXZ 100127c0 f   FindHighFlexRegionsAlgorithm.obj
 0001:000117d0       ??__FalgoLog@U2@@YAXXZ     100127d0 f   FindHighFlexRegionsAlgorithm.obj
 0001:000117e0       ??__FcmdLog@U2@@YAXXZ      100127e0 f   FindHighFlexRegionsAlgorithm.obj
 0001:000117f0       ??__FcoreLog@U2@@YAXXZ     100127f0 f   FindHighFlexRegionsAlgorithm.obj
 0001:00011800       ??__FioLog@U2@@YAXXZ       10012800 f   FindHighFlexRegionsAlgorithm.obj
 0001:00011810       ??__FperfLog@U2@@YAXXZ     10012810 f   FindHighFlexRegionsAlgorithm.obj
 0001:00011820       ??__FscriptLog@U2@@YAXXZ   10012820 f   FindHighFlexRegionsAlgorithm.obj
 0001:00011830       ??__FtaskLog@U2@@YAXXZ     10012830 f   FindHighFlexRegionsAlgorithm.obj
 0001:00011840       ??__FuiLog@U2@@YAXXZ       10012840 f   FindHighFlexRegionsAlgorithm.obj
 0001:00011850       ??__FuserActLog@U2@@YAXXZ  10012850 f   FindHighFlexRegionsAlgorithm.obj
 0001:00011860       ??__F?SETTINGS_PATH@HighFlexSettings@U2@@0VQString@@B@@YAXXZ 10012860 f   HighFlexSettings.obj
 0001:00011870       ??__F?SETTING_THRESHOLD@HighFlexSettings@U2@@0VQString@@B@@YAXXZ 10012870 f   HighFlexSettings.obj
 0001:00011880       ??__F?SETTING_WINDOW_SIZE@HighFlexSettings@U2@@0VQString@@B@@YAXXZ 10012880 f   HighFlexSettings.obj
 0001:00011890       ??__F?SETTING_WINDOW_STEP@HighFlexSettings@U2@@0VQString@@B@@YAXXZ 10012890 f   HighFlexSettings.obj
 0001:000118a0       ??__F?_Generic_object@?$_Error_objects@H@std@@2V_Generic_error_category@2@A@@YAXXZ 100128a0 f   HighFlexSettings.obj
 0001:000118b0       ??__F?_Iostream_object@?$_Error_objects@H@std@@2V_Iostream_error_category@2@A@@YAXXZ 100128b0 f   HighFlexSettings.obj
 0001:000118c0       ??__F?_System_object@?$_Error_objects@H@std@@2V_System_error_category@2@A@@YAXXZ 100128c0 f   HighFlexSettings.obj
 0001:000118d0       ??__FalgoLog@U2@@YAXXZ     100128d0 f   HighFlexSettings.obj
 0001:000118e0       ??__FcmdLog@U2@@YAXXZ      100128e0 f   HighFlexSettings.obj
 0001:000118f0       ??__FcoreLog@U2@@YAXXZ     100128f0 f   HighFlexSettings.obj
 0001:00011900       ??__FioLog@U2@@YAXXZ       10012900 f   HighFlexSettings.obj
 0001:00011910       ??__FperfLog@U2@@YAXXZ     10012910 f   HighFlexSettings.obj
 0001:00011920       ??__FscriptLog@U2@@YAXXZ   10012920 f   HighFlexSettings.obj
 0001:00011930       ??__FtaskLog@U2@@YAXXZ     10012930 f   HighFlexSettings.obj
 0001:00011940       ??__FuiLog@U2@@YAXXZ       10012940 f   HighFlexSettings.obj
 0001:00011950       ??__FuserActLog@U2@@YAXXZ  10012950 f   HighFlexSettings.obj
 0001:00011960       ??__F?_Generic_object@?$_Error_objects@H@std@@2V_Generic_error_category@2@A@@YAXXZ 10012960 f   moc_DNAFlexDialog.obj
 0001:00011970       ??__F?_Iostream_object@?$_Error_objects@H@std@@2V_Iostream_error_category@2@A@@YAXXZ 10012970 f   moc_DNAFlexDialog.obj
 0001:00011980       ??__F?_System_object@?$_Error_objects@H@std@@2V_System_error_category@2@A@@YAXXZ 10012980 f   moc_DNAFlexDialog.obj
 0001:00011990       ??__F?_Generic_object@?$_Error_objects@H@std@@2V_Generic_error_category@2@A@@YAXXZ 10012990 f   moc_DNAFlexGraph.obj
 0001:000119a0       ??__F?_Iostream_object@?$_Error_objects@H@std@@2V_Iostream_error_category@2@A@@YAXXZ 100129a0 f   moc_DNAFlexGraph.obj
 0001:000119b0       ??__F?_System_object@?$_Error_objects@H@std@@2V_System_error_category@2@A@@YAXXZ 100129b0 f   moc_DNAFlexGraph.obj
 0001:000119c0       ??__FService_DNAExport@U2@@YAXXZ 100129c0 f   moc_DNAFlexGraph.obj
 0001:000119d0       ??__FService_DNAGraphPack@U2@@YAXXZ 100129d0 f   moc_DNAFlexGraph.obj
 0001:000119e0       ??__FService_ExternalToolSupport@U2@@YAXXZ 100129e0 f   moc_DNAFlexGraph.obj
 0001:000119f0       ??__FService_GUITesting@U2@@YAXXZ 100129f0 f   moc_DNAFlexGraph.obj
 0001:00011a00       ??__FService_MaxCoreServiceId@U2@@YAXXZ 10012a00 f   moc_DNAFlexGraph.obj
 0001:00011a10       ??__FService_MinCoreServiceId@U2@@YAXXZ 10012a10 f   moc_DNAFlexGraph.obj
 0001:00011a20       ??__FService_PluginViewer@U2@@YAXXZ 10012a20 f   moc_DNAFlexGraph.obj
 0001:00011a30       ??__FService_Project@U2@@YAXXZ 10012a30 f   moc_DNAFlexGraph.obj
 0001:00011a40       ??__FService_ProjectView@U2@@YAXXZ 10012a40 f   moc_DNAFlexGraph.obj
 0001:00011a50       ??__FService_QueryDesigner@U2@@YAXXZ 10012a50 f   moc_DNAFlexGraph.obj
 0001:00011a60       ??__FService_ScriptRegistry@U2@@YAXXZ 10012a60 f   moc_DNAFlexGraph.obj
 0001:00011a70       ??__FService_TestRunner@U2@@YAXXZ 10012a70 f   moc_DNAFlexGraph.obj
 0001:00011a80       ??__FService_WorkflowDesigner@U2@@YAXXZ 10012a80 f   moc_DNAFlexGraph.obj
 0001:00011a90       ??__FalgoLog@U2@@YAXXZ     10012a90 f   moc_DNAFlexGraph.obj
 0001:00011aa0       ??__FcmdLog@U2@@YAXXZ      10012aa0 f   moc_DNAFlexGraph.obj
 0001:00011ab0       ??__FcoreLog@U2@@YAXXZ     10012ab0 f   moc_DNAFlexGraph.obj
 0001:00011ac0       ??__FioLog@U2@@YAXXZ       10012ac0 f   moc_DNAFlexGraph.obj
 0001:00011ad0       ??__FperfLog@U2@@YAXXZ     10012ad0 f   moc_DNAFlexGraph.obj
 0001:00011ae0       ??__FscriptLog@U2@@YAXXZ   10012ae0 f   moc_DNAFlexGraph.obj
 0001:00011af0       ??__FtaskLog@U2@@YAXXZ     10012af0 f   moc_DNAFlexGraph.obj
 0001:00011b00       ??__FuiLog@U2@@YAXXZ       10012b00 f   moc_DNAFlexGraph.obj
 0001:00011b10       ??__FuserActLog@U2@@YAXXZ  10012b10 f   moc_DNAFlexGraph.obj
 0001:00011b20       ??__F?_Generic_object@?$_Error_objects@H@std@@2V_Generic_error_category@2@A@@YAXXZ 10012b20 f   moc_DNAFlexPlugin.obj
 0001:00011b30       ??__F?_Iostream_object@?$_Error_objects@H@std@@2V_Iostream_error_category@2@A@@YAXXZ 10012b30 f   moc_DNAFlexPlugin.obj
 0001:00011b40       ??__F?_System_object@?$_Error_objects@H@std@@2V_System_error_category@2@A@@YAXXZ 10012b40 f   moc_DNAFlexPlugin.obj
 0001:00011b50       ??__FService_DNAExport@U2@@YAXXZ 10012b50 f   moc_DNAFlexPlugin.obj
 0001:00011b60       ??__FService_DNAGraphPack@U2@@YAXXZ 10012b60 f   moc_DNAFlexPlugin.obj
 0001:00011b70       ??__FService_ExternalToolSupport@U2@@YAXXZ 10012b70 f   moc_DNAFlexPlugin.obj
 0001:00011b80       ??__FService_GUITesting@U2@@YAXXZ 10012b80 f   moc_DNAFlexPlugin.obj
 0001:00011b90       ??__FService_MaxCoreServiceId@U2@@YAXXZ 10012b90 f   moc_DNAFlexPlugin.obj
 0001:00011ba0       ??__FService_MinCoreServiceId@U2@@YAXXZ 10012ba0 f   moc_DNAFlexPlugin.obj
 0001:00011bb0       ??__FService_PluginViewer@U2@@YAXXZ 10012bb0 f   moc_DNAFlexPlugin.obj
 0001:00011bc0       ??__FService_Project@U2@@YAXXZ 10012bc0 f   moc_DNAFlexPlugin.obj
 0001:00011bd0       ??__FService_ProjectView@U2@@YAXXZ 10012bd0 f   moc_DNAFlexPlugin.obj
 0001:00011be0       ??__FService_QueryDesigner@U2@@YAXXZ 10012be0 f   moc_DNAFlexPlugin.obj
 0001:00011bf0       ??__FService_ScriptRegistry@U2@@YAXXZ 10012bf0 f   moc_DNAFlexPlugin.obj
 0001:00011c00       ??__FService_TestRunner@U2@@YAXXZ 10012c00 f   moc_DNAFlexPlugin.obj
 0001:00011c10       ??__FService_WorkflowDesigner@U2@@YAXXZ 10012c10 f   moc_DNAFlexPlugin.obj
 0001:00011c20       ??__FalgoLog@U2@@YAXXZ     10012c20 f   moc_DNAFlexPlugin.obj
 0001:00011c30       ??__FcmdLog@U2@@YAXXZ      10012c30 f   moc_DNAFlexPlugin.obj
 0001:00011c40       ??__FcoreLog@U2@@YAXXZ     10012c40 f   moc_DNAFlexPlugin.obj
 0001:00011c50       ??__FioLog@U2@@YAXXZ       10012c50 f   moc_DNAFlexPlugin.obj
 0001:00011c60       ??__FperfLog@U2@@YAXXZ     10012c60 f   moc_DNAFlexPlugin.obj
 0001:00011c70       ??__FscriptLog@U2@@YAXXZ   10012c70 f   moc_DNAFlexPlugin.obj
 0001:00011c80       ??__FtaskLog@U2@@YAXXZ     10012c80 f   moc_DNAFlexPlugin.obj
 0001:00011c90       ??__FuiLog@U2@@YAXXZ       10012c90 f   moc_DNAFlexPlugin.obj
 0001:00011ca0       ??__FuserActLog@U2@@YAXXZ  10012ca0 f   moc_DNAFlexPlugin.obj
 0001:00011cb0       ??__F?_Generic_object@?$_Error_objects@H@std@@2V_Generic_error_category@2@A@@YAXXZ 10012cb0 f   moc_DNAFlexTask.obj
 0001:00011cc0       ??__F?_Iostream_object@?$_Error_objects@H@std@@2V_Iostream_error_category@2@A@@YAXXZ 10012cc0 f   moc_DNAFlexTask.obj
 0001:00011cd0       ??__F?_System_object@?$_Error_objects@H@std@@2V_System_error_category@2@A@@YAXXZ 10012cd0 f   moc_DNAFlexTask.obj
 0001:00011ce0       ??__FalgoLog@U2@@YAXXZ     10012ce0 f   moc_DNAFlexTask.obj
 0001:00011cf0       ??__FcmdLog@U2@@YAXXZ      10012cf0 f   moc_DNAFlexTask.obj
 0001:00011d00       ??__FcoreLog@U2@@YAXXZ     10012d00 f   moc_DNAFlexTask.obj
 0001:00011d10       ??__FioLog@U2@@YAXXZ       10012d10 f   moc_DNAFlexTask.obj
 0001:00011d20       ??__FperfLog@U2@@YAXXZ     10012d20 f   moc_DNAFlexTask.obj
 0001:00011d30       ??__FscriptLog@U2@@YAXXZ   10012d30 f   moc_DNAFlexTask.obj
 0001:00011d40       ??__FtaskLog@U2@@YAXXZ     10012d40 f   moc_DNAFlexTask.obj
 0001:00011d50       ??__FuiLog@U2@@YAXXZ       10012d50 f   moc_DNAFlexTask.obj
 0001:00011d60       ??__FuserActLog@U2@@YAXXZ  10012d60 f   moc_DNAFlexTask.obj
 0001:00011d70       ??__F?_Generic_object@?$_Error_objects@H@std@@2V_Generic_error_category@2@A@@YAXXZ 10012d70 f   moc_FindHighFlexRegions.obj
 0001:00011d80       ??__F?_Iostream_object@?$_Error_objects@H@std@@2V_Iostream_error_category@2@A@@YAXXZ 10012d80 f   moc_FindHighFlexRegions.obj
 0001:00011d90       ??__F?_System_object@?$_Error_objects@H@std@@2V_System_error_category@2@A@@YAXXZ 10012d90 f   moc_FindHighFlexRegions.obj
 0001:00011da0       ??__FalgoLog@U2@@YAXXZ     10012da0 f   moc_FindHighFlexRegions.obj
 0001:00011db0       ??__FcmdLog@U2@@YAXXZ      10012db0 f   moc_FindHighFlexRegions.obj
 0001:00011dc0       ??__FcoreLog@U2@@YAXXZ     10012dc0 f   moc_FindHighFlexRegions.obj
 0001:00011dd0       ??__FioLog@U2@@YAXXZ       10012dd0 f   moc_FindHighFlexRegions.obj
 0001:00011de0       ??__FperfLog@U2@@YAXXZ     10012de0 f   moc_FindHighFlexRegions.obj
 0001:00011df0       ??__FscriptLog@U2@@YAXXZ   10012df0 f   moc_FindHighFlexRegions.obj
 0001:00011e00       ??__FtaskLog@U2@@YAXXZ     10012e00 f   moc_FindHighFlexRegions.obj
 0001:00011e10       ??__FuiLog@U2@@YAXXZ       10012e10 f   moc_FindHighFlexRegions.obj
 0001:00011e20       ??__FuserActLog@U2@@YAXXZ  10012e20 f   moc_FindHighFlexRegions.obj
 0001:00011e30       ??__Fdummy@?A0xf1761197@@YAXXZ 10012e30 f   qrc_dna_flexibility.obj
 0002:000008bc       _algoLog$initializer$      100138bc     DNAFlexDialog.obj
 0002:000008c0       _cmdLog$initializer$       100138c0     DNAFlexDialog.obj
 0002:000008c4       _coreLog$initializer$      100138c4     DNAFlexDialog.obj
 0002:000008c8       _ioLog$initializer$        100138c8     DNAFlexDialog.obj
 0002:000008cc       _perfLog$initializer$      100138cc     DNAFlexDialog.obj
 0002:000008d0       _scriptLog$initializer$    100138d0     DNAFlexDialog.obj
 0002:000008d4       _taskLog$initializer$      100138d4     DNAFlexDialog.obj
 0002:000008d8       _uiLog$initializer$        100138d8     DNAFlexDialog.obj
 0002:000008dc       _userActLog$initializer$   100138dc     DNAFlexDialog.obj
 0002:000008e0       _Service_PluginViewer$initializer$ 100138e0     DNAFlexDialog.obj
 0002:000008e4       _Service_Project$initializer$ 100138e4     DNAFlexDialog.obj
 0002:000008e8       _Service_ProjectView$initializer$ 100138e8     DNAFlexDialog.obj
 0002:000008ec       _Service_DNAGraphPack$initializer$ 100138ec     DNAFlexDialog.obj
 0002:000008f0       _Service_DNAExport$initializer$ 100138f0     DNAFlexDialog.obj
 0002:000008f4       _Service_TestRunner$initializer$ 100138f4     DNAFlexDialog.obj
 0002:000008f8       _Service_ScriptRegistry$initializer$ 100138f8     DNAFlexDialog.obj
 0002:000008fc       _Service_ExternalToolSupport$initializer$ 100138fc     DNAFlexDialog.obj
 0002:00000900       _Service_GUITesting$initializer$ 10013900     DNAFlexDialog.obj
 0002:00000904       _Service_WorkflowDesigner$initializer$ 10013904     DNAFlexDialog.obj
 0002:00000908       _Service_QueryDesigner$initializer$ 10013908     DNAFlexDialog.obj
 0002:0000090c       _Service_MinCoreServiceId$initializer$ 1001390c     DNAFlexDialog.obj
 0002:00000910       _Service_MaxCoreServiceId$initializer$ 10013910     DNAFlexDialog.obj
 0002:00000914       ?_Generic_object$initializer$@?$_Error_objects@H@std@@2P6AXXZA 10013914     DNAFlexDialog.obj
 0002:00000918       ?_Iostream_object$initializer$@?$_Error_objects@H@std@@2P6AXXZA 10013918     DNAFlexDialog.obj
 0002:0000091c       ?_System_object$initializer$@?$_Error_objects@H@std@@2P6AXXZA 1001391c     DNAFlexDialog.obj
 0002:00000920       _Service_PluginViewer$initializer$ 10013920     DNAFlexGraph.obj
 0002:00000924       _Service_Project$initializer$ 10013924     DNAFlexGraph.obj
 0002:00000928       _Service_ProjectView$initializer$ 10013928     DNAFlexGraph.obj
 0002:0000092c       _Service_DNAGraphPack$initializer$ 1001392c     DNAFlexGraph.obj
 0002:00000930       _Service_DNAExport$initializer$ 10013930     DNAFlexGraph.obj
 0002:00000934       _Service_TestRunner$initializer$ 10013934     DNAFlexGraph.obj
 0002:00000938       _Service_ScriptRegistry$initializer$ 10013938     DNAFlexGraph.obj
 0002:0000093c       _Service_ExternalToolSupport$initializer$ 1001393c     DNAFlexGraph.obj
 0002:00000940       _Service_GUITesting$initializer$ 10013940     DNAFlexGraph.obj
 0002:00000944       _Service_WorkflowDesigner$initializer$ 10013944     DNAFlexGraph.obj
 0002:00000948       _Service_QueryDesigner$initializer$ 10013948     DNAFlexGraph.obj
 0002:0000094c       _Service_MinCoreServiceId$initializer$ 1001394c     DNAFlexGraph.obj
 0002:00000950       _Service_MaxCoreServiceId$initializer$ 10013950     DNAFlexGraph.obj
 0002:00000954       _algoLog$initializer$      10013954     DNAFlexGraph.obj
 0002:00000958       _cmdLog$initializer$       10013958     DNAFlexGraph.obj
 0002:0000095c       _coreLog$initializer$      1001395c     DNAFlexGraph.obj
 0002:00000960       _ioLog$initializer$        10013960     DNAFlexGraph.obj
 0002:00000964       _perfLog$initializer$      10013964     DNAFlexGraph.obj
 0002:00000968       _scriptLog$initializer$    10013968     DNAFlexGraph.obj
 0002:0000096c       _taskLog$initializer$      1001396c     DNAFlexGraph.obj
 0002:00000970       _uiLog$initializer$        10013970     DNAFlexGraph.obj
 0002:00000974       _userActLog$initializer$   10013974     DNAFlexGraph.obj
 0002:00000978       _Service_PluginViewer$initializer$ 10013978     DNAFlexGraphAlgorithm.obj
 0002:0000097c       _Service_Project$initializer$ 1001397c     DNAFlexGraphAlgorithm.obj
 0002:00000980       _Service_ProjectView$initializer$ 10013980     DNAFlexGraphAlgorithm.obj
 0002:00000984       _Service_DNAGraphPack$initializer$ 10013984     DNAFlexGraphAlgorithm.obj
 0002:00000988       _Service_DNAExport$initializer$ 10013988     DNAFlexGraphAlgorithm.obj
 0002:0000098c       _Service_TestRunner$initializer$ 1001398c     DNAFlexGraphAlgorithm.obj
 0002:00000990       _Service_ScriptRegistry$initializer$ 10013990     DNAFlexGraphAlgorithm.obj
 0002:00000994       _Service_ExternalToolSupport$initializer$ 10013994     DNAFlexGraphAlgorithm.obj
 0002:00000998       _Service_GUITesting$initializer$ 10013998     DNAFlexGraphAlgorithm.obj
 0002:0000099c       _Service_WorkflowDesigner$initializer$ 1001399c     DNAFlexGraphAlgorithm.obj
 0002:000009a0       _Service_QueryDesigner$initializer$ 100139a0     DNAFlexGraphAlgorithm.obj
 0002:000009a4       _Service_MinCoreServiceId$initializer$ 100139a4     DNAFlexGraphAlgorithm.obj
 0002:000009a8       _Service_MaxCoreServiceId$initializer$ 100139a8     DNAFlexGraphAlgorithm.obj
 0002:000009ac       _algoLog$initializer$      100139ac     DNAFlexGraphAlgorithm.obj
 0002:000009b0       _cmdLog$initializer$       100139b0     DNAFlexGraphAlgorithm.obj
 0002:000009b4       _coreLog$initializer$      100139b4     DNAFlexGraphAlgorithm.obj
 0002:000009b8       _ioLog$initializer$        100139b8     DNAFlexGraphAlgorithm.obj
 0002:000009bc       _perfLog$initializer$      100139bc     DNAFlexGraphAlgorithm.obj
 0002:000009c0       _scriptLog$initializer$    100139c0     DNAFlexGraphAlgorithm.obj
 0002:000009c4       _taskLog$initializer$      100139c4     DNAFlexGraphAlgorithm.obj
 0002:000009c8       _uiLog$initializer$        100139c8     DNAFlexGraphAlgorithm.obj
 0002:000009cc       _userActLog$initializer$   100139cc     DNAFlexGraphAlgorithm.obj
 0002:000009d0       _algoLog$initializer$      100139d0     DNAFlexPlugin.obj
 0002:000009d4       _cmdLog$initializer$       100139d4     DNAFlexPlugin.obj
 0002:000009d8       _coreLog$initializer$      100139d8     DNAFlexPlugin.obj
 0002:000009dc       _ioLog$initializer$        100139dc     DNAFlexPlugin.obj
 0002:000009e0       _perfLog$initializer$      100139e0     DNAFlexPlugin.obj
 0002:000009e4       _scriptLog$initializer$    100139e4     DNAFlexPlugin.obj
 0002:000009e8       _taskLog$initializer$      100139e8     DNAFlexPlugin.obj
 0002:000009ec       _uiLog$initializer$        100139ec     DNAFlexPlugin.obj
 0002:000009f0       _userActLog$initializer$   100139f0     DNAFlexPlugin.obj
 0002:000009f4       _Service_PluginViewer$initializer$ 100139f4     DNAFlexPlugin.obj
 0002:000009f8       _Service_Project$initializer$ 100139f8     DNAFlexPlugin.obj
 0002:000009fc       _Service_ProjectView$initializer$ 100139fc     DNAFlexPlugin.obj
 0002:00000a00       _Service_DNAGraphPack$initializer$ 10013a00     DNAFlexPlugin.obj
 0002:00000a04       _Service_DNAExport$initializer$ 10013a04     DNAFlexPlugin.obj
 0002:00000a08       _Service_TestRunner$initializer$ 10013a08     DNAFlexPlugin.obj
 0002:00000a0c       _Service_ScriptRegistry$initializer$ 10013a0c     DNAFlexPlugin.obj
 0002:00000a10       _Service_ExternalToolSupport$initializer$ 10013a10     DNAFlexPlugin.obj
 0002:00000a14       _Service_GUITesting$initializer$ 10013a14     DNAFlexPlugin.obj
 0002:00000a18       _Service_WorkflowDesigner$initializer$ 10013a18     DNAFlexPlugin.obj
 0002:00000a1c       _Service_QueryDesigner$initializer$ 10013a1c     DNAFlexPlugin.obj
 0002:00000a20       _Service_MinCoreServiceId$initializer$ 10013a20     DNAFlexPlugin.obj
 0002:00000a24       _Service_MaxCoreServiceId$initializer$ 10013a24     DNAFlexPlugin.obj
 0002:00000a28       _algoLog$initializer$      10013a28     DNAFlexTask.obj
 0002:00000a2c       _cmdLog$initializer$       10013a2c     DNAFlexTask.obj
 0002:00000a30       _coreLog$initializer$      10013a30     DNAFlexTask.obj
 0002:00000a34       _ioLog$initializer$        10013a34     DNAFlexTask.obj
 0002:00000a38       _perfLog$initializer$      10013a38     DNAFlexTask.obj
 0002:00000a3c       _scriptLog$initializer$    10013a3c     DNAFlexTask.obj
 0002:00000a40       _taskLog$initializer$      10013a40     DNAFlexTask.obj
 0002:00000a44       _uiLog$initializer$        10013a44     DNAFlexTask.obj
 0002:00000a48       _userActLog$initializer$   10013a48     DNAFlexTask.obj
 0002:00000a4c       _algoLog$initializer$      10013a4c     FindHighFlexRegions.obj
 0002:00000a50       _cmdLog$initializer$       10013a50     FindHighFlexRegions.obj
 0002:00000a54       _coreLog$initializer$      10013a54     FindHighFlexRegions.obj
 0002:00000a58       _ioLog$initializer$        10013a58     FindHighFlexRegions.obj
 0002:00000a5c       _perfLog$initializer$      10013a5c     FindHighFlexRegions.obj
 0002:00000a60       _scriptLog$initializer$    10013a60     FindHighFlexRegions.obj
 0002:00000a64       _taskLog$initializer$      10013a64     FindHighFlexRegions.obj
 0002:00000a68       _uiLog$initializer$        10013a68     FindHighFlexRegions.obj
 0002:00000a6c       _userActLog$initializer$   10013a6c     FindHighFlexRegions.obj
 0002:00000a70       _algoLog$initializer$      10013a70     FindHighFlexRegionsAlgorithm.obj
 0002:00000a74       _cmdLog$initializer$       10013a74     FindHighFlexRegionsAlgorithm.obj
 0002:00000a78       _coreLog$initializer$      10013a78     FindHighFlexRegionsAlgorithm.obj
 0002:00000a7c       _ioLog$initializer$        10013a7c     FindHighFlexRegionsAlgorithm.obj
 0002:00000a80       _perfLog$initializer$      10013a80     FindHighFlexRegionsAlgorithm.obj
 0002:00000a84       _scriptLog$initializer$    10013a84     FindHighFlexRegionsAlgorithm.obj
 0002:00000a88       _taskLog$initializer$      10013a88     FindHighFlexRegionsAlgorithm.obj
 0002:00000a8c       _uiLog$initializer$        10013a8c     FindHighFlexRegionsAlgorithm.obj
 0002:00000a90       _userActLog$initializer$   10013a90     FindHighFlexRegionsAlgorithm.obj
 0002:00000a94       _algoLog$initializer$      10013a94     HighFlexSettings.obj
 0002:00000a98       _cmdLog$initializer$       10013a98     HighFlexSettings.obj
 0002:00000a9c       _coreLog$initializer$      10013a9c     HighFlexSettings.obj
 0002:00000aa0       _ioLog$initializer$        10013aa0     HighFlexSettings.obj
 0002:00000aa4       _perfLog$initializer$      10013aa4     HighFlexSettings.obj
 0002:00000aa8       _scriptLog$initializer$    10013aa8     HighFlexSettings.obj
 0002:00000aac       _taskLog$initializer$      10013aac     HighFlexSettings.obj
 0002:00000ab0       _uiLog$initializer$        10013ab0     HighFlexSettings.obj
 0002:00000ab4       _userActLog$initializer$   10013ab4     HighFlexSettings.obj
 0002:00000ab8       ?SETTINGS_PATH$initializer$@HighFlexSettings@U2@@0P6AXXZA 10013ab8     HighFlexSettings.obj
 0002:00000abc       ?SETTING_WINDOW_SIZE$initializer$@HighFlexSettings@U2@@0P6AXXZA 10013abc     HighFlexSettings.obj
 0002:00000ac0       ?SETTING_WINDOW_STEP$initializer$@HighFlexSettings@U2@@0P6AXXZA 10013ac0     HighFlexSettings.obj
 0002:00000ac4       ?SETTING_THRESHOLD$initializer$@HighFlexSettings@U2@@0P6AXXZA 10013ac4     HighFlexSettings.obj
 0002:00000ac8       ?staticMetaObject$initializer$@DNAFlexDialog@U2@@2P6AXXZA 10013ac8     moc_DNAFlexDialog.obj
 0002:00000acc       _Service_PluginViewer$initializer$ 10013acc     moc_DNAFlexGraph.obj
 0002:00000ad0       _Service_Project$initializer$ 10013ad0     moc_DNAFlexGraph.obj
 0002:00000ad4       _Service_ProjectView$initializer$ 10013ad4     moc_DNAFlexGraph.obj
 0002:00000ad8       _Service_DNAGraphPack$initializer$ 10013ad8     moc_DNAFlexGraph.obj
 0002:00000adc       _Service_DNAExport$initializer$ 10013adc     moc_DNAFlexGraph.obj
 0002:00000ae0       _Service_TestRunner$initializer$ 10013ae0     moc_DNAFlexGraph.obj
 0002:00000ae4       _Service_ScriptRegistry$initializer$ 10013ae4     moc_DNAFlexGraph.obj
 0002:00000ae8       _Service_ExternalToolSupport$initializer$ 10013ae8     moc_DNAFlexGraph.obj
 0002:00000aec       _Service_GUITesting$initializer$ 10013aec     moc_DNAFlexGraph.obj
 0002:00000af0       _Service_WorkflowDesigner$initializer$ 10013af0     moc_DNAFlexGraph.obj
 0002:00000af4       _Service_QueryDesigner$initializer$ 10013af4     moc_DNAFlexGraph.obj
 0002:00000af8       _Service_MinCoreServiceId$initializer$ 10013af8     moc_DNAFlexGraph.obj
 0002:00000afc       _Service_MaxCoreServiceId$initializer$ 10013afc     moc_DNAFlexGraph.obj
 0002:00000b00       _algoLog$initializer$      10013b00     moc_DNAFlexGraph.obj
 0002:00000b04       _cmdLog$initializer$       10013b04     moc_DNAFlexGraph.obj
 0002:00000b08       _coreLog$initializer$      10013b08     moc_DNAFlexGraph.obj
 0002:00000b0c       _ioLog$initializer$        10013b0c     moc_DNAFlexGraph.obj
 0002:00000b10       _perfLog$initializer$      10013b10     moc_DNAFlexGraph.obj
 0002:00000b14       _scriptLog$initializer$    10013b14     moc_DNAFlexGraph.obj
 0002:00000b18       _taskLog$initializer$      10013b18     moc_DNAFlexGraph.obj
 0002:00000b1c       _uiLog$initializer$        10013b1c     moc_DNAFlexGraph.obj
 0002:00000b20       _userActLog$initializer$   10013b20     moc_DNAFlexGraph.obj
 0002:00000b24       ?staticMetaObject$initializer$@DNAFlexGraphFactory@U2@@2P6AXXZA 10013b24     moc_DNAFlexGraph.obj
 0002:00000b28       _Service_PluginViewer$initializer$ 10013b28     moc_DNAFlexPlugin.obj
 0002:00000b2c       _Service_Project$initializer$ 10013b2c     moc_DNAFlexPlugin.obj
 0002:00000b30       _Service_ProjectView$initializer$ 10013b30     moc_DNAFlexPlugin.obj
 0002:00000b34       _Service_DNAGraphPack$initializer$ 10013b34     moc_DNAFlexPlugin.obj
 0002:00000b38       _Service_DNAExport$initializer$ 10013b38     moc_DNAFlexPlugin.obj
 0002:00000b3c       _Service_TestRunner$initializer$ 10013b3c     moc_DNAFlexPlugin.obj
 0002:00000b40       _Service_ScriptRegistry$initializer$ 10013b40     moc_DNAFlexPlugin.obj
 0002:00000b44       _Service_ExternalToolSupport$initializer$ 10013b44     moc_DNAFlexPlugin.obj
 0002:00000b48       _Service_GUITesting$initializer$ 10013b48     moc_DNAFlexPlugin.obj
 0002:00000b4c       _Service_WorkflowDesigner$initializer$ 10013b4c     moc_DNAFlexPlugin.obj
 0002:00000b50       _Service_QueryDesigner$initializer$ 10013b50     moc_DNAFlexPlugin.obj
 0002:00000b54       _Service_MinCoreServiceId$initializer$ 10013b54     moc_DNAFlexPlugin.obj
 0002:00000b58       _Service_MaxCoreServiceId$initializer$ 10013b58     moc_DNAFlexPlugin.obj
 0002:00000b5c       _algoLog$initializer$      10013b5c     moc_DNAFlexPlugin.obj
 0002:00000b60       _cmdLog$initializer$       10013b60     moc_DNAFlexPlugin.obj
 0002:00000b64       _coreLog$initializer$      10013b64     moc_DNAFlexPlugin.obj
 0002:00000b68       _ioLog$initializer$        10013b68     moc_DNAFlexPlugin.obj
 0002:00000b6c       _perfLog$initializer$      10013b6c     moc_DNAFlexPlugin.obj
 0002:00000b70       _scriptLog$initializer$    10013b70     moc_DNAFlexPlugin.obj
 0002:00000b74       _taskLog$initializer$      10013b74     moc_DNAFlexPlugin.obj
 0002:00000b78       _uiLog$initializer$        10013b78     moc_DNAFlexPlugin.obj
 0002:00000b7c       _userActLog$initializer$   10013b7c     moc_DNAFlexPlugin.obj
 0002:00000b80       ?staticMetaObject$initializer$@DNAFlexPlugin@U2@@2P6AXXZA 10013b80     moc_DNAFlexPlugin.obj
 0002:00000b84       ?staticMetaObject$initializer$@DNAFlexViewContext@U2@@2P6AXXZA 10013b84     moc_DNAFlexPlugin.obj
 0002:00000b88       _algoLog$initializer$      10013b88     moc_DNAFlexTask.obj
 0002:00000b8c       _cmdLog$initializer$       10013b8c     moc_DNAFlexTask.obj
 0002:00000b90       _coreLog$initializer$      10013b90     moc_DNAFlexTask.obj
 0002:00000b94       _ioLog$initializer$        10013b94     moc_DNAFlexTask.obj
 0002:00000b98       _perfLog$initializer$      10013b98     moc_DNAFlexTask.obj
 0002:00000b9c       _scriptLog$initializer$    10013b9c     moc_DNAFlexTask.obj
 0002:00000ba0       _taskLog$initializer$      10013ba0     moc_DNAFlexTask.obj
 0002:00000ba4       _uiLog$initializer$        10013ba4     moc_DNAFlexTask.obj
 0002:00000ba8       _userActLog$initializer$   10013ba8     moc_DNAFlexTask.obj
 0002:00000bac       ?staticMetaObject$initializer$@DNAFlexTask@U2@@2P6AXXZA 10013bac     moc_DNAFlexTask.obj
 0002:00000bb0       _algoLog$initializer$      10013bb0     moc_FindHighFlexRegions.obj
 0002:00000bb4       _cmdLog$initializer$       10013bb4     moc_FindHighFlexRegions.obj
 0002:00000bb8       _coreLog$initializer$      10013bb8     moc_FindHighFlexRegions.obj
 0002:00000bbc       _ioLog$initializer$        10013bbc     moc_FindHighFlexRegions.obj
 0002:00000bc0       _perfLog$initializer$      10013bc0     moc_FindHighFlexRegions.obj
 0002:00000bc4       _scriptLog$initializer$    10013bc4     moc_FindHighFlexRegions.obj
 0002:00000bc8       _taskLog$initializer$      10013bc8     moc_FindHighFlexRegions.obj
 0002:00000bcc       _uiLog$initializer$        10013bcc     moc_FindHighFlexRegions.obj
 0002:00000bd0       _userActLog$initializer$   10013bd0     moc_FindHighFlexRegions.obj
 0002:00000bd4       ?staticMetaObject$initializer$@FindHighFlexRegions@U2@@2P6AXXZA 10013bd4     moc_FindHighFlexRegions.obj
 0002:00000bd8       _dummy$initializer$        10013bd8     qrc_dna_flexibility.obj
 0002:00000be4       _pcinit                    10013be4     MSVCRT:crtdll.obj
 0002:00000be8       _pinit                     10013be8     MSVCRT:atonexit.obj
 0002:0000171c       ?qstring_literal@?6???R<lambda_1cfb2c5c4119324300889144faedee2e>@@QBE?AVQString@@XZ@4U?$QStaticStringData@$0N@@@B 1001471c     DNAFlexDialog.obj
 0002:00001748       ?qstring_literal@?7???R<lambda_c54a255dbb70683bcc9e7ac18dc46ed1>@@QBE?AVQString@@XZ@4U?$QStaticStringData@$0O@@@B 10014748     DNAFlexDialog.obj
 0002:00001778       ?qstring_literal@?8???R<lambda_5c6a044f2f458955f0d06defa39d488f>@@QBE?AVQString@@XZ@4U?$QStaticStringData@$08@@B 10014778     DNAFlexDialog.obj
 0002:0000179c       ?qstring_literal@?9???R<lambda_458b0f23edea6d4478a012c5955cb606>@@QBE?AVQString@@XZ@4U?$QStaticStringData@$0BB@@@B 1001479c     DNAFlexDialog.obj
 0002:000017d0       ?qstring_literal@?L@???R<lambda_57a051c781f8d8c95caf7ca077bc5f12>@@QBE?AVQString@@XZ@4U?$QStaticStringData@$0BA@@@B 100147d0     DNAFlexDialog.obj
 0002:00001804       ?qstring_literal@?M@???R<lambda_707fe8b4ae45d9fe5ca46cd514e2687d>@@QBE?AVQString@@XZ@4U?$QStaticStringData@$0BF@@@B 10014804     DNAFlexDialog.obj
 0002:00001840       ?qstring_literal@?N@???R<lambda_8dadecbf2ac41c19a976dc614914c4ce>@@QBE?AVQString@@XZ@4U?$QStaticStringData@$0BA@@@B 10014840     DNAFlexDialog.obj
 0002:00001874       ?qstring_literal@?O@???R<lambda_00118d359345adf794be5d433703ad4b>@@QBE?AVQString@@XZ@4U?$QStaticStringData@$09@@B 10014874     DNAFlexDialog.obj
 0002:0000189c       ?qstring_literal@?P@???R<lambda_4717dcb402506f06d2b359e39d831609>@@QBE?AVQString@@XZ@4U?$QStaticStringData@$0N@@@B 1001489c     DNAFlexDialog.obj
 0002:000018c8       ?qstring_literal@?BA@???R<lambda_60c36b2ba8f6ac249075d3447a06946a>@@QBE?AVQString@@XZ@4U?$QStaticStringData@$0BB@@@B 100148c8     DNAFlexDialog.obj
 0002:000018fc       ?qstring_literal@?BB@???R<lambda_821a87b4b859d3d71973b8c7c9ac2d25>@@QBE?AVQString@@XZ@4U?$QStaticStringData@$0N@@@B 100148fc     DNAFlexDialog.obj
 0002:00001928       ?qstring_literal@?BC@???R<lambda_1d1eaa33596ff48552c744a4378a660b>@@QBE?AVQString@@XZ@4U?$QStaticStringData@$0BB@@@B 10014928     DNAFlexDialog.obj
 0002:0000195c       ?qstring_literal@?BD@???R<lambda_99cbfa8a2e2a089352d749da904ef1d2>@@QBE?AVQString@@XZ@4U?$QStaticStringData@$0M@@@B 1001495c     DNAFlexDialog.obj
 0002:00001988       ?qstring_literal@?BE@???R<lambda_f5440838e2e94d9a157f8927169bbc41>@@QBE?AVQString@@XZ@4U?$QStaticStringData@$0BG@@@B 10014988     DNAFlexDialog.obj
 0002:000019c8       ?qstring_literal@?BF@???R<lambda_17b0b2d6700668d280cd86f7b3fbe6a9>@@QBE?AVQString@@XZ@4U?$QStaticStringData@$0L@@@B 100149c8     DNAFlexDialog.obj
 0002:000019f0       ?qstring_literal@?BG@???R<lambda_7151c4947fd3098b290b8908712616f2>@@QBE?AVQString@@XZ@4U?$QStaticStringData@$0L@@@B 100149f0     DNAFlexDialog.obj
 0002:00001a18       ?qstring_literal@?BH@???R<lambda_2a848a472f6df9fe3550693bba86a84d>@@QBE?AVQString@@XZ@4U?$QStaticStringData@$08@@B 10014a18     DNAFlexDialog.obj
 0002:00001a3c       ?qstring_literal@?BI@???R<lambda_52ee9bd10a54360c0a60eb05b65cf928>@@QBE?AVQString@@XZ@4U?$QStaticStringData@$0BA@@@B 10014a3c     DNAFlexDialog.obj
 0002:00001a70       ?qstring_literal@?BJ@???R<lambda_eda4e94934f57365d954060c5e0ec9a8>@@QBE?AVQString@@XZ@4U?$QStaticStringData@$08@@B 10014a70     DNAFlexDialog.obj
 0002:000028c8       _qt_meta_stringdata_U2__DNAFlexDialog 100158c8     moc_DNAFlexDialog.obj
 0002:000029e0       _qt_meta_data_U2__DNAFlexDialog 100159e0     moc_DNAFlexDialog.obj
 0002:00002ae0       _qt_meta_stringdata_U2__DNAFlexGraphFactory 10015ae0     moc_DNAFlexGraph.obj
 0002:00002b08       _qt_meta_data_U2__DNAFlexGraphFactory 10015b08     moc_DNAFlexGraph.obj
 0002:00002b48       _qt_meta_stringdata_U2__DNAFlexPlugin 10015b48     moc_DNAFlexPlugin.obj
 0002:00002b6c       _qt_meta_data_U2__DNAFlexPlugin 10015b6c     moc_DNAFlexPlugin.obj
 0002:00002ba8       _qt_meta_stringdata_U2__DNAFlexViewContext 10015ba8     moc_DNAFlexPlugin.obj
 0002:00002c50       _qt_meta_data_U2__DNAFlexViewContext 10015c50     moc_DNAFlexPlugin.obj
 0002:00002cc4       _qt_meta_stringdata_U2__DNAFlexTask 10015cc4     moc_DNAFlexTask.obj
 0002:00002ce4       _qt_meta_data_U2__DNAFlexTask 10015ce4     moc_DNAFlexTask.obj
 0002:00002d20       _qt_meta_stringdata_U2__FindHighFlexRegions 10015d20     moc_FindHighFlexRegions.obj
 0002:00002d48       _qt_meta_data_U2__FindHighFlexRegions 10015d48     moc_FindHighFlexRegions.obj
 0002:00002da0       _qt_resource_data          10015da0     qrc_dna_flexibility.obj
 0002:00002f88       _qt_resource_name          10015f88     qrc_dna_flexibility.obj
 0002:00002fe4       _qt_resource_struct        10015fe4     qrc_dna_flexibility.obj
 0002:0000302c       _GS_ExceptionPointers      1001602c     MSVCRT:gs_report.obj
 0002:00004450       __catchsym$?_Copy@?$basic_string@DU?$char_traits@D@std@@V?$allocator@D@2@@std@@QAEXII@Z$5 10017450     DNAFlexDialog.obj
 0002:00004460       __catchsym$?_Copy@?$basic_string@DU?$char_traits@D@std@@V?$allocator@D@2@@std@@QAEXII@Z$4 10017460     DNAFlexDialog.obj
 0002:00004470       __unwindtable$?_Copy@?$basic_string@DU?$char_traits@D@std@@V?$allocator@D@2@@std@@QAEXII@Z 10017470     DNAFlexDialog.obj
 0002:00004490       __ehfuncinfo$?_Copy@?$basic_string@DU?$char_traits@D@std@@V?$allocator@D@2@@std@@QAEXII@Z 10017490     DNAFlexDialog.obj
 0002:000044b4       __tryblocktable$?_Copy@?$basic_string@DU?$char_traits@D@std@@V?$allocator@D@2@@std@@QAEXII@Z 100174b4     DNAFlexDialog.obj
 0002:000044dc       __ehfuncinfo$?setupUi@Ui_DNAFlexDialog@@QAEXPAVQDialog@@@Z 100174dc     DNAFlexDialog.obj
 0002:00004500       __unwindtable$?setupUi@Ui_DNAFlexDialog@@QAEXPAVQDialog@@@Z 10017500     DNAFlexDialog.obj
 0002:00004640       __ehfuncinfo$?retranslateUi@Ui_DNAFlexDialog@@QAEXPAVQDialog@@@Z 10017640     DNAFlexDialog.obj
 0002:00004664       __unwindtable$?retranslateUi@Ui_DNAFlexDialog@@QAEXPAVQDialog@@@Z 10017664     DNAFlexDialog.obj
 0002:000046bc       __ehfuncinfo$??0DNAFlexDialog@U2@@QAE@PAVADVSequenceObjectContext@1@@Z 100176bc     DNAFlexDialog.obj
 0002:000046e0       __unwindtable$??0DNAFlexDialog@U2@@QAE@PAVADVSequenceObjectContext@1@@Z 100176e0     DNAFlexDialog.obj
 0002:00004738       __ehfuncinfo$?accept@DNAFlexDialog@U2@@UAEXXZ 10017738     DNAFlexDialog.obj
 0002:0000475c       __unwindtable$?accept@DNAFlexDialog@U2@@UAEXXZ 1001775c     DNAFlexDialog.obj
 0002:000047c4       __unwindtable$??__EalgoLog@U2@@YAXXZ 100177c4     DNAFlexDialog.obj
 0002:000047cc       __ehfuncinfo$??__EalgoLog@U2@@YAXXZ 100177cc     DNAFlexDialog.obj
 0002:000047f0       __unwindtable$??__EcmdLog@U2@@YAXXZ 100177f0     DNAFlexDialog.obj
 0002:000047f8       __ehfuncinfo$??__EcmdLog@U2@@YAXXZ 100177f8     DNAFlexDialog.obj
 0002:0000481c       __unwindtable$??__EcoreLog@U2@@YAXXZ 1001781c     DNAFlexDialog.obj
 0002:00004824       __ehfuncinfo$??__EcoreLog@U2@@YAXXZ 10017824     DNAFlexDialog.obj
 0002:00004848       __unwindtable$??__EioLog@U2@@YAXXZ 10017848     DNAFlexDialog.obj
 0002:00004850       __ehfuncinfo$??__EioLog@U2@@YAXXZ 10017850     DNAFlexDialog.obj
 0002:00004874       __unwindtable$??__EperfLog@U2@@YAXXZ 10017874     DNAFlexDialog.obj
 0002:0000487c       __ehfuncinfo$??__EperfLog@U2@@YAXXZ 1001787c     DNAFlexDialog.obj
 0002:000048a0       __unwindtable$??__EscriptLog@U2@@YAXXZ 100178a0     DNAFlexDialog.obj
 0002:000048a8       __ehfuncinfo$??__EscriptLog@U2@@YAXXZ 100178a8     DNAFlexDialog.obj
 0002:000048cc       __unwindtable$??__EtaskLog@U2@@YAXXZ 100178cc     DNAFlexDialog.obj
 0002:000048d4       __ehfuncinfo$??__EtaskLog@U2@@YAXXZ 100178d4     DNAFlexDialog.obj
 0002:000048f8       __unwindtable$??__EuiLog@U2@@YAXXZ 100178f8     DNAFlexDialog.obj
 0002:00004900       __ehfuncinfo$??__EuiLog@U2@@YAXXZ 10017900     DNAFlexDialog.obj
 0002:00004924       __unwindtable$??__EuserActLog@U2@@YAXXZ 10017924     DNAFlexDialog.obj
 0002:0000492c       __ehfuncinfo$??__EuserActLog@U2@@YAXXZ 1001792c     DNAFlexDialog.obj
 0002:00004950       __unwindtable$?clone@?$QSharedDataPointer@VAnnotationData@U2@@@@IAEPAVAnnotationData@U2@@XZ 10017950     DNAFlexDialog.obj
 0002:00004958       __ehfuncinfo$?clone@?$QSharedDataPointer@VAnnotationData@U2@@@@IAEPAVAnnotationData@U2@@XZ 10017958     DNAFlexDialog.obj
 0002:0000497c       __unwindtable$?detach_helper@?$QSharedDataPointer@VAnnotationData@U2@@@@AAEXXZ 1001797c     DNAFlexDialog.obj
 0002:00004984       __ehfuncinfo$?detach_helper@?$QSharedDataPointer@VAnnotationData@U2@@@@AAEXXZ 10017984     DNAFlexDialog.obj
 0002:000049a8       __unwindtable$??__EalgoLog@U2@@YAXXZ 100179a8     DNAFlexGraph.obj
 0002:000049b0       __ehfuncinfo$??__EalgoLog@U2@@YAXXZ 100179b0     DNAFlexGraph.obj
 0002:000049d4       __unwindtable$??__EcmdLog@U2@@YAXXZ 100179d4     DNAFlexGraph.obj
 0002:000049dc       __ehfuncinfo$??__EcmdLog@U2@@YAXXZ 100179dc     DNAFlexGraph.obj
 0002:00004a00       __unwindtable$??__EcoreLog@U2@@YAXXZ 10017a00     DNAFlexGraph.obj
 0002:00004a08       __ehfuncinfo$??__EcoreLog@U2@@YAXXZ 10017a08     DNAFlexGraph.obj
 0002:00004a2c       __unwindtable$??__EioLog@U2@@YAXXZ 10017a2c     DNAFlexGraph.obj
 0002:00004a34       __ehfuncinfo$??__EioLog@U2@@YAXXZ 10017a34     DNAFlexGraph.obj
 0002:00004a58       __unwindtable$??__EperfLog@U2@@YAXXZ 10017a58     DNAFlexGraph.obj
 0002:00004a60       __ehfuncinfo$??__EperfLog@U2@@YAXXZ 10017a60     DNAFlexGraph.obj
 0002:00004a84       __unwindtable$??__EscriptLog@U2@@YAXXZ 10017a84     DNAFlexGraph.obj
 0002:00004a8c       __ehfuncinfo$??__EscriptLog@U2@@YAXXZ 10017a8c     DNAFlexGraph.obj
 0002:00004ab0       __unwindtable$??__EtaskLog@U2@@YAXXZ 10017ab0     DNAFlexGraph.obj
 0002:00004ab8       __ehfuncinfo$??__EtaskLog@U2@@YAXXZ 10017ab8     DNAFlexGraph.obj
 0002:00004adc       __unwindtable$??__EuiLog@U2@@YAXXZ 10017adc     DNAFlexGraph.obj
 0002:00004ae4       __ehfuncinfo$??__EuiLog@U2@@YAXXZ 10017ae4     DNAFlexGraph.obj
 0002:00004b08       __unwindtable$??__EuserActLog@U2@@YAXXZ 10017b08     DNAFlexGraph.obj
 0002:00004b10       __ehfuncinfo$??__EuserActLog@U2@@YAXXZ 10017b10     DNAFlexGraph.obj
 0002:00004b34       __catchsym$?append@?$QList@V?$QSharedPointer@VGSequenceGraphData@U2@@@@@@QAEXABV?$QSharedPointer@VGSequenceGraphData@U2@@@@@Z$9 10017b34     DNAFlexGraph.obj
 0002:00004b44       __catchsym$?append@?$QList@V?$QSharedPointer@VGSequenceGraphData@U2@@@@@@QAEXABV?$QSharedPointer@VGSequenceGraphData@U2@@@@@Z$8 10017b44     DNAFlexGraph.obj
 0002:00004b54       __ehfuncinfo$?append@?$QList@V?$QSharedPointer@VGSequenceGraphData@U2@@@@@@QAEXABV?$QSharedPointer@VGSequenceGraphData@U2@@@@@Z 10017b54     DNAFlexGraph.obj
 0002:00004b78       __tryblocktable$?append@?$QList@V?$QSharedPointer@VGSequenceGraphData@U2@@@@@@QAEXABV?$QSharedPointer@VGSequenceGraphData@U2@@@@@Z 10017b78     DNAFlexGraph.obj
 0002:00004ba0       __unwindtable$?append@?$QList@V?$QSharedPointer@VGSequenceGraphData@U2@@@@@@QAEXABV?$QSharedPointer@VGSequenceGraphData@U2@@@@@Z 10017ba0     DNAFlexGraph.obj
 0002:00004bd0       __catchsym$?detach_helper_grow@?$QList@V?$QSharedPointer@VGSequenceGraphData@U2@@@@@@AAEPAUNode@1@HH@Z$5 10017bd0     DNAFlexGraph.obj
 0002:00004be0       __catchsym$?detach_helper_grow@?$QList@V?$QSharedPointer@VGSequenceGraphData@U2@@@@@@AAEPAUNode@1@HH@Z$4 10017be0     DNAFlexGraph.obj
 0002:00004bf0       __unwindtable$?detach_helper_grow@?$QList@V?$QSharedPointer@VGSequenceGraphData@U2@@@@@@AAEPAUNode@1@HH@Z 10017bf0     DNAFlexGraph.obj
 0002:00004c10       __ehfuncinfo$?detach_helper_grow@?$QList@V?$QSharedPointer@VGSequenceGraphData@U2@@@@@@AAEPAUNode@1@HH@Z 10017c10     DNAFlexGraph.obj
 0002:00004c34       __tryblocktable$?detach_helper_grow@?$QList@V?$QSharedPointer@VGSequenceGraphData@U2@@@@@@AAEPAUNode@1@HH@Z 10017c34     DNAFlexGraph.obj
 0002:00004c5c       __catchsym$?node_copy@?$QList@V?$QSharedPointer@VGSequenceGraphData@U2@@@@@@AAEXPAUNode@1@00@Z$6 10017c5c     DNAFlexGraph.obj
 0002:00004c6c       __tryblocktable$?node_copy@?$QList@V?$QSharedPointer@VGSequenceGraphData@U2@@@@@@AAEXPAUNode@1@00@Z 10017c6c     DNAFlexGraph.obj
 0002:00004c80       __unwindtable$?node_copy@?$QList@V?$QSharedPointer@VGSequenceGraphData@U2@@@@@@AAEXPAUNode@1@00@Z 10017c80     DNAFlexGraph.obj
 0002:00004ca0       __ehfuncinfo$?node_copy@?$QList@V?$QSharedPointer@VGSequenceGraphData@U2@@@@@@AAEXPAUNode@1@00@Z 10017ca0     DNAFlexGraph.obj
 0002:00004cc4       __unwindtable$??0DNAFlexGraphFactory@U2@@QAE@PAVQObject@@@Z 10017cc4     DNAFlexGraph.obj
 0002:00004cdc       __ehfuncinfo$??0DNAFlexGraphFactory@U2@@QAE@PAVQObject@@@Z 10017cdc     DNAFlexGraph.obj
 0002:00004d00       __unwindtable$?createGraphs@DNAFlexGraphFactory@U2@@UAE?AV?$QList@V?$QSharedPointer@VGSequenceGraphData@U2@@@@@@PAVGSequenceGraphView@2@@Z 10017d00     DNAFlexGraph.obj
 0002:00004d20       __ehfuncinfo$?createGraphs@DNAFlexGraphFactory@U2@@UAE?AV?$QList@V?$QSharedPointer@VGSequenceGraphData@U2@@@@@@PAVGSequenceGraphView@2@@Z 10017d20     DNAFlexGraph.obj
 0002:00004d44       __unwindtable$?getDrawer@DNAFlexGraphFactory@U2@@UAEPAVGSequenceGraphDrawer@2@PAVGSequenceGraphView@2@@Z 10017d44     DNAFlexGraph.obj
 0002:00004d54       __ehfuncinfo$?getDrawer@DNAFlexGraphFactory@U2@@UAEPAVGSequenceGraphDrawer@2@PAVGSequenceGraphView@2@@Z 10017d54     DNAFlexGraph.obj
 0002:00004d78       __unwindtable$?isEnabled@DNAFlexGraphFactory@U2@@UBE_NPBVU2SequenceObject@2@@Z 10017d78     DNAFlexGraph.obj
 0002:00004d80       __ehfuncinfo$?isEnabled@DNAFlexGraphFactory@U2@@UBE_NPBVU2SequenceObject@2@@Z 10017d80     DNAFlexGraph.obj
 0002:00004da4       __unwindtable$??__EalgoLog@U2@@YAXXZ 10017da4     DNAFlexGraphAlgorithm.obj
 0002:00004dac       __ehfuncinfo$??__EalgoLog@U2@@YAXXZ 10017dac     DNAFlexGraphAlgorithm.obj
 0002:00004dd0       __unwindtable$??__EcmdLog@U2@@YAXXZ 10017dd0     DNAFlexGraphAlgorithm.obj
 0002:00004dd8       __ehfuncinfo$??__EcmdLog@U2@@YAXXZ 10017dd8     DNAFlexGraphAlgorithm.obj
 0002:00004dfc       __unwindtable$??__EcoreLog@U2@@YAXXZ 10017dfc     DNAFlexGraphAlgorithm.obj
 0002:00004e04       __ehfuncinfo$??__EcoreLog@U2@@YAXXZ 10017e04     DNAFlexGraphAlgorithm.obj
 0002:00004e28       __unwindtable$??__EioLog@U2@@YAXXZ 10017e28     DNAFlexGraphAlgorithm.obj
 0002:00004e30       __ehfuncinfo$??__EioLog@U2@@YAXXZ 10017e30     DNAFlexGraphAlgorithm.obj
 0002:00004e54       __unwindtable$??__EperfLog@U2@@YAXXZ 10017e54     DNAFlexGraphAlgorithm.obj
 0002:00004e5c       __ehfuncinfo$??__EperfLog@U2@@YAXXZ 10017e5c     DNAFlexGraphAlgorithm.obj
 0002:00004e80       __unwindtable$??__EscriptLog@U2@@YAXXZ 10017e80     DNAFlexGraphAlgorithm.obj
 0002:00004e88       __ehfuncinfo$??__EscriptLog@U2@@YAXXZ 10017e88     DNAFlexGraphAlgorithm.obj
 0002:00004eac       __unwindtable$??__EtaskLog@U2@@YAXXZ 10017eac     DNAFlexGraphAlgorithm.obj
 0002:00004eb4       __ehfuncinfo$??__EtaskLog@U2@@YAXXZ 10017eb4     DNAFlexGraphAlgorithm.obj
 0002:00004ed8       __unwindtable$??__EuiLog@U2@@YAXXZ 10017ed8     DNAFlexGraphAlgorithm.obj
 0002:00004ee0       __ehfuncinfo$??__EuiLog@U2@@YAXXZ 10017ee0     DNAFlexGraphAlgorithm.obj
 0002:00004f04       __unwindtable$??__EuserActLog@U2@@YAXXZ 10017f04     DNAFlexGraphAlgorithm.obj
 0002:00004f0c       __ehfuncinfo$??__EuserActLog@U2@@YAXXZ 10017f0c     DNAFlexGraphAlgorithm.obj
 0002:00004f30       __catchsym$?reallocData@?$QVector@M@@AAEXHHV?$QFlags@W4AllocationOption@QArrayData@@@@@Z$5 10017f30     DNAFlexGraphAlgorithm.obj
 0002:00004f40       __catchsym$?reallocData@?$QVector@M@@AAEXHHV?$QFlags@W4AllocationOption@QArrayData@@@@@Z$4 10017f40     DNAFlexGraphAlgorithm.obj
 0002:00004f50       __unwindtable$?reallocData@?$QVector@M@@AAEXHHV?$QFlags@W4AllocationOption@QArrayData@@@@@Z 10017f50     DNAFlexGraphAlgorithm.obj
 0002:00004f70       __ehfuncinfo$?reallocData@?$QVector@M@@AAEXHHV?$QFlags@W4AllocationOption@QArrayData@@@@@Z 10017f70     DNAFlexGraphAlgorithm.obj
 0002:00004f94       __tryblocktable$?reallocData@?$QVector@M@@AAEXHHV?$QFlags@W4AllocationOption@QArrayData@@@@@Z 10017f94     DNAFlexGraphAlgorithm.obj
 0002:00004fbc       __tryblocktable$?calculate@DNAFlexGraphAlgorithm@U2@@UAEXAAV?$QVector@M@@PAVU2SequenceObject@2@ABVU2Region@2@PBVGSequenceGraphWindowData@2@AAVU2OpStatus@2@@Z 10017fbc     DNAFlexGraphAlgorithm.obj
 0002:00004fd0       __catchsym$?calculate@DNAFlexGraphAlgorithm@U2@@UAEXAAV?$QVector@M@@PAVU2SequenceObject@2@ABVU2Region@2@PBVGSequenceGraphWindowData@2@AAVU2OpStatus@2@@Z$5 10017fd0     DNAFlexGraphAlgorithm.obj
 0002:00004ff0       __unwindtable$?calculate@DNAFlexGraphAlgorithm@U2@@UAEXAAV?$QVector@M@@PAVU2SequenceObject@2@ABVU2Region@2@PBVGSequenceGraphWindowData@2@AAVU2OpStatus@2@@Z 10017ff0     DNAFlexGraphAlgorithm.obj
 0002:00005010       __ehfuncinfo$?calculate@DNAFlexGraphAlgorithm@U2@@UAEXAAV?$QVector@M@@PAVU2SequenceObject@2@ABVU2Region@2@PBVGSequenceGraphWindowData@2@AAVU2OpStatus@2@@Z 10018010     DNAFlexGraphAlgorithm.obj
 0002:00005034       __unwindtable$??__EalgoLog@U2@@YAXXZ 10018034     DNAFlexPlugin.obj
 0002:0000503c       __ehfuncinfo$??__EalgoLog@U2@@YAXXZ 1001803c     DNAFlexPlugin.obj
 0002:00005060       __unwindtable$??__EcmdLog@U2@@YAXXZ 10018060     DNAFlexPlugin.obj
 0002:00005068       __ehfuncinfo$??__EcmdLog@U2@@YAXXZ 10018068     DNAFlexPlugin.obj
 0002:0000508c       __unwindtable$??__EcoreLog@U2@@YAXXZ 1001808c     DNAFlexPlugin.obj
 0002:00005094       __ehfuncinfo$??__EcoreLog@U2@@YAXXZ 10018094     DNAFlexPlugin.obj
 0002:000050b8       __unwindtable$??__EioLog@U2@@YAXXZ 100180b8     DNAFlexPlugin.obj
 0002:000050c0       __ehfuncinfo$??__EioLog@U2@@YAXXZ 100180c0     DNAFlexPlugin.obj
 0002:000050e4       __unwindtable$??__EperfLog@U2@@YAXXZ 100180e4     DNAFlexPlugin.obj
 0002:000050ec       __ehfuncinfo$??__EperfLog@U2@@YAXXZ 100180ec     DNAFlexPlugin.obj
 0002:00005110       __unwindtable$??__EscriptLog@U2@@YAXXZ 10018110     DNAFlexPlugin.obj
 0002:00005118       __ehfuncinfo$??__EscriptLog@U2@@YAXXZ 10018118     DNAFlexPlugin.obj
 0002:0000513c       __unwindtable$??__EtaskLog@U2@@YAXXZ 1001813c     DNAFlexPlugin.obj
 0002:00005144       __ehfuncinfo$??__EtaskLog@U2@@YAXXZ 10018144     DNAFlexPlugin.obj
 0002:00005168       __unwindtable$??__EuiLog@U2@@YAXXZ 10018168     DNAFlexPlugin.obj
 0002:00005170       __ehfuncinfo$??__EuiLog@U2@@YAXXZ 10018170     DNAFlexPlugin.obj
 0002:00005194       __unwindtable$??__EuserActLog@U2@@YAXXZ 10018194     DNAFlexPlugin.obj
 0002:0000519c       __ehfuncinfo$??__EuserActLog@U2@@YAXXZ 1001819c     DNAFlexPlugin.obj
 0002:000051c0       __catchsym$??0?$QList@PAVADVSequenceWidget@U2@@@@QAE@ABV0@@Z$2 100181c0     DNAFlexPlugin.obj
 0002:000051d0       __unwindtable$??0?$QList@PAVADVSequenceWidget@U2@@@@QAE@ABV0@@Z 100181d0     DNAFlexPlugin.obj
 0002:000051e0       __tryblocktable$??0?$QList@PAVADVSequenceWidget@U2@@@@QAE@ABV0@@Z 100181e0     DNAFlexPlugin.obj
 0002:000051f4       __ehfuncinfo$??0?$QList@PAVADVSequenceWidget@U2@@@@QAE@ABV0@@Z 100181f4     DNAFlexPlugin.obj
 0002:00005218       __ehfuncinfo$??0DNAFlexPlugin@U2@@QAE@XZ 10018218     DNAFlexPlugin.obj
 0002:0000523c       __unwindtable$??0DNAFlexPlugin@U2@@QAE@XZ 1001823c     DNAFlexPlugin.obj
 0002:0000526c       __unwindtable$??0DNAFlexViewContext@U2@@QAE@PAVQObject@@@Z 1001826c     DNAFlexPlugin.obj
 0002:0000528c       __ehfuncinfo$??0DNAFlexViewContext@U2@@QAE@PAVQObject@@@Z 1001828c     DNAFlexPlugin.obj
 0002:000052b0       __ehfuncinfo$?sl_showDNAFlexDialog@DNAFlexViewContext@U2@@AAEXXZ 100182b0     DNAFlexPlugin.obj
 0002:000052d4       __unwindtable$?sl_showDNAFlexDialog@DNAFlexViewContext@U2@@AAEXXZ 100182d4     DNAFlexPlugin.obj
 0002:0000535c       __unwindtable$?sl_sequenceWidgetAdded@DNAFlexViewContext@U2@@AAEXPAVADVSequenceWidget@2@@Z 1001835c     DNAFlexPlugin.obj
 0002:0000536c       __ehfuncinfo$?sl_sequenceWidgetAdded@DNAFlexViewContext@U2@@AAEXPAVADVSequenceWidget@2@@Z 1001836c     DNAFlexPlugin.obj
 0002:00005390       __ehfuncinfo$?initViewContext@DNAFlexViewContext@U2@@EAEXPAVGObjectView@2@@Z 10018390     DNAFlexPlugin.obj
 0002:000053b4       __unwindtable$?initViewContext@DNAFlexViewContext@U2@@EAEXPAVGObjectView@2@@Z 100183b4     DNAFlexPlugin.obj
 0002:00005404       __unwindtable$??1?$QObjectScopedPointer@VDNAFlexDialog@U2@@@U2@@QAE@XZ 10018404     DNAFlexPlugin.obj
 0002:0000540c       __ehfuncinfo$??1?$QObjectScopedPointer@VDNAFlexDialog@U2@@@U2@@QAE@XZ 1001840c     DNAFlexPlugin.obj
 0002:00005430       __catchsym$?reallocData@?$QVector@VU2Region@U2@@@@AAEXHHV?$QFlags@W4AllocationOption@QArrayData@@@@@Z$5 10018430     DNAFlexTask.obj
 0002:00005440       __catchsym$?reallocData@?$QVector@VU2Region@U2@@@@AAEXHHV?$QFlags@W4AllocationOption@QArrayData@@@@@Z$4 10018440     DNAFlexTask.obj
 0002:00005450       __unwindtable$?reallocData@?$QVector@VU2Region@U2@@@@AAEXHHV?$QFlags@W4AllocationOption@QArrayData@@@@@Z 10018450     DNAFlexTask.obj
 0002:00005470       __ehfuncinfo$?reallocData@?$QVector@VU2Region@U2@@@@AAEXHHV?$QFlags@W4AllocationOption@QArrayData@@@@@Z 10018470     DNAFlexTask.obj
 0002:00005494       __tryblocktable$?reallocData@?$QVector@VU2Region@U2@@@@AAEXHHV?$QFlags@W4AllocationOption@QArrayData@@@@@Z 10018494     DNAFlexTask.obj
 0002:000054bc       __unwindtable$?append@?$QVector@VU2Qualifier@U2@@@@QAEXABVU2Qualifier@U2@@@Z 100184bc     DNAFlexTask.obj
 0002:000054cc       __ehfuncinfo$?append@?$QVector@VU2Qualifier@U2@@@@QAEXABVU2Qualifier@U2@@@Z 100184cc     DNAFlexTask.obj
 0002:000054f0       __catchsym$?reallocData@?$QVector@VU2Qualifier@U2@@@@AAEXHHV?$QFlags@W4AllocationOption@QArrayData@@@@@Z$6 100184f0     DNAFlexTask.obj
 0002:00005500       __catchsym$?reallocData@?$QVector@VU2Qualifier@U2@@@@AAEXHHV?$QFlags@W4AllocationOption@QArrayData@@@@@Z$5 10018500     DNAFlexTask.obj
 0002:00005510       __ehfuncinfo$?reallocData@?$QVector@VU2Qualifier@U2@@@@AAEXHHV?$QFlags@W4AllocationOption@QArrayData@@@@@Z 10018510     DNAFlexTask.obj
 0002:00005534       __tryblocktable$?reallocData@?$QVector@VU2Qualifier@U2@@@@AAEXHHV?$QFlags@W4AllocationOption@QArrayData@@@@@Z 10018534     DNAFlexTask.obj
 0002:0000555c       __unwindtable$?reallocData@?$QVector@VU2Qualifier@U2@@@@AAEXHHV?$QFlags@W4AllocationOption@QArrayData@@@@@Z 1001855c     DNAFlexTask.obj
 0002:00005584       __unwindtable$?defaultConstruct@?$QVector@VU2Qualifier@U2@@@@AAEXPAVU2Qualifier@U2@@0@Z 10018584     DNAFlexTask.obj
 0002:0000558c       __ehfuncinfo$?defaultConstruct@?$QVector@VU2Qualifier@U2@@@@AAEXPAVU2Qualifier@U2@@0@Z 1001858c     DNAFlexTask.obj
 0002:000055b0       __catchsym$?append@?$QList@V?$QSharedDataPointer@VAnnotationData@U2@@@@@@QAEXABV?$QSharedDataPointer@VAnnotationData@U2@@@@@Z$12 100185b0     DNAFlexTask.obj
 0002:000055c0       __tryblocktable$?append@?$QList@V?$QSharedDataPointer@VAnnotationData@U2@@@@@@QAEXABV?$QSharedDataPointer@VAnnotationData@U2@@@@@Z 100185c0     DNAFlexTask.obj
 0002:000055d4       __ehfuncinfo$?append@?$QList@V?$QSharedDataPointer@VAnnotationData@U2@@@@@@QAEXABV?$QSharedDataPointer@VAnnotationData@U2@@@@@Z 100185d4     DNAFlexTask.obj
 0002:000055f8       __unwindtable$?append@?$QList@V?$QSharedDataPointer@VAnnotationData@U2@@@@@@QAEXABV?$QSharedDataPointer@VAnnotationData@U2@@@@@Z 100185f8     DNAFlexTask.obj
 0002:00005628       __catchsym$?detach_helper_grow@?$QList@V?$QSharedDataPointer@VAnnotationData@U2@@@@@@AAEPAUNode@1@HH@Z$5 10018628     DNAFlexTask.obj
 0002:00005638       __catchsym$?detach_helper_grow@?$QList@V?$QSharedDataPointer@VAnnotationData@U2@@@@@@AAEPAUNode@1@HH@Z$4 10018638     DNAFlexTask.obj
 0002:00005648       __unwindtable$?detach_helper_grow@?$QList@V?$QSharedDataPointer@VAnnotationData@U2@@@@@@AAEPAUNode@1@HH@Z 10018648     DNAFlexTask.obj
 0002:00005668       __ehfuncinfo$?detach_helper_grow@?$QList@V?$QSharedDataPointer@VAnnotationData@U2@@@@@@AAEPAUNode@1@HH@Z 10018668     DNAFlexTask.obj
 0002:0000568c       __tryblocktable$?detach_helper_grow@?$QList@V?$QSharedDataPointer@VAnnotationData@U2@@@@@@AAEPAUNode@1@HH@Z 1001868c     DNAFlexTask.obj
 0002:000056b4       __unwindtable$??__EalgoLog@U2@@YAXXZ 100186b4     DNAFlexTask.obj
 0002:000056bc       __ehfuncinfo$??__EalgoLog@U2@@YAXXZ 100186bc     DNAFlexTask.obj
 0002:000056e0       __unwindtable$??__EcmdLog@U2@@YAXXZ 100186e0     DNAFlexTask.obj
 0002:000056e8       __ehfuncinfo$??__EcmdLog@U2@@YAXXZ 100186e8     DNAFlexTask.obj
 0002:0000570c       __unwindtable$??__EcoreLog@U2@@YAXXZ 1001870c     DNAFlexTask.obj
 0002:00005714       __ehfuncinfo$??__EcoreLog@U2@@YAXXZ 10018714     DNAFlexTask.obj
 0002:00005738       __unwindtable$??__EioLog@U2@@YAXXZ 10018738     DNAFlexTask.obj
 0002:00005740       __ehfuncinfo$??__EioLog@U2@@YAXXZ 10018740     DNAFlexTask.obj
 0002:00005764       __unwindtable$??__EperfLog@U2@@YAXXZ 10018764     DNAFlexTask.obj
 0002:0000576c       __ehfuncinfo$??__EperfLog@U2@@YAXXZ 1001876c     DNAFlexTask.obj
 0002:00005790       __unwindtable$??__EscriptLog@U2@@YAXXZ 10018790     DNAFlexTask.obj
 0002:00005798       __ehfuncinfo$??__EscriptLog@U2@@YAXXZ 10018798     DNAFlexTask.obj
 0002:000057bc       __unwindtable$??__EtaskLog@U2@@YAXXZ 100187bc     DNAFlexTask.obj
 0002:000057c4       __ehfuncinfo$??__EtaskLog@U2@@YAXXZ 100187c4     DNAFlexTask.obj
 0002:000057e8       __unwindtable$??__EuiLog@U2@@YAXXZ 100187e8     DNAFlexTask.obj
 0002:000057f0       __ehfuncinfo$??__EuiLog@U2@@YAXXZ 100187f0     DNAFlexTask.obj
 0002:00005814       __unwindtable$??__EuserActLog@U2@@YAXXZ 10018814     DNAFlexTask.obj
 0002:0000581c       __ehfuncinfo$??__EuserActLog@U2@@YAXXZ 1001881c     DNAFlexTask.obj
 0002:00005840       __catchsym$?append@?$QList@PAVTask@U2@@@@QAEXABQAVTask@U2@@@Z$6 10018840     DNAFlexTask.obj
 0002:00005850       __tryblocktable$?append@?$QList@PAVTask@U2@@@@QAEXABQAVTask@U2@@@Z 10018850     DNAFlexTask.obj
 0002:00005864       __ehfuncinfo$?append@?$QList@PAVTask@U2@@@@QAEXABQAVTask@U2@@@Z 10018864     DNAFlexTask.obj
 0002:00005888       __unwindtable$?append@?$QList@PAVTask@U2@@@@QAEXABQAVTask@U2@@@Z 10018888     DNAFlexTask.obj
 0002:000058b8       __catchsym$?detach_helper_grow@?$QList@PAVTask@U2@@@@AAEPAUNode@1@HH@Z$5 100188b8     DNAFlexTask.obj
 0002:000058c8       __catchsym$?detach_helper_grow@?$QList@PAVTask@U2@@@@AAEPAUNode@1@HH@Z$4 100188c8     DNAFlexTask.obj
 0002:000058d8       __unwindtable$?detach_helper_grow@?$QList@PAVTask@U2@@@@AAEPAUNode@1@HH@Z 100188d8     DNAFlexTask.obj
 0002:000058f8       __ehfuncinfo$?detach_helper_grow@?$QList@PAVTask@U2@@@@AAEPAUNode@1@HH@Z 100188f8     DNAFlexTask.obj
 0002:0000591c       __tryblocktable$?detach_helper_grow@?$QList@PAVTask@U2@@@@AAEPAUNode@1@HH@Z 1001891c     DNAFlexTask.obj
 0002:00005944       __catchsym$??0?$QList@VHighFlexResult@U2@@@@QAE@ABV0@@Z$2 10018944     DNAFlexTask.obj
 0002:00005954       __unwindtable$??0?$QList@VHighFlexResult@U2@@@@QAE@ABV0@@Z 10018954     DNAFlexTask.obj
 0002:00005964       __tryblocktable$??0?$QList@VHighFlexResult@U2@@@@QAE@ABV0@@Z 10018964     DNAFlexTask.obj
 0002:00005978       __ehfuncinfo$??0?$QList@VHighFlexResult@U2@@@@QAE@ABV0@@Z 10018978     DNAFlexTask.obj
 0002:0000599c       __catchsym$?node_copy@?$QList@VHighFlexResult@U2@@@@AAEXPAUNode@1@00@Z$4 1001899c     DNAFlexTask.obj
 0002:000059ac       __tryblocktable$?node_copy@?$QList@VHighFlexResult@U2@@@@AAEXPAUNode@1@00@Z 100189ac     DNAFlexTask.obj
 0002:000059c0       __unwindtable$?node_copy@?$QList@VHighFlexResult@U2@@@@AAEXPAUNode@1@00@Z 100189c0     DNAFlexTask.obj
 0002:000059e0       __ehfuncinfo$?node_copy@?$QList@VHighFlexResult@U2@@@@AAEXPAUNode@1@00@Z 100189e0     DNAFlexTask.obj
 0002:00005a04       __ehfuncinfo$??0DNAFlexTask@U2@@QAE@ABVHighFlexSettings@1@PAVAnnotationTableObject@1@ABVQString@@22ABVDNASequence@1@@Z 10018a04     DNAFlexTask.obj
 0002:00005a28       __unwindtable$??0DNAFlexTask@U2@@QAE@ABVHighFlexSettings@1@PAVAnnotationTableObject@1@ABVQString@@22ABVDNASequence@1@@Z 10018a28     DNAFlexTask.obj
 0002:00005a70       __ehfuncinfo$?onSubTaskFinished@DNAFlexTask@U2@@UAE?AV?$QList@PAVTask@U2@@@@PAVTask@2@@Z 10018a70     DNAFlexTask.obj
 0002:00005a94       __unwindtable$?onSubTaskFinished@DNAFlexTask@U2@@UAE?AV?$QList@PAVTask@U2@@@@PAVTask@2@@Z 10018a94     DNAFlexTask.obj
 0002:00005afc       __ehfuncinfo$?getAnnotationsFromResults@DNAFlexTask@U2@@QAE?AV?$QList@V?$QSharedDataPointer@VAnnotationData@U2@@@@@@ABV?$QList@VHighFlexResult@U2@@@@@Z 10018afc     DNAFlexTask.obj
 0002:00005b20       __unwindtable$?getAnnotationsFromResults@DNAFlexTask@U2@@QAE?AV?$QList@V?$QSharedDataPointer@VAnnotationData@U2@@@@@@ABV?$QList@VHighFlexResult@U2@@@@@Z 10018b20     DNAFlexTask.obj
 0002:00005bb0       __ehfuncinfo$??1DNAFlexTask@U2@@UAE@XZ 10018bb0     DNAFlexTask.obj
 0002:00005bd4       __unwindtable$??1DNAFlexTask@U2@@UAE@XZ 10018bd4     DNAFlexTask.obj
 0002:00005bfc       __unwindtable$??__EalgoLog@U2@@YAXXZ 10018bfc     FindHighFlexRegions.obj
 0002:00005c04       __ehfuncinfo$??__EalgoLog@U2@@YAXXZ 10018c04     FindHighFlexRegions.obj
 0002:00005c28       __unwindtable$??__EcmdLog@U2@@YAXXZ 10018c28     FindHighFlexRegions.obj
 0002:00005c30       __ehfuncinfo$??__EcmdLog@U2@@YAXXZ 10018c30     FindHighFlexRegions.obj
 0002:00005c54       __unwindtable$??__EcoreLog@U2@@YAXXZ 10018c54     FindHighFlexRegions.obj
 0002:00005c5c       __ehfuncinfo$??__EcoreLog@U2@@YAXXZ 10018c5c     FindHighFlexRegions.obj
 0002:00005c80       __unwindtable$??__EioLog@U2@@YAXXZ 10018c80     FindHighFlexRegions.obj
 0002:00005c88       __ehfuncinfo$??__EioLog@U2@@YAXXZ 10018c88     FindHighFlexRegions.obj
 0002:00005cac       __unwindtable$??__EperfLog@U2@@YAXXZ 10018cac     FindHighFlexRegions.obj
 0002:00005cb4       __ehfuncinfo$??__EperfLog@U2@@YAXXZ 10018cb4     FindHighFlexRegions.obj
 0002:00005cd8       __unwindtable$??__EscriptLog@U2@@YAXXZ 10018cd8     FindHighFlexRegions.obj
 0002:00005ce0       __ehfuncinfo$??__EscriptLog@U2@@YAXXZ 10018ce0     FindHighFlexRegions.obj
 0002:00005d04       __unwindtable$??__EtaskLog@U2@@YAXXZ 10018d04     FindHighFlexRegions.obj
 0002:00005d0c       __ehfuncinfo$??__EtaskLog@U2@@YAXXZ 10018d0c     FindHighFlexRegions.obj
 0002:00005d30       __unwindtable$??__EuiLog@U2@@YAXXZ 10018d30     FindHighFlexRegions.obj
 0002:00005d38       __ehfuncinfo$??__EuiLog@U2@@YAXXZ 10018d38     FindHighFlexRegions.obj
 0002:00005d5c       __unwindtable$??__EuserActLog@U2@@YAXXZ 10018d5c     FindHighFlexRegions.obj
 0002:00005d64       __ehfuncinfo$??__EuserActLog@U2@@YAXXZ 10018d64     FindHighFlexRegions.obj
 0002:00005d88       __unwindtable$??0FindHighFlexRegions@U2@@QAE@ABVDNASequence@1@ABVHighFlexSettings@1@@Z 10018d88     FindHighFlexRegions.obj
 0002:00005da8       __ehfuncinfo$??0FindHighFlexRegions@U2@@QAE@ABVDNASequence@1@ABVHighFlexSettings@1@@Z 10018da8     FindHighFlexRegions.obj
 0002:00005dcc       __catchsym$?append@?$QList@VHighFlexResult@U2@@@@QAEXABVHighFlexResult@U2@@@Z$7 10018dcc     FindHighFlexRegions.obj
 0002:00005ddc       __catchsym$?append@?$QList@VHighFlexResult@U2@@@@QAEXABVHighFlexResult@U2@@@Z$6 10018ddc     FindHighFlexRegions.obj
 0002:00005dec       __ehfuncinfo$?append@?$QList@VHighFlexResult@U2@@@@QAEXABVHighFlexResult@U2@@@Z 10018dec     FindHighFlexRegions.obj
 0002:00005e10       __tryblocktable$?append@?$QList@VHighFlexResult@U2@@@@QAEXABVHighFlexResult@U2@@@Z 10018e10     FindHighFlexRegions.obj
 0002:00005e38       __unwindtable$?append@?$QList@VHighFlexResult@U2@@@@QAEXABVHighFlexResult@U2@@@Z 10018e38     FindHighFlexRegions.obj
 0002:00005e68       __catchsym$?detach_helper_grow@?$QList@VHighFlexResult@U2@@@@AAEPAUNode@1@HH@Z$5 10018e68     FindHighFlexRegions.obj
 0002:00005e78       __catchsym$?detach_helper_grow@?$QList@VHighFlexResult@U2@@@@AAEPAUNode@1@HH@Z$4 10018e78     FindHighFlexRegions.obj
 0002:00005e88       __unwindtable$?detach_helper_grow@?$QList@VHighFlexResult@U2@@@@AAEPAUNode@1@HH@Z 10018e88     FindHighFlexRegions.obj
 0002:00005ea8       __ehfuncinfo$?detach_helper_grow@?$QList@VHighFlexResult@U2@@@@AAEPAUNode@1@HH@Z 10018ea8     FindHighFlexRegions.obj
 0002:00005ecc       __tryblocktable$?detach_helper_grow@?$QList@VHighFlexResult@U2@@@@AAEPAUNode@1@HH@Z 10018ecc     FindHighFlexRegions.obj
 0002:00005ef4       __unwindtable$??1FindHighFlexRegions@U2@@UAE@XZ 10018ef4     FindHighFlexRegions.obj
 0002:00005f0c       __ehfuncinfo$??1FindHighFlexRegions@U2@@UAE@XZ 10018f0c     FindHighFlexRegions.obj
 0002:00005f30       __unwindtable$??_GFindHighFlexRegions@U2@@UAEPAXI@Z 10018f30     FindHighFlexRegions.obj
 0002:00005f48       __ehfuncinfo$??_GFindHighFlexRegions@U2@@UAEPAXI@Z 10018f48     FindHighFlexRegions.obj
 0002:00005f6c       __unwindtable$??__EalgoLog@U2@@YAXXZ 10018f6c     FindHighFlexRegionsAlgorithm.obj
 0002:00005f74       __ehfuncinfo$??__EalgoLog@U2@@YAXXZ 10018f74     FindHighFlexRegionsAlgorithm.obj
 0002:00005f98       __unwindtable$??__EcmdLog@U2@@YAXXZ 10018f98     FindHighFlexRegionsAlgorithm.obj
 0002:00005fa0       __ehfuncinfo$??__EcmdLog@U2@@YAXXZ 10018fa0     FindHighFlexRegionsAlgorithm.obj
 0002:00005fc4       __unwindtable$??__EcoreLog@U2@@YAXXZ 10018fc4     FindHighFlexRegionsAlgorithm.obj
 0002:00005fcc       __ehfuncinfo$??__EcoreLog@U2@@YAXXZ 10018fcc     FindHighFlexRegionsAlgorithm.obj
 0002:00005ff0       __unwindtable$??__EioLog@U2@@YAXXZ 10018ff0     FindHighFlexRegionsAlgorithm.obj
 0002:00005ff8       __ehfuncinfo$??__EioLog@U2@@YAXXZ 10018ff8     FindHighFlexRegionsAlgorithm.obj
 0002:0000601c       __unwindtable$??__EperfLog@U2@@YAXXZ 1001901c     FindHighFlexRegionsAlgorithm.obj
 0002:00006024       __ehfuncinfo$??__EperfLog@U2@@YAXXZ 10019024     FindHighFlexRegionsAlgorithm.obj
 0002:00006048       __unwindtable$??__EscriptLog@U2@@YAXXZ 10019048     FindHighFlexRegionsAlgorithm.obj
 0002:00006050       __ehfuncinfo$??__EscriptLog@U2@@YAXXZ 10019050     FindHighFlexRegionsAlgorithm.obj
 0002:00006074       __unwindtable$??__EtaskLog@U2@@YAXXZ 10019074     FindHighFlexRegionsAlgorithm.obj
 0002:0000607c       __ehfuncinfo$??__EtaskLog@U2@@YAXXZ 1001907c     FindHighFlexRegionsAlgorithm.obj
 0002:000060a0       __unwindtable$??__EuiLog@U2@@YAXXZ 100190a0     FindHighFlexRegionsAlgorithm.obj
 0002:000060a8       __ehfuncinfo$??__EuiLog@U2@@YAXXZ 100190a8     FindHighFlexRegionsAlgorithm.obj
 0002:000060cc       __unwindtable$??__EuserActLog@U2@@YAXXZ 100190cc     FindHighFlexRegionsAlgorithm.obj
 0002:000060d4       __ehfuncinfo$??__EuserActLog@U2@@YAXXZ 100190d4     FindHighFlexRegionsAlgorithm.obj
 0002:000060f8       __ehfuncinfo$?find@FindHighFlexRegionsAlgorithm@U2@@SAXPAVFindHighFlexRegionsListener@2@ABVHighFlexSettings@2@VQByteArray@@HAAH3@Z 100190f8     FindHighFlexRegionsAlgorithm.obj
 0002:0000611c       __unwindtable$?find@FindHighFlexRegionsAlgorithm@U2@@SAXPAVFindHighFlexRegionsListener@2@ABVHighFlexSettings@2@VQByteArray@@HAAH3@Z 1001911c     FindHighFlexRegionsAlgorithm.obj
 0002:00006184       __ehfuncinfo$?flexibilityAngle@FindHighFlexRegionsAlgorithm@U2@@SANDD@Z 10019184     FindHighFlexRegionsAlgorithm.obj
 0002:000061a8       __unwindtable$?flexibilityAngle@FindHighFlexRegionsAlgorithm@U2@@SANDD@Z 100191a8     FindHighFlexRegionsAlgorithm.obj
 0002:000061d8       __ehfuncinfo$?addToResults@FindHighFlexRegionsAlgorithm@U2@@CAXPAVFindHighFlexRegionsListener@2@ABVHighFlexResult@2@@Z 100191d8     FindHighFlexRegionsAlgorithm.obj
 0002:000061fc       __unwindtable$?addToResults@FindHighFlexRegionsAlgorithm@U2@@CAXPAVFindHighFlexRegionsListener@2@ABVHighFlexResult@2@@Z 100191fc     FindHighFlexRegionsAlgorithm.obj
 0002:0000622c       __unwindtable$??H@YA?BVQString@@ABV0@0@Z 1001922c     HighFlexSettings.obj
 0002:00006234       __ehfuncinfo$??H@YA?BVQString@@ABV0@0@Z 10019234     HighFlexSettings.obj
 0002:00006258       __unwindtable$??H@YA?BVQString@@ABV0@PBD@Z 10019258     HighFlexSettings.obj
 0002:00006268       __ehfuncinfo$??H@YA?BVQString@@ABV0@PBD@Z 10019268     HighFlexSettings.obj
 0002:0000628c       __ehfuncinfo$?restoreDefaults@HighFlexSettings@U2@@QAEXXZ 1001928c     HighFlexSettings.obj
 0002:000062b0       __unwindtable$?restoreDefaults@HighFlexSettings@U2@@QAEXXZ 100192b0     HighFlexSettings.obj
 0002:000062e0       __ehfuncinfo$?rememberSettings@HighFlexSettings@U2@@QAEXXZ 100192e0     HighFlexSettings.obj
 0002:00006304       __unwindtable$?rememberSettings@HighFlexSettings@U2@@QAEXXZ 10019304     HighFlexSettings.obj
 0002:0000634c       __ehfuncinfo$?restoreRememberedSettings@HighFlexSettings@U2@@AAE_NXZ 1001934c     HighFlexSettings.obj
 0002:00006370       __unwindtable$?restoreRememberedSettings@HighFlexSettings@U2@@AAE_NXZ 10019370     HighFlexSettings.obj
 0002:00006430       __unwindtable$??__EalgoLog@U2@@YAXXZ 10019430     HighFlexSettings.obj
 0002:00006438       __ehfuncinfo$??__EalgoLog@U2@@YAXXZ 10019438     HighFlexSettings.obj
 0002:0000645c       __unwindtable$??__EcmdLog@U2@@YAXXZ 1001945c     HighFlexSettings.obj
 0002:00006464       __ehfuncinfo$??__EcmdLog@U2@@YAXXZ 10019464     HighFlexSettings.obj
 0002:00006488       __unwindtable$??__EcoreLog@U2@@YAXXZ 10019488     HighFlexSettings.obj
 0002:00006490       __ehfuncinfo$??__EcoreLog@U2@@YAXXZ 10019490     HighFlexSettings.obj
 0002:000064b4       __unwindtable$??__EioLog@U2@@YAXXZ 100194b4     HighFlexSettings.obj
 0002:000064bc       __ehfuncinfo$??__EioLog@U2@@YAXXZ 100194bc     HighFlexSettings.obj
 0002:000064e0       __unwindtable$??__EperfLog@U2@@YAXXZ 100194e0     HighFlexSettings.obj
 0002:000064e8       __ehfuncinfo$??__EperfLog@U2@@YAXXZ 100194e8     HighFlexSettings.obj
 0002:0000650c       __unwindtable$??__EscriptLog@U2@@YAXXZ 1001950c     HighFlexSettings.obj
 0002:00006514       __ehfuncinfo$??__EscriptLog@U2@@YAXXZ 10019514     HighFlexSettings.obj
 0002:00006538       __unwindtable$??__EtaskLog@U2@@YAXXZ 10019538     HighFlexSettings.obj
 0002:00006540       __ehfuncinfo$??__EtaskLog@U2@@YAXXZ 10019540     HighFlexSettings.obj
 0002:00006564       __unwindtable$??__EuiLog@U2@@YAXXZ 10019564     HighFlexSettings.obj
 0002:0000656c       __ehfuncinfo$??__EuiLog@U2@@YAXXZ 1001956c     HighFlexSettings.obj
 0002:00006590       __unwindtable$??__EuserActLog@U2@@YAXXZ 10019590     HighFlexSettings.obj
 0002:00006598       __ehfuncinfo$??__EuserActLog@U2@@YAXXZ 10019598     HighFlexSettings.obj
 0002:000065bc       __unwindtable$??__EalgoLog@U2@@YAXXZ 100195bc     moc_DNAFlexGraph.obj
 0002:000065c4       __ehfuncinfo$??__EalgoLog@U2@@YAXXZ 100195c4     moc_DNAFlexGraph.obj
 0002:000065e8       __unwindtable$??__EcmdLog@U2@@YAXXZ 100195e8     moc_DNAFlexGraph.obj
 0002:000065f0       __ehfuncinfo$??__EcmdLog@U2@@YAXXZ 100195f0     moc_DNAFlexGraph.obj
 0002:00006614       __unwindtable$??__EcoreLog@U2@@YAXXZ 10019614     moc_DNAFlexGraph.obj
 0002:0000661c       __ehfuncinfo$??__EcoreLog@U2@@YAXXZ 1001961c     moc_DNAFlexGraph.obj
 0002:00006640       __unwindtable$??__EioLog@U2@@YAXXZ 10019640     moc_DNAFlexGraph.obj
 0002:00006648       __ehfuncinfo$??__EioLog@U2@@YAXXZ 10019648     moc_DNAFlexGraph.obj
 0002:0000666c       __unwindtable$??__EperfLog@U2@@YAXXZ 1001966c     moc_DNAFlexGraph.obj
 0002:00006674       __ehfuncinfo$??__EperfLog@U2@@YAXXZ 10019674     moc_DNAFlexGraph.obj
 0002:00006698       __unwindtable$??__EscriptLog@U2@@YAXXZ 10019698     moc_DNAFlexGraph.obj
 0002:000066a0       __ehfuncinfo$??__EscriptLog@U2@@YAXXZ 100196a0     moc_DNAFlexGraph.obj
 0002:000066c4       __unwindtable$??__EtaskLog@U2@@YAXXZ 100196c4     moc_DNAFlexGraph.obj
 0002:000066cc       __ehfuncinfo$??__EtaskLog@U2@@YAXXZ 100196cc     moc_DNAFlexGraph.obj
 0002:000066f0       __unwindtable$??__EuiLog@U2@@YAXXZ 100196f0     moc_DNAFlexGraph.obj
 0002:000066f8       __ehfuncinfo$??__EuiLog@U2@@YAXXZ 100196f8     moc_DNAFlexGraph.obj
 0002:0000671c       __unwindtable$??__EuserActLog@U2@@YAXXZ 1001971c     moc_DNAFlexGraph.obj
 0002:00006724       __ehfuncinfo$??__EuserActLog@U2@@YAXXZ 10019724     moc_DNAFlexGraph.obj
 0002:00006748       __unwindtable$??__EalgoLog@U2@@YAXXZ 10019748     moc_DNAFlexPlugin.obj
 0002:00006750       __ehfuncinfo$??__EalgoLog@U2@@YAXXZ 10019750     moc_DNAFlexPlugin.obj
 0002:00006774       __unwindtable$??__EcmdLog@U2@@YAXXZ 10019774     moc_DNAFlexPlugin.obj
 0002:0000677c       __ehfuncinfo$??__EcmdLog@U2@@YAXXZ 1001977c     moc_DNAFlexPlugin.obj
 0002:000067a0       __unwindtable$??__EcoreLog@U2@@YAXXZ 100197a0     moc_DNAFlexPlugin.obj
 0002:000067a8       __ehfuncinfo$??__EcoreLog@U2@@YAXXZ 100197a8     moc_DNAFlexPlugin.obj
 0002:000067cc       __unwindtable$??__EioLog@U2@@YAXXZ 100197cc     moc_DNAFlexPlugin.obj
 0002:000067d4       __ehfuncinfo$??__EioLog@U2@@YAXXZ 100197d4     moc_DNAFlexPlugin.obj
 0002:000067f8       __unwindtable$??__EperfLog@U2@@YAXXZ 100197f8     moc_DNAFlexPlugin.obj
 0002:00006800       __ehfuncinfo$??__EperfLog@U2@@YAXXZ 10019800     moc_DNAFlexPlugin.obj
 0002:00006824       __unwindtable$??__EscriptLog@U2@@YAXXZ 10019824     moc_DNAFlexPlugin.obj
 0002:0000682c       __ehfuncinfo$??__EscriptLog@U2@@YAXXZ 1001982c     moc_DNAFlexPlugin.obj
 0002:00006850       __unwindtable$??__EtaskLog@U2@@YAXXZ 10019850     moc_DNAFlexPlugin.obj
 0002:00006858       __ehfuncinfo$??__EtaskLog@U2@@YAXXZ 10019858     moc_DNAFlexPlugin.obj
 0002:0000687c       __unwindtable$??__EuiLog@U2@@YAXXZ 1001987c     moc_DNAFlexPlugin.obj
 0002:00006884       __ehfuncinfo$??__EuiLog@U2@@YAXXZ 10019884     moc_DNAFlexPlugin.obj
 0002:000068a8       __unwindtable$??__EuserActLog@U2@@YAXXZ 100198a8     moc_DNAFlexPlugin.obj
 0002:000068b0       __ehfuncinfo$??__EuserActLog@U2@@YAXXZ 100198b0     moc_DNAFlexPlugin.obj
 0002:000068d4       __unwindtable$?qt_metatype_id@?$QMetaTypeIdQObject@PAVADVSequenceWidget@U2@@$00@@SAHXZ 100198d4     moc_DNAFlexPlugin.obj
 0002:000068dc       __ehfuncinfo$?qt_metatype_id@?$QMetaTypeIdQObject@PAVADVSequenceWidget@U2@@$00@@SAHXZ 100198dc     moc_DNAFlexPlugin.obj
 0002:00006900       __unwindtable$??__EalgoLog@U2@@YAXXZ 10019900     moc_DNAFlexTask.obj
 0002:00006908       __ehfuncinfo$??__EalgoLog@U2@@YAXXZ 10019908     moc_DNAFlexTask.obj
 0002:0000692c       __unwindtable$??__EcmdLog@U2@@YAXXZ 1001992c     moc_DNAFlexTask.obj
 0002:00006934       __ehfuncinfo$??__EcmdLog@U2@@YAXXZ 10019934     moc_DNAFlexTask.obj
 0002:00006958       __unwindtable$??__EcoreLog@U2@@YAXXZ 10019958     moc_DNAFlexTask.obj
 0002:00006960       __ehfuncinfo$??__EcoreLog@U2@@YAXXZ 10019960     moc_DNAFlexTask.obj
 0002:00006984       __unwindtable$??__EioLog@U2@@YAXXZ 10019984     moc_DNAFlexTask.obj
 0002:0000698c       __ehfuncinfo$??__EioLog@U2@@YAXXZ 1001998c     moc_DNAFlexTask.obj
 0002:000069b0       __unwindtable$??__EperfLog@U2@@YAXXZ 100199b0     moc_DNAFlexTask.obj
 0002:000069b8       __ehfuncinfo$??__EperfLog@U2@@YAXXZ 100199b8     moc_DNAFlexTask.obj
 0002:000069dc       __unwindtable$??__EscriptLog@U2@@YAXXZ 100199dc     moc_DNAFlexTask.obj
 0002:000069e4       __ehfuncinfo$??__EscriptLog@U2@@YAXXZ 100199e4     moc_DNAFlexTask.obj
 0002:00006a08       __unwindtable$??__EtaskLog@U2@@YAXXZ 10019a08     moc_DNAFlexTask.obj
 0002:00006a10       __ehfuncinfo$??__EtaskLog@U2@@YAXXZ 10019a10     moc_DNAFlexTask.obj
 0002:00006a34       __unwindtable$??__EuiLog@U2@@YAXXZ 10019a34     moc_DNAFlexTask.obj
 0002:00006a3c       __ehfuncinfo$??__EuiLog@U2@@YAXXZ 10019a3c     moc_DNAFlexTask.obj
 0002:00006a60       __unwindtable$??__EuserActLog@U2@@YAXXZ 10019a60     moc_DNAFlexTask.obj
 0002:00006a68       __ehfuncinfo$??__EuserActLog@U2@@YAXXZ 10019a68     moc_DNAFlexTask.obj
 0002:00006a8c       __unwindtable$??__EalgoLog@U2@@YAXXZ 10019a8c     moc_FindHighFlexRegions.obj
 0002:00006a94       __ehfuncinfo$??__EalgoLog@U2@@YAXXZ 10019a94     moc_FindHighFlexRegions.obj
 0002:00006ab8       __unwindtable$??__EcmdLog@U2@@YAXXZ 10019ab8     moc_FindHighFlexRegions.obj
 0002:00006ac0       __ehfuncinfo$??__EcmdLog@U2@@YAXXZ 10019ac0     moc_FindHighFlexRegions.obj
 0002:00006ae4       __unwindtable$??__EcoreLog@U2@@YAXXZ 10019ae4     moc_FindHighFlexRegions.obj
 0002:00006aec       __ehfuncinfo$??__EcoreLog@U2@@YAXXZ 10019aec     moc_FindHighFlexRegions.obj
 0002:00006b10       __unwindtable$??__EioLog@U2@@YAXXZ 10019b10     moc_FindHighFlexRegions.obj
 0002:00006b18       __ehfuncinfo$??__EioLog@U2@@YAXXZ 10019b18     moc_FindHighFlexRegions.obj
 0002:00006b3c       __unwindtable$??__EperfLog@U2@@YAXXZ 10019b3c     moc_FindHighFlexRegions.obj
 0002:00006b44       __ehfuncinfo$??__EperfLog@U2@@YAXXZ 10019b44     moc_FindHighFlexRegions.obj
 0002:00006b68       __unwindtable$??__EscriptLog@U2@@YAXXZ 10019b68     moc_FindHighFlexRegions.obj
 0002:00006b70       __ehfuncinfo$??__EscriptLog@U2@@YAXXZ 10019b70     moc_FindHighFlexRegions.obj
 0002:00006b94       __unwindtable$??__EtaskLog@U2@@YAXXZ 10019b94     moc_FindHighFlexRegions.obj
 0002:00006b9c       __ehfuncinfo$??__EtaskLog@U2@@YAXXZ 10019b9c     moc_FindHighFlexRegions.obj
 0002:00006bc0       __unwindtable$??__EuiLog@U2@@YAXXZ 10019bc0     moc_FindHighFlexRegions.obj
 0002:00006bc8       __ehfuncinfo$??__EuiLog@U2@@YAXXZ 10019bc8     moc_FindHighFlexRegions.obj
 0002:00006bec       __unwindtable$??__EuserActLog@U2@@YAXXZ 10019bec     moc_FindHighFlexRegions.obj
 0002:00006bf4       __ehfuncinfo$??__EuserActLog@U2@@YAXXZ 10019bf4     moc_FindHighFlexRegions.obj
 0002:00006c18       __sehtable$__onexit        10019c18     MSVCRT:atonexit.obj
 0002:00006c38       __sehtable$___DllMainCRTStartup 10019c38     MSVCRT:crtdll.obj
 0002:00006c60       __sehtable$??_M@YGXPAXIHP6EX0@Z@Z 10019c60     MSVCRT:ehvecdtr.obj
 0002:00006c80       __sehtable$?__ArrayUnwind@@YGXPAXIHP6EX0@Z@Z 10019c80     MSVCRT:ehvecdtr.obj
 0002:00006ca0       __sehtable$__IsNonwritableInCurrentImage 10019ca0     MSVCRT:pesect.obj
 0002:00006cc0       .edata                     10019cc0     dna_flexibility.exp
 0002:00006ce8       rgpv                       10019ce8     dna_flexibility.exp
 0002:00006cec       rgszName                   10019cec     dna_flexibility.exp
 0002:00006cf0       rgwOrd                     10019cf0     dna_flexibility.exp
 0002:00006cf2       szName                     10019cf2     dna_flexibility.exp
 0002:00006d06       $N00001                    10019d06     dna_flexibility.exp
 0002:000083ae       .idata$6                   1001b3ae     U2Core:U2Core.dll
 0002:00008cbc       .idata$6                   1001bcbc     U2Gui:U2Gui.dll
 0002:0000962c       .idata$6                   1001c62c     U2View:U2View.dll
 0002:0000cb6e       .idata$6                   1001fb6e     Qt5Widgets:Qt5Widgets.dll
 0002:0000cbb2       .idata$6                   1001fbb2     Qt5Gui:Qt5Gui.dll
 0002:0000d6aa       .idata$6                   100206aa     Qt5Core:Qt5Core.dll
 0002:0000d750       .idata$6                   10020750     msvcprt:MSVCP120.dll
 0002:0000d7de       .idata$6                   100207de     MSVCRT:MSVCR120.dll
 0002:0000d9f2       .idata$6                   100209f2     kernel32:KERNEL32.dll
 0003:0000000c       _Service_PluginViewer      1002100c     DNAFlexDialog.obj
 0003:00000014       _Service_Project           10021014     DNAFlexDialog.obj
 0003:0000001c       _Service_ProjectView       1002101c     DNAFlexDialog.obj
 0003:00000024       _Service_DNAGraphPack      10021024     DNAFlexDialog.obj
 0003:0000002c       _Service_DNAExport         1002102c     DNAFlexDialog.obj
 0003:00000034       _Service_TestRunner        10021034     DNAFlexDialog.obj
 0003:0000003c       _Service_ScriptRegistry    1002103c     DNAFlexDialog.obj
 0003:00000044       _Service_ExternalToolSupport 10021044     DNAFlexDialog.obj
 0003:0000004c       _Service_GUITesting        1002104c     DNAFlexDialog.obj
 0003:00000054       _Service_WorkflowDesigner  10021054     DNAFlexDialog.obj
 0003:0000005c       _Service_QueryDesigner     1002105c     DNAFlexDialog.obj
 0003:00000064       _Service_MinCoreServiceId  10021064     DNAFlexDialog.obj
 0003:0000006c       _Service_MaxCoreServiceId  1002106c     DNAFlexDialog.obj
 0003:00000074       _Service_PluginViewer      10021074     DNAFlexGraph.obj
 0003:0000007c       _Service_Project           1002107c     DNAFlexGraph.obj
 0003:00000084       _Service_ProjectView       10021084     DNAFlexGraph.obj
 0003:0000008c       _Service_DNAGraphPack      1002108c     DNAFlexGraph.obj
 0003:00000094       _Service_DNAExport         10021094     DNAFlexGraph.obj
 0003:0000009c       _Service_TestRunner        1002109c     DNAFlexGraph.obj
 0003:000000a4       _Service_ScriptRegistry    100210a4     DNAFlexGraph.obj
 0003:000000ac       _Service_ExternalToolSupport 100210ac     DNAFlexGraph.obj
 0003:000000b4       _Service_GUITesting        100210b4     DNAFlexGraph.obj
 0003:000000bc       _Service_WorkflowDesigner  100210bc     DNAFlexGraph.obj
 0003:000000c4       _Service_QueryDesigner     100210c4     DNAFlexGraph.obj
 0003:000000cc       _Service_MinCoreServiceId  100210cc     DNAFlexGraph.obj
 0003:000000d4       _Service_MaxCoreServiceId  100210d4     DNAFlexGraph.obj
 0003:000000dc       _Service_PluginViewer      100210dc     DNAFlexGraphAlgorithm.obj
 0003:000000e4       _Service_Project           100210e4     DNAFlexGraphAlgorithm.obj
 0003:000000ec       _Service_ProjectView       100210ec     DNAFlexGraphAlgorithm.obj
 0003:000000f4       _Service_DNAGraphPack      100210f4     DNAFlexGraphAlgorithm.obj
 0003:000000fc       _Service_DNAExport         100210fc     DNAFlexGraphAlgorithm.obj
 0003:00000104       _Service_TestRunner        10021104     DNAFlexGraphAlgorithm.obj
 0003:0000010c       _Service_ScriptRegistry    1002110c     DNAFlexGraphAlgorithm.obj
 0003:00000114       _Service_ExternalToolSupport 10021114     DNAFlexGraphAlgorithm.obj
 0003:0000011c       _Service_GUITesting        1002111c     DNAFlexGraphAlgorithm.obj
 0003:00000124       _Service_WorkflowDesigner  10021124     DNAFlexGraphAlgorithm.obj
 0003:0000012c       _Service_QueryDesigner     1002112c     DNAFlexGraphAlgorithm.obj
 0003:00000134       _Service_MinCoreServiceId  10021134     DNAFlexGraphAlgorithm.obj
 0003:0000013c       _Service_MaxCoreServiceId  1002113c     DNAFlexGraphAlgorithm.obj
 0003:00000144       _Service_PluginViewer      10021144     DNAFlexPlugin.obj
 0003:0000014c       _Service_Project           1002114c     DNAFlexPlugin.obj
 0003:00000154       _Service_ProjectView       10021154     DNAFlexPlugin.obj
 0003:0000015c       _Service_DNAGraphPack      1002115c     DNAFlexPlugin.obj
 0003:00000164       _Service_DNAExport         10021164     DNAFlexPlugin.obj
 0003:0000016c       _Service_TestRunner        1002116c     DNAFlexPlugin.obj
 0003:00000174       _Service_ScriptRegistry    10021174     DNAFlexPlugin.obj
 0003:0000017c       _Service_ExternalToolSupport 1002117c     DNAFlexPlugin.obj
 0003:00000184       _Service_GUITesting        10021184     DNAFlexPlugin.obj
 0003:0000018c       _Service_WorkflowDesigner  1002118c     DNAFlexPlugin.obj
 0003:00000194       _Service_QueryDesigner     10021194     DNAFlexPlugin.obj
 0003:0000019c       _Service_MinCoreServiceId  1002119c     DNAFlexPlugin.obj
 0003:000001a4       _Service_MaxCoreServiceId  100211a4     DNAFlexPlugin.obj
 0003:000001c4       _Service_PluginViewer      100211c4     moc_DNAFlexGraph.obj
 0003:000001cc       _Service_Project           100211cc     moc_DNAFlexGraph.obj
 0003:000001d4       _Service_ProjectView       100211d4     moc_DNAFlexGraph.obj
 0003:000001dc       _Service_DNAGraphPack      100211dc     moc_DNAFlexGraph.obj
 0003:000001e4       _Service_DNAExport         100211e4     moc_DNAFlexGraph.obj
 0003:000001ec       _Service_TestRunner        100211ec     moc_DNAFlexGraph.obj
 0003:000001f4       _Service_ScriptRegistry    100211f4     moc_DNAFlexGraph.obj
 0003:000001fc       _Service_ExternalToolSupport 100211fc     moc_DNAFlexGraph.obj
 0003:00000204       _Service_GUITesting        10021204     moc_DNAFlexGraph.obj
 0003:0000020c       _Service_WorkflowDesigner  1002120c     moc_DNAFlexGraph.obj
 0003:00000214       _Service_QueryDesigner     10021214     moc_DNAFlexGraph.obj
 0003:0000021c       _Service_MinCoreServiceId  1002121c     moc_DNAFlexGraph.obj
 0003:00000224       _Service_MaxCoreServiceId  10021224     moc_DNAFlexGraph.obj
 0003:00000244       _Service_PluginViewer      10021244     moc_DNAFlexPlugin.obj
 0003:0000024c       _Service_Project           1002124c     moc_DNAFlexPlugin.obj
 0003:00000254       _Service_ProjectView       10021254     moc_DNAFlexPlugin.obj
 0003:0000025c       _Service_DNAGraphPack      1002125c     moc_DNAFlexPlugin.obj
 0003:00000264       _Service_DNAExport         10021264     moc_DNAFlexPlugin.obj
 0003:0000026c       _Service_TestRunner        1002126c     moc_DNAFlexPlugin.obj
 0003:00000274       _Service_ScriptRegistry    10021274     moc_DNAFlexPlugin.obj
 0003:0000027c       _Service_ExternalToolSupport 1002127c     moc_DNAFlexPlugin.obj
 0003:00000284       _Service_GUITesting        10021284     moc_DNAFlexPlugin.obj
 0003:0000028c       _Service_WorkflowDesigner  1002128c     moc_DNAFlexPlugin.obj
 0003:00000294       _Service_QueryDesigner     10021294     moc_DNAFlexPlugin.obj
 0003:0000029c       _Service_MinCoreServiceId  1002129c     moc_DNAFlexPlugin.obj
 0003:000002a4       _Service_MaxCoreServiceId  100212a4     moc_DNAFlexPlugin.obj
 0003:00000a10       __Tuple_alloc              10021a10     DNAFlexDialog.obj
 0003:00000a11       _ignore                    10021a11     DNAFlexDialog.obj
 0003:00000a12       _allocator_arg             10021a12     DNAFlexDialog.obj
 0003:00000a13       _piecewise_construct       10021a13     DNAFlexDialog.obj
 0003:00000a14       _taskLog                   10021a14     DNAFlexDialog.obj
 0003:00000a1c       _algoLog                   10021a1c     DNAFlexDialog.obj
 0003:00000a24       _userActLog                10021a24     DNAFlexDialog.obj
 0003:00000a2c       _ioLog                     10021a2c     DNAFlexDialog.obj
 0003:00000a34       _coreLog                   10021a34     DNAFlexDialog.obj
 0003:00000a3c       _uiLog                     10021a3c     DNAFlexDialog.obj
 0003:00000a44       _scriptLog                 10021a44     DNAFlexDialog.obj
 0003:00000a4c       _perfLog                   10021a4c     DNAFlexDialog.obj
 0003:00000a54       _cmdLog                    10021a54     DNAFlexDialog.obj
 0003:00000a64       __Tuple_alloc              10021a64     DNAFlexGraph.obj
 0003:00000a65       _ignore                    10021a65     DNAFlexGraph.obj
 0003:00000a66       _allocator_arg             10021a66     DNAFlexGraph.obj
 0003:00000a67       _piecewise_construct       10021a67     DNAFlexGraph.obj
 0003:00000a68       _taskLog                   10021a68     DNAFlexGraph.obj
 0003:00000a70       _algoLog                   10021a70     DNAFlexGraph.obj
 0003:00000a78       _userActLog                10021a78     DNAFlexGraph.obj
 0003:00000a80       _ioLog                     10021a80     DNAFlexGraph.obj
 0003:00000a88       _coreLog                   10021a88     DNAFlexGraph.obj
 0003:00000a90       _uiLog                     10021a90     DNAFlexGraph.obj
 0003:00000a98       _scriptLog                 10021a98     DNAFlexGraph.obj
 0003:00000aa0       _perfLog                   10021aa0     DNAFlexGraph.obj
 0003:00000aa8       _cmdLog                    10021aa8     DNAFlexGraph.obj
 0003:00000ab0       __Tuple_alloc              10021ab0     DNAFlexGraphAlgorithm.obj
 0003:00000ab1       _ignore                    10021ab1     DNAFlexGraphAlgorithm.obj
 0003:00000ab2       _allocator_arg             10021ab2     DNAFlexGraphAlgorithm.obj
 0003:00000ab3       _piecewise_construct       10021ab3     DNAFlexGraphAlgorithm.obj
 0003:00000ab4       _taskLog                   10021ab4     DNAFlexGraphAlgorithm.obj
 0003:00000abc       _algoLog                   10021abc     DNAFlexGraphAlgorithm.obj
 0003:00000ac4       _userActLog                10021ac4     DNAFlexGraphAlgorithm.obj
 0003:00000acc       _ioLog                     10021acc     DNAFlexGraphAlgorithm.obj
 0003:00000ad4       _coreLog                   10021ad4     DNAFlexGraphAlgorithm.obj
 0003:00000adc       _uiLog                     10021adc     DNAFlexGraphAlgorithm.obj
 0003:00000ae4       _scriptLog                 10021ae4     DNAFlexGraphAlgorithm.obj
 0003:00000aec       _perfLog                   10021aec     DNAFlexGraphAlgorithm.obj
 0003:00000af4       _cmdLog                    10021af4     DNAFlexGraphAlgorithm.obj
 0003:00000afc       __Tuple_alloc              10021afc     DNAFlexPlugin.obj
 0003:00000afd       _ignore                    10021afd     DNAFlexPlugin.obj
 0003:00000afe       _allocator_arg             10021afe     DNAFlexPlugin.obj
 0003:00000aff       _piecewise_construct       10021aff     DNAFlexPlugin.obj
 0003:00000b00       _taskLog                   10021b00     DNAFlexPlugin.obj
 0003:00000b08       _algoLog                   10021b08     DNAFlexPlugin.obj
 0003:00000b10       _userActLog                10021b10     DNAFlexPlugin.obj
 0003:00000b18       _ioLog                     10021b18     DNAFlexPlugin.obj
 0003:00000b20       _coreLog                   10021b20     DNAFlexPlugin.obj
 0003:00000b28       _uiLog                     10021b28     DNAFlexPlugin.obj
 0003:00000b30       _scriptLog                 10021b30     DNAFlexPlugin.obj
 0003:00000b38       _perfLog                   10021b38     DNAFlexPlugin.obj
 0003:00000b40       _cmdLog                    10021b40     DNAFlexPlugin.obj
 0003:00000b48       __Tuple_alloc              10021b48     DNAFlexTask.obj
 0003:00000b49       _ignore                    10021b49     DNAFlexTask.obj
 0003:00000b4a       _allocator_arg             10021b4a     DNAFlexTask.obj
 0003:00000b4b       _piecewise_construct       10021b4b     DNAFlexTask.obj
 0003:00000b4c       _taskLog                   10021b4c     DNAFlexTask.obj
 0003:00000b54       _algoLog                   10021b54     DNAFlexTask.obj
 0003:00000b5c       _userActLog                10021b5c     DNAFlexTask.obj
 0003:00000b64       _ioLog                     10021b64     DNAFlexTask.obj
 0003:00000b6c       _coreLog                   10021b6c     DNAFlexTask.obj
 0003:00000b74       _uiLog                     10021b74     DNAFlexTask.obj
 0003:00000b7c       _scriptLog                 10021b7c     DNAFlexTask.obj
 0003:00000b84       _perfLog                   10021b84     DNAFlexTask.obj
 0003:00000b8c       _cmdLog                    10021b8c     DNAFlexTask.obj
 0003:00000b94       __Tuple_alloc              10021b94     FindHighFlexRegions.obj
 0003:00000b95       _ignore                    10021b95     FindHighFlexRegions.obj
 0003:00000b96       _allocator_arg             10021b96     FindHighFlexRegions.obj
 0003:00000b97       _piecewise_construct       10021b97     FindHighFlexRegions.obj
 0003:00000b98       _taskLog                   10021b98     FindHighFlexRegions.obj
 0003:00000ba0       _algoLog                   10021ba0     FindHighFlexRegions.obj
 0003:00000ba8       _userActLog                10021ba8     FindHighFlexRegions.obj
 0003:00000bb0       _ioLog                     10021bb0     FindHighFlexRegions.obj
 0003:00000bb8       _coreLog                   10021bb8     FindHighFlexRegions.obj
 0003:00000bc0       _uiLog                     10021bc0     FindHighFlexRegions.obj
 0003:00000bc8       _scriptLog                 10021bc8     FindHighFlexRegions.obj
 0003:00000bd0       _perfLog                   10021bd0     FindHighFlexRegions.obj
 0003:00000bd8       _cmdLog                    10021bd8     FindHighFlexRegions.obj
 0003:00000be0       __Tuple_alloc              10021be0     FindHighFlexRegionsAlgorithm.obj
 0003:00000be1       _ignore                    10021be1     FindHighFlexRegionsAlgorithm.obj
 0003:00000be2       _allocator_arg             10021be2     FindHighFlexRegionsAlgorithm.obj
 0003:00000be3       _piecewise_construct       10021be3     FindHighFlexRegionsAlgorithm.obj
 0003:00000be4       _taskLog                   10021be4     FindHighFlexRegionsAlgorithm.obj
 0003:00000bec       _algoLog                   10021bec     FindHighFlexRegionsAlgorithm.obj
 0003:00000bf4       _userActLog                10021bf4     FindHighFlexRegionsAlgorithm.obj
 0003:00000bfc       _ioLog                     10021bfc     FindHighFlexRegionsAlgorithm.obj
 0003:00000c04       _coreLog                   10021c04     FindHighFlexRegionsAlgorithm.obj
 0003:00000c0c       _uiLog                     10021c0c     FindHighFlexRegionsAlgorithm.obj
 0003:00000c14       _scriptLog                 10021c14     FindHighFlexRegionsAlgorithm.obj
 0003:00000c1c       _perfLog                   10021c1c     FindHighFlexRegionsAlgorithm.obj
 0003:00000c24       _cmdLog                    10021c24     FindHighFlexRegionsAlgorithm.obj
 0003:00000c2c       __Tuple_alloc              10021c2c     HighFlexSettings.obj
 0003:00000c2d       _ignore                    10021c2d     HighFlexSettings.obj
 0003:00000c2e       _allocator_arg             10021c2e     HighFlexSettings.obj
 0003:00000c2f       _piecewise_construct       10021c2f     HighFlexSettings.obj
 0003:00000c30       _taskLog                   10021c30     HighFlexSettings.obj
 0003:00000c38       _algoLog                   10021c38     HighFlexSettings.obj
 0003:00000c44       _userActLog                10021c44     HighFlexSettings.obj
 0003:00000c4c       _ioLog                     10021c4c     HighFlexSettings.obj
 0003:00000c54       _coreLog                   10021c54     HighFlexSettings.obj
 0003:00000c5c       _uiLog                     10021c5c     HighFlexSettings.obj
 0003:00000c64       _scriptLog                 10021c64     HighFlexSettings.obj
 0003:00000c70       _perfLog                   10021c70     HighFlexSettings.obj
 0003:00000c7c       _cmdLog                    10021c7c     HighFlexSettings.obj
 0003:00000c88       __Tuple_alloc              10021c88     moc_DNAFlexDialog.obj
 0003:00000c89       _ignore                    10021c89     moc_DNAFlexDialog.obj
 0003:00000c8a       _allocator_arg             10021c8a     moc_DNAFlexDialog.obj
 0003:00000c8b       _piecewise_construct       10021c8b     moc_DNAFlexDialog.obj
 0003:00000c8c       __Tuple_alloc              10021c8c     moc_DNAFlexGraph.obj
 0003:00000c8d       _ignore                    10021c8d     moc_DNAFlexGraph.obj
 0003:00000c8e       _allocator_arg             10021c8e     moc_DNAFlexGraph.obj
 0003:00000c8f       _piecewise_construct       10021c8f     moc_DNAFlexGraph.obj
 0003:00000c90       _taskLog                   10021c90     moc_DNAFlexGraph.obj
 0003:00000c98       _algoLog                   10021c98     moc_DNAFlexGraph.obj
 0003:00000ca0       _userActLog                10021ca0     moc_DNAFlexGraph.obj
 0003:00000ca8       _ioLog                     10021ca8     moc_DNAFlexGraph.obj
 0003:00000cb0       _coreLog                   10021cb0     moc_DNAFlexGraph.obj
 0003:00000cb8       _uiLog                     10021cb8     moc_DNAFlexGraph.obj
 0003:00000cc0       _scriptLog                 10021cc0     moc_DNAFlexGraph.obj
 0003:00000cc8       _perfLog                   10021cc8     moc_DNAFlexGraph.obj
 0003:00000cd0       _cmdLog                    10021cd0     moc_DNAFlexGraph.obj
 0003:00000cd8       __Tuple_alloc              10021cd8     moc_DNAFlexPlugin.obj
 0003:00000cd9       _ignore                    10021cd9     moc_DNAFlexPlugin.obj
 0003:00000cda       _allocator_arg             10021cda     moc_DNAFlexPlugin.obj
 0003:00000cdb       _piecewise_construct       10021cdb     moc_DNAFlexPlugin.obj
 0003:00000cdc       _taskLog                   10021cdc     moc_DNAFlexPlugin.obj
 0003:00000ce4       _algoLog                   10021ce4     moc_DNAFlexPlugin.obj
 0003:00000cec       _userActLog                10021cec     moc_DNAFlexPlugin.obj
 0003:00000cf4       _ioLog                     10021cf4     moc_DNAFlexPlugin.obj
 0003:00000cfc       _coreLog                   10021cfc     moc_DNAFlexPlugin.obj
 0003:00000d04       _uiLog                     10021d04     moc_DNAFlexPlugin.obj
 0003:00000d0c       _scriptLog                 10021d0c     moc_DNAFlexPlugin.obj
 0003:00000d14       _perfLog                   10021d14     moc_DNAFlexPlugin.obj
 0003:00000d1c       _cmdLog                    10021d1c     moc_DNAFlexPlugin.obj
 0003:00000d28       __Tuple_alloc              10021d28     moc_DNAFlexTask.obj
 0003:00000d29       _ignore                    10021d29     moc_DNAFlexTask.obj
 0003:00000d2a       _allocator_arg             10021d2a     moc_DNAFlexTask.obj
 0003:00000d2b       _piecewise_construct       10021d2b     moc_DNAFlexTask.obj
 0003:00000d2c       _taskLog                   10021d2c     moc_DNAFlexTask.obj
 0003:00000d34       _algoLog                   10021d34     moc_DNAFlexTask.obj
 0003:00000d3c       _userActLog                10021d3c     moc_DNAFlexTask.obj
 0003:00000d44       _ioLog                     10021d44     moc_DNAFlexTask.obj
 0003:00000d4c       _coreLog                   10021d4c     moc_DNAFlexTask.obj
 0003:00000d54       _uiLog                     10021d54     moc_DNAFlexTask.obj
 0003:00000d5c       _scriptLog                 10021d5c     moc_DNAFlexTask.obj
 0003:00000d64       _perfLog                   10021d64     moc_DNAFlexTask.obj
 0003:00000d6c       _cmdLog                    10021d6c     moc_DNAFlexTask.obj
 0003:00000d74       __Tuple_alloc              10021d74     moc_FindHighFlexRegions.obj
 0003:00000d75       _ignore                    10021d75     moc_FindHighFlexRegions.obj
 0003:00000d76       _allocator_arg             10021d76     moc_FindHighFlexRegions.obj
 0003:00000d77       _piecewise_construct       10021d77     moc_FindHighFlexRegions.obj
 0003:00000d78       _taskLog                   10021d78     moc_FindHighFlexRegions.obj
 0003:00000d80       _algoLog                   10021d80     moc_FindHighFlexRegions.obj
 0003:00000d88       _userActLog                10021d88     moc_FindHighFlexRegions.obj
 0003:00000d90       _ioLog                     10021d90     moc_FindHighFlexRegions.obj
 0003:00000d98       _coreLog                   10021d98     moc_FindHighFlexRegions.obj
 0003:00000da0       _uiLog                     10021da0     moc_FindHighFlexRegions.obj
 0003:00000da8       _scriptLog                 10021da8     moc_FindHighFlexRegions.obj
 0003:00000db0       _perfLog                   10021db0     moc_FindHighFlexRegions.obj
 0003:00000db8       _cmdLog                    10021db8     moc_FindHighFlexRegions.obj
 0003:00000dc4       ___proc_attached           10021dc4     MSVCRT:crtdll.obj
 0003:00000dc8       _GS_ExceptionRecord        10021dc8     MSVCRT:gs_report.obj
 0003:00000e18       _GS_ContextRecord          10021e18     MSVCRT:gs_report.obj
 0003:000010e4       _DebuggerWasPresent        100220e4     MSVCRT:gs_report.obj
 0004:00000060       $R000000                   10023060     * linker generated manifest res *

 Exports

  ordinal    name

        1    _ugene_plugin_init
               exported name: ugene_plugin_init
